Archive member included to satisfy reference by file (symbol)

d:/lijie_tools/clion_cubemx/gcc-arm-none-eabi-10.3-2021.10/bin/../lib/gcc/arm-none-eabi/10.3.1/thumb/v7e-m/nofp\libgcc.a(_arm_muldf3.o)
                              CMakeFiles/H750_S15909.elf.dir/APP/DS18B20.c.obj (__aeabi_dmul)
d:/lijie_tools/clion_cubemx/gcc-arm-none-eabi-10.3-2021.10/bin/../lib/gcc/arm-none-eabi/10.3.1/thumb/v7e-m/nofp\libgcc.a(_arm_mulsf3.o)
                              CMakeFiles/H750_S15909.elf.dir/Core/Src/system_stm32h7xx.c.obj (__aeabi_fmul)
d:/lijie_tools/clion_cubemx/gcc-arm-none-eabi-10.3-2021.10/bin/../lib/gcc/arm-none-eabi/10.3.1/thumb/v7e-m/nofp\libgcc.a(_arm_addsubdf3.o)
                              CMakeFiles/H750_S15909.elf.dir/APP/data_analyse.c.obj (__aeabi_dadd)
d:/lijie_tools/clion_cubemx/gcc-arm-none-eabi-10.3-2021.10/bin/../lib/gcc/arm-none-eabi/10.3.1/thumb/v7e-m/nofp\libgcc.a(_arm_muldivdf3.o)
                              CMakeFiles/H750_S15909.elf.dir/APP/communication.c.obj (__aeabi_ddiv)
d:/lijie_tools/clion_cubemx/gcc-arm-none-eabi-10.3-2021.10/bin/../lib/gcc/arm-none-eabi/10.3.1/thumb/v7e-m/nofp\libgcc.a(_arm_cmpdf2.o)
                              CMakeFiles/H750_S15909.elf.dir/APP/communication.c.obj (__aeabi_dcmplt)
d:/lijie_tools/clion_cubemx/gcc-arm-none-eabi-10.3-2021.10/bin/../lib/gcc/arm-none-eabi/10.3.1/thumb/v7e-m/nofp\libgcc.a(_arm_fixdfsi.o)
                              CMakeFiles/H750_S15909.elf.dir/APP/communication.c.obj (__aeabi_d2iz)
d:/lijie_tools/clion_cubemx/gcc-arm-none-eabi-10.3-2021.10/bin/../lib/gcc/arm-none-eabi/10.3.1/thumb/v7e-m/nofp\libgcc.a(_arm_fixunsdfsi.o)
                              CMakeFiles/H750_S15909.elf.dir/APP/data_analyse.c.obj (__aeabi_d2uiz)
d:/lijie_tools/clion_cubemx/gcc-arm-none-eabi-10.3-2021.10/bin/../lib/gcc/arm-none-eabi/10.3.1/thumb/v7e-m/nofp\libgcc.a(_arm_truncdfsf2.o)
                              CMakeFiles/H750_S15909.elf.dir/APP/DS18B20.c.obj (__aeabi_d2f)
d:/lijie_tools/clion_cubemx/gcc-arm-none-eabi-10.3-2021.10/bin/../lib/gcc/arm-none-eabi/10.3.1/thumb/v7e-m/nofp\libgcc.a(_arm_addsubsf3.o)
                              CMakeFiles/H750_S15909.elf.dir/Core/Src/system_stm32h7xx.c.obj (__aeabi_fadd)
d:/lijie_tools/clion_cubemx/gcc-arm-none-eabi-10.3-2021.10/bin/../lib/gcc/arm-none-eabi/10.3.1/thumb/v7e-m/nofp\libgcc.a(_arm_muldivsf3.o)
                              CMakeFiles/H750_S15909.elf.dir/Core/Src/system_stm32h7xx.c.obj (__aeabi_fdiv)
d:/lijie_tools/clion_cubemx/gcc-arm-none-eabi-10.3-2021.10/bin/../lib/gcc/arm-none-eabi/10.3.1/thumb/v7e-m/nofp\libgcc.a(_arm_fixunssfsi.o)
                              CMakeFiles/H750_S15909.elf.dir/Core/Src/system_stm32h7xx.c.obj (__aeabi_f2uiz)
d:/lijie_tools/clion_cubemx/gcc-arm-none-eabi-10.3-2021.10/bin/../lib/gcc/arm-none-eabi/10.3.1/thumb/v7e-m/nofp\libgcc.a(_aeabi_uldivmod.o)
                              CMakeFiles/H750_S15909.elf.dir/Drivers/STM32H7xx_HAL_Driver/Src/stm32h7xx_hal_uart.c.obj (__aeabi_uldivmod)
d:/lijie_tools/clion_cubemx/gcc-arm-none-eabi-10.3-2021.10/bin/../lib/gcc/arm-none-eabi/10.3.1/thumb/v7e-m/nofp\libgcc.a(_udivmoddi4.o)
                              d:/lijie_tools/clion_cubemx/gcc-arm-none-eabi-10.3-2021.10/bin/../lib/gcc/arm-none-eabi/10.3.1/thumb/v7e-m/nofp\libgcc.a(_aeabi_uldivmod.o) (__udivmoddi4)
d:/lijie_tools/clion_cubemx/gcc-arm-none-eabi-10.3-2021.10/bin/../lib/gcc/arm-none-eabi/10.3.1/thumb/v7e-m/nofp\libgcc.a(_dvmd_tls.o)
                              d:/lijie_tools/clion_cubemx/gcc-arm-none-eabi-10.3-2021.10/bin/../lib/gcc/arm-none-eabi/10.3.1/thumb/v7e-m/nofp\libgcc.a(_aeabi_uldivmod.o) (__aeabi_ldiv0)
d:/lijie_tools/clion_cubemx/gcc-arm-none-eabi-10.3-2021.10/bin/../lib/gcc/arm-none-eabi/10.3.1/../../../../arm-none-eabi/lib/thumb/v7e-m/nofp\libg.a(lib_a-errno.o)
                              CMakeFiles/H750_S15909.elf.dir/Core/Src/syscalls.c.obj (__errno)
d:/lijie_tools/clion_cubemx/gcc-arm-none-eabi-10.3-2021.10/bin/../lib/gcc/arm-none-eabi/10.3.1/../../../../arm-none-eabi/lib/thumb/v7e-m/nofp\libg.a(lib_a-exit.o)
                              d:/lijie_tools/clion_cubemx/gcc-arm-none-eabi-10.3-2021.10/bin/../lib/gcc/arm-none-eabi/10.3.1/../../../../arm-none-eabi/lib/thumb/v7e-m/nofp/crt0.o (exit)
d:/lijie_tools/clion_cubemx/gcc-arm-none-eabi-10.3-2021.10/bin/../lib/gcc/arm-none-eabi/10.3.1/../../../../arm-none-eabi/lib/thumb/v7e-m/nofp\libg.a(lib_a-impure.o)
                              d:/lijie_tools/clion_cubemx/gcc-arm-none-eabi-10.3-2021.10/bin/../lib/gcc/arm-none-eabi/10.3.1/../../../../arm-none-eabi/lib/thumb/v7e-m/nofp\libg.a(lib_a-exit.o) (_global_impure_ptr)
d:/lijie_tools/clion_cubemx/gcc-arm-none-eabi-10.3-2021.10/bin/../lib/gcc/arm-none-eabi/10.3.1/../../../../arm-none-eabi/lib/thumb/v7e-m/nofp\libg.a(lib_a-init.o)
                              d:/lijie_tools/clion_cubemx/gcc-arm-none-eabi-10.3-2021.10/bin/../lib/gcc/arm-none-eabi/10.3.1/../../../../arm-none-eabi/lib/thumb/v7e-m/nofp/crt0.o (__libc_init_array)
d:/lijie_tools/clion_cubemx/gcc-arm-none-eabi-10.3-2021.10/bin/../lib/gcc/arm-none-eabi/10.3.1/../../../../arm-none-eabi/lib/thumb/v7e-m/nofp\libg.a(lib_a-memcpy.o)
                              CMakeFiles/H750_S15909.elf.dir/APP/IRIS_Method.c.obj (memcpy)
d:/lijie_tools/clion_cubemx/gcc-arm-none-eabi-10.3-2021.10/bin/../lib/gcc/arm-none-eabi/10.3.1/../../../../arm-none-eabi/lib/thumb/v7e-m/nofp\libg.a(lib_a-memset.o)
                              d:/lijie_tools/clion_cubemx/gcc-arm-none-eabi-10.3-2021.10/bin/../lib/gcc/arm-none-eabi/10.3.1/../../../../arm-none-eabi/lib/thumb/v7e-m/nofp/crt0.o (memset)
d:/lijie_tools/clion_cubemx/gcc-arm-none-eabi-10.3-2021.10/bin/../lib/gcc/arm-none-eabi/10.3.1/../../../../arm-none-eabi/lib/thumb/v7e-m/nofp\libg.a(lib_a-setvbuf.o)
                              CMakeFiles/H750_S15909.elf.dir/APP/mymain.c.obj (setvbuf)
d:/lijie_tools/clion_cubemx/gcc-arm-none-eabi-10.3-2021.10/bin/../lib/gcc/arm-none-eabi/10.3.1/../../../../arm-none-eabi/lib/thumb/v7e-m/nofp\libg.a(lib_a-__call_atexit.o)
                              d:/lijie_tools/clion_cubemx/gcc-arm-none-eabi-10.3-2021.10/bin/../lib/gcc/arm-none-eabi/10.3.1/../../../../arm-none-eabi/lib/thumb/v7e-m/nofp\libg.a(lib_a-exit.o) (__call_exitprocs)
d:/lijie_tools/clion_cubemx/gcc-arm-none-eabi-10.3-2021.10/bin/../lib/gcc/arm-none-eabi/10.3.1/../../../../arm-none-eabi/lib/thumb/v7e-m/nofp\libg.a(lib_a-atexit.o)
                              d:/lijie_tools/clion_cubemx/gcc-arm-none-eabi-10.3-2021.10/bin/../lib/gcc/arm-none-eabi/10.3.1/../../../../arm-none-eabi/lib/thumb/v7e-m/nofp\libg.a(lib_a-__call_atexit.o) (atexit)
d:/lijie_tools/clion_cubemx/gcc-arm-none-eabi-10.3-2021.10/bin/../lib/gcc/arm-none-eabi/10.3.1/../../../../arm-none-eabi/lib/thumb/v7e-m/nofp\libg.a(lib_a-fflush.o)
                              d:/lijie_tools/clion_cubemx/gcc-arm-none-eabi-10.3-2021.10/bin/../lib/gcc/arm-none-eabi/10.3.1/../../../../arm-none-eabi/lib/thumb/v7e-m/nofp\libg.a(lib_a-setvbuf.o) (_fflush_r)
d:/lijie_tools/clion_cubemx/gcc-arm-none-eabi-10.3-2021.10/bin/../lib/gcc/arm-none-eabi/10.3.1/../../../../arm-none-eabi/lib/thumb/v7e-m/nofp\libg.a(lib_a-findfp.o)
                              d:/lijie_tools/clion_cubemx/gcc-arm-none-eabi-10.3-2021.10/bin/../lib/gcc/arm-none-eabi/10.3.1/../../../../arm-none-eabi/lib/thumb/v7e-m/nofp\libg.a(lib_a-setvbuf.o) (__sinit)
d:/lijie_tools/clion_cubemx/gcc-arm-none-eabi-10.3-2021.10/bin/../lib/gcc/arm-none-eabi/10.3.1/../../../../arm-none-eabi/lib/thumb/v7e-m/nofp\libg.a(lib_a-fini.o)
                              d:/lijie_tools/clion_cubemx/gcc-arm-none-eabi-10.3-2021.10/bin/../lib/gcc/arm-none-eabi/10.3.1/../../../../arm-none-eabi/lib/thumb/v7e-m/nofp\libg.a(lib_a-__call_atexit.o) (__libc_fini_array)
d:/lijie_tools/clion_cubemx/gcc-arm-none-eabi-10.3-2021.10/bin/../lib/gcc/arm-none-eabi/10.3.1/../../../../arm-none-eabi/lib/thumb/v7e-m/nofp\libg.a(lib_a-freer.o)
                              d:/lijie_tools/clion_cubemx/gcc-arm-none-eabi-10.3-2021.10/bin/../lib/gcc/arm-none-eabi/10.3.1/../../../../arm-none-eabi/lib/thumb/v7e-m/nofp\libg.a(lib_a-setvbuf.o) (_free_r)
d:/lijie_tools/clion_cubemx/gcc-arm-none-eabi-10.3-2021.10/bin/../lib/gcc/arm-none-eabi/10.3.1/../../../../arm-none-eabi/lib/thumb/v7e-m/nofp\libg.a(lib_a-fwalk.o)
                              d:/lijie_tools/clion_cubemx/gcc-arm-none-eabi-10.3-2021.10/bin/../lib/gcc/arm-none-eabi/10.3.1/../../../../arm-none-eabi/lib/thumb/v7e-m/nofp\libg.a(lib_a-findfp.o) (_fwalk)
d:/lijie_tools/clion_cubemx/gcc-arm-none-eabi-10.3-2021.10/bin/../lib/gcc/arm-none-eabi/10.3.1/../../../../arm-none-eabi/lib/thumb/v7e-m/nofp\libg.a(lib_a-lock.o)
                              d:/lijie_tools/clion_cubemx/gcc-arm-none-eabi-10.3-2021.10/bin/../lib/gcc/arm-none-eabi/10.3.1/../../../../arm-none-eabi/lib/thumb/v7e-m/nofp\libg.a(lib_a-findfp.o) (__retarget_lock_init_recursive)
d:/lijie_tools/clion_cubemx/gcc-arm-none-eabi-10.3-2021.10/bin/../lib/gcc/arm-none-eabi/10.3.1/../../../../arm-none-eabi/lib/thumb/v7e-m/nofp\libg.a(lib_a-makebuf.o)
                              d:/lijie_tools/clion_cubemx/gcc-arm-none-eabi-10.3-2021.10/bin/../lib/gcc/arm-none-eabi/10.3.1/../../../../arm-none-eabi/lib/thumb/v7e-m/nofp\libg.a(lib_a-setvbuf.o) (__swhatbuf_r)
d:/lijie_tools/clion_cubemx/gcc-arm-none-eabi-10.3-2021.10/bin/../lib/gcc/arm-none-eabi/10.3.1/../../../../arm-none-eabi/lib/thumb/v7e-m/nofp\libg.a(lib_a-malloc.o)
                              d:/lijie_tools/clion_cubemx/gcc-arm-none-eabi-10.3-2021.10/bin/../lib/gcc/arm-none-eabi/10.3.1/../../../../arm-none-eabi/lib/thumb/v7e-m/nofp\libg.a(lib_a-setvbuf.o) (malloc)
d:/lijie_tools/clion_cubemx/gcc-arm-none-eabi-10.3-2021.10/bin/../lib/gcc/arm-none-eabi/10.3.1/../../../../arm-none-eabi/lib/thumb/v7e-m/nofp\libg.a(lib_a-mallocr.o)
                              d:/lijie_tools/clion_cubemx/gcc-arm-none-eabi-10.3-2021.10/bin/../lib/gcc/arm-none-eabi/10.3.1/../../../../arm-none-eabi/lib/thumb/v7e-m/nofp\libg.a(lib_a-findfp.o) (_malloc_r)
d:/lijie_tools/clion_cubemx/gcc-arm-none-eabi-10.3-2021.10/bin/../lib/gcc/arm-none-eabi/10.3.1/../../../../arm-none-eabi/lib/thumb/v7e-m/nofp\libg.a(lib_a-mlock.o)
                              d:/lijie_tools/clion_cubemx/gcc-arm-none-eabi-10.3-2021.10/bin/../lib/gcc/arm-none-eabi/10.3.1/../../../../arm-none-eabi/lib/thumb/v7e-m/nofp\libg.a(lib_a-freer.o) (__malloc_lock)
d:/lijie_tools/clion_cubemx/gcc-arm-none-eabi-10.3-2021.10/bin/../lib/gcc/arm-none-eabi/10.3.1/../../../../arm-none-eabi/lib/thumb/v7e-m/nofp\libg.a(lib_a-sbrkr.o)
                              d:/lijie_tools/clion_cubemx/gcc-arm-none-eabi-10.3-2021.10/bin/../lib/gcc/arm-none-eabi/10.3.1/../../../../arm-none-eabi/lib/thumb/v7e-m/nofp\libg.a(lib_a-freer.o) (_sbrk_r)
d:/lijie_tools/clion_cubemx/gcc-arm-none-eabi-10.3-2021.10/bin/../lib/gcc/arm-none-eabi/10.3.1/../../../../arm-none-eabi/lib/thumb/v7e-m/nofp\libg.a(lib_a-stdio.o)
                              d:/lijie_tools/clion_cubemx/gcc-arm-none-eabi-10.3-2021.10/bin/../lib/gcc/arm-none-eabi/10.3.1/../../../../arm-none-eabi/lib/thumb/v7e-m/nofp\libg.a(lib_a-findfp.o) (__sread)
d:/lijie_tools/clion_cubemx/gcc-arm-none-eabi-10.3-2021.10/bin/../lib/gcc/arm-none-eabi/10.3.1/../../../../arm-none-eabi/lib/thumb/v7e-m/nofp\libg.a(lib_a-writer.o)
                              d:/lijie_tools/clion_cubemx/gcc-arm-none-eabi-10.3-2021.10/bin/../lib/gcc/arm-none-eabi/10.3.1/../../../../arm-none-eabi/lib/thumb/v7e-m/nofp\libg.a(lib_a-stdio.o) (_write_r)
d:/lijie_tools/clion_cubemx/gcc-arm-none-eabi-10.3-2021.10/bin/../lib/gcc/arm-none-eabi/10.3.1/../../../../arm-none-eabi/lib/thumb/v7e-m/nofp\libg.a(lib_a-__atexit.o)
                              d:/lijie_tools/clion_cubemx/gcc-arm-none-eabi-10.3-2021.10/bin/../lib/gcc/arm-none-eabi/10.3.1/../../../../arm-none-eabi/lib/thumb/v7e-m/nofp\libg.a(lib_a-atexit.o) (__register_exitproc)
d:/lijie_tools/clion_cubemx/gcc-arm-none-eabi-10.3-2021.10/bin/../lib/gcc/arm-none-eabi/10.3.1/../../../../arm-none-eabi/lib/thumb/v7e-m/nofp\libg.a(lib_a-closer.o)
                              d:/lijie_tools/clion_cubemx/gcc-arm-none-eabi-10.3-2021.10/bin/../lib/gcc/arm-none-eabi/10.3.1/../../../../arm-none-eabi/lib/thumb/v7e-m/nofp\libg.a(lib_a-stdio.o) (_close_r)
d:/lijie_tools/clion_cubemx/gcc-arm-none-eabi-10.3-2021.10/bin/../lib/gcc/arm-none-eabi/10.3.1/../../../../arm-none-eabi/lib/thumb/v7e-m/nofp\libg.a(lib_a-fclose.o)
                              d:/lijie_tools/clion_cubemx/gcc-arm-none-eabi-10.3-2021.10/bin/../lib/gcc/arm-none-eabi/10.3.1/../../../../arm-none-eabi/lib/thumb/v7e-m/nofp\libg.a(lib_a-findfp.o) (_fclose_r)
d:/lijie_tools/clion_cubemx/gcc-arm-none-eabi-10.3-2021.10/bin/../lib/gcc/arm-none-eabi/10.3.1/../../../../arm-none-eabi/lib/thumb/v7e-m/nofp\libg.a(lib_a-fstatr.o)
                              d:/lijie_tools/clion_cubemx/gcc-arm-none-eabi-10.3-2021.10/bin/../lib/gcc/arm-none-eabi/10.3.1/../../../../arm-none-eabi/lib/thumb/v7e-m/nofp\libg.a(lib_a-makebuf.o) (_fstat_r)
d:/lijie_tools/clion_cubemx/gcc-arm-none-eabi-10.3-2021.10/bin/../lib/gcc/arm-none-eabi/10.3.1/../../../../arm-none-eabi/lib/thumb/v7e-m/nofp\libg.a(lib_a-isattyr.o)
                              d:/lijie_tools/clion_cubemx/gcc-arm-none-eabi-10.3-2021.10/bin/../lib/gcc/arm-none-eabi/10.3.1/../../../../arm-none-eabi/lib/thumb/v7e-m/nofp\libg.a(lib_a-makebuf.o) (_isatty_r)
d:/lijie_tools/clion_cubemx/gcc-arm-none-eabi-10.3-2021.10/bin/../lib/gcc/arm-none-eabi/10.3.1/../../../../arm-none-eabi/lib/thumb/v7e-m/nofp\libg.a(lib_a-lseekr.o)
                              d:/lijie_tools/clion_cubemx/gcc-arm-none-eabi-10.3-2021.10/bin/../lib/gcc/arm-none-eabi/10.3.1/../../../../arm-none-eabi/lib/thumb/v7e-m/nofp\libg.a(lib_a-stdio.o) (_lseek_r)
d:/lijie_tools/clion_cubemx/gcc-arm-none-eabi-10.3-2021.10/bin/../lib/gcc/arm-none-eabi/10.3.1/../../../../arm-none-eabi/lib/thumb/v7e-m/nofp\libg.a(lib_a-readr.o)
                              d:/lijie_tools/clion_cubemx/gcc-arm-none-eabi-10.3-2021.10/bin/../lib/gcc/arm-none-eabi/10.3.1/../../../../arm-none-eabi/lib/thumb/v7e-m/nofp\libg.a(lib_a-stdio.o) (_read_r)
d:/lijie_tools/clion_cubemx/gcc-arm-none-eabi-10.3-2021.10/bin/../lib/gcc/arm-none-eabi/10.3.1/../../../../arm-none-eabi/lib/thumb/v7e-m/nofp\libg.a(lib_a-reent.o)
                              d:/lijie_tools/clion_cubemx/gcc-arm-none-eabi-10.3-2021.10/bin/../lib/gcc/arm-none-eabi/10.3.1/../../../../arm-none-eabi/lib/thumb/v7e-m/nofp\libg.a(lib_a-sbrkr.o) (errno)
d:/lijie_tools/clion_cubemx/gcc-arm-none-eabi-10.3-2021.10/bin/../lib/gcc/arm-none-eabi/10.3.1/../../../../arm-none-eabi/lib/thumb/v7e-m/nofp\libm.a(lib_a-s_round.o)
                              CMakeFiles/H750_S15909.elf.dir/APP/data_analyse.c.obj (round)
d:/lijie_tools/clion_cubemx/gcc-arm-none-eabi-10.3-2021.10/bin/../lib/gcc/arm-none-eabi/10.3.1/../../../../arm-none-eabi/lib/thumb/v7e-m/nofp\libm.a(lib_a-w_exp.o)
                              CMakeFiles/H750_S15909.elf.dir/APP/data_analyse.c.obj (exp)
d:/lijie_tools/clion_cubemx/gcc-arm-none-eabi-10.3-2021.10/bin/../lib/gcc/arm-none-eabi/10.3.1/../../../../arm-none-eabi/lib/thumb/v7e-m/nofp\libm.a(lib_a-e_exp.o)
                              d:/lijie_tools/clion_cubemx/gcc-arm-none-eabi-10.3-2021.10/bin/../lib/gcc/arm-none-eabi/10.3.1/../../../../arm-none-eabi/lib/thumb/v7e-m/nofp\libm.a(lib_a-w_exp.o) (__ieee754_exp)
d:/lijie_tools/clion_cubemx/gcc-arm-none-eabi-10.3-2021.10/bin/../lib/gcc/arm-none-eabi/10.3.1/../../../../arm-none-eabi/lib/thumb/v7e-m/nofp\libm.a(lib_a-math_err.o)
                              d:/lijie_tools/clion_cubemx/gcc-arm-none-eabi-10.3-2021.10/bin/../lib/gcc/arm-none-eabi/10.3.1/../../../../arm-none-eabi/lib/thumb/v7e-m/nofp\libm.a(lib_a-e_exp.o) (__math_uflow)
d:/lijie_tools/clion_cubemx/gcc-arm-none-eabi-10.3-2021.10/bin/../lib/gcc/arm-none-eabi/10.3.1/../../../../arm-none-eabi/lib/thumb/v7e-m/nofp\libm.a(lib_a-s_finite.o)
                              d:/lijie_tools/clion_cubemx/gcc-arm-none-eabi-10.3-2021.10/bin/../lib/gcc/arm-none-eabi/10.3.1/../../../../arm-none-eabi/lib/thumb/v7e-m/nofp\libm.a(lib_a-w_exp.o) (finite)
d:/lijie_tools/clion_cubemx/gcc-arm-none-eabi-10.3-2021.10/bin/../lib/gcc/arm-none-eabi/10.3.1/thumb/v7e-m/nofp\libgcc.a(_arm_unorddf2.o)
                              d:/lijie_tools/clion_cubemx/gcc-arm-none-eabi-10.3-2021.10/bin/../lib/gcc/arm-none-eabi/10.3.1/../../../../arm-none-eabi/lib/thumb/v7e-m/nofp\libm.a(lib_a-math_err.o) (__aeabi_dcmpun)

Discarded input sections

 .text          0x00000000        0x0 d:/lijie_tools/clion_cubemx/gcc-arm-none-eabi-10.3-2021.10/bin/../lib/gcc/arm-none-eabi/10.3.1/thumb/v7e-m/nofp/crti.o
 .data          0x00000000        0x0 d:/lijie_tools/clion_cubemx/gcc-arm-none-eabi-10.3-2021.10/bin/../lib/gcc/arm-none-eabi/10.3.1/thumb/v7e-m/nofp/crti.o
 .bss           0x00000000        0x0 d:/lijie_tools/clion_cubemx/gcc-arm-none-eabi-10.3-2021.10/bin/../lib/gcc/arm-none-eabi/10.3.1/thumb/v7e-m/nofp/crti.o
 .data          0x00000000        0x4 d:/lijie_tools/clion_cubemx/gcc-arm-none-eabi-10.3-2021.10/bin/../lib/gcc/arm-none-eabi/10.3.1/thumb/v7e-m/nofp/crtbegin.o
 .rodata        0x00000000       0x24 d:/lijie_tools/clion_cubemx/gcc-arm-none-eabi-10.3-2021.10/bin/../lib/gcc/arm-none-eabi/10.3.1/thumb/v7e-m/nofp/crtbegin.o
 .text          0x00000000       0x7c d:/lijie_tools/clion_cubemx/gcc-arm-none-eabi-10.3-2021.10/bin/../lib/gcc/arm-none-eabi/10.3.1/../../../../arm-none-eabi/lib/thumb/v7e-m/nofp/crt0.o
 .data          0x00000000        0x0 d:/lijie_tools/clion_cubemx/gcc-arm-none-eabi-10.3-2021.10/bin/../lib/gcc/arm-none-eabi/10.3.1/../../../../arm-none-eabi/lib/thumb/v7e-m/nofp/crt0.o
 .bss           0x00000000        0x0 d:/lijie_tools/clion_cubemx/gcc-arm-none-eabi-10.3-2021.10/bin/../lib/gcc/arm-none-eabi/10.3.1/../../../../arm-none-eabi/lib/thumb/v7e-m/nofp/crt0.o
 .ARM.extab     0x00000000        0x0 d:/lijie_tools/clion_cubemx/gcc-arm-none-eabi-10.3-2021.10/bin/../lib/gcc/arm-none-eabi/10.3.1/../../../../arm-none-eabi/lib/thumb/v7e-m/nofp/crt0.o
 .ARM.exidx     0x00000000       0x10 d:/lijie_tools/clion_cubemx/gcc-arm-none-eabi-10.3-2021.10/bin/../lib/gcc/arm-none-eabi/10.3.1/../../../../arm-none-eabi/lib/thumb/v7e-m/nofp/crt0.o
 .ARM.attributes
                0x00000000       0x1c d:/lijie_tools/clion_cubemx/gcc-arm-none-eabi-10.3-2021.10/bin/../lib/gcc/arm-none-eabi/10.3.1/../../../../arm-none-eabi/lib/thumb/v7e-m/nofp/crt0.o
 .text          0x00000000        0x0 CMakeFiles/H750_S15909.elf.dir/APP/DS18B20.c.obj
 .data          0x00000000        0x0 CMakeFiles/H750_S15909.elf.dir/APP/DS18B20.c.obj
 .bss           0x00000000        0x0 CMakeFiles/H750_S15909.elf.dir/APP/DS18B20.c.obj
 .text.DS18B20_Write_Bit
                0x00000000       0x58 CMakeFiles/H750_S15909.elf.dir/APP/DS18B20.c.obj
 .text          0x00000000        0x0 CMakeFiles/H750_S15909.elf.dir/APP/IRIS_Method.c.obj
 .data          0x00000000        0x0 CMakeFiles/H750_S15909.elf.dir/APP/IRIS_Method.c.obj
 .bss           0x00000000        0x0 CMakeFiles/H750_S15909.elf.dir/APP/IRIS_Method.c.obj
 .text.IRIS_Cut_Befor_Header
                0x00000000       0x54 CMakeFiles/H750_S15909.elf.dir/APP/IRIS_Method.c.obj
 .text.IRIS_Protocol_Unpack
                0x00000000       0xa4 CMakeFiles/H750_S15909.elf.dir/APP/IRIS_Method.c.obj
 .text.IRIS_Check_Data_Valid
                0x00000000       0x78 CMakeFiles/H750_S15909.elf.dir/APP/IRIS_Method.c.obj
 .text          0x00000000        0x0 CMakeFiles/H750_S15909.elf.dir/APP/LED.c.obj
 .data          0x00000000        0x0 CMakeFiles/H750_S15909.elf.dir/APP/LED.c.obj
 .bss           0x00000000        0x0 CMakeFiles/H750_S15909.elf.dir/APP/LED.c.obj
 .text.led_init
                0x00000000       0x4c CMakeFiles/H750_S15909.elf.dir/APP/LED.c.obj
 .debug_info    0x00000000      0x5f6 CMakeFiles/H750_S15909.elf.dir/APP/LED.c.obj
 .debug_abbrev  0x00000000      0x143 CMakeFiles/H750_S15909.elf.dir/APP/LED.c.obj
 .debug_aranges
                0x00000000       0x20 CMakeFiles/H750_S15909.elf.dir/APP/LED.c.obj
 .debug_ranges  0x00000000       0x10 CMakeFiles/H750_S15909.elf.dir/APP/LED.c.obj
 .debug_line    0x00000000      0x1d9 CMakeFiles/H750_S15909.elf.dir/APP/LED.c.obj
 .debug_str     0x00000000      0x489 CMakeFiles/H750_S15909.elf.dir/APP/LED.c.obj
 .comment       0x00000000       0x4a CMakeFiles/H750_S15909.elf.dir/APP/LED.c.obj
 .debug_frame   0x00000000       0x2c CMakeFiles/H750_S15909.elf.dir/APP/LED.c.obj
 .ARM.attributes
                0x00000000       0x2e CMakeFiles/H750_S15909.elf.dir/APP/LED.c.obj
 .text          0x00000000        0x0 CMakeFiles/H750_S15909.elf.dir/APP/Shutter.c.obj
 .data          0x00000000        0x0 CMakeFiles/H750_S15909.elf.dir/APP/Shutter.c.obj
 .bss           0x00000000        0x0 CMakeFiles/H750_S15909.elf.dir/APP/Shutter.c.obj
 .text.Shutter_Init
                0x00000000       0x48 CMakeFiles/H750_S15909.elf.dir/APP/Shutter.c.obj
 .text          0x00000000        0x0 CMakeFiles/H750_S15909.elf.dir/APP/communication.c.obj
 .data          0x00000000        0x0 CMakeFiles/H750_S15909.elf.dir/APP/communication.c.obj
 .bss           0x00000000        0x0 CMakeFiles/H750_S15909.elf.dir/APP/communication.c.obj
 .text          0x00000000        0x0 CMakeFiles/H750_S15909.elf.dir/APP/data_analyse.c.obj
 .data          0x00000000        0x0 CMakeFiles/H750_S15909.elf.dir/APP/data_analyse.c.obj
 .bss           0x00000000        0x0 CMakeFiles/H750_S15909.elf.dir/APP/data_analyse.c.obj
 .text          0x00000000        0x0 CMakeFiles/H750_S15909.elf.dir/APP/delay.c.obj
 .data          0x00000000        0x0 CMakeFiles/H750_S15909.elf.dir/APP/delay.c.obj
 .bss           0x00000000        0x0 CMakeFiles/H750_S15909.elf.dir/APP/delay.c.obj
 .text          0x00000000        0x0 CMakeFiles/H750_S15909.elf.dir/APP/mymain.c.obj
 .data          0x00000000        0x0 CMakeFiles/H750_S15909.elf.dir/APP/mymain.c.obj
 .bss           0x00000000        0x0 CMakeFiles/H750_S15909.elf.dir/APP/mymain.c.obj
 .text          0x00000000        0x0 CMakeFiles/H750_S15909.elf.dir/APP/usart1_tx_dma.c.obj
 .data          0x00000000        0x0 CMakeFiles/H750_S15909.elf.dir/APP/usart1_tx_dma.c.obj
 .bss           0x00000000        0x0 CMakeFiles/H750_S15909.elf.dir/APP/usart1_tx_dma.c.obj
 .text          0x00000000        0x0 CMakeFiles/H750_S15909.elf.dir/Core/Src/dma.c.obj
 .data          0x00000000        0x0 CMakeFiles/H750_S15909.elf.dir/Core/Src/dma.c.obj
 .bss           0x00000000        0x0 CMakeFiles/H750_S15909.elf.dir/Core/Src/dma.c.obj
 .text          0x00000000        0x0 CMakeFiles/H750_S15909.elf.dir/Core/Src/gpio.c.obj
 .data          0x00000000        0x0 CMakeFiles/H750_S15909.elf.dir/Core/Src/gpio.c.obj
 .bss           0x00000000        0x0 CMakeFiles/H750_S15909.elf.dir/Core/Src/gpio.c.obj
 .text          0x00000000        0x0 CMakeFiles/H750_S15909.elf.dir/Core/Src/main.c.obj
 .data          0x00000000        0x0 CMakeFiles/H750_S15909.elf.dir/Core/Src/main.c.obj
 .bss           0x00000000        0x0 CMakeFiles/H750_S15909.elf.dir/Core/Src/main.c.obj
 .text          0x00000000        0x0 CMakeFiles/H750_S15909.elf.dir/Core/Src/stm32h7xx_hal_msp.c.obj
 .data          0x00000000        0x0 CMakeFiles/H750_S15909.elf.dir/Core/Src/stm32h7xx_hal_msp.c.obj
 .bss           0x00000000        0x0 CMakeFiles/H750_S15909.elf.dir/Core/Src/stm32h7xx_hal_msp.c.obj
 .text          0x00000000        0x0 CMakeFiles/H750_S15909.elf.dir/Core/Src/stm32h7xx_it.c.obj
 .data          0x00000000        0x0 CMakeFiles/H750_S15909.elf.dir/Core/Src/stm32h7xx_it.c.obj
 .bss           0x00000000        0x0 CMakeFiles/H750_S15909.elf.dir/Core/Src/stm32h7xx_it.c.obj
 .text          0x00000000        0x0 CMakeFiles/H750_S15909.elf.dir/Core/Src/syscalls.c.obj
 .data          0x00000000        0x0 CMakeFiles/H750_S15909.elf.dir/Core/Src/syscalls.c.obj
 .bss           0x00000000        0x0 CMakeFiles/H750_S15909.elf.dir/Core/Src/syscalls.c.obj
 .text.initialise_monitor_handles
                0x00000000        0x2 CMakeFiles/H750_S15909.elf.dir/Core/Src/syscalls.c.obj
 .text._getpid  0x00000000        0x4 CMakeFiles/H750_S15909.elf.dir/Core/Src/syscalls.c.obj
 .text._kill    0x00000000       0x10 CMakeFiles/H750_S15909.elf.dir/Core/Src/syscalls.c.obj
 .text._exit    0x00000000        0xc CMakeFiles/H750_S15909.elf.dir/Core/Src/syscalls.c.obj
 .text._write   0x00000000       0x1c CMakeFiles/H750_S15909.elf.dir/Core/Src/syscalls.c.obj
 .text._isatty  0x00000000        0x4 CMakeFiles/H750_S15909.elf.dir/Core/Src/syscalls.c.obj
 .text._open    0x00000000        0xa CMakeFiles/H750_S15909.elf.dir/Core/Src/syscalls.c.obj
 .text._wait    0x00000000       0x10 CMakeFiles/H750_S15909.elf.dir/Core/Src/syscalls.c.obj
 .text._unlink  0x00000000       0x10 CMakeFiles/H750_S15909.elf.dir/Core/Src/syscalls.c.obj
 .text._times   0x00000000        0x6 CMakeFiles/H750_S15909.elf.dir/Core/Src/syscalls.c.obj
 .text._stat    0x00000000        0xa CMakeFiles/H750_S15909.elf.dir/Core/Src/syscalls.c.obj
 .text._link    0x00000000       0x10 CMakeFiles/H750_S15909.elf.dir/Core/Src/syscalls.c.obj
 .text._fork    0x00000000       0x10 CMakeFiles/H750_S15909.elf.dir/Core/Src/syscalls.c.obj
 .text._execve  0x00000000       0x10 CMakeFiles/H750_S15909.elf.dir/Core/Src/syscalls.c.obj
 .bss.__env     0x00000000        0x4 CMakeFiles/H750_S15909.elf.dir/Core/Src/syscalls.c.obj
 .data.environ  0x00000000        0x4 CMakeFiles/H750_S15909.elf.dir/Core/Src/syscalls.c.obj
 .text          0x00000000        0x0 CMakeFiles/H750_S15909.elf.dir/Core/Src/sysmem.c.obj
 .data          0x00000000        0x0 CMakeFiles/H750_S15909.elf.dir/Core/Src/sysmem.c.obj
 .bss           0x00000000        0x0 CMakeFiles/H750_S15909.elf.dir/Core/Src/sysmem.c.obj
 .text          0x00000000        0x0 CMakeFiles/H750_S15909.elf.dir/Core/Src/system_stm32h7xx.c.obj
 .data          0x00000000        0x0 CMakeFiles/H750_S15909.elf.dir/Core/Src/system_stm32h7xx.c.obj
 .bss           0x00000000        0x0 CMakeFiles/H750_S15909.elf.dir/Core/Src/system_stm32h7xx.c.obj
 .text.SystemCoreClockUpdate
                0x00000000      0x238 CMakeFiles/H750_S15909.elf.dir/Core/Src/system_stm32h7xx.c.obj
 .text          0x00000000        0x0 CMakeFiles/H750_S15909.elf.dir/Core/Src/tim.c.obj
 .data          0x00000000        0x0 CMakeFiles/H750_S15909.elf.dir/Core/Src/tim.c.obj
 .bss           0x00000000        0x0 CMakeFiles/H750_S15909.elf.dir/Core/Src/tim.c.obj
 .text.HAL_TIM_Base_MspDeInit
                0x00000000       0x24 CMakeFiles/H750_S15909.elf.dir/Core/Src/tim.c.obj
 .text          0x00000000        0x0 CMakeFiles/H750_S15909.elf.dir/Core/Src/usart.c.obj
 .data          0x00000000        0x0 CMakeFiles/H750_S15909.elf.dir/Core/Src/usart.c.obj
 .bss           0x00000000        0x0 CMakeFiles/H750_S15909.elf.dir/Core/Src/usart.c.obj
 .text.HAL_UART_MspDeInit
                0x00000000       0x64 CMakeFiles/H750_S15909.elf.dir/Core/Src/usart.c.obj
 .text          0x00000000       0x14 CMakeFiles/H750_S15909.elf.dir/Core/Startup/startup_stm32h750vbtx.s.obj
 .data          0x00000000        0x0 CMakeFiles/H750_S15909.elf.dir/Core/Startup/startup_stm32h750vbtx.s.obj
 .bss           0x00000000        0x0 CMakeFiles/H750_S15909.elf.dir/Core/Startup/startup_stm32h750vbtx.s.obj
 .text          0x00000000        0x0 CMakeFiles/H750_S15909.elf.dir/Drivers/STM32H7xx_HAL_Driver/Src/stm32h7xx_hal.c.obj
 .data          0x00000000        0x0 CMakeFiles/H750_S15909.elf.dir/Drivers/STM32H7xx_HAL_Driver/Src/stm32h7xx_hal.c.obj
 .bss           0x00000000        0x0 CMakeFiles/H750_S15909.elf.dir/Drivers/STM32H7xx_HAL_Driver/Src/stm32h7xx_hal.c.obj
 .text.HAL_MspInit
                0x00000000        0x2 CMakeFiles/H750_S15909.elf.dir/Drivers/STM32H7xx_HAL_Driver/Src/stm32h7xx_hal.c.obj
 .text.HAL_MspDeInit
                0x00000000        0x2 CMakeFiles/H750_S15909.elf.dir/Drivers/STM32H7xx_HAL_Driver/Src/stm32h7xx_hal.c.obj
 .text.HAL_DeInit
                0x00000000       0x84 CMakeFiles/H750_S15909.elf.dir/Drivers/STM32H7xx_HAL_Driver/Src/stm32h7xx_hal.c.obj
 .text.HAL_GetTickPrio
                0x00000000        0xc CMakeFiles/H750_S15909.elf.dir/Drivers/STM32H7xx_HAL_Driver/Src/stm32h7xx_hal.c.obj
 .text.HAL_SetTickFreq
                0x00000000       0x2c CMakeFiles/H750_S15909.elf.dir/Drivers/STM32H7xx_HAL_Driver/Src/stm32h7xx_hal.c.obj
 .text.HAL_GetTickFreq
                0x00000000        0xc CMakeFiles/H750_S15909.elf.dir/Drivers/STM32H7xx_HAL_Driver/Src/stm32h7xx_hal.c.obj
 .text.HAL_SuspendTick
                0x00000000        0xe CMakeFiles/H750_S15909.elf.dir/Drivers/STM32H7xx_HAL_Driver/Src/stm32h7xx_hal.c.obj
 .text.HAL_ResumeTick
                0x00000000        0xe CMakeFiles/H750_S15909.elf.dir/Drivers/STM32H7xx_HAL_Driver/Src/stm32h7xx_hal.c.obj
 .text.HAL_GetHalVersion
                0x00000000        0x8 CMakeFiles/H750_S15909.elf.dir/Drivers/STM32H7xx_HAL_Driver/Src/stm32h7xx_hal.c.obj
 .text.HAL_GetDEVID
                0x00000000       0x10 CMakeFiles/H750_S15909.elf.dir/Drivers/STM32H7xx_HAL_Driver/Src/stm32h7xx_hal.c.obj
 .text.HAL_GetUIDw0
                0x00000000        0xc CMakeFiles/H750_S15909.elf.dir/Drivers/STM32H7xx_HAL_Driver/Src/stm32h7xx_hal.c.obj
 .text.HAL_GetUIDw1
                0x00000000        0xc CMakeFiles/H750_S15909.elf.dir/Drivers/STM32H7xx_HAL_Driver/Src/stm32h7xx_hal.c.obj
 .text.HAL_GetUIDw2
                0x00000000        0xc CMakeFiles/H750_S15909.elf.dir/Drivers/STM32H7xx_HAL_Driver/Src/stm32h7xx_hal.c.obj
 .text.HAL_SYSCFG_VREFBUF_VoltageScalingConfig
                0x00000000       0x14 CMakeFiles/H750_S15909.elf.dir/Drivers/STM32H7xx_HAL_Driver/Src/stm32h7xx_hal.c.obj
 .text.HAL_SYSCFG_VREFBUF_HighImpedanceConfig
                0x00000000       0x14 CMakeFiles/H750_S15909.elf.dir/Drivers/STM32H7xx_HAL_Driver/Src/stm32h7xx_hal.c.obj
 .text.HAL_SYSCFG_VREFBUF_TrimmingConfig
                0x00000000       0x14 CMakeFiles/H750_S15909.elf.dir/Drivers/STM32H7xx_HAL_Driver/Src/stm32h7xx_hal.c.obj
 .text.HAL_SYSCFG_EnableVREFBUF
                0x00000000       0x34 CMakeFiles/H750_S15909.elf.dir/Drivers/STM32H7xx_HAL_Driver/Src/stm32h7xx_hal.c.obj
 .text.HAL_SYSCFG_DisableVREFBUF
                0x00000000       0x10 CMakeFiles/H750_S15909.elf.dir/Drivers/STM32H7xx_HAL_Driver/Src/stm32h7xx_hal.c.obj
 .text.HAL_SYSCFG_ETHInterfaceSelect
                0x00000000       0x14 CMakeFiles/H750_S15909.elf.dir/Drivers/STM32H7xx_HAL_Driver/Src/stm32h7xx_hal.c.obj
 .text.HAL_SYSCFG_AnalogSwitchConfig
                0x00000000       0x14 CMakeFiles/H750_S15909.elf.dir/Drivers/STM32H7xx_HAL_Driver/Src/stm32h7xx_hal.c.obj
 .text.HAL_SYSCFG_EnableBOOST
                0x00000000       0x10 CMakeFiles/H750_S15909.elf.dir/Drivers/STM32H7xx_HAL_Driver/Src/stm32h7xx_hal.c.obj
 .text.HAL_SYSCFG_DisableBOOST
                0x00000000       0x10 CMakeFiles/H750_S15909.elf.dir/Drivers/STM32H7xx_HAL_Driver/Src/stm32h7xx_hal.c.obj
 .text.HAL_SYSCFG_CM7BootAddConfig
                0x00000000       0x34 CMakeFiles/H750_S15909.elf.dir/Drivers/STM32H7xx_HAL_Driver/Src/stm32h7xx_hal.c.obj
 .text.HAL_EnableCompensationCell
                0x00000000       0x10 CMakeFiles/H750_S15909.elf.dir/Drivers/STM32H7xx_HAL_Driver/Src/stm32h7xx_hal.c.obj
 .text.HAL_DisableCompensationCell
                0x00000000       0x10 CMakeFiles/H750_S15909.elf.dir/Drivers/STM32H7xx_HAL_Driver/Src/stm32h7xx_hal.c.obj
 .text.HAL_SYSCFG_EnableIOSpeedOptimize
                0x00000000       0x10 CMakeFiles/H750_S15909.elf.dir/Drivers/STM32H7xx_HAL_Driver/Src/stm32h7xx_hal.c.obj
 .text.HAL_SYSCFG_DisableIOSpeedOptimize
                0x00000000       0x10 CMakeFiles/H750_S15909.elf.dir/Drivers/STM32H7xx_HAL_Driver/Src/stm32h7xx_hal.c.obj
 .text.HAL_SYSCFG_CompensationCodeSelect
                0x00000000       0x14 CMakeFiles/H750_S15909.elf.dir/Drivers/STM32H7xx_HAL_Driver/Src/stm32h7xx_hal.c.obj
 .text.HAL_SYSCFG_CompensationCodeConfig
                0x00000000       0x18 CMakeFiles/H750_S15909.elf.dir/Drivers/STM32H7xx_HAL_Driver/Src/stm32h7xx_hal.c.obj
 .text.HAL_DBGMCU_EnableDBGSleepMode
                0x00000000       0x10 CMakeFiles/H750_S15909.elf.dir/Drivers/STM32H7xx_HAL_Driver/Src/stm32h7xx_hal.c.obj
 .text.HAL_DBGMCU_DisableDBGSleepMode
                0x00000000       0x10 CMakeFiles/H750_S15909.elf.dir/Drivers/STM32H7xx_HAL_Driver/Src/stm32h7xx_hal.c.obj
 .text.HAL_DBGMCU_EnableDBGStopMode
                0x00000000       0x10 CMakeFiles/H750_S15909.elf.dir/Drivers/STM32H7xx_HAL_Driver/Src/stm32h7xx_hal.c.obj
 .text.HAL_DBGMCU_DisableDBGStopMode
                0x00000000       0x10 CMakeFiles/H750_S15909.elf.dir/Drivers/STM32H7xx_HAL_Driver/Src/stm32h7xx_hal.c.obj
 .text.HAL_DBGMCU_EnableDBGStandbyMode
                0x00000000       0x10 CMakeFiles/H750_S15909.elf.dir/Drivers/STM32H7xx_HAL_Driver/Src/stm32h7xx_hal.c.obj
 .text.HAL_DBGMCU_DisableDBGStandbyMode
                0x00000000       0x10 CMakeFiles/H750_S15909.elf.dir/Drivers/STM32H7xx_HAL_Driver/Src/stm32h7xx_hal.c.obj
 .text.HAL_SetFMCMemorySwappingConfig
                0x00000000       0x14 CMakeFiles/H750_S15909.elf.dir/Drivers/STM32H7xx_HAL_Driver/Src/stm32h7xx_hal.c.obj
 .text.HAL_GetFMCMemorySwappingConfig
                0x00000000       0x10 CMakeFiles/H750_S15909.elf.dir/Drivers/STM32H7xx_HAL_Driver/Src/stm32h7xx_hal.c.obj
 .text.HAL_EXTI_EdgeConfig
                0x00000000       0x54 CMakeFiles/H750_S15909.elf.dir/Drivers/STM32H7xx_HAL_Driver/Src/stm32h7xx_hal.c.obj
 .text.HAL_EXTI_GenerateSWInterrupt
                0x00000000       0x20 CMakeFiles/H750_S15909.elf.dir/Drivers/STM32H7xx_HAL_Driver/Src/stm32h7xx_hal.c.obj
 .text.HAL_EXTI_D1_ClearFlag
                0x00000000       0x18 CMakeFiles/H750_S15909.elf.dir/Drivers/STM32H7xx_HAL_Driver/Src/stm32h7xx_hal.c.obj
 .text.HAL_EXTI_D1_EventInputConfig
                0x00000000       0x84 CMakeFiles/H750_S15909.elf.dir/Drivers/STM32H7xx_HAL_Driver/Src/stm32h7xx_hal.c.obj
 .text.HAL_EXTI_D3_EventInputConfig
                0x00000000       0x7c CMakeFiles/H750_S15909.elf.dir/Drivers/STM32H7xx_HAL_Driver/Src/stm32h7xx_hal.c.obj
 .text          0x00000000        0x0 CMakeFiles/H750_S15909.elf.dir/Drivers/STM32H7xx_HAL_Driver/Src/stm32h7xx_hal_cortex.c.obj
 .data          0x00000000        0x0 CMakeFiles/H750_S15909.elf.dir/Drivers/STM32H7xx_HAL_Driver/Src/stm32h7xx_hal_cortex.c.obj
 .bss           0x00000000        0x0 CMakeFiles/H750_S15909.elf.dir/Drivers/STM32H7xx_HAL_Driver/Src/stm32h7xx_hal_cortex.c.obj
 .text.HAL_NVIC_DisableIRQ
                0x00000000       0x24 CMakeFiles/H750_S15909.elf.dir/Drivers/STM32H7xx_HAL_Driver/Src/stm32h7xx_hal_cortex.c.obj
 .text.HAL_NVIC_SystemReset
                0x00000000       0x24 CMakeFiles/H750_S15909.elf.dir/Drivers/STM32H7xx_HAL_Driver/Src/stm32h7xx_hal_cortex.c.obj
 .text.HAL_MPU_Disable
                0x00000000       0x1c CMakeFiles/H750_S15909.elf.dir/Drivers/STM32H7xx_HAL_Driver/Src/stm32h7xx_hal_cortex.c.obj
 .text.HAL_MPU_Enable
                0x00000000       0x20 CMakeFiles/H750_S15909.elf.dir/Drivers/STM32H7xx_HAL_Driver/Src/stm32h7xx_hal_cortex.c.obj
 .text.HAL_MPU_ConfigRegion
                0x00000000       0x60 CMakeFiles/H750_S15909.elf.dir/Drivers/STM32H7xx_HAL_Driver/Src/stm32h7xx_hal_cortex.c.obj
 .text.HAL_NVIC_GetPriorityGrouping
                0x00000000       0x10 CMakeFiles/H750_S15909.elf.dir/Drivers/STM32H7xx_HAL_Driver/Src/stm32h7xx_hal_cortex.c.obj
 .text.HAL_NVIC_GetPriority
                0x00000000       0x5c CMakeFiles/H750_S15909.elf.dir/Drivers/STM32H7xx_HAL_Driver/Src/stm32h7xx_hal_cortex.c.obj
 .text.HAL_NVIC_SetPendingIRQ
                0x00000000       0x1c CMakeFiles/H750_S15909.elf.dir/Drivers/STM32H7xx_HAL_Driver/Src/stm32h7xx_hal_cortex.c.obj
 .text.HAL_NVIC_GetPendingIRQ
                0x00000000       0x24 CMakeFiles/H750_S15909.elf.dir/Drivers/STM32H7xx_HAL_Driver/Src/stm32h7xx_hal_cortex.c.obj
 .text.HAL_NVIC_ClearPendingIRQ
                0x00000000       0x1c CMakeFiles/H750_S15909.elf.dir/Drivers/STM32H7xx_HAL_Driver/Src/stm32h7xx_hal_cortex.c.obj
 .text.HAL_NVIC_GetActive
                0x00000000       0x24 CMakeFiles/H750_S15909.elf.dir/Drivers/STM32H7xx_HAL_Driver/Src/stm32h7xx_hal_cortex.c.obj
 .text.HAL_SYSTICK_CLKSourceConfig
                0x00000000       0x20 CMakeFiles/H750_S15909.elf.dir/Drivers/STM32H7xx_HAL_Driver/Src/stm32h7xx_hal_cortex.c.obj
 .text.HAL_SYSTICK_Callback
                0x00000000        0x2 CMakeFiles/H750_S15909.elf.dir/Drivers/STM32H7xx_HAL_Driver/Src/stm32h7xx_hal_cortex.c.obj
 .text.HAL_SYSTICK_IRQHandler
                0x00000000        0x8 CMakeFiles/H750_S15909.elf.dir/Drivers/STM32H7xx_HAL_Driver/Src/stm32h7xx_hal_cortex.c.obj
 .text.HAL_GetCurrentCPUID
                0x00000000        0x4 CMakeFiles/H750_S15909.elf.dir/Drivers/STM32H7xx_HAL_Driver/Src/stm32h7xx_hal_cortex.c.obj
 .text          0x00000000        0x0 CMakeFiles/H750_S15909.elf.dir/Drivers/STM32H7xx_HAL_Driver/Src/stm32h7xx_hal_dma.c.obj
 .data          0x00000000        0x0 CMakeFiles/H750_S15909.elf.dir/Drivers/STM32H7xx_HAL_Driver/Src/stm32h7xx_hal_dma.c.obj
 .bss           0x00000000        0x0 CMakeFiles/H750_S15909.elf.dir/Drivers/STM32H7xx_HAL_Driver/Src/stm32h7xx_hal_dma.c.obj
 .text.HAL_DMA_Start
                0x00000000      0x148 CMakeFiles/H750_S15909.elf.dir/Drivers/STM32H7xx_HAL_Driver/Src/stm32h7xx_hal_dma.c.obj
 .text.HAL_DMA_PollForTransfer
                0x00000000      0x450 CMakeFiles/H750_S15909.elf.dir/Drivers/STM32H7xx_HAL_Driver/Src/stm32h7xx_hal_dma.c.obj
 .text.HAL_DMA_RegisterCallback
                0x00000000       0x60 CMakeFiles/H750_S15909.elf.dir/Drivers/STM32H7xx_HAL_Driver/Src/stm32h7xx_hal_dma.c.obj
 .text.HAL_DMA_UnRegisterCallback
                0x00000000       0x76 CMakeFiles/H750_S15909.elf.dir/Drivers/STM32H7xx_HAL_Driver/Src/stm32h7xx_hal_dma.c.obj
 .text.HAL_DMA_GetState
                0x00000000        0x6 CMakeFiles/H750_S15909.elf.dir/Drivers/STM32H7xx_HAL_Driver/Src/stm32h7xx_hal_dma.c.obj
 .text          0x00000000        0x0 CMakeFiles/H750_S15909.elf.dir/Drivers/STM32H7xx_HAL_Driver/Src/stm32h7xx_hal_dma_ex.c.obj
 .data          0x00000000        0x0 CMakeFiles/H750_S15909.elf.dir/Drivers/STM32H7xx_HAL_Driver/Src/stm32h7xx_hal_dma_ex.c.obj
 .bss           0x00000000        0x0 CMakeFiles/H750_S15909.elf.dir/Drivers/STM32H7xx_HAL_Driver/Src/stm32h7xx_hal_dma_ex.c.obj
 .text.DMA_MultiBufferSetConfig
                0x00000000       0xa8 CMakeFiles/H750_S15909.elf.dir/Drivers/STM32H7xx_HAL_Driver/Src/stm32h7xx_hal_dma_ex.c.obj
 .text.HAL_DMAEx_MultiBufferStart
                0x00000000      0x218 CMakeFiles/H750_S15909.elf.dir/Drivers/STM32H7xx_HAL_Driver/Src/stm32h7xx_hal_dma_ex.c.obj
 .text.HAL_DMAEx_MultiBufferStart_IT
                0x00000000      0x398 CMakeFiles/H750_S15909.elf.dir/Drivers/STM32H7xx_HAL_Driver/Src/stm32h7xx_hal_dma_ex.c.obj
 .text.HAL_DMAEx_ChangeMemory
                0x00000000       0x88 CMakeFiles/H750_S15909.elf.dir/Drivers/STM32H7xx_HAL_Driver/Src/stm32h7xx_hal_dma_ex.c.obj
 .text.HAL_DMAEx_ConfigMuxSync
                0x00000000       0x70 CMakeFiles/H750_S15909.elf.dir/Drivers/STM32H7xx_HAL_Driver/Src/stm32h7xx_hal_dma_ex.c.obj
 .text.HAL_DMAEx_ConfigMuxRequestGenerator
                0x00000000       0x58 CMakeFiles/H750_S15909.elf.dir/Drivers/STM32H7xx_HAL_Driver/Src/stm32h7xx_hal_dma_ex.c.obj
 .text.HAL_DMAEx_EnableMuxRequestGenerator
                0x00000000       0x1e CMakeFiles/H750_S15909.elf.dir/Drivers/STM32H7xx_HAL_Driver/Src/stm32h7xx_hal_dma_ex.c.obj
 .text.HAL_DMAEx_DisableMuxRequestGenerator
                0x00000000       0x1e CMakeFiles/H750_S15909.elf.dir/Drivers/STM32H7xx_HAL_Driver/Src/stm32h7xx_hal_dma_ex.c.obj
 .text.HAL_DMAEx_MUX_IRQHandler
                0x00000000       0x5a CMakeFiles/H750_S15909.elf.dir/Drivers/STM32H7xx_HAL_Driver/Src/stm32h7xx_hal_dma_ex.c.obj
 .debug_info    0x00000000      0x961 CMakeFiles/H750_S15909.elf.dir/Drivers/STM32H7xx_HAL_Driver/Src/stm32h7xx_hal_dma_ex.c.obj
 .debug_abbrev  0x00000000      0x207 CMakeFiles/H750_S15909.elf.dir/Drivers/STM32H7xx_HAL_Driver/Src/stm32h7xx_hal_dma_ex.c.obj
 .debug_loc     0x00000000      0x7df CMakeFiles/H750_S15909.elf.dir/Drivers/STM32H7xx_HAL_Driver/Src/stm32h7xx_hal_dma_ex.c.obj
 .debug_aranges
                0x00000000       0x60 CMakeFiles/H750_S15909.elf.dir/Drivers/STM32H7xx_HAL_Driver/Src/stm32h7xx_hal_dma_ex.c.obj
 .debug_ranges  0x00000000       0x50 CMakeFiles/H750_S15909.elf.dir/Drivers/STM32H7xx_HAL_Driver/Src/stm32h7xx_hal_dma_ex.c.obj
 .debug_line    0x00000000      0xc25 CMakeFiles/H750_S15909.elf.dir/Drivers/STM32H7xx_HAL_Driver/Src/stm32h7xx_hal_dma_ex.c.obj
 .debug_str     0x00000000      0x814 CMakeFiles/H750_S15909.elf.dir/Drivers/STM32H7xx_HAL_Driver/Src/stm32h7xx_hal_dma_ex.c.obj
 .comment       0x00000000       0x4a CMakeFiles/H750_S15909.elf.dir/Drivers/STM32H7xx_HAL_Driver/Src/stm32h7xx_hal_dma_ex.c.obj
 .debug_frame   0x00000000      0x104 CMakeFiles/H750_S15909.elf.dir/Drivers/STM32H7xx_HAL_Driver/Src/stm32h7xx_hal_dma_ex.c.obj
 .ARM.attributes
                0x00000000       0x2e CMakeFiles/H750_S15909.elf.dir/Drivers/STM32H7xx_HAL_Driver/Src/stm32h7xx_hal_dma_ex.c.obj
 .text          0x00000000        0x0 CMakeFiles/H750_S15909.elf.dir/Drivers/STM32H7xx_HAL_Driver/Src/stm32h7xx_hal_exti.c.obj
 .data          0x00000000        0x0 CMakeFiles/H750_S15909.elf.dir/Drivers/STM32H7xx_HAL_Driver/Src/stm32h7xx_hal_exti.c.obj
 .bss           0x00000000        0x0 CMakeFiles/H750_S15909.elf.dir/Drivers/STM32H7xx_HAL_Driver/Src/stm32h7xx_hal_exti.c.obj
 .text.HAL_EXTI_SetConfigLine
                0x00000000      0x144 CMakeFiles/H750_S15909.elf.dir/Drivers/STM32H7xx_HAL_Driver/Src/stm32h7xx_hal_exti.c.obj
 .text.HAL_EXTI_GetConfigLine
                0x00000000      0x10c CMakeFiles/H750_S15909.elf.dir/Drivers/STM32H7xx_HAL_Driver/Src/stm32h7xx_hal_exti.c.obj
 .text.HAL_EXTI_ClearConfigLine
                0x00000000       0xec CMakeFiles/H750_S15909.elf.dir/Drivers/STM32H7xx_HAL_Driver/Src/stm32h7xx_hal_exti.c.obj
 .text.HAL_EXTI_RegisterCallback
                0x00000000       0x12 CMakeFiles/H750_S15909.elf.dir/Drivers/STM32H7xx_HAL_Driver/Src/stm32h7xx_hal_exti.c.obj
 .text.HAL_EXTI_GetHandle
                0x00000000        0xc CMakeFiles/H750_S15909.elf.dir/Drivers/STM32H7xx_HAL_Driver/Src/stm32h7xx_hal_exti.c.obj
 .text.HAL_EXTI_IRQHandler
                0x00000000       0x2c CMakeFiles/H750_S15909.elf.dir/Drivers/STM32H7xx_HAL_Driver/Src/stm32h7xx_hal_exti.c.obj
 .text.HAL_EXTI_GetPending
                0x00000000       0x20 CMakeFiles/H750_S15909.elf.dir/Drivers/STM32H7xx_HAL_Driver/Src/stm32h7xx_hal_exti.c.obj
 .text.HAL_EXTI_ClearPending
                0x00000000       0x1c CMakeFiles/H750_S15909.elf.dir/Drivers/STM32H7xx_HAL_Driver/Src/stm32h7xx_hal_exti.c.obj
 .text.HAL_EXTI_GenerateSWI
                0x00000000       0x1c CMakeFiles/H750_S15909.elf.dir/Drivers/STM32H7xx_HAL_Driver/Src/stm32h7xx_hal_exti.c.obj
 .debug_info    0x00000000      0xa76 CMakeFiles/H750_S15909.elf.dir/Drivers/STM32H7xx_HAL_Driver/Src/stm32h7xx_hal_exti.c.obj
 .debug_abbrev  0x00000000      0x1e2 CMakeFiles/H750_S15909.elf.dir/Drivers/STM32H7xx_HAL_Driver/Src/stm32h7xx_hal_exti.c.obj
 .debug_loc     0x00000000      0xde3 CMakeFiles/H750_S15909.elf.dir/Drivers/STM32H7xx_HAL_Driver/Src/stm32h7xx_hal_exti.c.obj
 .debug_aranges
                0x00000000       0x60 CMakeFiles/H750_S15909.elf.dir/Drivers/STM32H7xx_HAL_Driver/Src/stm32h7xx_hal_exti.c.obj
 .debug_ranges  0x00000000       0x50 CMakeFiles/H750_S15909.elf.dir/Drivers/STM32H7xx_HAL_Driver/Src/stm32h7xx_hal_exti.c.obj
 .debug_line    0x00000000      0x8f6 CMakeFiles/H750_S15909.elf.dir/Drivers/STM32H7xx_HAL_Driver/Src/stm32h7xx_hal_exti.c.obj
 .debug_str     0x00000000      0x52e CMakeFiles/H750_S15909.elf.dir/Drivers/STM32H7xx_HAL_Driver/Src/stm32h7xx_hal_exti.c.obj
 .comment       0x00000000       0x4a CMakeFiles/H750_S15909.elf.dir/Drivers/STM32H7xx_HAL_Driver/Src/stm32h7xx_hal_exti.c.obj
 .debug_frame   0x00000000      0x100 CMakeFiles/H750_S15909.elf.dir/Drivers/STM32H7xx_HAL_Driver/Src/stm32h7xx_hal_exti.c.obj
 .ARM.attributes
                0x00000000       0x2e CMakeFiles/H750_S15909.elf.dir/Drivers/STM32H7xx_HAL_Driver/Src/stm32h7xx_hal_exti.c.obj
 .text          0x00000000        0x0 CMakeFiles/H750_S15909.elf.dir/Drivers/STM32H7xx_HAL_Driver/Src/stm32h7xx_hal_flash.c.obj
 .data          0x00000000        0x0 CMakeFiles/H750_S15909.elf.dir/Drivers/STM32H7xx_HAL_Driver/Src/stm32h7xx_hal_flash.c.obj
 .bss           0x00000000        0x0 CMakeFiles/H750_S15909.elf.dir/Drivers/STM32H7xx_HAL_Driver/Src/stm32h7xx_hal_flash.c.obj
 .text.HAL_FLASH_EndOfOperationCallback
                0x00000000        0x2 CMakeFiles/H750_S15909.elf.dir/Drivers/STM32H7xx_HAL_Driver/Src/stm32h7xx_hal_flash.c.obj
 .text.HAL_FLASH_OperationErrorCallback
                0x00000000        0x2 CMakeFiles/H750_S15909.elf.dir/Drivers/STM32H7xx_HAL_Driver/Src/stm32h7xx_hal_flash.c.obj
 .text.HAL_FLASH_IRQHandler
                0x00000000      0x100 CMakeFiles/H750_S15909.elf.dir/Drivers/STM32H7xx_HAL_Driver/Src/stm32h7xx_hal_flash.c.obj
 .text.HAL_FLASH_Unlock
                0x00000000       0x34 CMakeFiles/H750_S15909.elf.dir/Drivers/STM32H7xx_HAL_Driver/Src/stm32h7xx_hal_flash.c.obj
 .text.HAL_FLASH_Lock
                0x00000000       0x20 CMakeFiles/H750_S15909.elf.dir/Drivers/STM32H7xx_HAL_Driver/Src/stm32h7xx_hal_flash.c.obj
 .text.HAL_FLASH_OB_Unlock
                0x00000000       0x34 CMakeFiles/H750_S15909.elf.dir/Drivers/STM32H7xx_HAL_Driver/Src/stm32h7xx_hal_flash.c.obj
 .text.HAL_FLASH_OB_Lock
                0x00000000       0x20 CMakeFiles/H750_S15909.elf.dir/Drivers/STM32H7xx_HAL_Driver/Src/stm32h7xx_hal_flash.c.obj
 .text.HAL_FLASH_GetError
                0x00000000        0xc CMakeFiles/H750_S15909.elf.dir/Drivers/STM32H7xx_HAL_Driver/Src/stm32h7xx_hal_flash.c.obj
 .text.FLASH_WaitForLastOperation
                0x00000000       0x84 CMakeFiles/H750_S15909.elf.dir/Drivers/STM32H7xx_HAL_Driver/Src/stm32h7xx_hal_flash.c.obj
 .text.HAL_FLASH_Program
                0x00000000       0x88 CMakeFiles/H750_S15909.elf.dir/Drivers/STM32H7xx_HAL_Driver/Src/stm32h7xx_hal_flash.c.obj
 .text.HAL_FLASH_Program_IT
                0x00000000       0x88 CMakeFiles/H750_S15909.elf.dir/Drivers/STM32H7xx_HAL_Driver/Src/stm32h7xx_hal_flash.c.obj
 .text.FLASH_OB_WaitForLastOperation
                0x00000000       0x60 CMakeFiles/H750_S15909.elf.dir/Drivers/STM32H7xx_HAL_Driver/Src/stm32h7xx_hal_flash.c.obj
 .text.FLASH_CRC_WaitForLastOperation
                0x00000000       0x74 CMakeFiles/H750_S15909.elf.dir/Drivers/STM32H7xx_HAL_Driver/Src/stm32h7xx_hal_flash.c.obj
 .text.HAL_FLASH_OB_Launch
                0x00000000       0x2c CMakeFiles/H750_S15909.elf.dir/Drivers/STM32H7xx_HAL_Driver/Src/stm32h7xx_hal_flash.c.obj
 .bss.pFlash    0x00000000       0x1c CMakeFiles/H750_S15909.elf.dir/Drivers/STM32H7xx_HAL_Driver/Src/stm32h7xx_hal_flash.c.obj
 .debug_info    0x00000000      0xa90 CMakeFiles/H750_S15909.elf.dir/Drivers/STM32H7xx_HAL_Driver/Src/stm32h7xx_hal_flash.c.obj
 .debug_abbrev  0x00000000      0x289 CMakeFiles/H750_S15909.elf.dir/Drivers/STM32H7xx_HAL_Driver/Src/stm32h7xx_hal_flash.c.obj
 .debug_loc     0x00000000      0x72d CMakeFiles/H750_S15909.elf.dir/Drivers/STM32H7xx_HAL_Driver/Src/stm32h7xx_hal_flash.c.obj
 .debug_aranges
                0x00000000       0x88 CMakeFiles/H750_S15909.elf.dir/Drivers/STM32H7xx_HAL_Driver/Src/stm32h7xx_hal_flash.c.obj
 .debug_ranges  0x00000000       0x78 CMakeFiles/H750_S15909.elf.dir/Drivers/STM32H7xx_HAL_Driver/Src/stm32h7xx_hal_flash.c.obj
 .debug_line    0x00000000      0x906 CMakeFiles/H750_S15909.elf.dir/Drivers/STM32H7xx_HAL_Driver/Src/stm32h7xx_hal_flash.c.obj
 .debug_str     0x00000000      0x716 CMakeFiles/H750_S15909.elf.dir/Drivers/STM32H7xx_HAL_Driver/Src/stm32h7xx_hal_flash.c.obj
 .comment       0x00000000       0x4a CMakeFiles/H750_S15909.elf.dir/Drivers/STM32H7xx_HAL_Driver/Src/stm32h7xx_hal_flash.c.obj
 .debug_frame   0x00000000      0x148 CMakeFiles/H750_S15909.elf.dir/Drivers/STM32H7xx_HAL_Driver/Src/stm32h7xx_hal_flash.c.obj
 .ARM.attributes
                0x00000000       0x2e CMakeFiles/H750_S15909.elf.dir/Drivers/STM32H7xx_HAL_Driver/Src/stm32h7xx_hal_flash.c.obj
 .text          0x00000000        0x0 CMakeFiles/H750_S15909.elf.dir/Drivers/STM32H7xx_HAL_Driver/Src/stm32h7xx_hal_flash_ex.c.obj
 .data          0x00000000        0x0 CMakeFiles/H750_S15909.elf.dir/Drivers/STM32H7xx_HAL_Driver/Src/stm32h7xx_hal_flash_ex.c.obj
 .bss           0x00000000        0x0 CMakeFiles/H750_S15909.elf.dir/Drivers/STM32H7xx_HAL_Driver/Src/stm32h7xx_hal_flash_ex.c.obj
 .text.FLASH_MassErase
                0x00000000       0x24 CMakeFiles/H750_S15909.elf.dir/Drivers/STM32H7xx_HAL_Driver/Src/stm32h7xx_hal_flash_ex.c.obj
 .text.FLASH_OB_EnableWRP
                0x00000000       0x18 CMakeFiles/H750_S15909.elf.dir/Drivers/STM32H7xx_HAL_Driver/Src/stm32h7xx_hal_flash_ex.c.obj
 .text.FLASH_OB_DisableWRP
                0x00000000       0x18 CMakeFiles/H750_S15909.elf.dir/Drivers/STM32H7xx_HAL_Driver/Src/stm32h7xx_hal_flash_ex.c.obj
 .text.FLASH_OB_GetWRP
                0x00000000       0x24 CMakeFiles/H750_S15909.elf.dir/Drivers/STM32H7xx_HAL_Driver/Src/stm32h7xx_hal_flash_ex.c.obj
 .text.FLASH_OB_RDPConfig
                0x00000000       0x14 CMakeFiles/H750_S15909.elf.dir/Drivers/STM32H7xx_HAL_Driver/Src/stm32h7xx_hal_flash_ex.c.obj
 .text.FLASH_OB_GetRDP
                0x00000000       0x20 CMakeFiles/H750_S15909.elf.dir/Drivers/STM32H7xx_HAL_Driver/Src/stm32h7xx_hal_flash_ex.c.obj
 .text.FLASH_OB_UserConfig
                0x00000000       0xa0 CMakeFiles/H750_S15909.elf.dir/Drivers/STM32H7xx_HAL_Driver/Src/stm32h7xx_hal_flash_ex.c.obj
 .text.FLASH_OB_GetUser
                0x00000000       0x14 CMakeFiles/H750_S15909.elf.dir/Drivers/STM32H7xx_HAL_Driver/Src/stm32h7xx_hal_flash_ex.c.obj
 .text.FLASH_OB_PCROPConfig
                0x00000000       0x24 CMakeFiles/H750_S15909.elf.dir/Drivers/STM32H7xx_HAL_Driver/Src/stm32h7xx_hal_flash_ex.c.obj
 .text.FLASH_OB_GetPCROP
                0x00000000       0x40 CMakeFiles/H750_S15909.elf.dir/Drivers/STM32H7xx_HAL_Driver/Src/stm32h7xx_hal_flash_ex.c.obj
 .text.FLASH_OB_BOR_LevelConfig
                0x00000000       0x14 CMakeFiles/H750_S15909.elf.dir/Drivers/STM32H7xx_HAL_Driver/Src/stm32h7xx_hal_flash_ex.c.obj
 .text.FLASH_OB_GetBOR
                0x00000000       0x10 CMakeFiles/H750_S15909.elf.dir/Drivers/STM32H7xx_HAL_Driver/Src/stm32h7xx_hal_flash_ex.c.obj
 .text.FLASH_OB_BootAddConfig
                0x00000000       0x34 CMakeFiles/H750_S15909.elf.dir/Drivers/STM32H7xx_HAL_Driver/Src/stm32h7xx_hal_flash_ex.c.obj
 .text.FLASH_OB_GetBootAdd
                0x00000000       0x18 CMakeFiles/H750_S15909.elf.dir/Drivers/STM32H7xx_HAL_Driver/Src/stm32h7xx_hal_flash_ex.c.obj
 .text.FLASH_OB_SecureAreaConfig
                0x00000000       0x28 CMakeFiles/H750_S15909.elf.dir/Drivers/STM32H7xx_HAL_Driver/Src/stm32h7xx_hal_flash_ex.c.obj
 .text.FLASH_OB_GetSecureArea
                0x00000000       0x40 CMakeFiles/H750_S15909.elf.dir/Drivers/STM32H7xx_HAL_Driver/Src/stm32h7xx_hal_flash_ex.c.obj
 .text.FLASH_CRC_AddSector
                0x00000000       0x20 CMakeFiles/H750_S15909.elf.dir/Drivers/STM32H7xx_HAL_Driver/Src/stm32h7xx_hal_flash_ex.c.obj
 .text.FLASH_CRC_SelectAddress
                0x00000000       0x14 CMakeFiles/H750_S15909.elf.dir/Drivers/STM32H7xx_HAL_Driver/Src/stm32h7xx_hal_flash_ex.c.obj
 .text.HAL_FLASHEx_OBProgram
                0x00000000       0xcc CMakeFiles/H750_S15909.elf.dir/Drivers/STM32H7xx_HAL_Driver/Src/stm32h7xx_hal_flash_ex.c.obj
 .text.HAL_FLASHEx_OBGetConfig
                0x00000000       0x6e CMakeFiles/H750_S15909.elf.dir/Drivers/STM32H7xx_HAL_Driver/Src/stm32h7xx_hal_flash_ex.c.obj
 .text.HAL_FLASHEx_Unlock_Bank1
                0x00000000       0x34 CMakeFiles/H750_S15909.elf.dir/Drivers/STM32H7xx_HAL_Driver/Src/stm32h7xx_hal_flash_ex.c.obj
 .text.HAL_FLASHEx_Lock_Bank1
                0x00000000       0x14 CMakeFiles/H750_S15909.elf.dir/Drivers/STM32H7xx_HAL_Driver/Src/stm32h7xx_hal_flash_ex.c.obj
 .text.HAL_FLASHEx_ComputeCRC
                0x00000000       0xb4 CMakeFiles/H750_S15909.elf.dir/Drivers/STM32H7xx_HAL_Driver/Src/stm32h7xx_hal_flash_ex.c.obj
 .text.FLASH_Erase_Sector
                0x00000000       0x24 CMakeFiles/H750_S15909.elf.dir/Drivers/STM32H7xx_HAL_Driver/Src/stm32h7xx_hal_flash_ex.c.obj
 .text.HAL_FLASHEx_Erase
                0x00000000       0xc8 CMakeFiles/H750_S15909.elf.dir/Drivers/STM32H7xx_HAL_Driver/Src/stm32h7xx_hal_flash_ex.c.obj
 .text.HAL_FLASHEx_Erase_IT
                0x00000000       0x98 CMakeFiles/H750_S15909.elf.dir/Drivers/STM32H7xx_HAL_Driver/Src/stm32h7xx_hal_flash_ex.c.obj
 .debug_info    0x00000000      0xfb1 CMakeFiles/H750_S15909.elf.dir/Drivers/STM32H7xx_HAL_Driver/Src/stm32h7xx_hal_flash_ex.c.obj
 .debug_abbrev  0x00000000      0x273 CMakeFiles/H750_S15909.elf.dir/Drivers/STM32H7xx_HAL_Driver/Src/stm32h7xx_hal_flash_ex.c.obj
 .debug_loc     0x00000000      0x906 CMakeFiles/H750_S15909.elf.dir/Drivers/STM32H7xx_HAL_Driver/Src/stm32h7xx_hal_flash_ex.c.obj
 .debug_aranges
                0x00000000       0xe8 CMakeFiles/H750_S15909.elf.dir/Drivers/STM32H7xx_HAL_Driver/Src/stm32h7xx_hal_flash_ex.c.obj
 .debug_ranges  0x00000000       0xd8 CMakeFiles/H750_S15909.elf.dir/Drivers/STM32H7xx_HAL_Driver/Src/stm32h7xx_hal_flash_ex.c.obj
 .debug_line    0x00000000      0xb71 CMakeFiles/H750_S15909.elf.dir/Drivers/STM32H7xx_HAL_Driver/Src/stm32h7xx_hal_flash_ex.c.obj
 .debug_str     0x00000000      0x996 CMakeFiles/H750_S15909.elf.dir/Drivers/STM32H7xx_HAL_Driver/Src/stm32h7xx_hal_flash_ex.c.obj
 .comment       0x00000000       0x4a CMakeFiles/H750_S15909.elf.dir/Drivers/STM32H7xx_HAL_Driver/Src/stm32h7xx_hal_flash_ex.c.obj
 .debug_frame   0x00000000      0x214 CMakeFiles/H750_S15909.elf.dir/Drivers/STM32H7xx_HAL_Driver/Src/stm32h7xx_hal_flash_ex.c.obj
 .ARM.attributes
                0x00000000       0x2e CMakeFiles/H750_S15909.elf.dir/Drivers/STM32H7xx_HAL_Driver/Src/stm32h7xx_hal_flash_ex.c.obj
 .text          0x00000000        0x0 CMakeFiles/H750_S15909.elf.dir/Drivers/STM32H7xx_HAL_Driver/Src/stm32h7xx_hal_gpio.c.obj
 .data          0x00000000        0x0 CMakeFiles/H750_S15909.elf.dir/Drivers/STM32H7xx_HAL_Driver/Src/stm32h7xx_hal_gpio.c.obj
 .bss           0x00000000        0x0 CMakeFiles/H750_S15909.elf.dir/Drivers/STM32H7xx_HAL_Driver/Src/stm32h7xx_hal_gpio.c.obj
 .text.HAL_GPIO_DeInit
                0x00000000      0x150 CMakeFiles/H750_S15909.elf.dir/Drivers/STM32H7xx_HAL_Driver/Src/stm32h7xx_hal_gpio.c.obj
 .text.HAL_GPIO_TogglePin
                0x00000000       0x12 CMakeFiles/H750_S15909.elf.dir/Drivers/STM32H7xx_HAL_Driver/Src/stm32h7xx_hal_gpio.c.obj
 .text.HAL_GPIO_LockPin
                0x00000000       0x2e CMakeFiles/H750_S15909.elf.dir/Drivers/STM32H7xx_HAL_Driver/Src/stm32h7xx_hal_gpio.c.obj
 .text.HAL_GPIO_EXTI_Callback
                0x00000000        0x2 CMakeFiles/H750_S15909.elf.dir/Drivers/STM32H7xx_HAL_Driver/Src/stm32h7xx_hal_gpio.c.obj
 .text          0x00000000        0x0 CMakeFiles/H750_S15909.elf.dir/Drivers/STM32H7xx_HAL_Driver/Src/stm32h7xx_hal_hsem.c.obj
 .data          0x00000000        0x0 CMakeFiles/H750_S15909.elf.dir/Drivers/STM32H7xx_HAL_Driver/Src/stm32h7xx_hal_hsem.c.obj
 .bss           0x00000000        0x0 CMakeFiles/H750_S15909.elf.dir/Drivers/STM32H7xx_HAL_Driver/Src/stm32h7xx_hal_hsem.c.obj
 .text.HAL_HSEM_Take
                0x00000000       0x24 CMakeFiles/H750_S15909.elf.dir/Drivers/STM32H7xx_HAL_Driver/Src/stm32h7xx_hal_hsem.c.obj
 .text.HAL_HSEM_FastTake
                0x00000000       0x20 CMakeFiles/H750_S15909.elf.dir/Drivers/STM32H7xx_HAL_Driver/Src/stm32h7xx_hal_hsem.c.obj
 .text.HAL_HSEM_IsSemTaken
                0x00000000       0x18 CMakeFiles/H750_S15909.elf.dir/Drivers/STM32H7xx_HAL_Driver/Src/stm32h7xx_hal_hsem.c.obj
 .text.HAL_HSEM_Release
                0x00000000       0x10 CMakeFiles/H750_S15909.elf.dir/Drivers/STM32H7xx_HAL_Driver/Src/stm32h7xx_hal_hsem.c.obj
 .text.HAL_HSEM_ReleaseAll
                0x00000000       0x14 CMakeFiles/H750_S15909.elf.dir/Drivers/STM32H7xx_HAL_Driver/Src/stm32h7xx_hal_hsem.c.obj
 .text.HAL_HSEM_SetClearKey
                0x00000000       0x18 CMakeFiles/H750_S15909.elf.dir/Drivers/STM32H7xx_HAL_Driver/Src/stm32h7xx_hal_hsem.c.obj
 .text.HAL_HSEM_GetClearKey
                0x00000000       0x10 CMakeFiles/H750_S15909.elf.dir/Drivers/STM32H7xx_HAL_Driver/Src/stm32h7xx_hal_hsem.c.obj
 .text.HAL_HSEM_ActivateNotification
                0x00000000       0x10 CMakeFiles/H750_S15909.elf.dir/Drivers/STM32H7xx_HAL_Driver/Src/stm32h7xx_hal_hsem.c.obj
 .text.HAL_HSEM_DeactivateNotification
                0x00000000       0x10 CMakeFiles/H750_S15909.elf.dir/Drivers/STM32H7xx_HAL_Driver/Src/stm32h7xx_hal_hsem.c.obj
 .text.HAL_HSEM_FreeCallback
                0x00000000        0x2 CMakeFiles/H750_S15909.elf.dir/Drivers/STM32H7xx_HAL_Driver/Src/stm32h7xx_hal_hsem.c.obj
 .text.HAL_HSEM_IRQHandler
                0x00000000       0x1c CMakeFiles/H750_S15909.elf.dir/Drivers/STM32H7xx_HAL_Driver/Src/stm32h7xx_hal_hsem.c.obj
 .debug_info    0x00000000      0x3dd CMakeFiles/H750_S15909.elf.dir/Drivers/STM32H7xx_HAL_Driver/Src/stm32h7xx_hal_hsem.c.obj
 .debug_abbrev  0x00000000      0x1e7 CMakeFiles/H750_S15909.elf.dir/Drivers/STM32H7xx_HAL_Driver/Src/stm32h7xx_hal_hsem.c.obj
 .debug_loc     0x00000000      0x117 CMakeFiles/H750_S15909.elf.dir/Drivers/STM32H7xx_HAL_Driver/Src/stm32h7xx_hal_hsem.c.obj
 .debug_aranges
                0x00000000       0x70 CMakeFiles/H750_S15909.elf.dir/Drivers/STM32H7xx_HAL_Driver/Src/stm32h7xx_hal_hsem.c.obj
 .debug_ranges  0x00000000       0x60 CMakeFiles/H750_S15909.elf.dir/Drivers/STM32H7xx_HAL_Driver/Src/stm32h7xx_hal_hsem.c.obj
 .debug_line    0x00000000      0x354 CMakeFiles/H750_S15909.elf.dir/Drivers/STM32H7xx_HAL_Driver/Src/stm32h7xx_hal_hsem.c.obj
 .debug_str     0x00000000      0x38c CMakeFiles/H750_S15909.elf.dir/Drivers/STM32H7xx_HAL_Driver/Src/stm32h7xx_hal_hsem.c.obj
 .comment       0x00000000       0x4a CMakeFiles/H750_S15909.elf.dir/Drivers/STM32H7xx_HAL_Driver/Src/stm32h7xx_hal_hsem.c.obj
 .debug_frame   0x00000000       0xc8 CMakeFiles/H750_S15909.elf.dir/Drivers/STM32H7xx_HAL_Driver/Src/stm32h7xx_hal_hsem.c.obj
 .ARM.attributes
                0x00000000       0x2e CMakeFiles/H750_S15909.elf.dir/Drivers/STM32H7xx_HAL_Driver/Src/stm32h7xx_hal_hsem.c.obj
 .text          0x00000000        0x0 CMakeFiles/H750_S15909.elf.dir/Drivers/STM32H7xx_HAL_Driver/Src/stm32h7xx_hal_i2c.c.obj
 .data          0x00000000        0x0 CMakeFiles/H750_S15909.elf.dir/Drivers/STM32H7xx_HAL_Driver/Src/stm32h7xx_hal_i2c.c.obj
 .bss           0x00000000        0x0 CMakeFiles/H750_S15909.elf.dir/Drivers/STM32H7xx_HAL_Driver/Src/stm32h7xx_hal_i2c.c.obj
 .text.I2C_Flush_TXDR
                0x00000000       0x22 CMakeFiles/H750_S15909.elf.dir/Drivers/STM32H7xx_HAL_Driver/Src/stm32h7xx_hal_i2c.c.obj
 .text.I2C_TransferConfig
                0x00000000       0x3a CMakeFiles/H750_S15909.elf.dir/Drivers/STM32H7xx_HAL_Driver/Src/stm32h7xx_hal_i2c.c.obj
 .text.I2C_Enable_IRQ
                0x00000000       0x74 CMakeFiles/H750_S15909.elf.dir/Drivers/STM32H7xx_HAL_Driver/Src/stm32h7xx_hal_i2c.c.obj
 .text.I2C_Disable_IRQ
                0x00000000       0x70 CMakeFiles/H750_S15909.elf.dir/Drivers/STM32H7xx_HAL_Driver/Src/stm32h7xx_hal_i2c.c.obj
 .text.I2C_ConvertOtherXferOptions
                0x00000000       0x1e CMakeFiles/H750_S15909.elf.dir/Drivers/STM32H7xx_HAL_Driver/Src/stm32h7xx_hal_i2c.c.obj
 .text.I2C_IsErrorOccurred
                0x00000000      0x130 CMakeFiles/H750_S15909.elf.dir/Drivers/STM32H7xx_HAL_Driver/Src/stm32h7xx_hal_i2c.c.obj
 .text.I2C_WaitOnTXISFlagUntilTimeout
                0x00000000       0x56 CMakeFiles/H750_S15909.elf.dir/Drivers/STM32H7xx_HAL_Driver/Src/stm32h7xx_hal_i2c.c.obj
 .text.I2C_WaitOnFlagUntilTimeout
                0x00000000       0x5a CMakeFiles/H750_S15909.elf.dir/Drivers/STM32H7xx_HAL_Driver/Src/stm32h7xx_hal_i2c.c.obj
 .text.I2C_RequestMemoryWrite
                0x00000000       0x7c CMakeFiles/H750_S15909.elf.dir/Drivers/STM32H7xx_HAL_Driver/Src/stm32h7xx_hal_i2c.c.obj
 .text.I2C_RequestMemoryRead
                0x00000000       0x78 CMakeFiles/H750_S15909.elf.dir/Drivers/STM32H7xx_HAL_Driver/Src/stm32h7xx_hal_i2c.c.obj
 .text.I2C_WaitOnSTOPFlagUntilTimeout
                0x00000000       0x50 CMakeFiles/H750_S15909.elf.dir/Drivers/STM32H7xx_HAL_Driver/Src/stm32h7xx_hal_i2c.c.obj
 .text.I2C_WaitOnRXNEFlagUntilTimeout
                0x00000000       0xae CMakeFiles/H750_S15909.elf.dir/Drivers/STM32H7xx_HAL_Driver/Src/stm32h7xx_hal_i2c.c.obj
 .text.HAL_I2C_MspInit
                0x00000000        0x2 CMakeFiles/H750_S15909.elf.dir/Drivers/STM32H7xx_HAL_Driver/Src/stm32h7xx_hal_i2c.c.obj
 .text.HAL_I2C_Init
                0x00000000       0xbc CMakeFiles/H750_S15909.elf.dir/Drivers/STM32H7xx_HAL_Driver/Src/stm32h7xx_hal_i2c.c.obj
 .text.HAL_I2C_MspDeInit
                0x00000000        0x2 CMakeFiles/H750_S15909.elf.dir/Drivers/STM32H7xx_HAL_Driver/Src/stm32h7xx_hal_i2c.c.obj
 .text.HAL_I2C_DeInit
                0x00000000       0x32 CMakeFiles/H750_S15909.elf.dir/Drivers/STM32H7xx_HAL_Driver/Src/stm32h7xx_hal_i2c.c.obj
 .text.HAL_I2C_Master_Transmit
                0x00000000      0x17c CMakeFiles/H750_S15909.elf.dir/Drivers/STM32H7xx_HAL_Driver/Src/stm32h7xx_hal_i2c.c.obj
 .text.HAL_I2C_Master_Receive
                0x00000000      0x17c CMakeFiles/H750_S15909.elf.dir/Drivers/STM32H7xx_HAL_Driver/Src/stm32h7xx_hal_i2c.c.obj
 .text.HAL_I2C_Slave_Transmit
                0x00000000      0x1b0 CMakeFiles/H750_S15909.elf.dir/Drivers/STM32H7xx_HAL_Driver/Src/stm32h7xx_hal_i2c.c.obj
 .text.HAL_I2C_Slave_Receive
                0x00000000      0x184 CMakeFiles/H750_S15909.elf.dir/Drivers/STM32H7xx_HAL_Driver/Src/stm32h7xx_hal_i2c.c.obj
 .text.HAL_I2C_Master_Transmit_IT
                0x00000000       0x98 CMakeFiles/H750_S15909.elf.dir/Drivers/STM32H7xx_HAL_Driver/Src/stm32h7xx_hal_i2c.c.obj
 .text.HAL_I2C_Master_Receive_IT
                0x00000000       0x98 CMakeFiles/H750_S15909.elf.dir/Drivers/STM32H7xx_HAL_Driver/Src/stm32h7xx_hal_i2c.c.obj
 .text.HAL_I2C_Slave_Transmit_IT
                0x00000000       0x64 CMakeFiles/H750_S15909.elf.dir/Drivers/STM32H7xx_HAL_Driver/Src/stm32h7xx_hal_i2c.c.obj
 .text.HAL_I2C_Slave_Receive_IT
                0x00000000       0x64 CMakeFiles/H750_S15909.elf.dir/Drivers/STM32H7xx_HAL_Driver/Src/stm32h7xx_hal_i2c.c.obj
 .text.HAL_I2C_Master_Transmit_DMA
                0x00000000      0x154 CMakeFiles/H750_S15909.elf.dir/Drivers/STM32H7xx_HAL_Driver/Src/stm32h7xx_hal_i2c.c.obj
 .text.HAL_I2C_Master_Receive_DMA
                0x00000000      0x150 CMakeFiles/H750_S15909.elf.dir/Drivers/STM32H7xx_HAL_Driver/Src/stm32h7xx_hal_i2c.c.obj
 .text.HAL_I2C_Slave_Transmit_DMA
                0x00000000       0xf0 CMakeFiles/H750_S15909.elf.dir/Drivers/STM32H7xx_HAL_Driver/Src/stm32h7xx_hal_i2c.c.obj
 .text.HAL_I2C_Slave_Receive_DMA
                0x00000000       0xf4 CMakeFiles/H750_S15909.elf.dir/Drivers/STM32H7xx_HAL_Driver/Src/stm32h7xx_hal_i2c.c.obj
 .text.HAL_I2C_Mem_Write
                0x00000000      0x1aa CMakeFiles/H750_S15909.elf.dir/Drivers/STM32H7xx_HAL_Driver/Src/stm32h7xx_hal_i2c.c.obj
 .text.HAL_I2C_Mem_Read
                0x00000000      0x1b0 CMakeFiles/H750_S15909.elf.dir/Drivers/STM32H7xx_HAL_Driver/Src/stm32h7xx_hal_i2c.c.obj
 .text.HAL_I2C_Mem_Write_IT
                0x00000000       0xe4 CMakeFiles/H750_S15909.elf.dir/Drivers/STM32H7xx_HAL_Driver/Src/stm32h7xx_hal_i2c.c.obj
 .text.HAL_I2C_Mem_Read_IT
                0x00000000       0xe8 CMakeFiles/H750_S15909.elf.dir/Drivers/STM32H7xx_HAL_Driver/Src/stm32h7xx_hal_i2c.c.obj
 .text.HAL_I2C_Mem_Write_DMA
                0x00000000      0x168 CMakeFiles/H750_S15909.elf.dir/Drivers/STM32H7xx_HAL_Driver/Src/stm32h7xx_hal_i2c.c.obj
 .text.HAL_I2C_Mem_Read_DMA
                0x00000000      0x16c CMakeFiles/H750_S15909.elf.dir/Drivers/STM32H7xx_HAL_Driver/Src/stm32h7xx_hal_i2c.c.obj
 .text.HAL_I2C_IsDeviceReady
                0x00000000      0x16c CMakeFiles/H750_S15909.elf.dir/Drivers/STM32H7xx_HAL_Driver/Src/stm32h7xx_hal_i2c.c.obj
 .text.HAL_I2C_Master_Seq_Transmit_IT
                0x00000000       0xb4 CMakeFiles/H750_S15909.elf.dir/Drivers/STM32H7xx_HAL_Driver/Src/stm32h7xx_hal_i2c.c.obj
 .text.HAL_I2C_Master_Seq_Transmit_DMA
                0x00000000      0x174 CMakeFiles/H750_S15909.elf.dir/Drivers/STM32H7xx_HAL_Driver/Src/stm32h7xx_hal_i2c.c.obj
 .text.HAL_I2C_Master_Seq_Receive_IT
                0x00000000       0xb4 CMakeFiles/H750_S15909.elf.dir/Drivers/STM32H7xx_HAL_Driver/Src/stm32h7xx_hal_i2c.c.obj
 .text.HAL_I2C_Master_Seq_Receive_DMA
                0x00000000      0x174 CMakeFiles/H750_S15909.elf.dir/Drivers/STM32H7xx_HAL_Driver/Src/stm32h7xx_hal_i2c.c.obj
 .text.HAL_I2C_Slave_Seq_Transmit_IT
                0x00000000       0xdc CMakeFiles/H750_S15909.elf.dir/Drivers/STM32H7xx_HAL_Driver/Src/stm32h7xx_hal_i2c.c.obj
 .text.HAL_I2C_Slave_Seq_Transmit_DMA
                0x00000000      0x1a4 CMakeFiles/H750_S15909.elf.dir/Drivers/STM32H7xx_HAL_Driver/Src/stm32h7xx_hal_i2c.c.obj
 .text.HAL_I2C_Slave_Seq_Receive_IT
                0x00000000       0xdc CMakeFiles/H750_S15909.elf.dir/Drivers/STM32H7xx_HAL_Driver/Src/stm32h7xx_hal_i2c.c.obj
 .text.HAL_I2C_Slave_Seq_Receive_DMA
                0x00000000      0x1a4 CMakeFiles/H750_S15909.elf.dir/Drivers/STM32H7xx_HAL_Driver/Src/stm32h7xx_hal_i2c.c.obj
 .text.HAL_I2C_EnableListen_IT
                0x00000000       0x2c CMakeFiles/H750_S15909.elf.dir/Drivers/STM32H7xx_HAL_Driver/Src/stm32h7xx_hal_i2c.c.obj
 .text.HAL_I2C_DisableListen_IT
                0x00000000       0x3a CMakeFiles/H750_S15909.elf.dir/Drivers/STM32H7xx_HAL_Driver/Src/stm32h7xx_hal_i2c.c.obj
 .text.HAL_I2C_Master_Abort_IT
                0x00000000       0x84 CMakeFiles/H750_S15909.elf.dir/Drivers/STM32H7xx_HAL_Driver/Src/stm32h7xx_hal_i2c.c.obj
 .text.HAL_I2C_EV_IRQHandler
                0x00000000       0x10 CMakeFiles/H750_S15909.elf.dir/Drivers/STM32H7xx_HAL_Driver/Src/stm32h7xx_hal_i2c.c.obj
 .text.HAL_I2C_MasterTxCpltCallback
                0x00000000        0x2 CMakeFiles/H750_S15909.elf.dir/Drivers/STM32H7xx_HAL_Driver/Src/stm32h7xx_hal_i2c.c.obj
 .text.HAL_I2C_MasterRxCpltCallback
                0x00000000        0x2 CMakeFiles/H750_S15909.elf.dir/Drivers/STM32H7xx_HAL_Driver/Src/stm32h7xx_hal_i2c.c.obj
 .text.I2C_ITMasterSeqCplt
                0x00000000       0x54 CMakeFiles/H750_S15909.elf.dir/Drivers/STM32H7xx_HAL_Driver/Src/stm32h7xx_hal_i2c.c.obj
 .text.HAL_I2C_SlaveTxCpltCallback
                0x00000000        0x2 CMakeFiles/H750_S15909.elf.dir/Drivers/STM32H7xx_HAL_Driver/Src/stm32h7xx_hal_i2c.c.obj
 .text.HAL_I2C_SlaveRxCpltCallback
                0x00000000        0x2 CMakeFiles/H750_S15909.elf.dir/Drivers/STM32H7xx_HAL_Driver/Src/stm32h7xx_hal_i2c.c.obj
 .text.I2C_ITSlaveSeqCplt
                0x00000000       0x82 CMakeFiles/H750_S15909.elf.dir/Drivers/STM32H7xx_HAL_Driver/Src/stm32h7xx_hal_i2c.c.obj
 .text.I2C_DMASlaveTransmitCplt
                0x00000000       0x22 CMakeFiles/H750_S15909.elf.dir/Drivers/STM32H7xx_HAL_Driver/Src/stm32h7xx_hal_i2c.c.obj
 .text.I2C_DMASlaveReceiveCplt
                0x00000000       0xa0 CMakeFiles/H750_S15909.elf.dir/Drivers/STM32H7xx_HAL_Driver/Src/stm32h7xx_hal_i2c.c.obj
 .text.HAL_I2C_AddrCallback
                0x00000000        0x2 CMakeFiles/H750_S15909.elf.dir/Drivers/STM32H7xx_HAL_Driver/Src/stm32h7xx_hal_i2c.c.obj
 .text.I2C_ITAddrCplt
                0x00000000       0xa0 CMakeFiles/H750_S15909.elf.dir/Drivers/STM32H7xx_HAL_Driver/Src/stm32h7xx_hal_i2c.c.obj
 .text.HAL_I2C_ListenCpltCallback
                0x00000000        0x2 CMakeFiles/H750_S15909.elf.dir/Drivers/STM32H7xx_HAL_Driver/Src/stm32h7xx_hal_i2c.c.obj
 .text.I2C_ITListenCplt
                0x00000000       0x68 CMakeFiles/H750_S15909.elf.dir/Drivers/STM32H7xx_HAL_Driver/Src/stm32h7xx_hal_i2c.c.obj
 .text.HAL_I2C_MemTxCpltCallback
                0x00000000        0x2 CMakeFiles/H750_S15909.elf.dir/Drivers/STM32H7xx_HAL_Driver/Src/stm32h7xx_hal_i2c.c.obj
 .text.HAL_I2C_MemRxCpltCallback
                0x00000000        0x2 CMakeFiles/H750_S15909.elf.dir/Drivers/STM32H7xx_HAL_Driver/Src/stm32h7xx_hal_i2c.c.obj
 .text.HAL_I2C_ErrorCallback
                0x00000000        0x2 CMakeFiles/H750_S15909.elf.dir/Drivers/STM32H7xx_HAL_Driver/Src/stm32h7xx_hal_i2c.c.obj
 .text.HAL_I2C_AbortCpltCallback
                0x00000000        0x2 CMakeFiles/H750_S15909.elf.dir/Drivers/STM32H7xx_HAL_Driver/Src/stm32h7xx_hal_i2c.c.obj
 .text.I2C_TreatErrorCallback
                0x00000000       0x2e CMakeFiles/H750_S15909.elf.dir/Drivers/STM32H7xx_HAL_Driver/Src/stm32h7xx_hal_i2c.c.obj
 .text.I2C_ITError
                0x00000000      0x108 CMakeFiles/H750_S15909.elf.dir/Drivers/STM32H7xx_HAL_Driver/Src/stm32h7xx_hal_i2c.c.obj
 .text.I2C_ITSlaveCplt
                0x00000000      0x244 CMakeFiles/H750_S15909.elf.dir/Drivers/STM32H7xx_HAL_Driver/Src/stm32h7xx_hal_i2c.c.obj
 .text.I2C_Slave_ISR_IT
                0x00000000      0x150 CMakeFiles/H750_S15909.elf.dir/Drivers/STM32H7xx_HAL_Driver/Src/stm32h7xx_hal_i2c.c.obj
 .text.I2C_ITMasterCplt
                0x00000000      0x12e CMakeFiles/H750_S15909.elf.dir/Drivers/STM32H7xx_HAL_Driver/Src/stm32h7xx_hal_i2c.c.obj
 .text.I2C_Master_ISR_IT
                0x00000000      0x180 CMakeFiles/H750_S15909.elf.dir/Drivers/STM32H7xx_HAL_Driver/Src/stm32h7xx_hal_i2c.c.obj
 .text.I2C_Slave_ISR_DMA
                0x00000000      0x220 CMakeFiles/H750_S15909.elf.dir/Drivers/STM32H7xx_HAL_Driver/Src/stm32h7xx_hal_i2c.c.obj
 .text.I2C_Master_ISR_DMA
                0x00000000      0x142 CMakeFiles/H750_S15909.elf.dir/Drivers/STM32H7xx_HAL_Driver/Src/stm32h7xx_hal_i2c.c.obj
 .text.I2C_DMAError
                0x00000000      0x138 CMakeFiles/H750_S15909.elf.dir/Drivers/STM32H7xx_HAL_Driver/Src/stm32h7xx_hal_i2c.c.obj
 .text.I2C_DMAMasterTransmitCplt
                0x00000000       0x5a CMakeFiles/H750_S15909.elf.dir/Drivers/STM32H7xx_HAL_Driver/Src/stm32h7xx_hal_i2c.c.obj
 .text.I2C_DMAMasterReceiveCplt
                0x00000000       0x5a CMakeFiles/H750_S15909.elf.dir/Drivers/STM32H7xx_HAL_Driver/Src/stm32h7xx_hal_i2c.c.obj
 .text.HAL_I2C_ER_IRQHandler
                0x00000000       0x6a CMakeFiles/H750_S15909.elf.dir/Drivers/STM32H7xx_HAL_Driver/Src/stm32h7xx_hal_i2c.c.obj
 .text.I2C_DMAAbort
                0x00000000       0x1a CMakeFiles/H750_S15909.elf.dir/Drivers/STM32H7xx_HAL_Driver/Src/stm32h7xx_hal_i2c.c.obj
 .text.HAL_I2C_GetState
                0x00000000        0x6 CMakeFiles/H750_S15909.elf.dir/Drivers/STM32H7xx_HAL_Driver/Src/stm32h7xx_hal_i2c.c.obj
 .text.HAL_I2C_GetMode
                0x00000000        0x6 CMakeFiles/H750_S15909.elf.dir/Drivers/STM32H7xx_HAL_Driver/Src/stm32h7xx_hal_i2c.c.obj
 .text.HAL_I2C_GetError
                0x00000000        0x4 CMakeFiles/H750_S15909.elf.dir/Drivers/STM32H7xx_HAL_Driver/Src/stm32h7xx_hal_i2c.c.obj
 .debug_info    0x00000000     0x4233 CMakeFiles/H750_S15909.elf.dir/Drivers/STM32H7xx_HAL_Driver/Src/stm32h7xx_hal_i2c.c.obj
 .debug_abbrev  0x00000000      0x252 CMakeFiles/H750_S15909.elf.dir/Drivers/STM32H7xx_HAL_Driver/Src/stm32h7xx_hal_i2c.c.obj
 .debug_loc     0x00000000     0x47c7 CMakeFiles/H750_S15909.elf.dir/Drivers/STM32H7xx_HAL_Driver/Src/stm32h7xx_hal_i2c.c.obj
 .debug_aranges
                0x00000000      0x290 CMakeFiles/H750_S15909.elf.dir/Drivers/STM32H7xx_HAL_Driver/Src/stm32h7xx_hal_i2c.c.obj
 .debug_ranges  0x00000000      0x280 CMakeFiles/H750_S15909.elf.dir/Drivers/STM32H7xx_HAL_Driver/Src/stm32h7xx_hal_i2c.c.obj
 .debug_line    0x00000000     0x4c71 CMakeFiles/H750_S15909.elf.dir/Drivers/STM32H7xx_HAL_Driver/Src/stm32h7xx_hal_i2c.c.obj
 .debug_str     0x00000000     0x1168 CMakeFiles/H750_S15909.elf.dir/Drivers/STM32H7xx_HAL_Driver/Src/stm32h7xx_hal_i2c.c.obj
 .comment       0x00000000       0x4a CMakeFiles/H750_S15909.elf.dir/Drivers/STM32H7xx_HAL_Driver/Src/stm32h7xx_hal_i2c.c.obj
 .debug_frame   0x00000000      0x938 CMakeFiles/H750_S15909.elf.dir/Drivers/STM32H7xx_HAL_Driver/Src/stm32h7xx_hal_i2c.c.obj
 .ARM.attributes
                0x00000000       0x2e CMakeFiles/H750_S15909.elf.dir/Drivers/STM32H7xx_HAL_Driver/Src/stm32h7xx_hal_i2c.c.obj
 .text          0x00000000        0x0 CMakeFiles/H750_S15909.elf.dir/Drivers/STM32H7xx_HAL_Driver/Src/stm32h7xx_hal_i2c_ex.c.obj
 .data          0x00000000        0x0 CMakeFiles/H750_S15909.elf.dir/Drivers/STM32H7xx_HAL_Driver/Src/stm32h7xx_hal_i2c_ex.c.obj
 .bss           0x00000000        0x0 CMakeFiles/H750_S15909.elf.dir/Drivers/STM32H7xx_HAL_Driver/Src/stm32h7xx_hal_i2c_ex.c.obj
 .text.HAL_I2CEx_ConfigAnalogFilter
                0x00000000       0x5c CMakeFiles/H750_S15909.elf.dir/Drivers/STM32H7xx_HAL_Driver/Src/stm32h7xx_hal_i2c_ex.c.obj
 .text.HAL_I2CEx_ConfigDigitalFilter
                0x00000000       0x58 CMakeFiles/H750_S15909.elf.dir/Drivers/STM32H7xx_HAL_Driver/Src/stm32h7xx_hal_i2c_ex.c.obj
 .text.HAL_I2CEx_EnableWakeUp
                0x00000000       0x54 CMakeFiles/H750_S15909.elf.dir/Drivers/STM32H7xx_HAL_Driver/Src/stm32h7xx_hal_i2c_ex.c.obj
 .text.HAL_I2CEx_DisableWakeUp
                0x00000000       0x54 CMakeFiles/H750_S15909.elf.dir/Drivers/STM32H7xx_HAL_Driver/Src/stm32h7xx_hal_i2c_ex.c.obj
 .text.HAL_I2CEx_EnableFastModePlus
                0x00000000       0x30 CMakeFiles/H750_S15909.elf.dir/Drivers/STM32H7xx_HAL_Driver/Src/stm32h7xx_hal_i2c_ex.c.obj
 .text.HAL_I2CEx_DisableFastModePlus
                0x00000000       0x34 CMakeFiles/H750_S15909.elf.dir/Drivers/STM32H7xx_HAL_Driver/Src/stm32h7xx_hal_i2c_ex.c.obj
 .debug_info    0x00000000      0xe56 CMakeFiles/H750_S15909.elf.dir/Drivers/STM32H7xx_HAL_Driver/Src/stm32h7xx_hal_i2c_ex.c.obj
 .debug_abbrev  0x00000000      0x1e4 CMakeFiles/H750_S15909.elf.dir/Drivers/STM32H7xx_HAL_Driver/Src/stm32h7xx_hal_i2c_ex.c.obj
 .debug_loc     0x00000000      0x202 CMakeFiles/H750_S15909.elf.dir/Drivers/STM32H7xx_HAL_Driver/Src/stm32h7xx_hal_i2c_ex.c.obj
 .debug_aranges
                0x00000000       0x48 CMakeFiles/H750_S15909.elf.dir/Drivers/STM32H7xx_HAL_Driver/Src/stm32h7xx_hal_i2c_ex.c.obj
 .debug_ranges  0x00000000       0x38 CMakeFiles/H750_S15909.elf.dir/Drivers/STM32H7xx_HAL_Driver/Src/stm32h7xx_hal_i2c_ex.c.obj
 .debug_line    0x00000000      0x4fb CMakeFiles/H750_S15909.elf.dir/Drivers/STM32H7xx_HAL_Driver/Src/stm32h7xx_hal_i2c_ex.c.obj
 .debug_str     0x00000000      0xb5d CMakeFiles/H750_S15909.elf.dir/Drivers/STM32H7xx_HAL_Driver/Src/stm32h7xx_hal_i2c_ex.c.obj
 .comment       0x00000000       0x4a CMakeFiles/H750_S15909.elf.dir/Drivers/STM32H7xx_HAL_Driver/Src/stm32h7xx_hal_i2c_ex.c.obj
 .debug_frame   0x00000000       0x80 CMakeFiles/H750_S15909.elf.dir/Drivers/STM32H7xx_HAL_Driver/Src/stm32h7xx_hal_i2c_ex.c.obj
 .ARM.attributes
                0x00000000       0x2e CMakeFiles/H750_S15909.elf.dir/Drivers/STM32H7xx_HAL_Driver/Src/stm32h7xx_hal_i2c_ex.c.obj
 .text          0x00000000        0x0 CMakeFiles/H750_S15909.elf.dir/Drivers/STM32H7xx_HAL_Driver/Src/stm32h7xx_hal_mdma.c.obj
 .data          0x00000000        0x0 CMakeFiles/H750_S15909.elf.dir/Drivers/STM32H7xx_HAL_Driver/Src/stm32h7xx_hal_mdma.c.obj
 .bss           0x00000000        0x0 CMakeFiles/H750_S15909.elf.dir/Drivers/STM32H7xx_HAL_Driver/Src/stm32h7xx_hal_mdma.c.obj
 .text.MDMA_SetConfig
                0x00000000       0x88 CMakeFiles/H750_S15909.elf.dir/Drivers/STM32H7xx_HAL_Driver/Src/stm32h7xx_hal_mdma.c.obj
 .text.MDMA_Init
                0x00000000       0xb8 CMakeFiles/H750_S15909.elf.dir/Drivers/STM32H7xx_HAL_Driver/Src/stm32h7xx_hal_mdma.c.obj
 .text.HAL_MDMA_Init
                0x00000000       0x60 CMakeFiles/H750_S15909.elf.dir/Drivers/STM32H7xx_HAL_Driver/Src/stm32h7xx_hal_mdma.c.obj
 .text.HAL_MDMA_DeInit
                0x00000000       0x56 CMakeFiles/H750_S15909.elf.dir/Drivers/STM32H7xx_HAL_Driver/Src/stm32h7xx_hal_mdma.c.obj
 .text.HAL_MDMA_ConfigPostRequestMask
                0x00000000       0x66 CMakeFiles/H750_S15909.elf.dir/Drivers/STM32H7xx_HAL_Driver/Src/stm32h7xx_hal_mdma.c.obj
 .text.HAL_MDMA_RegisterCallback
                0x00000000       0x64 CMakeFiles/H750_S15909.elf.dir/Drivers/STM32H7xx_HAL_Driver/Src/stm32h7xx_hal_mdma.c.obj
 .text.HAL_MDMA_UnRegisterCallback
                0x00000000       0x76 CMakeFiles/H750_S15909.elf.dir/Drivers/STM32H7xx_HAL_Driver/Src/stm32h7xx_hal_mdma.c.obj
 .text.HAL_MDMA_LinkedList_CreateNode
                0x00000000      0x10e CMakeFiles/H750_S15909.elf.dir/Drivers/STM32H7xx_HAL_Driver/Src/stm32h7xx_hal_mdma.c.obj
 .text.HAL_MDMA_LinkedList_AddNode
                0x00000000       0xe8 CMakeFiles/H750_S15909.elf.dir/Drivers/STM32H7xx_HAL_Driver/Src/stm32h7xx_hal_mdma.c.obj
 .text.HAL_MDMA_LinkedList_RemoveNode
                0x00000000       0xd2 CMakeFiles/H750_S15909.elf.dir/Drivers/STM32H7xx_HAL_Driver/Src/stm32h7xx_hal_mdma.c.obj
 .text.HAL_MDMA_LinkedList_EnableCircularMode
                0x00000000       0x56 CMakeFiles/H750_S15909.elf.dir/Drivers/STM32H7xx_HAL_Driver/Src/stm32h7xx_hal_mdma.c.obj
 .text.HAL_MDMA_LinkedList_DisableCircularMode
                0x00000000       0x52 CMakeFiles/H750_S15909.elf.dir/Drivers/STM32H7xx_HAL_Driver/Src/stm32h7xx_hal_mdma.c.obj
 .text.HAL_MDMA_Start
                0x00000000       0x78 CMakeFiles/H750_S15909.elf.dir/Drivers/STM32H7xx_HAL_Driver/Src/stm32h7xx_hal_mdma.c.obj
 .text.HAL_MDMA_Start_IT
                0x00000000       0xac CMakeFiles/H750_S15909.elf.dir/Drivers/STM32H7xx_HAL_Driver/Src/stm32h7xx_hal_mdma.c.obj
 .text.HAL_MDMA_Abort
                0x00000000       0x7c CMakeFiles/H750_S15909.elf.dir/Drivers/STM32H7xx_HAL_Driver/Src/stm32h7xx_hal_mdma.c.obj
 .text.HAL_MDMA_Abort_IT
                0x00000000       0x2c CMakeFiles/H750_S15909.elf.dir/Drivers/STM32H7xx_HAL_Driver/Src/stm32h7xx_hal_mdma.c.obj
 .text.HAL_MDMA_PollForTransfer
                0x00000000      0x122 CMakeFiles/H750_S15909.elf.dir/Drivers/STM32H7xx_HAL_Driver/Src/stm32h7xx_hal_mdma.c.obj
 .text.HAL_MDMA_GenerateSWRequest
                0x00000000       0x40 CMakeFiles/H750_S15909.elf.dir/Drivers/STM32H7xx_HAL_Driver/Src/stm32h7xx_hal_mdma.c.obj
 .text.HAL_MDMA_IRQHandler
                0x00000000      0x1b4 CMakeFiles/H750_S15909.elf.dir/Drivers/STM32H7xx_HAL_Driver/Src/stm32h7xx_hal_mdma.c.obj
 .text.HAL_MDMA_GetState
                0x00000000        0x6 CMakeFiles/H750_S15909.elf.dir/Drivers/STM32H7xx_HAL_Driver/Src/stm32h7xx_hal_mdma.c.obj
 .text.HAL_MDMA_GetError
                0x00000000        0x4 CMakeFiles/H750_S15909.elf.dir/Drivers/STM32H7xx_HAL_Driver/Src/stm32h7xx_hal_mdma.c.obj
 .debug_info    0x00000000      0xec5 CMakeFiles/H750_S15909.elf.dir/Drivers/STM32H7xx_HAL_Driver/Src/stm32h7xx_hal_mdma.c.obj
 .debug_abbrev  0x00000000      0x23a CMakeFiles/H750_S15909.elf.dir/Drivers/STM32H7xx_HAL_Driver/Src/stm32h7xx_hal_mdma.c.obj
 .debug_loc     0x00000000     0x11a3 CMakeFiles/H750_S15909.elf.dir/Drivers/STM32H7xx_HAL_Driver/Src/stm32h7xx_hal_mdma.c.obj
 .debug_aranges
                0x00000000       0xc0 CMakeFiles/H750_S15909.elf.dir/Drivers/STM32H7xx_HAL_Driver/Src/stm32h7xx_hal_mdma.c.obj
 .debug_ranges  0x00000000       0xb0 CMakeFiles/H750_S15909.elf.dir/Drivers/STM32H7xx_HAL_Driver/Src/stm32h7xx_hal_mdma.c.obj
 .debug_line    0x00000000     0x14c2 CMakeFiles/H750_S15909.elf.dir/Drivers/STM32H7xx_HAL_Driver/Src/stm32h7xx_hal_mdma.c.obj
 .debug_str     0x00000000      0xa4b CMakeFiles/H750_S15909.elf.dir/Drivers/STM32H7xx_HAL_Driver/Src/stm32h7xx_hal_mdma.c.obj
 .comment       0x00000000       0x4a CMakeFiles/H750_S15909.elf.dir/Drivers/STM32H7xx_HAL_Driver/Src/stm32h7xx_hal_mdma.c.obj
 .debug_frame   0x00000000      0x264 CMakeFiles/H750_S15909.elf.dir/Drivers/STM32H7xx_HAL_Driver/Src/stm32h7xx_hal_mdma.c.obj
 .ARM.attributes
                0x00000000       0x2e CMakeFiles/H750_S15909.elf.dir/Drivers/STM32H7xx_HAL_Driver/Src/stm32h7xx_hal_mdma.c.obj
 .text          0x00000000        0x0 CMakeFiles/H750_S15909.elf.dir/Drivers/STM32H7xx_HAL_Driver/Src/stm32h7xx_hal_pwr.c.obj
 .data          0x00000000        0x0 CMakeFiles/H750_S15909.elf.dir/Drivers/STM32H7xx_HAL_Driver/Src/stm32h7xx_hal_pwr.c.obj
 .bss           0x00000000        0x0 CMakeFiles/H750_S15909.elf.dir/Drivers/STM32H7xx_HAL_Driver/Src/stm32h7xx_hal_pwr.c.obj
 .text.HAL_PWR_DeInit
                0x00000000        0x2 CMakeFiles/H750_S15909.elf.dir/Drivers/STM32H7xx_HAL_Driver/Src/stm32h7xx_hal_pwr.c.obj
 .text.HAL_PWR_EnableBkUpAccess
                0x00000000       0x10 CMakeFiles/H750_S15909.elf.dir/Drivers/STM32H7xx_HAL_Driver/Src/stm32h7xx_hal_pwr.c.obj
 .text.HAL_PWR_DisableBkUpAccess
                0x00000000       0x10 CMakeFiles/H750_S15909.elf.dir/Drivers/STM32H7xx_HAL_Driver/Src/stm32h7xx_hal_pwr.c.obj
 .text.HAL_PWR_ConfigPVD
                0x00000000       0xa0 CMakeFiles/H750_S15909.elf.dir/Drivers/STM32H7xx_HAL_Driver/Src/stm32h7xx_hal_pwr.c.obj
 .text.HAL_PWR_EnablePVD
                0x00000000       0x10 CMakeFiles/H750_S15909.elf.dir/Drivers/STM32H7xx_HAL_Driver/Src/stm32h7xx_hal_pwr.c.obj
 .text.HAL_PWR_DisablePVD
                0x00000000       0x10 CMakeFiles/H750_S15909.elf.dir/Drivers/STM32H7xx_HAL_Driver/Src/stm32h7xx_hal_pwr.c.obj
 .text.HAL_PWR_EnableWakeUpPin
                0x00000000       0x18 CMakeFiles/H750_S15909.elf.dir/Drivers/STM32H7xx_HAL_Driver/Src/stm32h7xx_hal_pwr.c.obj
 .text.HAL_PWR_DisableWakeUpPin
                0x00000000       0x14 CMakeFiles/H750_S15909.elf.dir/Drivers/STM32H7xx_HAL_Driver/Src/stm32h7xx_hal_pwr.c.obj
 .text.HAL_PWR_EnterSLEEPMode
                0x00000000       0x1c CMakeFiles/H750_S15909.elf.dir/Drivers/STM32H7xx_HAL_Driver/Src/stm32h7xx_hal_pwr.c.obj
 .text.HAL_PWR_EnterSTOPMode
                0x00000000       0x4c CMakeFiles/H750_S15909.elf.dir/Drivers/STM32H7xx_HAL_Driver/Src/stm32h7xx_hal_pwr.c.obj
 .text.HAL_PWR_EnterSTANDBYMode
                0x00000000       0x30 CMakeFiles/H750_S15909.elf.dir/Drivers/STM32H7xx_HAL_Driver/Src/stm32h7xx_hal_pwr.c.obj
 .text.HAL_PWR_EnableSleepOnExit
                0x00000000       0x10 CMakeFiles/H750_S15909.elf.dir/Drivers/STM32H7xx_HAL_Driver/Src/stm32h7xx_hal_pwr.c.obj
 .text.HAL_PWR_DisableSleepOnExit
                0x00000000       0x10 CMakeFiles/H750_S15909.elf.dir/Drivers/STM32H7xx_HAL_Driver/Src/stm32h7xx_hal_pwr.c.obj
 .text.HAL_PWR_EnableSEVOnPend
                0x00000000       0x10 CMakeFiles/H750_S15909.elf.dir/Drivers/STM32H7xx_HAL_Driver/Src/stm32h7xx_hal_pwr.c.obj
 .text.HAL_PWR_DisableSEVOnPend
                0x00000000       0x10 CMakeFiles/H750_S15909.elf.dir/Drivers/STM32H7xx_HAL_Driver/Src/stm32h7xx_hal_pwr.c.obj
 .text.HAL_PWR_PVDCallback
                0x00000000        0x2 CMakeFiles/H750_S15909.elf.dir/Drivers/STM32H7xx_HAL_Driver/Src/stm32h7xx_hal_pwr.c.obj
 .text.HAL_PWR_PVD_IRQHandler
                0x00000000       0x28 CMakeFiles/H750_S15909.elf.dir/Drivers/STM32H7xx_HAL_Driver/Src/stm32h7xx_hal_pwr.c.obj
 .debug_info    0x00000000      0x984 CMakeFiles/H750_S15909.elf.dir/Drivers/STM32H7xx_HAL_Driver/Src/stm32h7xx_hal_pwr.c.obj
 .debug_abbrev  0x00000000      0x189 CMakeFiles/H750_S15909.elf.dir/Drivers/STM32H7xx_HAL_Driver/Src/stm32h7xx_hal_pwr.c.obj
 .debug_loc     0x00000000       0x57 CMakeFiles/H750_S15909.elf.dir/Drivers/STM32H7xx_HAL_Driver/Src/stm32h7xx_hal_pwr.c.obj
 .debug_aranges
                0x00000000       0xa0 CMakeFiles/H750_S15909.elf.dir/Drivers/STM32H7xx_HAL_Driver/Src/stm32h7xx_hal_pwr.c.obj
 .debug_ranges  0x00000000       0x90 CMakeFiles/H750_S15909.elf.dir/Drivers/STM32H7xx_HAL_Driver/Src/stm32h7xx_hal_pwr.c.obj
 .debug_line    0x00000000      0x482 CMakeFiles/H750_S15909.elf.dir/Drivers/STM32H7xx_HAL_Driver/Src/stm32h7xx_hal_pwr.c.obj
 .debug_str     0x00000000      0x633 CMakeFiles/H750_S15909.elf.dir/Drivers/STM32H7xx_HAL_Driver/Src/stm32h7xx_hal_pwr.c.obj
 .comment       0x00000000       0x4a CMakeFiles/H750_S15909.elf.dir/Drivers/STM32H7xx_HAL_Driver/Src/stm32h7xx_hal_pwr.c.obj
 .debug_frame   0x00000000      0x128 CMakeFiles/H750_S15909.elf.dir/Drivers/STM32H7xx_HAL_Driver/Src/stm32h7xx_hal_pwr.c.obj
 .ARM.attributes
                0x00000000       0x2e CMakeFiles/H750_S15909.elf.dir/Drivers/STM32H7xx_HAL_Driver/Src/stm32h7xx_hal_pwr.c.obj
 .text          0x00000000        0x0 CMakeFiles/H750_S15909.elf.dir/Drivers/STM32H7xx_HAL_Driver/Src/stm32h7xx_hal_pwr_ex.c.obj
 .data          0x00000000        0x0 CMakeFiles/H750_S15909.elf.dir/Drivers/STM32H7xx_HAL_Driver/Src/stm32h7xx_hal_pwr_ex.c.obj
 .bss           0x00000000        0x0 CMakeFiles/H750_S15909.elf.dir/Drivers/STM32H7xx_HAL_Driver/Src/stm32h7xx_hal_pwr_ex.c.obj
 .text.HAL_PWREx_GetSupplyConfig
                0x00000000       0x10 CMakeFiles/H750_S15909.elf.dir/Drivers/STM32H7xx_HAL_Driver/Src/stm32h7xx_hal_pwr_ex.c.obj
 .text.HAL_PWREx_ControlVoltageScaling
                0x00000000       0xd4 CMakeFiles/H750_S15909.elf.dir/Drivers/STM32H7xx_HAL_Driver/Src/stm32h7xx_hal_pwr_ex.c.obj
 .text.HAL_PWREx_GetVoltageRange
                0x00000000       0x10 CMakeFiles/H750_S15909.elf.dir/Drivers/STM32H7xx_HAL_Driver/Src/stm32h7xx_hal_pwr_ex.c.obj
 .text.HAL_PWREx_ControlStopModeVoltageScaling
                0x00000000       0x14 CMakeFiles/H750_S15909.elf.dir/Drivers/STM32H7xx_HAL_Driver/Src/stm32h7xx_hal_pwr_ex.c.obj
 .text.HAL_PWREx_GetStopModeVoltageRange
                0x00000000       0x10 CMakeFiles/H750_S15909.elf.dir/Drivers/STM32H7xx_HAL_Driver/Src/stm32h7xx_hal_pwr_ex.c.obj
 .text.HAL_PWREx_EnterSTOPMode
                0x00000000       0x68 CMakeFiles/H750_S15909.elf.dir/Drivers/STM32H7xx_HAL_Driver/Src/stm32h7xx_hal_pwr_ex.c.obj
 .text.HAL_PWREx_ClearPendingEvent
                0x00000000        0x4 CMakeFiles/H750_S15909.elf.dir/Drivers/STM32H7xx_HAL_Driver/Src/stm32h7xx_hal_pwr_ex.c.obj
 .text.HAL_PWREx_EnterSTANDBYMode
                0x00000000       0x40 CMakeFiles/H750_S15909.elf.dir/Drivers/STM32H7xx_HAL_Driver/Src/stm32h7xx_hal_pwr_ex.c.obj
 .text.HAL_PWREx_ConfigD3Domain
                0x00000000       0x14 CMakeFiles/H750_S15909.elf.dir/Drivers/STM32H7xx_HAL_Driver/Src/stm32h7xx_hal_pwr_ex.c.obj
 .text.HAL_PWREx_EnableFlashPowerDown
                0x00000000       0x10 CMakeFiles/H750_S15909.elf.dir/Drivers/STM32H7xx_HAL_Driver/Src/stm32h7xx_hal_pwr_ex.c.obj
 .text.HAL_PWREx_DisableFlashPowerDown
                0x00000000       0x10 CMakeFiles/H750_S15909.elf.dir/Drivers/STM32H7xx_HAL_Driver/Src/stm32h7xx_hal_pwr_ex.c.obj
 .text.HAL_PWREx_EnableWakeUpPin
                0x00000000       0xa8 CMakeFiles/H750_S15909.elf.dir/Drivers/STM32H7xx_HAL_Driver/Src/stm32h7xx_hal_pwr_ex.c.obj
 .text.HAL_PWREx_DisableWakeUpPin
                0x00000000       0x10 CMakeFiles/H750_S15909.elf.dir/Drivers/STM32H7xx_HAL_Driver/Src/stm32h7xx_hal_pwr_ex.c.obj
 .text.HAL_PWREx_GetWakeupFlag
                0x00000000        0xc CMakeFiles/H750_S15909.elf.dir/Drivers/STM32H7xx_HAL_Driver/Src/stm32h7xx_hal_pwr_ex.c.obj
 .text.HAL_PWREx_ClearWakeupFlag
                0x00000000       0x1c CMakeFiles/H750_S15909.elf.dir/Drivers/STM32H7xx_HAL_Driver/Src/stm32h7xx_hal_pwr_ex.c.obj
 .text.HAL_PWREx_WKUP1_Callback
                0x00000000        0x2 CMakeFiles/H750_S15909.elf.dir/Drivers/STM32H7xx_HAL_Driver/Src/stm32h7xx_hal_pwr_ex.c.obj
 .text.HAL_PWREx_WKUP2_Callback
                0x00000000        0x2 CMakeFiles/H750_S15909.elf.dir/Drivers/STM32H7xx_HAL_Driver/Src/stm32h7xx_hal_pwr_ex.c.obj
 .text.HAL_PWREx_WKUP3_Callback
                0x00000000        0x2 CMakeFiles/H750_S15909.elf.dir/Drivers/STM32H7xx_HAL_Driver/Src/stm32h7xx_hal_pwr_ex.c.obj
 .text.HAL_PWREx_WKUP4_Callback
                0x00000000        0x2 CMakeFiles/H750_S15909.elf.dir/Drivers/STM32H7xx_HAL_Driver/Src/stm32h7xx_hal_pwr_ex.c.obj
 .text.HAL_PWREx_WKUP5_Callback
                0x00000000        0x2 CMakeFiles/H750_S15909.elf.dir/Drivers/STM32H7xx_HAL_Driver/Src/stm32h7xx_hal_pwr_ex.c.obj
 .text.HAL_PWREx_WKUP6_Callback
                0x00000000        0x2 CMakeFiles/H750_S15909.elf.dir/Drivers/STM32H7xx_HAL_Driver/Src/stm32h7xx_hal_pwr_ex.c.obj
 .text.HAL_PWREx_WAKEUP_PIN_IRQHandler
                0x00000000       0x98 CMakeFiles/H750_S15909.elf.dir/Drivers/STM32H7xx_HAL_Driver/Src/stm32h7xx_hal_pwr_ex.c.obj
 .text.HAL_PWREx_EnableBkUpReg
                0x00000000       0x34 CMakeFiles/H750_S15909.elf.dir/Drivers/STM32H7xx_HAL_Driver/Src/stm32h7xx_hal_pwr_ex.c.obj
 .text.HAL_PWREx_DisableBkUpReg
                0x00000000       0x34 CMakeFiles/H750_S15909.elf.dir/Drivers/STM32H7xx_HAL_Driver/Src/stm32h7xx_hal_pwr_ex.c.obj
 .text.HAL_PWREx_EnableUSBReg
                0x00000000       0x34 CMakeFiles/H750_S15909.elf.dir/Drivers/STM32H7xx_HAL_Driver/Src/stm32h7xx_hal_pwr_ex.c.obj
 .text.HAL_PWREx_DisableUSBReg
                0x00000000       0x34 CMakeFiles/H750_S15909.elf.dir/Drivers/STM32H7xx_HAL_Driver/Src/stm32h7xx_hal_pwr_ex.c.obj
 .text.HAL_PWREx_EnableUSBVoltageDetector
                0x00000000       0x10 CMakeFiles/H750_S15909.elf.dir/Drivers/STM32H7xx_HAL_Driver/Src/stm32h7xx_hal_pwr_ex.c.obj
 .text.HAL_PWREx_DisableUSBVoltageDetector
                0x00000000       0x10 CMakeFiles/H750_S15909.elf.dir/Drivers/STM32H7xx_HAL_Driver/Src/stm32h7xx_hal_pwr_ex.c.obj
 .text.HAL_PWREx_EnableBatteryCharging
                0x00000000       0x1c CMakeFiles/H750_S15909.elf.dir/Drivers/STM32H7xx_HAL_Driver/Src/stm32h7xx_hal_pwr_ex.c.obj
 .text.HAL_PWREx_DisableBatteryCharging
                0x00000000       0x10 CMakeFiles/H750_S15909.elf.dir/Drivers/STM32H7xx_HAL_Driver/Src/stm32h7xx_hal_pwr_ex.c.obj
 .text.HAL_PWREx_EnableMonitoring
                0x00000000       0x10 CMakeFiles/H750_S15909.elf.dir/Drivers/STM32H7xx_HAL_Driver/Src/stm32h7xx_hal_pwr_ex.c.obj
 .text.HAL_PWREx_DisableMonitoring
                0x00000000       0x10 CMakeFiles/H750_S15909.elf.dir/Drivers/STM32H7xx_HAL_Driver/Src/stm32h7xx_hal_pwr_ex.c.obj
 .text.HAL_PWREx_GetTemperatureLevel
                0x00000000       0x1c CMakeFiles/H750_S15909.elf.dir/Drivers/STM32H7xx_HAL_Driver/Src/stm32h7xx_hal_pwr_ex.c.obj
 .text.HAL_PWREx_GetVBATLevel
                0x00000000       0x1c CMakeFiles/H750_S15909.elf.dir/Drivers/STM32H7xx_HAL_Driver/Src/stm32h7xx_hal_pwr_ex.c.obj
 .text.HAL_PWREx_ConfigAVD
                0x00000000       0x98 CMakeFiles/H750_S15909.elf.dir/Drivers/STM32H7xx_HAL_Driver/Src/stm32h7xx_hal_pwr_ex.c.obj
 .text.HAL_PWREx_EnableAVD
                0x00000000       0x10 CMakeFiles/H750_S15909.elf.dir/Drivers/STM32H7xx_HAL_Driver/Src/stm32h7xx_hal_pwr_ex.c.obj
 .text.HAL_PWREx_DisableAVD
                0x00000000       0x10 CMakeFiles/H750_S15909.elf.dir/Drivers/STM32H7xx_HAL_Driver/Src/stm32h7xx_hal_pwr_ex.c.obj
 .text.HAL_PWREx_AVDCallback
                0x00000000        0x2 CMakeFiles/H750_S15909.elf.dir/Drivers/STM32H7xx_HAL_Driver/Src/stm32h7xx_hal_pwr_ex.c.obj
 .text.HAL_PWREx_PVD_AVD_IRQHandler
                0x00000000       0x64 CMakeFiles/H750_S15909.elf.dir/Drivers/STM32H7xx_HAL_Driver/Src/stm32h7xx_hal_pwr_ex.c.obj
 .text          0x00000000        0x0 CMakeFiles/H750_S15909.elf.dir/Drivers/STM32H7xx_HAL_Driver/Src/stm32h7xx_hal_rcc.c.obj
 .data          0x00000000        0x0 CMakeFiles/H750_S15909.elf.dir/Drivers/STM32H7xx_HAL_Driver/Src/stm32h7xx_hal_rcc.c.obj
 .bss           0x00000000        0x0 CMakeFiles/H750_S15909.elf.dir/Drivers/STM32H7xx_HAL_Driver/Src/stm32h7xx_hal_rcc.c.obj
 .text.HAL_RCC_DeInit
                0x00000000      0x1cc CMakeFiles/H750_S15909.elf.dir/Drivers/STM32H7xx_HAL_Driver/Src/stm32h7xx_hal_rcc.c.obj
 .text.HAL_RCC_MCOConfig
                0x00000000       0xa4 CMakeFiles/H750_S15909.elf.dir/Drivers/STM32H7xx_HAL_Driver/Src/stm32h7xx_hal_rcc.c.obj
 .text.HAL_RCC_EnableCSS
                0x00000000       0x10 CMakeFiles/H750_S15909.elf.dir/Drivers/STM32H7xx_HAL_Driver/Src/stm32h7xx_hal_rcc.c.obj
 .text.HAL_RCC_DisableCSS
                0x00000000       0x10 CMakeFiles/H750_S15909.elf.dir/Drivers/STM32H7xx_HAL_Driver/Src/stm32h7xx_hal_rcc.c.obj
 .text.HAL_RCC_GetOscConfig
                0x00000000      0x154 CMakeFiles/H750_S15909.elf.dir/Drivers/STM32H7xx_HAL_Driver/Src/stm32h7xx_hal_rcc.c.obj
 .text.HAL_RCC_GetClockConfig
                0x00000000       0x54 CMakeFiles/H750_S15909.elf.dir/Drivers/STM32H7xx_HAL_Driver/Src/stm32h7xx_hal_rcc.c.obj
 .text.HAL_RCC_CSSCallback
                0x00000000        0x2 CMakeFiles/H750_S15909.elf.dir/Drivers/STM32H7xx_HAL_Driver/Src/stm32h7xx_hal_rcc.c.obj
 .text.HAL_RCC_NMI_IRQHandler
                0x00000000       0x20 CMakeFiles/H750_S15909.elf.dir/Drivers/STM32H7xx_HAL_Driver/Src/stm32h7xx_hal_rcc.c.obj
 .text          0x00000000        0x0 CMakeFiles/H750_S15909.elf.dir/Drivers/STM32H7xx_HAL_Driver/Src/stm32h7xx_hal_rcc_ex.c.obj
 .data          0x00000000        0x0 CMakeFiles/H750_S15909.elf.dir/Drivers/STM32H7xx_HAL_Driver/Src/stm32h7xx_hal_rcc_ex.c.obj
 .bss           0x00000000        0x0 CMakeFiles/H750_S15909.elf.dir/Drivers/STM32H7xx_HAL_Driver/Src/stm32h7xx_hal_rcc_ex.c.obj
 .text.HAL_RCCEx_GetPeriphCLKConfig
                0x00000000      0x1cc CMakeFiles/H750_S15909.elf.dir/Drivers/STM32H7xx_HAL_Driver/Src/stm32h7xx_hal_rcc_ex.c.obj
 .text.HAL_RCCEx_GetD1PCLK1Freq
                0x00000000       0x24 CMakeFiles/H750_S15909.elf.dir/Drivers/STM32H7xx_HAL_Driver/Src/stm32h7xx_hal_rcc_ex.c.obj
 .text.HAL_RCCEx_GetPLL1ClockFreq
                0x00000000      0x234 CMakeFiles/H750_S15909.elf.dir/Drivers/STM32H7xx_HAL_Driver/Src/stm32h7xx_hal_rcc_ex.c.obj
 .text.HAL_RCCEx_GetPeriphCLKFreq
                0x00000000      0x614 CMakeFiles/H750_S15909.elf.dir/Drivers/STM32H7xx_HAL_Driver/Src/stm32h7xx_hal_rcc_ex.c.obj
 .text.HAL_RCCEx_GetD1SysClockFreq
                0x00000000       0x44 CMakeFiles/H750_S15909.elf.dir/Drivers/STM32H7xx_HAL_Driver/Src/stm32h7xx_hal_rcc_ex.c.obj
 .text.HAL_RCCEx_EnableLSECSS
                0x00000000       0x10 CMakeFiles/H750_S15909.elf.dir/Drivers/STM32H7xx_HAL_Driver/Src/stm32h7xx_hal_rcc_ex.c.obj
 .text.HAL_RCCEx_DisableLSECSS
                0x00000000       0x18 CMakeFiles/H750_S15909.elf.dir/Drivers/STM32H7xx_HAL_Driver/Src/stm32h7xx_hal_rcc_ex.c.obj
 .text.HAL_RCCEx_EnableLSECSS_IT
                0x00000000       0x30 CMakeFiles/H750_S15909.elf.dir/Drivers/STM32H7xx_HAL_Driver/Src/stm32h7xx_hal_rcc_ex.c.obj
 .text.HAL_RCCEx_WakeUpStopCLKConfig
                0x00000000       0x14 CMakeFiles/H750_S15909.elf.dir/Drivers/STM32H7xx_HAL_Driver/Src/stm32h7xx_hal_rcc_ex.c.obj
 .text.HAL_RCCEx_KerWakeUpStopCLKConfig
                0x00000000       0x14 CMakeFiles/H750_S15909.elf.dir/Drivers/STM32H7xx_HAL_Driver/Src/stm32h7xx_hal_rcc_ex.c.obj
 .text.HAL_RCCEx_WWDGxSysResetConfig
                0x00000000       0x14 CMakeFiles/H750_S15909.elf.dir/Drivers/STM32H7xx_HAL_Driver/Src/stm32h7xx_hal_rcc_ex.c.obj
 .text.HAL_RCCEx_CRSConfig
                0x00000000       0x74 CMakeFiles/H750_S15909.elf.dir/Drivers/STM32H7xx_HAL_Driver/Src/stm32h7xx_hal_rcc_ex.c.obj
 .text.HAL_RCCEx_CRSSoftwareSynchronizationGenerate
                0x00000000       0x10 CMakeFiles/H750_S15909.elf.dir/Drivers/STM32H7xx_HAL_Driver/Src/stm32h7xx_hal_rcc_ex.c.obj
 .text.HAL_RCCEx_CRSGetSynchronizationInfo
                0x00000000       0x24 CMakeFiles/H750_S15909.elf.dir/Drivers/STM32H7xx_HAL_Driver/Src/stm32h7xx_hal_rcc_ex.c.obj
 .text.HAL_RCCEx_CRSWaitSynchronization
                0x00000000       0xac CMakeFiles/H750_S15909.elf.dir/Drivers/STM32H7xx_HAL_Driver/Src/stm32h7xx_hal_rcc_ex.c.obj
 .text.HAL_RCCEx_CRS_SyncOkCallback
                0x00000000        0x2 CMakeFiles/H750_S15909.elf.dir/Drivers/STM32H7xx_HAL_Driver/Src/stm32h7xx_hal_rcc_ex.c.obj
 .text.HAL_RCCEx_CRS_SyncWarnCallback
                0x00000000        0x2 CMakeFiles/H750_S15909.elf.dir/Drivers/STM32H7xx_HAL_Driver/Src/stm32h7xx_hal_rcc_ex.c.obj
 .text.HAL_RCCEx_CRS_ExpectedSyncCallback
                0x00000000        0x2 CMakeFiles/H750_S15909.elf.dir/Drivers/STM32H7xx_HAL_Driver/Src/stm32h7xx_hal_rcc_ex.c.obj
 .text.HAL_RCCEx_CRS_ErrorCallback
                0x00000000        0x2 CMakeFiles/H750_S15909.elf.dir/Drivers/STM32H7xx_HAL_Driver/Src/stm32h7xx_hal_rcc_ex.c.obj
 .text.HAL_RCCEx_CRS_IRQHandler
                0x00000000       0x88 CMakeFiles/H750_S15909.elf.dir/Drivers/STM32H7xx_HAL_Driver/Src/stm32h7xx_hal_rcc_ex.c.obj
 .text.HAL_RCCEx_LSECSS_Callback
                0x00000000        0x2 CMakeFiles/H750_S15909.elf.dir/Drivers/STM32H7xx_HAL_Driver/Src/stm32h7xx_hal_rcc_ex.c.obj
 .text.HAL_RCCEx_LSECSS_IRQHandler
                0x00000000       0x20 CMakeFiles/H750_S15909.elf.dir/Drivers/STM32H7xx_HAL_Driver/Src/stm32h7xx_hal_rcc_ex.c.obj
 .text          0x00000000        0x0 CMakeFiles/H750_S15909.elf.dir/Drivers/STM32H7xx_HAL_Driver/Src/stm32h7xx_hal_tim.c.obj
 .data          0x00000000        0x0 CMakeFiles/H750_S15909.elf.dir/Drivers/STM32H7xx_HAL_Driver/Src/stm32h7xx_hal_tim.c.obj
 .bss           0x00000000        0x0 CMakeFiles/H750_S15909.elf.dir/Drivers/STM32H7xx_HAL_Driver/Src/stm32h7xx_hal_tim.c.obj
 .text.TIM_OC1_SetConfig
                0x00000000       0xa8 CMakeFiles/H750_S15909.elf.dir/Drivers/STM32H7xx_HAL_Driver/Src/stm32h7xx_hal_tim.c.obj
 .text.TIM_OC3_SetConfig
                0x00000000       0x94 CMakeFiles/H750_S15909.elf.dir/Drivers/STM32H7xx_HAL_Driver/Src/stm32h7xx_hal_tim.c.obj
 .text.TIM_OC4_SetConfig
                0x00000000       0x74 CMakeFiles/H750_S15909.elf.dir/Drivers/STM32H7xx_HAL_Driver/Src/stm32h7xx_hal_tim.c.obj
 .text.TIM_OC5_SetConfig
                0x00000000       0x74 CMakeFiles/H750_S15909.elf.dir/Drivers/STM32H7xx_HAL_Driver/Src/stm32h7xx_hal_tim.c.obj
 .text.TIM_OC6_SetConfig
                0x00000000       0x74 CMakeFiles/H750_S15909.elf.dir/Drivers/STM32H7xx_HAL_Driver/Src/stm32h7xx_hal_tim.c.obj
 .text.TIM_TI2_SetConfig
                0x00000000       0x36 CMakeFiles/H750_S15909.elf.dir/Drivers/STM32H7xx_HAL_Driver/Src/stm32h7xx_hal_tim.c.obj
 .text.TIM_TI3_SetConfig
                0x00000000       0x36 CMakeFiles/H750_S15909.elf.dir/Drivers/STM32H7xx_HAL_Driver/Src/stm32h7xx_hal_tim.c.obj
 .text.TIM_TI4_SetConfig
                0x00000000       0x36 CMakeFiles/H750_S15909.elf.dir/Drivers/STM32H7xx_HAL_Driver/Src/stm32h7xx_hal_tim.c.obj
 .text.HAL_TIM_Base_MspInit
                0x00000000        0x2 CMakeFiles/H750_S15909.elf.dir/Drivers/STM32H7xx_HAL_Driver/Src/stm32h7xx_hal_tim.c.obj
 .text.HAL_TIM_Base_MspDeInit
                0x00000000        0x2 CMakeFiles/H750_S15909.elf.dir/Drivers/STM32H7xx_HAL_Driver/Src/stm32h7xx_hal_tim.c.obj
 .text.HAL_TIM_Base_DeInit
                0x00000000       0x66 CMakeFiles/H750_S15909.elf.dir/Drivers/STM32H7xx_HAL_Driver/Src/stm32h7xx_hal_tim.c.obj
 .text.HAL_TIM_Base_Stop
                0x00000000       0x28 CMakeFiles/H750_S15909.elf.dir/Drivers/STM32H7xx_HAL_Driver/Src/stm32h7xx_hal_tim.c.obj
 .text.HAL_TIM_Base_Start_IT
                0x00000000       0x90 CMakeFiles/H750_S15909.elf.dir/Drivers/STM32H7xx_HAL_Driver/Src/stm32h7xx_hal_tim.c.obj
 .text.HAL_TIM_Base_Stop_IT
                0x00000000       0x32 CMakeFiles/H750_S15909.elf.dir/Drivers/STM32H7xx_HAL_Driver/Src/stm32h7xx_hal_tim.c.obj
 .text.HAL_TIM_Base_Start_DMA
                0x00000000       0xe4 CMakeFiles/H750_S15909.elf.dir/Drivers/STM32H7xx_HAL_Driver/Src/stm32h7xx_hal_tim.c.obj
 .text.HAL_TIM_Base_Stop_DMA
                0x00000000       0x3c CMakeFiles/H750_S15909.elf.dir/Drivers/STM32H7xx_HAL_Driver/Src/stm32h7xx_hal_tim.c.obj
 .text.HAL_TIM_OC_MspInit
                0x00000000        0x2 CMakeFiles/H750_S15909.elf.dir/Drivers/STM32H7xx_HAL_Driver/Src/stm32h7xx_hal_tim.c.obj
 .text.HAL_TIM_OC_MspDeInit
                0x00000000        0x2 CMakeFiles/H750_S15909.elf.dir/Drivers/STM32H7xx_HAL_Driver/Src/stm32h7xx_hal_tim.c.obj
 .text.HAL_TIM_OC_DeInit
                0x00000000       0x66 CMakeFiles/H750_S15909.elf.dir/Drivers/STM32H7xx_HAL_Driver/Src/stm32h7xx_hal_tim.c.obj
 .text.HAL_TIM_PWM_MspInit
                0x00000000        0x2 CMakeFiles/H750_S15909.elf.dir/Drivers/STM32H7xx_HAL_Driver/Src/stm32h7xx_hal_tim.c.obj
 .text.HAL_TIM_PWM_MspDeInit
                0x00000000        0x2 CMakeFiles/H750_S15909.elf.dir/Drivers/STM32H7xx_HAL_Driver/Src/stm32h7xx_hal_tim.c.obj
 .text.HAL_TIM_PWM_DeInit
                0x00000000       0x66 CMakeFiles/H750_S15909.elf.dir/Drivers/STM32H7xx_HAL_Driver/Src/stm32h7xx_hal_tim.c.obj
 .text.HAL_TIM_IC_MspInit
                0x00000000        0x2 CMakeFiles/H750_S15909.elf.dir/Drivers/STM32H7xx_HAL_Driver/Src/stm32h7xx_hal_tim.c.obj
 .text.HAL_TIM_IC_MspDeInit
                0x00000000        0x2 CMakeFiles/H750_S15909.elf.dir/Drivers/STM32H7xx_HAL_Driver/Src/stm32h7xx_hal_tim.c.obj
 .text.HAL_TIM_IC_DeInit
                0x00000000       0x66 CMakeFiles/H750_S15909.elf.dir/Drivers/STM32H7xx_HAL_Driver/Src/stm32h7xx_hal_tim.c.obj
 .text.HAL_TIM_OnePulse_MspInit
                0x00000000        0x2 CMakeFiles/H750_S15909.elf.dir/Drivers/STM32H7xx_HAL_Driver/Src/stm32h7xx_hal_tim.c.obj
 .text.HAL_TIM_OnePulse_MspDeInit
                0x00000000        0x2 CMakeFiles/H750_S15909.elf.dir/Drivers/STM32H7xx_HAL_Driver/Src/stm32h7xx_hal_tim.c.obj
 .text.HAL_TIM_OnePulse_DeInit
                0x00000000       0x4e CMakeFiles/H750_S15909.elf.dir/Drivers/STM32H7xx_HAL_Driver/Src/stm32h7xx_hal_tim.c.obj
 .text.HAL_TIM_Encoder_MspInit
                0x00000000        0x2 CMakeFiles/H750_S15909.elf.dir/Drivers/STM32H7xx_HAL_Driver/Src/stm32h7xx_hal_tim.c.obj
 .text.HAL_TIM_Encoder_MspDeInit
                0x00000000        0x2 CMakeFiles/H750_S15909.elf.dir/Drivers/STM32H7xx_HAL_Driver/Src/stm32h7xx_hal_tim.c.obj
 .text.HAL_TIM_Encoder_DeInit
                0x00000000       0x4e CMakeFiles/H750_S15909.elf.dir/Drivers/STM32H7xx_HAL_Driver/Src/stm32h7xx_hal_tim.c.obj
 .text.HAL_TIM_DMABurst_MultiWriteStart
                0x00000000      0x1ac CMakeFiles/H750_S15909.elf.dir/Drivers/STM32H7xx_HAL_Driver/Src/stm32h7xx_hal_tim.c.obj
 .text.HAL_TIM_DMABurst_WriteStart
                0x00000000       0x16 CMakeFiles/H750_S15909.elf.dir/Drivers/STM32H7xx_HAL_Driver/Src/stm32h7xx_hal_tim.c.obj
 .text.HAL_TIM_DMABurst_WriteStop
                0x00000000       0x84 CMakeFiles/H750_S15909.elf.dir/Drivers/STM32H7xx_HAL_Driver/Src/stm32h7xx_hal_tim.c.obj
 .text.HAL_TIM_DMABurst_MultiReadStart
                0x00000000      0x1b0 CMakeFiles/H750_S15909.elf.dir/Drivers/STM32H7xx_HAL_Driver/Src/stm32h7xx_hal_tim.c.obj
 .text.HAL_TIM_DMABurst_ReadStart
                0x00000000       0x16 CMakeFiles/H750_S15909.elf.dir/Drivers/STM32H7xx_HAL_Driver/Src/stm32h7xx_hal_tim.c.obj
 .text.HAL_TIM_DMABurst_ReadStop
                0x00000000       0x84 CMakeFiles/H750_S15909.elf.dir/Drivers/STM32H7xx_HAL_Driver/Src/stm32h7xx_hal_tim.c.obj
 .text.HAL_TIM_GenerateEvent
                0x00000000       0x2a CMakeFiles/H750_S15909.elf.dir/Drivers/STM32H7xx_HAL_Driver/Src/stm32h7xx_hal_tim.c.obj
 .text.HAL_TIM_ConfigTI1Input
                0x00000000       0x10 CMakeFiles/H750_S15909.elf.dir/Drivers/STM32H7xx_HAL_Driver/Src/stm32h7xx_hal_tim.c.obj
 .text.HAL_TIM_ReadCapturedValue
                0x00000000       0x32 CMakeFiles/H750_S15909.elf.dir/Drivers/STM32H7xx_HAL_Driver/Src/stm32h7xx_hal_tim.c.obj
 .text.HAL_TIM_PeriodElapsedCallback
                0x00000000        0x2 CMakeFiles/H750_S15909.elf.dir/Drivers/STM32H7xx_HAL_Driver/Src/stm32h7xx_hal_tim.c.obj
 .text.TIM_DMAPeriodElapsedCplt
                0x00000000       0x16 CMakeFiles/H750_S15909.elf.dir/Drivers/STM32H7xx_HAL_Driver/Src/stm32h7xx_hal_tim.c.obj
 .text.HAL_TIM_PeriodElapsedHalfCpltCallback
                0x00000000        0x2 CMakeFiles/H750_S15909.elf.dir/Drivers/STM32H7xx_HAL_Driver/Src/stm32h7xx_hal_tim.c.obj
 .text.TIM_DMAPeriodElapsedHalfCplt
                0x00000000        0xa CMakeFiles/H750_S15909.elf.dir/Drivers/STM32H7xx_HAL_Driver/Src/stm32h7xx_hal_tim.c.obj
 .text.HAL_TIM_OC_DelayElapsedCallback
                0x00000000        0x2 CMakeFiles/H750_S15909.elf.dir/Drivers/STM32H7xx_HAL_Driver/Src/stm32h7xx_hal_tim.c.obj
 .text.HAL_TIM_IC_CaptureCallback
                0x00000000        0x2 CMakeFiles/H750_S15909.elf.dir/Drivers/STM32H7xx_HAL_Driver/Src/stm32h7xx_hal_tim.c.obj
 .text.TIM_DMACaptureCplt
                0x00000000       0x80 CMakeFiles/H750_S15909.elf.dir/Drivers/STM32H7xx_HAL_Driver/Src/stm32h7xx_hal_tim.c.obj
 .text.HAL_TIM_IC_CaptureHalfCpltCallback
                0x00000000        0x2 CMakeFiles/H750_S15909.elf.dir/Drivers/STM32H7xx_HAL_Driver/Src/stm32h7xx_hal_tim.c.obj
 .text.TIM_DMACaptureHalfCplt
                0x00000000       0x3e CMakeFiles/H750_S15909.elf.dir/Drivers/STM32H7xx_HAL_Driver/Src/stm32h7xx_hal_tim.c.obj
 .text.HAL_TIM_PWM_PulseFinishedCallback
                0x00000000        0x2 CMakeFiles/H750_S15909.elf.dir/Drivers/STM32H7xx_HAL_Driver/Src/stm32h7xx_hal_tim.c.obj
 .text.TIM_DMADelayPulseCplt
                0x00000000       0x70 CMakeFiles/H750_S15909.elf.dir/Drivers/STM32H7xx_HAL_Driver/Src/stm32h7xx_hal_tim.c.obj
 .text.HAL_TIM_PWM_PulseFinishedHalfCpltCallback
                0x00000000        0x2 CMakeFiles/H750_S15909.elf.dir/Drivers/STM32H7xx_HAL_Driver/Src/stm32h7xx_hal_tim.c.obj
 .text.TIM_DMADelayPulseHalfCplt
                0x00000000       0x3e CMakeFiles/H750_S15909.elf.dir/Drivers/STM32H7xx_HAL_Driver/Src/stm32h7xx_hal_tim.c.obj
 .text.HAL_TIM_TriggerCallback
                0x00000000        0x2 CMakeFiles/H750_S15909.elf.dir/Drivers/STM32H7xx_HAL_Driver/Src/stm32h7xx_hal_tim.c.obj
 .text.HAL_TIM_IRQHandler
                0x00000000      0x19a CMakeFiles/H750_S15909.elf.dir/Drivers/STM32H7xx_HAL_Driver/Src/stm32h7xx_hal_tim.c.obj
 .text.TIM_DMATriggerCplt
                0x00000000       0x16 CMakeFiles/H750_S15909.elf.dir/Drivers/STM32H7xx_HAL_Driver/Src/stm32h7xx_hal_tim.c.obj
 .text.HAL_TIM_TriggerHalfCpltCallback
                0x00000000        0x2 CMakeFiles/H750_S15909.elf.dir/Drivers/STM32H7xx_HAL_Driver/Src/stm32h7xx_hal_tim.c.obj
 .text.TIM_DMATriggerHalfCplt
                0x00000000        0xa CMakeFiles/H750_S15909.elf.dir/Drivers/STM32H7xx_HAL_Driver/Src/stm32h7xx_hal_tim.c.obj
 .text.HAL_TIM_ErrorCallback
                0x00000000        0x2 CMakeFiles/H750_S15909.elf.dir/Drivers/STM32H7xx_HAL_Driver/Src/stm32h7xx_hal_tim.c.obj
 .text.TIM_DMAError
                0x00000000       0x5c CMakeFiles/H750_S15909.elf.dir/Drivers/STM32H7xx_HAL_Driver/Src/stm32h7xx_hal_tim.c.obj
 .text.HAL_TIM_Base_GetState
                0x00000000        0x6 CMakeFiles/H750_S15909.elf.dir/Drivers/STM32H7xx_HAL_Driver/Src/stm32h7xx_hal_tim.c.obj
 .text.HAL_TIM_OC_GetState
                0x00000000        0x6 CMakeFiles/H750_S15909.elf.dir/Drivers/STM32H7xx_HAL_Driver/Src/stm32h7xx_hal_tim.c.obj
 .text.HAL_TIM_PWM_GetState
                0x00000000        0x6 CMakeFiles/H750_S15909.elf.dir/Drivers/STM32H7xx_HAL_Driver/Src/stm32h7xx_hal_tim.c.obj
 .text.HAL_TIM_IC_GetState
                0x00000000        0x6 CMakeFiles/H750_S15909.elf.dir/Drivers/STM32H7xx_HAL_Driver/Src/stm32h7xx_hal_tim.c.obj
 .text.HAL_TIM_OnePulse_GetState
                0x00000000        0x6 CMakeFiles/H750_S15909.elf.dir/Drivers/STM32H7xx_HAL_Driver/Src/stm32h7xx_hal_tim.c.obj
 .text.HAL_TIM_Encoder_GetState
                0x00000000        0x6 CMakeFiles/H750_S15909.elf.dir/Drivers/STM32H7xx_HAL_Driver/Src/stm32h7xx_hal_tim.c.obj
 .text.HAL_TIM_GetActiveChannel
                0x00000000        0x4 CMakeFiles/H750_S15909.elf.dir/Drivers/STM32H7xx_HAL_Driver/Src/stm32h7xx_hal_tim.c.obj
 .text.HAL_TIM_GetChannelState
                0x00000000       0x42 CMakeFiles/H750_S15909.elf.dir/Drivers/STM32H7xx_HAL_Driver/Src/stm32h7xx_hal_tim.c.obj
 .text.HAL_TIM_DMABurstState
                0x00000000        0x6 CMakeFiles/H750_S15909.elf.dir/Drivers/STM32H7xx_HAL_Driver/Src/stm32h7xx_hal_tim.c.obj
 .text.HAL_TIM_OC_Init
                0x00000000       0x60 CMakeFiles/H750_S15909.elf.dir/Drivers/STM32H7xx_HAL_Driver/Src/stm32h7xx_hal_tim.c.obj
 .text.HAL_TIM_PWM_Init
                0x00000000       0x60 CMakeFiles/H750_S15909.elf.dir/Drivers/STM32H7xx_HAL_Driver/Src/stm32h7xx_hal_tim.c.obj
 .text.HAL_TIM_IC_Init
                0x00000000       0x60 CMakeFiles/H750_S15909.elf.dir/Drivers/STM32H7xx_HAL_Driver/Src/stm32h7xx_hal_tim.c.obj
 .text.HAL_TIM_OnePulse_Init
                0x00000000       0x5c CMakeFiles/H750_S15909.elf.dir/Drivers/STM32H7xx_HAL_Driver/Src/stm32h7xx_hal_tim.c.obj
 .text.HAL_TIM_Encoder_Init
                0x00000000       0xbc CMakeFiles/H750_S15909.elf.dir/Drivers/STM32H7xx_HAL_Driver/Src/stm32h7xx_hal_tim.c.obj
 .text.TIM_OC2_SetConfig
                0x00000000       0x94 CMakeFiles/H750_S15909.elf.dir/Drivers/STM32H7xx_HAL_Driver/Src/stm32h7xx_hal_tim.c.obj
 .text.HAL_TIM_OC_ConfigChannel
                0x00000000       0x7a CMakeFiles/H750_S15909.elf.dir/Drivers/STM32H7xx_HAL_Driver/Src/stm32h7xx_hal_tim.c.obj
 .text.HAL_TIM_PWM_ConfigChannel
                0x00000000      0x13a CMakeFiles/H750_S15909.elf.dir/Drivers/STM32H7xx_HAL_Driver/Src/stm32h7xx_hal_tim.c.obj
 .text.TIM_TI1_SetConfig
                0x00000000       0x94 CMakeFiles/H750_S15909.elf.dir/Drivers/STM32H7xx_HAL_Driver/Src/stm32h7xx_hal_tim.c.obj
 .text.HAL_TIM_IC_ConfigChannel
                0x00000000       0xc4 CMakeFiles/H750_S15909.elf.dir/Drivers/STM32H7xx_HAL_Driver/Src/stm32h7xx_hal_tim.c.obj
 .text.HAL_TIM_OnePulse_ConfigChannel
                0x00000000      0x104 CMakeFiles/H750_S15909.elf.dir/Drivers/STM32H7xx_HAL_Driver/Src/stm32h7xx_hal_tim.c.obj
 .text.HAL_TIM_ConfigOCrefClear
                0x00000000      0x144 CMakeFiles/H750_S15909.elf.dir/Drivers/STM32H7xx_HAL_Driver/Src/stm32h7xx_hal_tim.c.obj
 .text.TIM_SlaveTimer_SetConfig
                0x00000000      0x150 CMakeFiles/H750_S15909.elf.dir/Drivers/STM32H7xx_HAL_Driver/Src/stm32h7xx_hal_tim.c.obj
 .text.HAL_TIM_SlaveConfigSynchro
                0x00000000       0x52 CMakeFiles/H750_S15909.elf.dir/Drivers/STM32H7xx_HAL_Driver/Src/stm32h7xx_hal_tim.c.obj
 .text.HAL_TIM_SlaveConfigSynchro_IT
                0x00000000       0x52 CMakeFiles/H750_S15909.elf.dir/Drivers/STM32H7xx_HAL_Driver/Src/stm32h7xx_hal_tim.c.obj
 .text.TIM_CCxChannelCmd
                0x00000000       0x1e CMakeFiles/H750_S15909.elf.dir/Drivers/STM32H7xx_HAL_Driver/Src/stm32h7xx_hal_tim.c.obj
 .text.HAL_TIM_OC_Start
                0x00000000      0x168 CMakeFiles/H750_S15909.elf.dir/Drivers/STM32H7xx_HAL_Driver/Src/stm32h7xx_hal_tim.c.obj
 .text.HAL_TIM_OC_Stop
                0x00000000       0xbc CMakeFiles/H750_S15909.elf.dir/Drivers/STM32H7xx_HAL_Driver/Src/stm32h7xx_hal_tim.c.obj
 .text.HAL_TIM_OC_Start_IT
                0x00000000      0x1b0 CMakeFiles/H750_S15909.elf.dir/Drivers/STM32H7xx_HAL_Driver/Src/stm32h7xx_hal_tim.c.obj
 .text.HAL_TIM_OC_Stop_IT
                0x00000000      0x110 CMakeFiles/H750_S15909.elf.dir/Drivers/STM32H7xx_HAL_Driver/Src/stm32h7xx_hal_tim.c.obj
 .text.HAL_TIM_OC_Start_DMA
                0x00000000      0x300 CMakeFiles/H750_S15909.elf.dir/Drivers/STM32H7xx_HAL_Driver/Src/stm32h7xx_hal_tim.c.obj
 .text.HAL_TIM_OC_Stop_DMA
                0x00000000      0x128 CMakeFiles/H750_S15909.elf.dir/Drivers/STM32H7xx_HAL_Driver/Src/stm32h7xx_hal_tim.c.obj
 .text.HAL_TIM_PWM_Start
                0x00000000      0x168 CMakeFiles/H750_S15909.elf.dir/Drivers/STM32H7xx_HAL_Driver/Src/stm32h7xx_hal_tim.c.obj
 .text.HAL_TIM_PWM_Stop
                0x00000000       0xbc CMakeFiles/H750_S15909.elf.dir/Drivers/STM32H7xx_HAL_Driver/Src/stm32h7xx_hal_tim.c.obj
 .text.HAL_TIM_PWM_Start_IT
                0x00000000      0x1b0 CMakeFiles/H750_S15909.elf.dir/Drivers/STM32H7xx_HAL_Driver/Src/stm32h7xx_hal_tim.c.obj
 .text.HAL_TIM_PWM_Stop_IT
                0x00000000      0x110 CMakeFiles/H750_S15909.elf.dir/Drivers/STM32H7xx_HAL_Driver/Src/stm32h7xx_hal_tim.c.obj
 .text.HAL_TIM_PWM_Start_DMA
                0x00000000      0x300 CMakeFiles/H750_S15909.elf.dir/Drivers/STM32H7xx_HAL_Driver/Src/stm32h7xx_hal_tim.c.obj
 .text.HAL_TIM_PWM_Stop_DMA
                0x00000000      0x128 CMakeFiles/H750_S15909.elf.dir/Drivers/STM32H7xx_HAL_Driver/Src/stm32h7xx_hal_tim.c.obj
 .text.HAL_TIM_IC_Start
                0x00000000      0x168 CMakeFiles/H750_S15909.elf.dir/Drivers/STM32H7xx_HAL_Driver/Src/stm32h7xx_hal_tim.c.obj
 .text.HAL_TIM_IC_Stop
                0x00000000       0x98 CMakeFiles/H750_S15909.elf.dir/Drivers/STM32H7xx_HAL_Driver/Src/stm32h7xx_hal_tim.c.obj
 .text.HAL_TIM_IC_Start_IT
                0x00000000      0x1b0 CMakeFiles/H750_S15909.elf.dir/Drivers/STM32H7xx_HAL_Driver/Src/stm32h7xx_hal_tim.c.obj
 .text.HAL_TIM_IC_Stop_IT
                0x00000000       0xe8 CMakeFiles/H750_S15909.elf.dir/Drivers/STM32H7xx_HAL_Driver/Src/stm32h7xx_hal_tim.c.obj
 .text.HAL_TIM_IC_Start_DMA
                0x00000000      0x28c CMakeFiles/H750_S15909.elf.dir/Drivers/STM32H7xx_HAL_Driver/Src/stm32h7xx_hal_tim.c.obj
 .text.HAL_TIM_IC_Stop_DMA
                0x00000000      0x100 CMakeFiles/H750_S15909.elf.dir/Drivers/STM32H7xx_HAL_Driver/Src/stm32h7xx_hal_tim.c.obj
 .text.HAL_TIM_OnePulse_Start
                0x00000000       0x9c CMakeFiles/H750_S15909.elf.dir/Drivers/STM32H7xx_HAL_Driver/Src/stm32h7xx_hal_tim.c.obj
 .text.HAL_TIM_OnePulse_Stop
                0x00000000       0x98 CMakeFiles/H750_S15909.elf.dir/Drivers/STM32H7xx_HAL_Driver/Src/stm32h7xx_hal_tim.c.obj
 .text.HAL_TIM_OnePulse_Start_IT
                0x00000000       0xb4 CMakeFiles/H750_S15909.elf.dir/Drivers/STM32H7xx_HAL_Driver/Src/stm32h7xx_hal_tim.c.obj
 .text.HAL_TIM_OnePulse_Stop_IT
                0x00000000       0xac CMakeFiles/H750_S15909.elf.dir/Drivers/STM32H7xx_HAL_Driver/Src/stm32h7xx_hal_tim.c.obj
 .text.HAL_TIM_Encoder_Start
                0x00000000       0xc8 CMakeFiles/H750_S15909.elf.dir/Drivers/STM32H7xx_HAL_Driver/Src/stm32h7xx_hal_tim.c.obj
 .text.HAL_TIM_Encoder_Stop
                0x00000000       0xde CMakeFiles/H750_S15909.elf.dir/Drivers/STM32H7xx_HAL_Driver/Src/stm32h7xx_hal_tim.c.obj
 .text.HAL_TIM_Encoder_Start_IT
                0x00000000       0xf4 CMakeFiles/H750_S15909.elf.dir/Drivers/STM32H7xx_HAL_Driver/Src/stm32h7xx_hal_tim.c.obj
 .text.HAL_TIM_Encoder_Stop_IT
                0x00000000      0x108 CMakeFiles/H750_S15909.elf.dir/Drivers/STM32H7xx_HAL_Driver/Src/stm32h7xx_hal_tim.c.obj
 .text.HAL_TIM_Encoder_Start_DMA
                0x00000000      0x258 CMakeFiles/H750_S15909.elf.dir/Drivers/STM32H7xx_HAL_Driver/Src/stm32h7xx_hal_tim.c.obj
 .text.HAL_TIM_Encoder_Stop_DMA
                0x00000000      0x122 CMakeFiles/H750_S15909.elf.dir/Drivers/STM32H7xx_HAL_Driver/Src/stm32h7xx_hal_tim.c.obj
 .text          0x00000000        0x0 CMakeFiles/H750_S15909.elf.dir/Drivers/STM32H7xx_HAL_Driver/Src/stm32h7xx_hal_tim_ex.c.obj
 .data          0x00000000        0x0 CMakeFiles/H750_S15909.elf.dir/Drivers/STM32H7xx_HAL_Driver/Src/stm32h7xx_hal_tim_ex.c.obj
 .bss           0x00000000        0x0 CMakeFiles/H750_S15909.elf.dir/Drivers/STM32H7xx_HAL_Driver/Src/stm32h7xx_hal_tim_ex.c.obj
 .text.TIM_CCxNChannelCmd
                0x00000000       0x1e CMakeFiles/H750_S15909.elf.dir/Drivers/STM32H7xx_HAL_Driver/Src/stm32h7xx_hal_tim_ex.c.obj
 .text.TIM_DMAErrorCCxN
                0x00000000       0x44 CMakeFiles/H750_S15909.elf.dir/Drivers/STM32H7xx_HAL_Driver/Src/stm32h7xx_hal_tim_ex.c.obj
 .text.TIM_DMADelayPulseNCplt
                0x00000000       0x70 CMakeFiles/H750_S15909.elf.dir/Drivers/STM32H7xx_HAL_Driver/Src/stm32h7xx_hal_tim_ex.c.obj
 .text.HAL_TIMEx_HallSensor_MspInit
                0x00000000        0x2 CMakeFiles/H750_S15909.elf.dir/Drivers/STM32H7xx_HAL_Driver/Src/stm32h7xx_hal_tim_ex.c.obj
 .text.HAL_TIMEx_HallSensor_Init
                0x00000000       0xdc CMakeFiles/H750_S15909.elf.dir/Drivers/STM32H7xx_HAL_Driver/Src/stm32h7xx_hal_tim_ex.c.obj
 .text.HAL_TIMEx_HallSensor_MspDeInit
                0x00000000        0x2 CMakeFiles/H750_S15909.elf.dir/Drivers/STM32H7xx_HAL_Driver/Src/stm32h7xx_hal_tim_ex.c.obj
 .text.HAL_TIMEx_HallSensor_DeInit
                0x00000000       0x4e CMakeFiles/H750_S15909.elf.dir/Drivers/STM32H7xx_HAL_Driver/Src/stm32h7xx_hal_tim_ex.c.obj
 .text.HAL_TIMEx_HallSensor_Start
                0x00000000       0xc8 CMakeFiles/H750_S15909.elf.dir/Drivers/STM32H7xx_HAL_Driver/Src/stm32h7xx_hal_tim_ex.c.obj
 .text.HAL_TIMEx_HallSensor_Stop
                0x00000000       0x42 CMakeFiles/H750_S15909.elf.dir/Drivers/STM32H7xx_HAL_Driver/Src/stm32h7xx_hal_tim_ex.c.obj
 .text.HAL_TIMEx_HallSensor_Start_IT
                0x00000000       0xd4 CMakeFiles/H750_S15909.elf.dir/Drivers/STM32H7xx_HAL_Driver/Src/stm32h7xx_hal_tim_ex.c.obj
 .text.HAL_TIMEx_HallSensor_Stop_IT
                0x00000000       0x4c CMakeFiles/H750_S15909.elf.dir/Drivers/STM32H7xx_HAL_Driver/Src/stm32h7xx_hal_tim_ex.c.obj
 .text.HAL_TIMEx_HallSensor_Start_DMA
                0x00000000      0x100 CMakeFiles/H750_S15909.elf.dir/Drivers/STM32H7xx_HAL_Driver/Src/stm32h7xx_hal_tim_ex.c.obj
 .text.HAL_TIMEx_HallSensor_Stop_DMA
                0x00000000       0x4a CMakeFiles/H750_S15909.elf.dir/Drivers/STM32H7xx_HAL_Driver/Src/stm32h7xx_hal_tim_ex.c.obj
 .text.HAL_TIMEx_OCN_Start
                0x00000000      0x100 CMakeFiles/H750_S15909.elf.dir/Drivers/STM32H7xx_HAL_Driver/Src/stm32h7xx_hal_tim_ex.c.obj
 .text.HAL_TIMEx_OCN_Stop
                0x00000000       0x76 CMakeFiles/H750_S15909.elf.dir/Drivers/STM32H7xx_HAL_Driver/Src/stm32h7xx_hal_tim_ex.c.obj
 .text.HAL_TIMEx_OCN_Start_IT
                0x00000000      0x138 CMakeFiles/H750_S15909.elf.dir/Drivers/STM32H7xx_HAL_Driver/Src/stm32h7xx_hal_tim_ex.c.obj
 .text.HAL_TIMEx_OCN_Stop_IT
                0x00000000       0xc2 CMakeFiles/H750_S15909.elf.dir/Drivers/STM32H7xx_HAL_Driver/Src/stm32h7xx_hal_tim_ex.c.obj
 .text.HAL_TIMEx_OCN_Start_DMA
                0x00000000      0x228 CMakeFiles/H750_S15909.elf.dir/Drivers/STM32H7xx_HAL_Driver/Src/stm32h7xx_hal_tim_ex.c.obj
 .text.HAL_TIMEx_OCN_Stop_DMA
                0x00000000       0xc0 CMakeFiles/H750_S15909.elf.dir/Drivers/STM32H7xx_HAL_Driver/Src/stm32h7xx_hal_tim_ex.c.obj
 .text.HAL_TIMEx_PWMN_Start
                0x00000000      0x100 CMakeFiles/H750_S15909.elf.dir/Drivers/STM32H7xx_HAL_Driver/Src/stm32h7xx_hal_tim_ex.c.obj
 .text.HAL_TIMEx_PWMN_Stop
                0x00000000       0x76 CMakeFiles/H750_S15909.elf.dir/Drivers/STM32H7xx_HAL_Driver/Src/stm32h7xx_hal_tim_ex.c.obj
 .text.HAL_TIMEx_PWMN_Start_IT
                0x00000000      0x138 CMakeFiles/H750_S15909.elf.dir/Drivers/STM32H7xx_HAL_Driver/Src/stm32h7xx_hal_tim_ex.c.obj
 .text.HAL_TIMEx_PWMN_Stop_IT
                0x00000000       0xc2 CMakeFiles/H750_S15909.elf.dir/Drivers/STM32H7xx_HAL_Driver/Src/stm32h7xx_hal_tim_ex.c.obj
 .text.HAL_TIMEx_PWMN_Start_DMA
                0x00000000      0x228 CMakeFiles/H750_S15909.elf.dir/Drivers/STM32H7xx_HAL_Driver/Src/stm32h7xx_hal_tim_ex.c.obj
 .text.HAL_TIMEx_PWMN_Stop_DMA
                0x00000000       0xc0 CMakeFiles/H750_S15909.elf.dir/Drivers/STM32H7xx_HAL_Driver/Src/stm32h7xx_hal_tim_ex.c.obj
 .text.HAL_TIMEx_OnePulseN_Start
                0x00000000       0x7a CMakeFiles/H750_S15909.elf.dir/Drivers/STM32H7xx_HAL_Driver/Src/stm32h7xx_hal_tim_ex.c.obj
 .text.HAL_TIMEx_OnePulseN_Stop
                0x00000000       0x72 CMakeFiles/H750_S15909.elf.dir/Drivers/STM32H7xx_HAL_Driver/Src/stm32h7xx_hal_tim_ex.c.obj
 .text.HAL_TIMEx_OnePulseN_Start_IT
                0x00000000       0x90 CMakeFiles/H750_S15909.elf.dir/Drivers/STM32H7xx_HAL_Driver/Src/stm32h7xx_hal_tim_ex.c.obj
 .text.HAL_TIMEx_OnePulseN_Stop_IT
                0x00000000       0x86 CMakeFiles/H750_S15909.elf.dir/Drivers/STM32H7xx_HAL_Driver/Src/stm32h7xx_hal_tim_ex.c.obj
 .text.HAL_TIMEx_ConfigCommutEvent
                0x00000000       0x94 CMakeFiles/H750_S15909.elf.dir/Drivers/STM32H7xx_HAL_Driver/Src/stm32h7xx_hal_tim_ex.c.obj
 .text.HAL_TIMEx_ConfigCommutEvent_IT
                0x00000000       0x94 CMakeFiles/H750_S15909.elf.dir/Drivers/STM32H7xx_HAL_Driver/Src/stm32h7xx_hal_tim_ex.c.obj
 .text.HAL_TIMEx_ConfigCommutEvent_DMA
                0x00000000       0xb0 CMakeFiles/H750_S15909.elf.dir/Drivers/STM32H7xx_HAL_Driver/Src/stm32h7xx_hal_tim_ex.c.obj
 .text.HAL_TIMEx_ConfigBreakDeadTime
                0x00000000       0x90 CMakeFiles/H750_S15909.elf.dir/Drivers/STM32H7xx_HAL_Driver/Src/stm32h7xx_hal_tim_ex.c.obj
 .text.HAL_TIMEx_ConfigBreakInput
                0x00000000       0xd2 CMakeFiles/H750_S15909.elf.dir/Drivers/STM32H7xx_HAL_Driver/Src/stm32h7xx_hal_tim_ex.c.obj
 .text.HAL_TIMEx_RemapConfig
                0x00000000       0x28 CMakeFiles/H750_S15909.elf.dir/Drivers/STM32H7xx_HAL_Driver/Src/stm32h7xx_hal_tim_ex.c.obj
 .text.HAL_TIMEx_TISelection
                0x00000000       0x74 CMakeFiles/H750_S15909.elf.dir/Drivers/STM32H7xx_HAL_Driver/Src/stm32h7xx_hal_tim_ex.c.obj
 .text.HAL_TIMEx_GroupChannel5
                0x00000000       0x3c CMakeFiles/H750_S15909.elf.dir/Drivers/STM32H7xx_HAL_Driver/Src/stm32h7xx_hal_tim_ex.c.obj
 .text.HAL_TIMEx_CommutCallback
                0x00000000        0x2 CMakeFiles/H750_S15909.elf.dir/Drivers/STM32H7xx_HAL_Driver/Src/stm32h7xx_hal_tim_ex.c.obj
 .text.TIMEx_DMACommutationCplt
                0x00000000       0x10 CMakeFiles/H750_S15909.elf.dir/Drivers/STM32H7xx_HAL_Driver/Src/stm32h7xx_hal_tim_ex.c.obj
 .text.HAL_TIMEx_CommutHalfCpltCallback
                0x00000000        0x2 CMakeFiles/H750_S15909.elf.dir/Drivers/STM32H7xx_HAL_Driver/Src/stm32h7xx_hal_tim_ex.c.obj
 .text.TIMEx_DMACommutationHalfCplt
                0x00000000       0x10 CMakeFiles/H750_S15909.elf.dir/Drivers/STM32H7xx_HAL_Driver/Src/stm32h7xx_hal_tim_ex.c.obj
 .text.HAL_TIMEx_BreakCallback
                0x00000000        0x2 CMakeFiles/H750_S15909.elf.dir/Drivers/STM32H7xx_HAL_Driver/Src/stm32h7xx_hal_tim_ex.c.obj
 .text.HAL_TIMEx_Break2Callback
                0x00000000        0x2 CMakeFiles/H750_S15909.elf.dir/Drivers/STM32H7xx_HAL_Driver/Src/stm32h7xx_hal_tim_ex.c.obj
 .text.HAL_TIMEx_HallSensor_GetState
                0x00000000        0x6 CMakeFiles/H750_S15909.elf.dir/Drivers/STM32H7xx_HAL_Driver/Src/stm32h7xx_hal_tim_ex.c.obj
 .text.HAL_TIMEx_GetChannelNState
                0x00000000       0x2a CMakeFiles/H750_S15909.elf.dir/Drivers/STM32H7xx_HAL_Driver/Src/stm32h7xx_hal_tim_ex.c.obj
 .text          0x00000000        0x0 CMakeFiles/H750_S15909.elf.dir/Drivers/STM32H7xx_HAL_Driver/Src/stm32h7xx_hal_uart.c.obj
 .data          0x00000000        0x0 CMakeFiles/H750_S15909.elf.dir/Drivers/STM32H7xx_HAL_Driver/Src/stm32h7xx_hal_uart.c.obj
 .bss           0x00000000        0x0 CMakeFiles/H750_S15909.elf.dir/Drivers/STM32H7xx_HAL_Driver/Src/stm32h7xx_hal_uart.c.obj
 .text.UART_TxISR_8BIT
                0x00000000       0x56 CMakeFiles/H750_S15909.elf.dir/Drivers/STM32H7xx_HAL_Driver/Src/stm32h7xx_hal_uart.c.obj
 .text.UART_TxISR_16BIT
                0x00000000       0x5a CMakeFiles/H750_S15909.elf.dir/Drivers/STM32H7xx_HAL_Driver/Src/stm32h7xx_hal_uart.c.obj
 .text.UART_TxISR_8BIT_FIFOEN
                0x00000000       0x74 CMakeFiles/H750_S15909.elf.dir/Drivers/STM32H7xx_HAL_Driver/Src/stm32h7xx_hal_uart.c.obj
 .text.UART_TxISR_16BIT_FIFOEN
                0x00000000       0x78 CMakeFiles/H750_S15909.elf.dir/Drivers/STM32H7xx_HAL_Driver/Src/stm32h7xx_hal_uart.c.obj
 .text.HAL_UART_MspInit
                0x00000000        0x2 CMakeFiles/H750_S15909.elf.dir/Drivers/STM32H7xx_HAL_Driver/Src/stm32h7xx_hal_uart.c.obj
 .text.HAL_UART_MspDeInit
                0x00000000        0x2 CMakeFiles/H750_S15909.elf.dir/Drivers/STM32H7xx_HAL_Driver/Src/stm32h7xx_hal_uart.c.obj
 .text.HAL_UART_DeInit
                0x00000000       0x42 CMakeFiles/H750_S15909.elf.dir/Drivers/STM32H7xx_HAL_Driver/Src/stm32h7xx_hal_uart.c.obj
 .text.HAL_UART_Transmit_IT
                0x00000000       0xc8 CMakeFiles/H750_S15909.elf.dir/Drivers/STM32H7xx_HAL_Driver/Src/stm32h7xx_hal_uart.c.obj
 .text.HAL_UART_DMAPause
                0x00000000       0xa2 CMakeFiles/H750_S15909.elf.dir/Drivers/STM32H7xx_HAL_Driver/Src/stm32h7xx_hal_uart.c.obj
 .text.HAL_UART_DMAResume
                0x00000000       0x94 CMakeFiles/H750_S15909.elf.dir/Drivers/STM32H7xx_HAL_Driver/Src/stm32h7xx_hal_uart.c.obj
 .text.HAL_UART_Abort
                0x00000000      0x11c CMakeFiles/H750_S15909.elf.dir/Drivers/STM32H7xx_HAL_Driver/Src/stm32h7xx_hal_uart.c.obj
 .text.HAL_UART_AbortTransmit
                0x00000000       0x98 CMakeFiles/H750_S15909.elf.dir/Drivers/STM32H7xx_HAL_Driver/Src/stm32h7xx_hal_uart.c.obj
 .text.HAL_UART_AbortReceive
                0x00000000       0xb4 CMakeFiles/H750_S15909.elf.dir/Drivers/STM32H7xx_HAL_Driver/Src/stm32h7xx_hal_uart.c.obj
 .text.HAL_UART_RxCpltCallback
                0x00000000        0x2 CMakeFiles/H750_S15909.elf.dir/Drivers/STM32H7xx_HAL_Driver/Src/stm32h7xx_hal_uart.c.obj
 .text.HAL_UART_AbortCpltCallback
                0x00000000        0x2 CMakeFiles/H750_S15909.elf.dir/Drivers/STM32H7xx_HAL_Driver/Src/stm32h7xx_hal_uart.c.obj
 .text.HAL_UART_Abort_IT
                0x00000000      0x14c CMakeFiles/H750_S15909.elf.dir/Drivers/STM32H7xx_HAL_Driver/Src/stm32h7xx_hal_uart.c.obj
 .text.UART_DMARxAbortCallback
                0x00000000       0x42 CMakeFiles/H750_S15909.elf.dir/Drivers/STM32H7xx_HAL_Driver/Src/stm32h7xx_hal_uart.c.obj
 .text.UART_DMATxAbortCallback
                0x00000000       0x4e CMakeFiles/H750_S15909.elf.dir/Drivers/STM32H7xx_HAL_Driver/Src/stm32h7xx_hal_uart.c.obj
 .text.HAL_UART_AbortTransmitCpltCallback
                0x00000000        0x2 CMakeFiles/H750_S15909.elf.dir/Drivers/STM32H7xx_HAL_Driver/Src/stm32h7xx_hal_uart.c.obj
 .text.HAL_UART_AbortTransmit_IT
                0x00000000       0xac CMakeFiles/H750_S15909.elf.dir/Drivers/STM32H7xx_HAL_Driver/Src/stm32h7xx_hal_uart.c.obj
 .text.UART_DMATxOnlyAbortCallback
                0x00000000       0x2a CMakeFiles/H750_S15909.elf.dir/Drivers/STM32H7xx_HAL_Driver/Src/stm32h7xx_hal_uart.c.obj
 .text.HAL_UART_AbortReceiveCpltCallback
                0x00000000        0x2 CMakeFiles/H750_S15909.elf.dir/Drivers/STM32H7xx_HAL_Driver/Src/stm32h7xx_hal_uart.c.obj
 .text.HAL_UART_AbortReceive_IT
                0x00000000       0xd0 CMakeFiles/H750_S15909.elf.dir/Drivers/STM32H7xx_HAL_Driver/Src/stm32h7xx_hal_uart.c.obj
 .text.UART_DMARxOnlyAbortCallback
                0x00000000       0x28 CMakeFiles/H750_S15909.elf.dir/Drivers/STM32H7xx_HAL_Driver/Src/stm32h7xx_hal_uart.c.obj
 .text.HAL_UART_ReceiverTimeout_Config
                0x00000000       0x18 CMakeFiles/H750_S15909.elf.dir/Drivers/STM32H7xx_HAL_Driver/Src/stm32h7xx_hal_uart.c.obj
 .text.HAL_UART_EnableReceiverTimeout
                0x00000000       0x4c CMakeFiles/H750_S15909.elf.dir/Drivers/STM32H7xx_HAL_Driver/Src/stm32h7xx_hal_uart.c.obj
 .text.HAL_UART_DisableReceiverTimeout
                0x00000000       0x4c CMakeFiles/H750_S15909.elf.dir/Drivers/STM32H7xx_HAL_Driver/Src/stm32h7xx_hal_uart.c.obj
 .text.HAL_MultiProcessor_EnterMuteMode
                0x00000000        0xc CMakeFiles/H750_S15909.elf.dir/Drivers/STM32H7xx_HAL_Driver/Src/stm32h7xx_hal_uart.c.obj
 .text.HAL_HalfDuplex_EnableTransmitter
                0x00000000       0x4c CMakeFiles/H750_S15909.elf.dir/Drivers/STM32H7xx_HAL_Driver/Src/stm32h7xx_hal_uart.c.obj
 .text.HAL_HalfDuplex_EnableReceiver
                0x00000000       0x4c CMakeFiles/H750_S15909.elf.dir/Drivers/STM32H7xx_HAL_Driver/Src/stm32h7xx_hal_uart.c.obj
 .text.HAL_LIN_SendBreak
                0x00000000       0x32 CMakeFiles/H750_S15909.elf.dir/Drivers/STM32H7xx_HAL_Driver/Src/stm32h7xx_hal_uart.c.obj
 .text.HAL_UART_GetState
                0x00000000        0xc CMakeFiles/H750_S15909.elf.dir/Drivers/STM32H7xx_HAL_Driver/Src/stm32h7xx_hal_uart.c.obj
 .text.HAL_UART_GetError
                0x00000000        0x6 CMakeFiles/H750_S15909.elf.dir/Drivers/STM32H7xx_HAL_Driver/Src/stm32h7xx_hal_uart.c.obj
 .text.HAL_UART_Receive
                0x00000000      0x128 CMakeFiles/H750_S15909.elf.dir/Drivers/STM32H7xx_HAL_Driver/Src/stm32h7xx_hal_uart.c.obj
 .text.HAL_HalfDuplex_Init
                0x00000000       0x72 CMakeFiles/H750_S15909.elf.dir/Drivers/STM32H7xx_HAL_Driver/Src/stm32h7xx_hal_uart.c.obj
 .text.HAL_LIN_Init
                0x00000000       0x96 CMakeFiles/H750_S15909.elf.dir/Drivers/STM32H7xx_HAL_Driver/Src/stm32h7xx_hal_uart.c.obj
 .text.HAL_MultiProcessor_Init
                0x00000000       0x8e CMakeFiles/H750_S15909.elf.dir/Drivers/STM32H7xx_HAL_Driver/Src/stm32h7xx_hal_uart.c.obj
 .text.HAL_MultiProcessor_EnableMuteMode
                0x00000000       0x38 CMakeFiles/H750_S15909.elf.dir/Drivers/STM32H7xx_HAL_Driver/Src/stm32h7xx_hal_uart.c.obj
 .text.HAL_MultiProcessor_DisableMuteMode
                0x00000000       0x38 CMakeFiles/H750_S15909.elf.dir/Drivers/STM32H7xx_HAL_Driver/Src/stm32h7xx_hal_uart.c.obj
 .text          0x00000000        0x0 CMakeFiles/H750_S15909.elf.dir/Drivers/STM32H7xx_HAL_Driver/Src/stm32h7xx_hal_uart_ex.c.obj
 .data          0x00000000        0x0 CMakeFiles/H750_S15909.elf.dir/Drivers/STM32H7xx_HAL_Driver/Src/stm32h7xx_hal_uart_ex.c.obj
 .bss           0x00000000        0x0 CMakeFiles/H750_S15909.elf.dir/Drivers/STM32H7xx_HAL_Driver/Src/stm32h7xx_hal_uart_ex.c.obj
 .text.UARTEx_Wakeup_AddressConfig
                0x00000000       0x2e CMakeFiles/H750_S15909.elf.dir/Drivers/STM32H7xx_HAL_Driver/Src/stm32h7xx_hal_uart_ex.c.obj
 .text.HAL_RS485Ex_Init
                0x00000000       0x88 CMakeFiles/H750_S15909.elf.dir/Drivers/STM32H7xx_HAL_Driver/Src/stm32h7xx_hal_uart_ex.c.obj
 .text.HAL_MultiProcessorEx_AddressLength_Set
                0x00000000       0x38 CMakeFiles/H750_S15909.elf.dir/Drivers/STM32H7xx_HAL_Driver/Src/stm32h7xx_hal_uart_ex.c.obj
 .text.HAL_UARTEx_StopModeWakeUpSourceConfig
                0x00000000       0x82 CMakeFiles/H750_S15909.elf.dir/Drivers/STM32H7xx_HAL_Driver/Src/stm32h7xx_hal_uart_ex.c.obj
 .text.HAL_UARTEx_EnableStopMode
                0x00000000       0x2e CMakeFiles/H750_S15909.elf.dir/Drivers/STM32H7xx_HAL_Driver/Src/stm32h7xx_hal_uart_ex.c.obj
 .text.HAL_UARTEx_DisableStopMode
                0x00000000       0x2e CMakeFiles/H750_S15909.elf.dir/Drivers/STM32H7xx_HAL_Driver/Src/stm32h7xx_hal_uart_ex.c.obj
 .text.HAL_UARTEx_EnableFifoMode
                0x00000000       0x48 CMakeFiles/H750_S15909.elf.dir/Drivers/STM32H7xx_HAL_Driver/Src/stm32h7xx_hal_uart_ex.c.obj
 .text.HAL_UARTEx_ReceiveToIdle
                0x00000000      0x170 CMakeFiles/H750_S15909.elf.dir/Drivers/STM32H7xx_HAL_Driver/Src/stm32h7xx_hal_uart_ex.c.obj
 .text.HAL_UARTEx_ReceiveToIdle_IT
                0x00000000       0x5a CMakeFiles/H750_S15909.elf.dir/Drivers/STM32H7xx_HAL_Driver/Src/stm32h7xx_hal_uart_ex.c.obj
 .text.HAL_UARTEx_ReceiveToIdle_DMA
                0x00000000       0x5a CMakeFiles/H750_S15909.elf.dir/Drivers/STM32H7xx_HAL_Driver/Src/stm32h7xx_hal_uart_ex.c.obj
 .text          0x00000000      0x254 d:/lijie_tools/clion_cubemx/gcc-arm-none-eabi-10.3-2021.10/bin/../lib/gcc/arm-none-eabi/10.3.1/thumb/v7e-m/nofp\libgcc.a(_arm_muldf3.o)
 .data          0x00000000        0x0 d:/lijie_tools/clion_cubemx/gcc-arm-none-eabi-10.3-2021.10/bin/../lib/gcc/arm-none-eabi/10.3.1/thumb/v7e-m/nofp\libgcc.a(_arm_muldf3.o)
 .bss           0x00000000        0x0 d:/lijie_tools/clion_cubemx/gcc-arm-none-eabi-10.3-2021.10/bin/../lib/gcc/arm-none-eabi/10.3.1/thumb/v7e-m/nofp\libgcc.a(_arm_muldf3.o)
 .debug_frame   0x00000000       0x30 d:/lijie_tools/clion_cubemx/gcc-arm-none-eabi-10.3-2021.10/bin/../lib/gcc/arm-none-eabi/10.3.1/thumb/v7e-m/nofp\libgcc.a(_arm_muldf3.o)
 .ARM.attributes
                0x00000000       0x1e d:/lijie_tools/clion_cubemx/gcc-arm-none-eabi-10.3-2021.10/bin/../lib/gcc/arm-none-eabi/10.3.1/thumb/v7e-m/nofp\libgcc.a(_arm_muldf3.o)
 .text          0x00000000      0x168 d:/lijie_tools/clion_cubemx/gcc-arm-none-eabi-10.3-2021.10/bin/../lib/gcc/arm-none-eabi/10.3.1/thumb/v7e-m/nofp\libgcc.a(_arm_mulsf3.o)
 .data          0x00000000        0x0 d:/lijie_tools/clion_cubemx/gcc-arm-none-eabi-10.3-2021.10/bin/../lib/gcc/arm-none-eabi/10.3.1/thumb/v7e-m/nofp\libgcc.a(_arm_mulsf3.o)
 .bss           0x00000000        0x0 d:/lijie_tools/clion_cubemx/gcc-arm-none-eabi-10.3-2021.10/bin/../lib/gcc/arm-none-eabi/10.3.1/thumb/v7e-m/nofp\libgcc.a(_arm_mulsf3.o)
 .debug_frame   0x00000000       0x24 d:/lijie_tools/clion_cubemx/gcc-arm-none-eabi-10.3-2021.10/bin/../lib/gcc/arm-none-eabi/10.3.1/thumb/v7e-m/nofp\libgcc.a(_arm_mulsf3.o)
 .ARM.attributes
                0x00000000       0x1e d:/lijie_tools/clion_cubemx/gcc-arm-none-eabi-10.3-2021.10/bin/../lib/gcc/arm-none-eabi/10.3.1/thumb/v7e-m/nofp\libgcc.a(_arm_mulsf3.o)
 .data          0x00000000        0x0 d:/lijie_tools/clion_cubemx/gcc-arm-none-eabi-10.3-2021.10/bin/../lib/gcc/arm-none-eabi/10.3.1/thumb/v7e-m/nofp\libgcc.a(_arm_addsubdf3.o)
 .bss           0x00000000        0x0 d:/lijie_tools/clion_cubemx/gcc-arm-none-eabi-10.3-2021.10/bin/../lib/gcc/arm-none-eabi/10.3.1/thumb/v7e-m/nofp\libgcc.a(_arm_addsubdf3.o)
 .data          0x00000000        0x0 d:/lijie_tools/clion_cubemx/gcc-arm-none-eabi-10.3-2021.10/bin/../lib/gcc/arm-none-eabi/10.3.1/thumb/v7e-m/nofp\libgcc.a(_arm_muldivdf3.o)
 .bss           0x00000000        0x0 d:/lijie_tools/clion_cubemx/gcc-arm-none-eabi-10.3-2021.10/bin/../lib/gcc/arm-none-eabi/10.3.1/thumb/v7e-m/nofp\libgcc.a(_arm_muldivdf3.o)
 .data          0x00000000        0x0 d:/lijie_tools/clion_cubemx/gcc-arm-none-eabi-10.3-2021.10/bin/../lib/gcc/arm-none-eabi/10.3.1/thumb/v7e-m/nofp\libgcc.a(_arm_cmpdf2.o)
 .bss           0x00000000        0x0 d:/lijie_tools/clion_cubemx/gcc-arm-none-eabi-10.3-2021.10/bin/../lib/gcc/arm-none-eabi/10.3.1/thumb/v7e-m/nofp\libgcc.a(_arm_cmpdf2.o)
 .data          0x00000000        0x0 d:/lijie_tools/clion_cubemx/gcc-arm-none-eabi-10.3-2021.10/bin/../lib/gcc/arm-none-eabi/10.3.1/thumb/v7e-m/nofp\libgcc.a(_arm_fixdfsi.o)
 .bss           0x00000000        0x0 d:/lijie_tools/clion_cubemx/gcc-arm-none-eabi-10.3-2021.10/bin/../lib/gcc/arm-none-eabi/10.3.1/thumb/v7e-m/nofp\libgcc.a(_arm_fixdfsi.o)
 .data          0x00000000        0x0 d:/lijie_tools/clion_cubemx/gcc-arm-none-eabi-10.3-2021.10/bin/../lib/gcc/arm-none-eabi/10.3.1/thumb/v7e-m/nofp\libgcc.a(_arm_fixunsdfsi.o)
 .bss           0x00000000        0x0 d:/lijie_tools/clion_cubemx/gcc-arm-none-eabi-10.3-2021.10/bin/../lib/gcc/arm-none-eabi/10.3.1/thumb/v7e-m/nofp\libgcc.a(_arm_fixunsdfsi.o)
 .data          0x00000000        0x0 d:/lijie_tools/clion_cubemx/gcc-arm-none-eabi-10.3-2021.10/bin/../lib/gcc/arm-none-eabi/10.3.1/thumb/v7e-m/nofp\libgcc.a(_arm_truncdfsf2.o)
 .bss           0x00000000        0x0 d:/lijie_tools/clion_cubemx/gcc-arm-none-eabi-10.3-2021.10/bin/../lib/gcc/arm-none-eabi/10.3.1/thumb/v7e-m/nofp\libgcc.a(_arm_truncdfsf2.o)
 .data          0x00000000        0x0 d:/lijie_tools/clion_cubemx/gcc-arm-none-eabi-10.3-2021.10/bin/../lib/gcc/arm-none-eabi/10.3.1/thumb/v7e-m/nofp\libgcc.a(_arm_addsubsf3.o)
 .bss           0x00000000        0x0 d:/lijie_tools/clion_cubemx/gcc-arm-none-eabi-10.3-2021.10/bin/../lib/gcc/arm-none-eabi/10.3.1/thumb/v7e-m/nofp\libgcc.a(_arm_addsubsf3.o)
 .data          0x00000000        0x0 d:/lijie_tools/clion_cubemx/gcc-arm-none-eabi-10.3-2021.10/bin/../lib/gcc/arm-none-eabi/10.3.1/thumb/v7e-m/nofp\libgcc.a(_arm_muldivsf3.o)
 .bss           0x00000000        0x0 d:/lijie_tools/clion_cubemx/gcc-arm-none-eabi-10.3-2021.10/bin/../lib/gcc/arm-none-eabi/10.3.1/thumb/v7e-m/nofp\libgcc.a(_arm_muldivsf3.o)
 .data          0x00000000        0x0 d:/lijie_tools/clion_cubemx/gcc-arm-none-eabi-10.3-2021.10/bin/../lib/gcc/arm-none-eabi/10.3.1/thumb/v7e-m/nofp\libgcc.a(_arm_fixunssfsi.o)
 .bss           0x00000000        0x0 d:/lijie_tools/clion_cubemx/gcc-arm-none-eabi-10.3-2021.10/bin/../lib/gcc/arm-none-eabi/10.3.1/thumb/v7e-m/nofp\libgcc.a(_arm_fixunssfsi.o)
 .data          0x00000000        0x0 d:/lijie_tools/clion_cubemx/gcc-arm-none-eabi-10.3-2021.10/bin/../lib/gcc/arm-none-eabi/10.3.1/thumb/v7e-m/nofp\libgcc.a(_aeabi_uldivmod.o)
 .bss           0x00000000        0x0 d:/lijie_tools/clion_cubemx/gcc-arm-none-eabi-10.3-2021.10/bin/../lib/gcc/arm-none-eabi/10.3.1/thumb/v7e-m/nofp\libgcc.a(_aeabi_uldivmod.o)
 .data          0x00000000        0x0 d:/lijie_tools/clion_cubemx/gcc-arm-none-eabi-10.3-2021.10/bin/../lib/gcc/arm-none-eabi/10.3.1/thumb/v7e-m/nofp\libgcc.a(_udivmoddi4.o)
 .bss           0x00000000        0x0 d:/lijie_tools/clion_cubemx/gcc-arm-none-eabi-10.3-2021.10/bin/../lib/gcc/arm-none-eabi/10.3.1/thumb/v7e-m/nofp\libgcc.a(_udivmoddi4.o)
 .ARM.extab     0x00000000        0x0 d:/lijie_tools/clion_cubemx/gcc-arm-none-eabi-10.3-2021.10/bin/../lib/gcc/arm-none-eabi/10.3.1/thumb/v7e-m/nofp\libgcc.a(_udivmoddi4.o)
 .data          0x00000000        0x0 d:/lijie_tools/clion_cubemx/gcc-arm-none-eabi-10.3-2021.10/bin/../lib/gcc/arm-none-eabi/10.3.1/thumb/v7e-m/nofp\libgcc.a(_dvmd_tls.o)
 .bss           0x00000000        0x0 d:/lijie_tools/clion_cubemx/gcc-arm-none-eabi-10.3-2021.10/bin/../lib/gcc/arm-none-eabi/10.3.1/thumb/v7e-m/nofp\libgcc.a(_dvmd_tls.o)
 .text          0x00000000        0x0 d:/lijie_tools/clion_cubemx/gcc-arm-none-eabi-10.3-2021.10/bin/../lib/gcc/arm-none-eabi/10.3.1/../../../../arm-none-eabi/lib/thumb/v7e-m/nofp\libg.a(lib_a-errno.o)
 .data          0x00000000        0x0 d:/lijie_tools/clion_cubemx/gcc-arm-none-eabi-10.3-2021.10/bin/../lib/gcc/arm-none-eabi/10.3.1/../../../../arm-none-eabi/lib/thumb/v7e-m/nofp\libg.a(lib_a-errno.o)
 .bss           0x00000000        0x0 d:/lijie_tools/clion_cubemx/gcc-arm-none-eabi-10.3-2021.10/bin/../lib/gcc/arm-none-eabi/10.3.1/../../../../arm-none-eabi/lib/thumb/v7e-m/nofp\libg.a(lib_a-errno.o)
 .text          0x00000000        0x0 d:/lijie_tools/clion_cubemx/gcc-arm-none-eabi-10.3-2021.10/bin/../lib/gcc/arm-none-eabi/10.3.1/../../../../arm-none-eabi/lib/thumb/v7e-m/nofp\libg.a(lib_a-exit.o)
 .data          0x00000000        0x0 d:/lijie_tools/clion_cubemx/gcc-arm-none-eabi-10.3-2021.10/bin/../lib/gcc/arm-none-eabi/10.3.1/../../../../arm-none-eabi/lib/thumb/v7e-m/nofp\libg.a(lib_a-exit.o)
 .bss           0x00000000        0x0 d:/lijie_tools/clion_cubemx/gcc-arm-none-eabi-10.3-2021.10/bin/../lib/gcc/arm-none-eabi/10.3.1/../../../../arm-none-eabi/lib/thumb/v7e-m/nofp\libg.a(lib_a-exit.o)
 .text.exit     0x00000000       0x20 d:/lijie_tools/clion_cubemx/gcc-arm-none-eabi-10.3-2021.10/bin/../lib/gcc/arm-none-eabi/10.3.1/../../../../arm-none-eabi/lib/thumb/v7e-m/nofp\libg.a(lib_a-exit.o)
 .debug_frame   0x00000000       0x28 d:/lijie_tools/clion_cubemx/gcc-arm-none-eabi-10.3-2021.10/bin/../lib/gcc/arm-none-eabi/10.3.1/../../../../arm-none-eabi/lib/thumb/v7e-m/nofp\libg.a(lib_a-exit.o)
 .ARM.attributes
                0x00000000       0x2e d:/lijie_tools/clion_cubemx/gcc-arm-none-eabi-10.3-2021.10/bin/../lib/gcc/arm-none-eabi/10.3.1/../../../../arm-none-eabi/lib/thumb/v7e-m/nofp\libg.a(lib_a-exit.o)
 .text          0x00000000        0x0 d:/lijie_tools/clion_cubemx/gcc-arm-none-eabi-10.3-2021.10/bin/../lib/gcc/arm-none-eabi/10.3.1/../../../../arm-none-eabi/lib/thumb/v7e-m/nofp\libg.a(lib_a-impure.o)
 .data          0x00000000        0x0 d:/lijie_tools/clion_cubemx/gcc-arm-none-eabi-10.3-2021.10/bin/../lib/gcc/arm-none-eabi/10.3.1/../../../../arm-none-eabi/lib/thumb/v7e-m/nofp\libg.a(lib_a-impure.o)
 .bss           0x00000000        0x0 d:/lijie_tools/clion_cubemx/gcc-arm-none-eabi-10.3-2021.10/bin/../lib/gcc/arm-none-eabi/10.3.1/../../../../arm-none-eabi/lib/thumb/v7e-m/nofp\libg.a(lib_a-impure.o)
 .text          0x00000000        0x0 d:/lijie_tools/clion_cubemx/gcc-arm-none-eabi-10.3-2021.10/bin/../lib/gcc/arm-none-eabi/10.3.1/../../../../arm-none-eabi/lib/thumb/v7e-m/nofp\libg.a(lib_a-init.o)
 .data          0x00000000        0x0 d:/lijie_tools/clion_cubemx/gcc-arm-none-eabi-10.3-2021.10/bin/../lib/gcc/arm-none-eabi/10.3.1/../../../../arm-none-eabi/lib/thumb/v7e-m/nofp\libg.a(lib_a-init.o)
 .bss           0x00000000        0x0 d:/lijie_tools/clion_cubemx/gcc-arm-none-eabi-10.3-2021.10/bin/../lib/gcc/arm-none-eabi/10.3.1/../../../../arm-none-eabi/lib/thumb/v7e-m/nofp\libg.a(lib_a-init.o)
 .data          0x00000000        0x0 d:/lijie_tools/clion_cubemx/gcc-arm-none-eabi-10.3-2021.10/bin/../lib/gcc/arm-none-eabi/10.3.1/../../../../arm-none-eabi/lib/thumb/v7e-m/nofp\libg.a(lib_a-memcpy.o)
 .bss           0x00000000        0x0 d:/lijie_tools/clion_cubemx/gcc-arm-none-eabi-10.3-2021.10/bin/../lib/gcc/arm-none-eabi/10.3.1/../../../../arm-none-eabi/lib/thumb/v7e-m/nofp\libg.a(lib_a-memcpy.o)
 .text          0x00000000        0x0 d:/lijie_tools/clion_cubemx/gcc-arm-none-eabi-10.3-2021.10/bin/../lib/gcc/arm-none-eabi/10.3.1/../../../../arm-none-eabi/lib/thumb/v7e-m/nofp\libg.a(lib_a-memset.o)
 .data          0x00000000        0x0 d:/lijie_tools/clion_cubemx/gcc-arm-none-eabi-10.3-2021.10/bin/../lib/gcc/arm-none-eabi/10.3.1/../../../../arm-none-eabi/lib/thumb/v7e-m/nofp\libg.a(lib_a-memset.o)
 .bss           0x00000000        0x0 d:/lijie_tools/clion_cubemx/gcc-arm-none-eabi-10.3-2021.10/bin/../lib/gcc/arm-none-eabi/10.3.1/../../../../arm-none-eabi/lib/thumb/v7e-m/nofp\libg.a(lib_a-memset.o)
 .text          0x00000000        0x0 d:/lijie_tools/clion_cubemx/gcc-arm-none-eabi-10.3-2021.10/bin/../lib/gcc/arm-none-eabi/10.3.1/../../../../arm-none-eabi/lib/thumb/v7e-m/nofp\libg.a(lib_a-setvbuf.o)
 .data          0x00000000        0x0 d:/lijie_tools/clion_cubemx/gcc-arm-none-eabi-10.3-2021.10/bin/../lib/gcc/arm-none-eabi/10.3.1/../../../../arm-none-eabi/lib/thumb/v7e-m/nofp\libg.a(lib_a-setvbuf.o)
 .bss           0x00000000        0x0 d:/lijie_tools/clion_cubemx/gcc-arm-none-eabi-10.3-2021.10/bin/../lib/gcc/arm-none-eabi/10.3.1/../../../../arm-none-eabi/lib/thumb/v7e-m/nofp\libg.a(lib_a-setvbuf.o)
 .text          0x00000000        0x0 d:/lijie_tools/clion_cubemx/gcc-arm-none-eabi-10.3-2021.10/bin/../lib/gcc/arm-none-eabi/10.3.1/../../../../arm-none-eabi/lib/thumb/v7e-m/nofp\libg.a(lib_a-__call_atexit.o)
 .data          0x00000000        0x0 d:/lijie_tools/clion_cubemx/gcc-arm-none-eabi-10.3-2021.10/bin/../lib/gcc/arm-none-eabi/10.3.1/../../../../arm-none-eabi/lib/thumb/v7e-m/nofp\libg.a(lib_a-__call_atexit.o)
 .bss           0x00000000        0x0 d:/lijie_tools/clion_cubemx/gcc-arm-none-eabi-10.3-2021.10/bin/../lib/gcc/arm-none-eabi/10.3.1/../../../../arm-none-eabi/lib/thumb/v7e-m/nofp\libg.a(lib_a-__call_atexit.o)
 .text.__call_exitprocs
                0x00000000       0xc4 d:/lijie_tools/clion_cubemx/gcc-arm-none-eabi-10.3-2021.10/bin/../lib/gcc/arm-none-eabi/10.3.1/../../../../arm-none-eabi/lib/thumb/v7e-m/nofp\libg.a(lib_a-__call_atexit.o)
 .text          0x00000000        0x0 d:/lijie_tools/clion_cubemx/gcc-arm-none-eabi-10.3-2021.10/bin/../lib/gcc/arm-none-eabi/10.3.1/../../../../arm-none-eabi/lib/thumb/v7e-m/nofp\libg.a(lib_a-atexit.o)
 .data          0x00000000        0x0 d:/lijie_tools/clion_cubemx/gcc-arm-none-eabi-10.3-2021.10/bin/../lib/gcc/arm-none-eabi/10.3.1/../../../../arm-none-eabi/lib/thumb/v7e-m/nofp\libg.a(lib_a-atexit.o)
 .bss           0x00000000        0x0 d:/lijie_tools/clion_cubemx/gcc-arm-none-eabi-10.3-2021.10/bin/../lib/gcc/arm-none-eabi/10.3.1/../../../../arm-none-eabi/lib/thumb/v7e-m/nofp\libg.a(lib_a-atexit.o)
 .text          0x00000000        0x0 d:/lijie_tools/clion_cubemx/gcc-arm-none-eabi-10.3-2021.10/bin/../lib/gcc/arm-none-eabi/10.3.1/../../../../arm-none-eabi/lib/thumb/v7e-m/nofp\libg.a(lib_a-fflush.o)
 .data          0x00000000        0x0 d:/lijie_tools/clion_cubemx/gcc-arm-none-eabi-10.3-2021.10/bin/../lib/gcc/arm-none-eabi/10.3.1/../../../../arm-none-eabi/lib/thumb/v7e-m/nofp\libg.a(lib_a-fflush.o)
 .bss           0x00000000        0x0 d:/lijie_tools/clion_cubemx/gcc-arm-none-eabi-10.3-2021.10/bin/../lib/gcc/arm-none-eabi/10.3.1/../../../../arm-none-eabi/lib/thumb/v7e-m/nofp\libg.a(lib_a-fflush.o)
 .text.fflush   0x00000000       0x74 d:/lijie_tools/clion_cubemx/gcc-arm-none-eabi-10.3-2021.10/bin/../lib/gcc/arm-none-eabi/10.3.1/../../../../arm-none-eabi/lib/thumb/v7e-m/nofp\libg.a(lib_a-fflush.o)
 .text          0x00000000        0x0 d:/lijie_tools/clion_cubemx/gcc-arm-none-eabi-10.3-2021.10/bin/../lib/gcc/arm-none-eabi/10.3.1/../../../../arm-none-eabi/lib/thumb/v7e-m/nofp\libg.a(lib_a-findfp.o)
 .data          0x00000000        0x0 d:/lijie_tools/clion_cubemx/gcc-arm-none-eabi-10.3-2021.10/bin/../lib/gcc/arm-none-eabi/10.3.1/../../../../arm-none-eabi/lib/thumb/v7e-m/nofp\libg.a(lib_a-findfp.o)
 .bss           0x00000000        0x0 d:/lijie_tools/clion_cubemx/gcc-arm-none-eabi-10.3-2021.10/bin/../lib/gcc/arm-none-eabi/10.3.1/../../../../arm-none-eabi/lib/thumb/v7e-m/nofp\libg.a(lib_a-findfp.o)
 .text.__fp_lock
                0x00000000       0x1c d:/lijie_tools/clion_cubemx/gcc-arm-none-eabi-10.3-2021.10/bin/../lib/gcc/arm-none-eabi/10.3.1/../../../../arm-none-eabi/lib/thumb/v7e-m/nofp\libg.a(lib_a-findfp.o)
 .text.__fp_unlock
                0x00000000       0x1c d:/lijie_tools/clion_cubemx/gcc-arm-none-eabi-10.3-2021.10/bin/../lib/gcc/arm-none-eabi/10.3.1/../../../../arm-none-eabi/lib/thumb/v7e-m/nofp\libg.a(lib_a-findfp.o)
 .text.__sfmoreglue
                0x00000000       0x30 d:/lijie_tools/clion_cubemx/gcc-arm-none-eabi-10.3-2021.10/bin/../lib/gcc/arm-none-eabi/10.3.1/../../../../arm-none-eabi/lib/thumb/v7e-m/nofp\libg.a(lib_a-findfp.o)
 .text._cleanup
                0x00000000       0x14 d:/lijie_tools/clion_cubemx/gcc-arm-none-eabi-10.3-2021.10/bin/../lib/gcc/arm-none-eabi/10.3.1/../../../../arm-none-eabi/lib/thumb/v7e-m/nofp\libg.a(lib_a-findfp.o)
 .text.__sfp    0x00000000       0xc8 d:/lijie_tools/clion_cubemx/gcc-arm-none-eabi-10.3-2021.10/bin/../lib/gcc/arm-none-eabi/10.3.1/../../../../arm-none-eabi/lib/thumb/v7e-m/nofp\libg.a(lib_a-findfp.o)
 .text.__sinit_lock_acquire
                0x00000000        0xc d:/lijie_tools/clion_cubemx/gcc-arm-none-eabi-10.3-2021.10/bin/../lib/gcc/arm-none-eabi/10.3.1/../../../../arm-none-eabi/lib/thumb/v7e-m/nofp\libg.a(lib_a-findfp.o)
 .text.__sinit_lock_release
                0x00000000        0xc d:/lijie_tools/clion_cubemx/gcc-arm-none-eabi-10.3-2021.10/bin/../lib/gcc/arm-none-eabi/10.3.1/../../../../arm-none-eabi/lib/thumb/v7e-m/nofp\libg.a(lib_a-findfp.o)
 .text.__fp_lock_all
                0x00000000       0x24 d:/lijie_tools/clion_cubemx/gcc-arm-none-eabi-10.3-2021.10/bin/../lib/gcc/arm-none-eabi/10.3.1/../../../../arm-none-eabi/lib/thumb/v7e-m/nofp\libg.a(lib_a-findfp.o)
 .text.__fp_unlock_all
                0x00000000       0x24 d:/lijie_tools/clion_cubemx/gcc-arm-none-eabi-10.3-2021.10/bin/../lib/gcc/arm-none-eabi/10.3.1/../../../../arm-none-eabi/lib/thumb/v7e-m/nofp\libg.a(lib_a-findfp.o)
 .text          0x00000000        0x0 d:/lijie_tools/clion_cubemx/gcc-arm-none-eabi-10.3-2021.10/bin/../lib/gcc/arm-none-eabi/10.3.1/../../../../arm-none-eabi/lib/thumb/v7e-m/nofp\libg.a(lib_a-fini.o)
 .data          0x00000000        0x0 d:/lijie_tools/clion_cubemx/gcc-arm-none-eabi-10.3-2021.10/bin/../lib/gcc/arm-none-eabi/10.3.1/../../../../arm-none-eabi/lib/thumb/v7e-m/nofp\libg.a(lib_a-fini.o)
 .bss           0x00000000        0x0 d:/lijie_tools/clion_cubemx/gcc-arm-none-eabi-10.3-2021.10/bin/../lib/gcc/arm-none-eabi/10.3.1/../../../../arm-none-eabi/lib/thumb/v7e-m/nofp\libg.a(lib_a-fini.o)
 .text          0x00000000        0x0 d:/lijie_tools/clion_cubemx/gcc-arm-none-eabi-10.3-2021.10/bin/../lib/gcc/arm-none-eabi/10.3.1/../../../../arm-none-eabi/lib/thumb/v7e-m/nofp\libg.a(lib_a-freer.o)
 .data          0x00000000        0x0 d:/lijie_tools/clion_cubemx/gcc-arm-none-eabi-10.3-2021.10/bin/../lib/gcc/arm-none-eabi/10.3.1/../../../../arm-none-eabi/lib/thumb/v7e-m/nofp\libg.a(lib_a-freer.o)
 .bss           0x00000000        0x0 d:/lijie_tools/clion_cubemx/gcc-arm-none-eabi-10.3-2021.10/bin/../lib/gcc/arm-none-eabi/10.3.1/../../../../arm-none-eabi/lib/thumb/v7e-m/nofp\libg.a(lib_a-freer.o)
 .text          0x00000000        0x0 d:/lijie_tools/clion_cubemx/gcc-arm-none-eabi-10.3-2021.10/bin/../lib/gcc/arm-none-eabi/10.3.1/../../../../arm-none-eabi/lib/thumb/v7e-m/nofp\libg.a(lib_a-fwalk.o)
 .data          0x00000000        0x0 d:/lijie_tools/clion_cubemx/gcc-arm-none-eabi-10.3-2021.10/bin/../lib/gcc/arm-none-eabi/10.3.1/../../../../arm-none-eabi/lib/thumb/v7e-m/nofp\libg.a(lib_a-fwalk.o)
 .bss           0x00000000        0x0 d:/lijie_tools/clion_cubemx/gcc-arm-none-eabi-10.3-2021.10/bin/../lib/gcc/arm-none-eabi/10.3.1/../../../../arm-none-eabi/lib/thumb/v7e-m/nofp\libg.a(lib_a-fwalk.o)
 .text._fwalk   0x00000000       0x40 d:/lijie_tools/clion_cubemx/gcc-arm-none-eabi-10.3-2021.10/bin/../lib/gcc/arm-none-eabi/10.3.1/../../../../arm-none-eabi/lib/thumb/v7e-m/nofp\libg.a(lib_a-fwalk.o)
 .text          0x00000000        0x0 d:/lijie_tools/clion_cubemx/gcc-arm-none-eabi-10.3-2021.10/bin/../lib/gcc/arm-none-eabi/10.3.1/../../../../arm-none-eabi/lib/thumb/v7e-m/nofp\libg.a(lib_a-lock.o)
 .data          0x00000000        0x0 d:/lijie_tools/clion_cubemx/gcc-arm-none-eabi-10.3-2021.10/bin/../lib/gcc/arm-none-eabi/10.3.1/../../../../arm-none-eabi/lib/thumb/v7e-m/nofp\libg.a(lib_a-lock.o)
 .bss           0x00000000        0x0 d:/lijie_tools/clion_cubemx/gcc-arm-none-eabi-10.3-2021.10/bin/../lib/gcc/arm-none-eabi/10.3.1/../../../../arm-none-eabi/lib/thumb/v7e-m/nofp\libg.a(lib_a-lock.o)
 .text.__retarget_lock_init
                0x00000000        0x4 d:/lijie_tools/clion_cubemx/gcc-arm-none-eabi-10.3-2021.10/bin/../lib/gcc/arm-none-eabi/10.3.1/../../../../arm-none-eabi/lib/thumb/v7e-m/nofp\libg.a(lib_a-lock.o)
 .text.__retarget_lock_close
                0x00000000        0x4 d:/lijie_tools/clion_cubemx/gcc-arm-none-eabi-10.3-2021.10/bin/../lib/gcc/arm-none-eabi/10.3.1/../../../../arm-none-eabi/lib/thumb/v7e-m/nofp\libg.a(lib_a-lock.o)
 .text.__retarget_lock_acquire
                0x00000000        0x4 d:/lijie_tools/clion_cubemx/gcc-arm-none-eabi-10.3-2021.10/bin/../lib/gcc/arm-none-eabi/10.3.1/../../../../arm-none-eabi/lib/thumb/v7e-m/nofp\libg.a(lib_a-lock.o)
 .text.__retarget_lock_try_acquire
                0x00000000        0x4 d:/lijie_tools/clion_cubemx/gcc-arm-none-eabi-10.3-2021.10/bin/../lib/gcc/arm-none-eabi/10.3.1/../../../../arm-none-eabi/lib/thumb/v7e-m/nofp\libg.a(lib_a-lock.o)
 .text.__retarget_lock_try_acquire_recursive
                0x00000000        0x4 d:/lijie_tools/clion_cubemx/gcc-arm-none-eabi-10.3-2021.10/bin/../lib/gcc/arm-none-eabi/10.3.1/../../../../arm-none-eabi/lib/thumb/v7e-m/nofp\libg.a(lib_a-lock.o)
 .text.__retarget_lock_release
                0x00000000        0x4 d:/lijie_tools/clion_cubemx/gcc-arm-none-eabi-10.3-2021.10/bin/../lib/gcc/arm-none-eabi/10.3.1/../../../../arm-none-eabi/lib/thumb/v7e-m/nofp\libg.a(lib_a-lock.o)
 .bss.__lock___arc4random_mutex
                0x00000000        0x1 d:/lijie_tools/clion_cubemx/gcc-arm-none-eabi-10.3-2021.10/bin/../lib/gcc/arm-none-eabi/10.3.1/../../../../arm-none-eabi/lib/thumb/v7e-m/nofp\libg.a(lib_a-lock.o)
 .bss.__lock___at_quick_exit_mutex
                0x00000000        0x1 d:/lijie_tools/clion_cubemx/gcc-arm-none-eabi-10.3-2021.10/bin/../lib/gcc/arm-none-eabi/10.3.1/../../../../arm-none-eabi/lib/thumb/v7e-m/nofp\libg.a(lib_a-lock.o)
 .bss.__lock___dd_hash_mutex
                0x00000000        0x1 d:/lijie_tools/clion_cubemx/gcc-arm-none-eabi-10.3-2021.10/bin/../lib/gcc/arm-none-eabi/10.3.1/../../../../arm-none-eabi/lib/thumb/v7e-m/nofp\libg.a(lib_a-lock.o)
 .bss.__lock___env_recursive_mutex
                0x00000000        0x1 d:/lijie_tools/clion_cubemx/gcc-arm-none-eabi-10.3-2021.10/bin/../lib/gcc/arm-none-eabi/10.3.1/../../../../arm-none-eabi/lib/thumb/v7e-m/nofp\libg.a(lib_a-lock.o)
 .bss.__lock___tz_mutex
                0x00000000        0x1 d:/lijie_tools/clion_cubemx/gcc-arm-none-eabi-10.3-2021.10/bin/../lib/gcc/arm-none-eabi/10.3.1/../../../../arm-none-eabi/lib/thumb/v7e-m/nofp\libg.a(lib_a-lock.o)
 .text          0x00000000        0x0 d:/lijie_tools/clion_cubemx/gcc-arm-none-eabi-10.3-2021.10/bin/../lib/gcc/arm-none-eabi/10.3.1/../../../../arm-none-eabi/lib/thumb/v7e-m/nofp\libg.a(lib_a-makebuf.o)
 .data          0x00000000        0x0 d:/lijie_tools/clion_cubemx/gcc-arm-none-eabi-10.3-2021.10/bin/../lib/gcc/arm-none-eabi/10.3.1/../../../../arm-none-eabi/lib/thumb/v7e-m/nofp\libg.a(lib_a-makebuf.o)
 .bss           0x00000000        0x0 d:/lijie_tools/clion_cubemx/gcc-arm-none-eabi-10.3-2021.10/bin/../lib/gcc/arm-none-eabi/10.3.1/../../../../arm-none-eabi/lib/thumb/v7e-m/nofp\libg.a(lib_a-makebuf.o)
 .text.__smakebuf_r
                0x00000000       0xe0 d:/lijie_tools/clion_cubemx/gcc-arm-none-eabi-10.3-2021.10/bin/../lib/gcc/arm-none-eabi/10.3.1/../../../../arm-none-eabi/lib/thumb/v7e-m/nofp\libg.a(lib_a-makebuf.o)
 .text          0x00000000        0x0 d:/lijie_tools/clion_cubemx/gcc-arm-none-eabi-10.3-2021.10/bin/../lib/gcc/arm-none-eabi/10.3.1/../../../../arm-none-eabi/lib/thumb/v7e-m/nofp\libg.a(lib_a-malloc.o)
 .data          0x00000000        0x0 d:/lijie_tools/clion_cubemx/gcc-arm-none-eabi-10.3-2021.10/bin/../lib/gcc/arm-none-eabi/10.3.1/../../../../arm-none-eabi/lib/thumb/v7e-m/nofp\libg.a(lib_a-malloc.o)
 .bss           0x00000000        0x0 d:/lijie_tools/clion_cubemx/gcc-arm-none-eabi-10.3-2021.10/bin/../lib/gcc/arm-none-eabi/10.3.1/../../../../arm-none-eabi/lib/thumb/v7e-m/nofp\libg.a(lib_a-malloc.o)
 .text.free     0x00000000       0x10 d:/lijie_tools/clion_cubemx/gcc-arm-none-eabi-10.3-2021.10/bin/../lib/gcc/arm-none-eabi/10.3.1/../../../../arm-none-eabi/lib/thumb/v7e-m/nofp\libg.a(lib_a-malloc.o)
 .text          0x00000000        0x0 d:/lijie_tools/clion_cubemx/gcc-arm-none-eabi-10.3-2021.10/bin/../lib/gcc/arm-none-eabi/10.3.1/../../../../arm-none-eabi/lib/thumb/v7e-m/nofp\libg.a(lib_a-mallocr.o)
 .data          0x00000000        0x0 d:/lijie_tools/clion_cubemx/gcc-arm-none-eabi-10.3-2021.10/bin/../lib/gcc/arm-none-eabi/10.3.1/../../../../arm-none-eabi/lib/thumb/v7e-m/nofp\libg.a(lib_a-mallocr.o)
 .bss           0x00000000        0x0 d:/lijie_tools/clion_cubemx/gcc-arm-none-eabi-10.3-2021.10/bin/../lib/gcc/arm-none-eabi/10.3.1/../../../../arm-none-eabi/lib/thumb/v7e-m/nofp\libg.a(lib_a-mallocr.o)
 .text          0x00000000        0x0 d:/lijie_tools/clion_cubemx/gcc-arm-none-eabi-10.3-2021.10/bin/../lib/gcc/arm-none-eabi/10.3.1/../../../../arm-none-eabi/lib/thumb/v7e-m/nofp\libg.a(lib_a-mlock.o)
 .data          0x00000000        0x0 d:/lijie_tools/clion_cubemx/gcc-arm-none-eabi-10.3-2021.10/bin/../lib/gcc/arm-none-eabi/10.3.1/../../../../arm-none-eabi/lib/thumb/v7e-m/nofp\libg.a(lib_a-mlock.o)
 .bss           0x00000000        0x0 d:/lijie_tools/clion_cubemx/gcc-arm-none-eabi-10.3-2021.10/bin/../lib/gcc/arm-none-eabi/10.3.1/../../../../arm-none-eabi/lib/thumb/v7e-m/nofp\libg.a(lib_a-mlock.o)
 .text          0x00000000        0x0 d:/lijie_tools/clion_cubemx/gcc-arm-none-eabi-10.3-2021.10/bin/../lib/gcc/arm-none-eabi/10.3.1/../../../../arm-none-eabi/lib/thumb/v7e-m/nofp\libg.a(lib_a-sbrkr.o)
 .data          0x00000000        0x0 d:/lijie_tools/clion_cubemx/gcc-arm-none-eabi-10.3-2021.10/bin/../lib/gcc/arm-none-eabi/10.3.1/../../../../arm-none-eabi/lib/thumb/v7e-m/nofp\libg.a(lib_a-sbrkr.o)
 .bss           0x00000000        0x0 d:/lijie_tools/clion_cubemx/gcc-arm-none-eabi-10.3-2021.10/bin/../lib/gcc/arm-none-eabi/10.3.1/../../../../arm-none-eabi/lib/thumb/v7e-m/nofp\libg.a(lib_a-sbrkr.o)
 .text          0x00000000        0x0 d:/lijie_tools/clion_cubemx/gcc-arm-none-eabi-10.3-2021.10/bin/../lib/gcc/arm-none-eabi/10.3.1/../../../../arm-none-eabi/lib/thumb/v7e-m/nofp\libg.a(lib_a-stdio.o)
 .data          0x00000000        0x0 d:/lijie_tools/clion_cubemx/gcc-arm-none-eabi-10.3-2021.10/bin/../lib/gcc/arm-none-eabi/10.3.1/../../../../arm-none-eabi/lib/thumb/v7e-m/nofp\libg.a(lib_a-stdio.o)
 .bss           0x00000000        0x0 d:/lijie_tools/clion_cubemx/gcc-arm-none-eabi-10.3-2021.10/bin/../lib/gcc/arm-none-eabi/10.3.1/../../../../arm-none-eabi/lib/thumb/v7e-m/nofp\libg.a(lib_a-stdio.o)
 .text.__seofread
                0x00000000        0x4 d:/lijie_tools/clion_cubemx/gcc-arm-none-eabi-10.3-2021.10/bin/../lib/gcc/arm-none-eabi/10.3.1/../../../../arm-none-eabi/lib/thumb/v7e-m/nofp\libg.a(lib_a-stdio.o)
 .text          0x00000000        0x0 d:/lijie_tools/clion_cubemx/gcc-arm-none-eabi-10.3-2021.10/bin/../lib/gcc/arm-none-eabi/10.3.1/../../../../arm-none-eabi/lib/thumb/v7e-m/nofp\libg.a(lib_a-writer.o)
 .data          0x00000000        0x0 d:/lijie_tools/clion_cubemx/gcc-arm-none-eabi-10.3-2021.10/bin/../lib/gcc/arm-none-eabi/10.3.1/../../../../arm-none-eabi/lib/thumb/v7e-m/nofp\libg.a(lib_a-writer.o)
 .bss           0x00000000        0x0 d:/lijie_tools/clion_cubemx/gcc-arm-none-eabi-10.3-2021.10/bin/../lib/gcc/arm-none-eabi/10.3.1/../../../../arm-none-eabi/lib/thumb/v7e-m/nofp\libg.a(lib_a-writer.o)
 .text          0x00000000        0x0 d:/lijie_tools/clion_cubemx/gcc-arm-none-eabi-10.3-2021.10/bin/../lib/gcc/arm-none-eabi/10.3.1/../../../../arm-none-eabi/lib/thumb/v7e-m/nofp\libg.a(lib_a-__atexit.o)
 .data          0x00000000        0x0 d:/lijie_tools/clion_cubemx/gcc-arm-none-eabi-10.3-2021.10/bin/../lib/gcc/arm-none-eabi/10.3.1/../../../../arm-none-eabi/lib/thumb/v7e-m/nofp\libg.a(lib_a-__atexit.o)
 .bss           0x00000000        0x0 d:/lijie_tools/clion_cubemx/gcc-arm-none-eabi-10.3-2021.10/bin/../lib/gcc/arm-none-eabi/10.3.1/../../../../arm-none-eabi/lib/thumb/v7e-m/nofp\libg.a(lib_a-__atexit.o)
 .text          0x00000000        0x0 d:/lijie_tools/clion_cubemx/gcc-arm-none-eabi-10.3-2021.10/bin/../lib/gcc/arm-none-eabi/10.3.1/../../../../arm-none-eabi/lib/thumb/v7e-m/nofp\libg.a(lib_a-closer.o)
 .data          0x00000000        0x0 d:/lijie_tools/clion_cubemx/gcc-arm-none-eabi-10.3-2021.10/bin/../lib/gcc/arm-none-eabi/10.3.1/../../../../arm-none-eabi/lib/thumb/v7e-m/nofp\libg.a(lib_a-closer.o)
 .bss           0x00000000        0x0 d:/lijie_tools/clion_cubemx/gcc-arm-none-eabi-10.3-2021.10/bin/../lib/gcc/arm-none-eabi/10.3.1/../../../../arm-none-eabi/lib/thumb/v7e-m/nofp\libg.a(lib_a-closer.o)
 .text          0x00000000        0x0 d:/lijie_tools/clion_cubemx/gcc-arm-none-eabi-10.3-2021.10/bin/../lib/gcc/arm-none-eabi/10.3.1/../../../../arm-none-eabi/lib/thumb/v7e-m/nofp\libg.a(lib_a-fclose.o)
 .data          0x00000000        0x0 d:/lijie_tools/clion_cubemx/gcc-arm-none-eabi-10.3-2021.10/bin/../lib/gcc/arm-none-eabi/10.3.1/../../../../arm-none-eabi/lib/thumb/v7e-m/nofp\libg.a(lib_a-fclose.o)
 .bss           0x00000000        0x0 d:/lijie_tools/clion_cubemx/gcc-arm-none-eabi-10.3-2021.10/bin/../lib/gcc/arm-none-eabi/10.3.1/../../../../arm-none-eabi/lib/thumb/v7e-m/nofp\libg.a(lib_a-fclose.o)
 .text.fclose   0x00000000       0x10 d:/lijie_tools/clion_cubemx/gcc-arm-none-eabi-10.3-2021.10/bin/../lib/gcc/arm-none-eabi/10.3.1/../../../../arm-none-eabi/lib/thumb/v7e-m/nofp\libg.a(lib_a-fclose.o)
 .text          0x00000000        0x0 d:/lijie_tools/clion_cubemx/gcc-arm-none-eabi-10.3-2021.10/bin/../lib/gcc/arm-none-eabi/10.3.1/../../../../arm-none-eabi/lib/thumb/v7e-m/nofp\libg.a(lib_a-fstatr.o)
 .data          0x00000000        0x0 d:/lijie_tools/clion_cubemx/gcc-arm-none-eabi-10.3-2021.10/bin/../lib/gcc/arm-none-eabi/10.3.1/../../../../arm-none-eabi/lib/thumb/v7e-m/nofp\libg.a(lib_a-fstatr.o)
 .bss           0x00000000        0x0 d:/lijie_tools/clion_cubemx/gcc-arm-none-eabi-10.3-2021.10/bin/../lib/gcc/arm-none-eabi/10.3.1/../../../../arm-none-eabi/lib/thumb/v7e-m/nofp\libg.a(lib_a-fstatr.o)
 .text          0x00000000        0x0 d:/lijie_tools/clion_cubemx/gcc-arm-none-eabi-10.3-2021.10/bin/../lib/gcc/arm-none-eabi/10.3.1/../../../../arm-none-eabi/lib/thumb/v7e-m/nofp\libg.a(lib_a-isattyr.o)
 .data          0x00000000        0x0 d:/lijie_tools/clion_cubemx/gcc-arm-none-eabi-10.3-2021.10/bin/../lib/gcc/arm-none-eabi/10.3.1/../../../../arm-none-eabi/lib/thumb/v7e-m/nofp\libg.a(lib_a-isattyr.o)
 .bss           0x00000000        0x0 d:/lijie_tools/clion_cubemx/gcc-arm-none-eabi-10.3-2021.10/bin/../lib/gcc/arm-none-eabi/10.3.1/../../../../arm-none-eabi/lib/thumb/v7e-m/nofp\libg.a(lib_a-isattyr.o)
 .text._isatty_r
                0x00000000       0x24 d:/lijie_tools/clion_cubemx/gcc-arm-none-eabi-10.3-2021.10/bin/../lib/gcc/arm-none-eabi/10.3.1/../../../../arm-none-eabi/lib/thumb/v7e-m/nofp\libg.a(lib_a-isattyr.o)
 .debug_frame   0x00000000       0x2c d:/lijie_tools/clion_cubemx/gcc-arm-none-eabi-10.3-2021.10/bin/../lib/gcc/arm-none-eabi/10.3.1/../../../../arm-none-eabi/lib/thumb/v7e-m/nofp\libg.a(lib_a-isattyr.o)
 .ARM.attributes
                0x00000000       0x2e d:/lijie_tools/clion_cubemx/gcc-arm-none-eabi-10.3-2021.10/bin/../lib/gcc/arm-none-eabi/10.3.1/../../../../arm-none-eabi/lib/thumb/v7e-m/nofp\libg.a(lib_a-isattyr.o)
 .text          0x00000000        0x0 d:/lijie_tools/clion_cubemx/gcc-arm-none-eabi-10.3-2021.10/bin/../lib/gcc/arm-none-eabi/10.3.1/../../../../arm-none-eabi/lib/thumb/v7e-m/nofp\libg.a(lib_a-lseekr.o)
 .data          0x00000000        0x0 d:/lijie_tools/clion_cubemx/gcc-arm-none-eabi-10.3-2021.10/bin/../lib/gcc/arm-none-eabi/10.3.1/../../../../arm-none-eabi/lib/thumb/v7e-m/nofp\libg.a(lib_a-lseekr.o)
 .bss           0x00000000        0x0 d:/lijie_tools/clion_cubemx/gcc-arm-none-eabi-10.3-2021.10/bin/../lib/gcc/arm-none-eabi/10.3.1/../../../../arm-none-eabi/lib/thumb/v7e-m/nofp\libg.a(lib_a-lseekr.o)
 .text          0x00000000        0x0 d:/lijie_tools/clion_cubemx/gcc-arm-none-eabi-10.3-2021.10/bin/../lib/gcc/arm-none-eabi/10.3.1/../../../../arm-none-eabi/lib/thumb/v7e-m/nofp\libg.a(lib_a-readr.o)
 .data          0x00000000        0x0 d:/lijie_tools/clion_cubemx/gcc-arm-none-eabi-10.3-2021.10/bin/../lib/gcc/arm-none-eabi/10.3.1/../../../../arm-none-eabi/lib/thumb/v7e-m/nofp\libg.a(lib_a-readr.o)
 .bss           0x00000000        0x0 d:/lijie_tools/clion_cubemx/gcc-arm-none-eabi-10.3-2021.10/bin/../lib/gcc/arm-none-eabi/10.3.1/../../../../arm-none-eabi/lib/thumb/v7e-m/nofp\libg.a(lib_a-readr.o)
 .text          0x00000000        0x0 d:/lijie_tools/clion_cubemx/gcc-arm-none-eabi-10.3-2021.10/bin/../lib/gcc/arm-none-eabi/10.3.1/../../../../arm-none-eabi/lib/thumb/v7e-m/nofp\libg.a(lib_a-reent.o)
 .data          0x00000000        0x0 d:/lijie_tools/clion_cubemx/gcc-arm-none-eabi-10.3-2021.10/bin/../lib/gcc/arm-none-eabi/10.3.1/../../../../arm-none-eabi/lib/thumb/v7e-m/nofp\libg.a(lib_a-reent.o)
 .bss           0x00000000        0x0 d:/lijie_tools/clion_cubemx/gcc-arm-none-eabi-10.3-2021.10/bin/../lib/gcc/arm-none-eabi/10.3.1/../../../../arm-none-eabi/lib/thumb/v7e-m/nofp\libg.a(lib_a-reent.o)
 .text.cleanup_glue
                0x00000000       0x48 d:/lijie_tools/clion_cubemx/gcc-arm-none-eabi-10.3-2021.10/bin/../lib/gcc/arm-none-eabi/10.3.1/../../../../arm-none-eabi/lib/thumb/v7e-m/nofp\libg.a(lib_a-reent.o)
 .text._reclaim_reent
                0x00000000       0x90 d:/lijie_tools/clion_cubemx/gcc-arm-none-eabi-10.3-2021.10/bin/../lib/gcc/arm-none-eabi/10.3.1/../../../../arm-none-eabi/lib/thumb/v7e-m/nofp\libg.a(lib_a-reent.o)
 .text          0x00000000        0x0 d:/lijie_tools/clion_cubemx/gcc-arm-none-eabi-10.3-2021.10/bin/../lib/gcc/arm-none-eabi/10.3.1/thumb/v7e-m/nofp/crtend.o
 .data          0x00000000        0x0 d:/lijie_tools/clion_cubemx/gcc-arm-none-eabi-10.3-2021.10/bin/../lib/gcc/arm-none-eabi/10.3.1/thumb/v7e-m/nofp/crtend.o
 .bss           0x00000000        0x0 d:/lijie_tools/clion_cubemx/gcc-arm-none-eabi-10.3-2021.10/bin/../lib/gcc/arm-none-eabi/10.3.1/thumb/v7e-m/nofp/crtend.o
 .rodata        0x00000000       0x24 d:/lijie_tools/clion_cubemx/gcc-arm-none-eabi-10.3-2021.10/bin/../lib/gcc/arm-none-eabi/10.3.1/thumb/v7e-m/nofp/crtend.o
 .eh_frame      0x00000000        0x4 d:/lijie_tools/clion_cubemx/gcc-arm-none-eabi-10.3-2021.10/bin/../lib/gcc/arm-none-eabi/10.3.1/thumb/v7e-m/nofp/crtend.o
 .ARM.attributes
                0x00000000       0x2e d:/lijie_tools/clion_cubemx/gcc-arm-none-eabi-10.3-2021.10/bin/../lib/gcc/arm-none-eabi/10.3.1/thumb/v7e-m/nofp/crtend.o
 .text          0x00000000        0x0 d:/lijie_tools/clion_cubemx/gcc-arm-none-eabi-10.3-2021.10/bin/../lib/gcc/arm-none-eabi/10.3.1/thumb/v7e-m/nofp/crtn.o
 .data          0x00000000        0x0 d:/lijie_tools/clion_cubemx/gcc-arm-none-eabi-10.3-2021.10/bin/../lib/gcc/arm-none-eabi/10.3.1/thumb/v7e-m/nofp/crtn.o
 .bss           0x00000000        0x0 d:/lijie_tools/clion_cubemx/gcc-arm-none-eabi-10.3-2021.10/bin/../lib/gcc/arm-none-eabi/10.3.1/thumb/v7e-m/nofp/crtn.o
 .text          0x00000000        0x0 d:/lijie_tools/clion_cubemx/gcc-arm-none-eabi-10.3-2021.10/bin/../lib/gcc/arm-none-eabi/10.3.1/../../../../arm-none-eabi/lib/thumb/v7e-m/nofp\libm.a(lib_a-s_round.o)
 .data          0x00000000        0x0 d:/lijie_tools/clion_cubemx/gcc-arm-none-eabi-10.3-2021.10/bin/../lib/gcc/arm-none-eabi/10.3.1/../../../../arm-none-eabi/lib/thumb/v7e-m/nofp\libm.a(lib_a-s_round.o)
 .bss           0x00000000        0x0 d:/lijie_tools/clion_cubemx/gcc-arm-none-eabi-10.3-2021.10/bin/../lib/gcc/arm-none-eabi/10.3.1/../../../../arm-none-eabi/lib/thumb/v7e-m/nofp\libm.a(lib_a-s_round.o)
 .debug_frame   0x00000000       0x2c d:/lijie_tools/clion_cubemx/gcc-arm-none-eabi-10.3-2021.10/bin/../lib/gcc/arm-none-eabi/10.3.1/../../../../arm-none-eabi/lib/thumb/v7e-m/nofp\libm.a(lib_a-s_round.o)
 .ARM.attributes
                0x00000000       0x2e d:/lijie_tools/clion_cubemx/gcc-arm-none-eabi-10.3-2021.10/bin/../lib/gcc/arm-none-eabi/10.3.1/../../../../arm-none-eabi/lib/thumb/v7e-m/nofp\libm.a(lib_a-s_round.o)
 .text          0x00000000        0x0 d:/lijie_tools/clion_cubemx/gcc-arm-none-eabi-10.3-2021.10/bin/../lib/gcc/arm-none-eabi/10.3.1/../../../../arm-none-eabi/lib/thumb/v7e-m/nofp\libm.a(lib_a-w_exp.o)
 .data          0x00000000        0x0 d:/lijie_tools/clion_cubemx/gcc-arm-none-eabi-10.3-2021.10/bin/../lib/gcc/arm-none-eabi/10.3.1/../../../../arm-none-eabi/lib/thumb/v7e-m/nofp\libm.a(lib_a-w_exp.o)
 .bss           0x00000000        0x0 d:/lijie_tools/clion_cubemx/gcc-arm-none-eabi-10.3-2021.10/bin/../lib/gcc/arm-none-eabi/10.3.1/../../../../arm-none-eabi/lib/thumb/v7e-m/nofp\libm.a(lib_a-w_exp.o)
 .debug_frame   0x00000000       0x30 d:/lijie_tools/clion_cubemx/gcc-arm-none-eabi-10.3-2021.10/bin/../lib/gcc/arm-none-eabi/10.3.1/../../../../arm-none-eabi/lib/thumb/v7e-m/nofp\libm.a(lib_a-w_exp.o)
 .ARM.attributes
                0x00000000       0x2e d:/lijie_tools/clion_cubemx/gcc-arm-none-eabi-10.3-2021.10/bin/../lib/gcc/arm-none-eabi/10.3.1/../../../../arm-none-eabi/lib/thumb/v7e-m/nofp\libm.a(lib_a-w_exp.o)
 .text          0x00000000        0x0 d:/lijie_tools/clion_cubemx/gcc-arm-none-eabi-10.3-2021.10/bin/../lib/gcc/arm-none-eabi/10.3.1/../../../../arm-none-eabi/lib/thumb/v7e-m/nofp\libm.a(lib_a-e_exp.o)
 .data          0x00000000        0x0 d:/lijie_tools/clion_cubemx/gcc-arm-none-eabi-10.3-2021.10/bin/../lib/gcc/arm-none-eabi/10.3.1/../../../../arm-none-eabi/lib/thumb/v7e-m/nofp\libm.a(lib_a-e_exp.o)
 .bss           0x00000000        0x0 d:/lijie_tools/clion_cubemx/gcc-arm-none-eabi-10.3-2021.10/bin/../lib/gcc/arm-none-eabi/10.3.1/../../../../arm-none-eabi/lib/thumb/v7e-m/nofp\libm.a(lib_a-e_exp.o)
 .debug_frame   0x00000000       0x74 d:/lijie_tools/clion_cubemx/gcc-arm-none-eabi-10.3-2021.10/bin/../lib/gcc/arm-none-eabi/10.3.1/../../../../arm-none-eabi/lib/thumb/v7e-m/nofp\libm.a(lib_a-e_exp.o)
 .ARM.attributes
                0x00000000       0x2e d:/lijie_tools/clion_cubemx/gcc-arm-none-eabi-10.3-2021.10/bin/../lib/gcc/arm-none-eabi/10.3.1/../../../../arm-none-eabi/lib/thumb/v7e-m/nofp\libm.a(lib_a-e_exp.o)
 .text          0x00000000        0x0 d:/lijie_tools/clion_cubemx/gcc-arm-none-eabi-10.3-2021.10/bin/../lib/gcc/arm-none-eabi/10.3.1/../../../../arm-none-eabi/lib/thumb/v7e-m/nofp\libm.a(lib_a-math_err.o)
 .data          0x00000000        0x0 d:/lijie_tools/clion_cubemx/gcc-arm-none-eabi-10.3-2021.10/bin/../lib/gcc/arm-none-eabi/10.3.1/../../../../arm-none-eabi/lib/thumb/v7e-m/nofp\libm.a(lib_a-math_err.o)
 .bss           0x00000000        0x0 d:/lijie_tools/clion_cubemx/gcc-arm-none-eabi-10.3-2021.10/bin/../lib/gcc/arm-none-eabi/10.3.1/../../../../arm-none-eabi/lib/thumb/v7e-m/nofp\libm.a(lib_a-math_err.o)
 .text.__math_may_uflow
                0x00000000        0xc d:/lijie_tools/clion_cubemx/gcc-arm-none-eabi-10.3-2021.10/bin/../lib/gcc/arm-none-eabi/10.3.1/../../../../arm-none-eabi/lib/thumb/v7e-m/nofp\libm.a(lib_a-math_err.o)
 .text.__math_divzero
                0x00000000       0x34 d:/lijie_tools/clion_cubemx/gcc-arm-none-eabi-10.3-2021.10/bin/../lib/gcc/arm-none-eabi/10.3.1/../../../../arm-none-eabi/lib/thumb/v7e-m/nofp\libm.a(lib_a-math_err.o)
 .text.__math_invalid
                0x00000000       0x3c d:/lijie_tools/clion_cubemx/gcc-arm-none-eabi-10.3-2021.10/bin/../lib/gcc/arm-none-eabi/10.3.1/../../../../arm-none-eabi/lib/thumb/v7e-m/nofp\libm.a(lib_a-math_err.o)
 .text.__math_check_uflow
                0x00000000       0x24 d:/lijie_tools/clion_cubemx/gcc-arm-none-eabi-10.3-2021.10/bin/../lib/gcc/arm-none-eabi/10.3.1/../../../../arm-none-eabi/lib/thumb/v7e-m/nofp\libm.a(lib_a-math_err.o)
 .text.__math_check_oflow
                0x00000000       0x44 d:/lijie_tools/clion_cubemx/gcc-arm-none-eabi-10.3-2021.10/bin/../lib/gcc/arm-none-eabi/10.3.1/../../../../arm-none-eabi/lib/thumb/v7e-m/nofp\libm.a(lib_a-math_err.o)
 .debug_frame   0x00000000      0x11c d:/lijie_tools/clion_cubemx/gcc-arm-none-eabi-10.3-2021.10/bin/../lib/gcc/arm-none-eabi/10.3.1/../../../../arm-none-eabi/lib/thumb/v7e-m/nofp\libm.a(lib_a-math_err.o)
 .ARM.attributes
                0x00000000       0x2e d:/lijie_tools/clion_cubemx/gcc-arm-none-eabi-10.3-2021.10/bin/../lib/gcc/arm-none-eabi/10.3.1/../../../../arm-none-eabi/lib/thumb/v7e-m/nofp\libm.a(lib_a-math_err.o)
 .text          0x00000000        0x0 d:/lijie_tools/clion_cubemx/gcc-arm-none-eabi-10.3-2021.10/bin/../lib/gcc/arm-none-eabi/10.3.1/../../../../arm-none-eabi/lib/thumb/v7e-m/nofp\libm.a(lib_a-s_finite.o)
 .data          0x00000000        0x0 d:/lijie_tools/clion_cubemx/gcc-arm-none-eabi-10.3-2021.10/bin/../lib/gcc/arm-none-eabi/10.3.1/../../../../arm-none-eabi/lib/thumb/v7e-m/nofp\libm.a(lib_a-s_finite.o)
 .bss           0x00000000        0x0 d:/lijie_tools/clion_cubemx/gcc-arm-none-eabi-10.3-2021.10/bin/../lib/gcc/arm-none-eabi/10.3.1/../../../../arm-none-eabi/lib/thumb/v7e-m/nofp\libm.a(lib_a-s_finite.o)
 .debug_frame   0x00000000       0x20 d:/lijie_tools/clion_cubemx/gcc-arm-none-eabi-10.3-2021.10/bin/../lib/gcc/arm-none-eabi/10.3.1/../../../../arm-none-eabi/lib/thumb/v7e-m/nofp\libm.a(lib_a-s_finite.o)
 .ARM.attributes
                0x00000000       0x2e d:/lijie_tools/clion_cubemx/gcc-arm-none-eabi-10.3-2021.10/bin/../lib/gcc/arm-none-eabi/10.3.1/../../../../arm-none-eabi/lib/thumb/v7e-m/nofp\libm.a(lib_a-s_finite.o)
 .text          0x00000000       0x2c d:/lijie_tools/clion_cubemx/gcc-arm-none-eabi-10.3-2021.10/bin/../lib/gcc/arm-none-eabi/10.3.1/thumb/v7e-m/nofp\libgcc.a(_arm_unorddf2.o)
 .data          0x00000000        0x0 d:/lijie_tools/clion_cubemx/gcc-arm-none-eabi-10.3-2021.10/bin/../lib/gcc/arm-none-eabi/10.3.1/thumb/v7e-m/nofp\libgcc.a(_arm_unorddf2.o)
 .bss           0x00000000        0x0 d:/lijie_tools/clion_cubemx/gcc-arm-none-eabi-10.3-2021.10/bin/../lib/gcc/arm-none-eabi/10.3.1/thumb/v7e-m/nofp\libgcc.a(_arm_unorddf2.o)
 .debug_frame   0x00000000       0x20 d:/lijie_tools/clion_cubemx/gcc-arm-none-eabi-10.3-2021.10/bin/../lib/gcc/arm-none-eabi/10.3.1/thumb/v7e-m/nofp\libgcc.a(_arm_unorddf2.o)
 .ARM.attributes
                0x00000000       0x1e d:/lijie_tools/clion_cubemx/gcc-arm-none-eabi-10.3-2021.10/bin/../lib/gcc/arm-none-eabi/10.3.1/thumb/v7e-m/nofp\libgcc.a(_arm_unorddf2.o)

Memory Configuration

Name             Origin             Length             Attributes
FLASH            0x08000000         0x00020000         xr
DTCMRAM          0x20000000         0x00020000         xrw
RAM_D1           0x24000000         0x00080000         xrw
RAM_D2           0x30000000         0x00048000         xrw
RAM_D3           0x38000000         0x00010000         xrw
ITCMRAM          0x00000000         0x00010000         xrw
*default*        0x00000000         0xffffffff

Linker script and memory map

LOAD d:/lijie_tools/clion_cubemx/gcc-arm-none-eabi-10.3-2021.10/bin/../lib/gcc/arm-none-eabi/10.3.1/thumb/v7e-m/nofp/crti.o
LOAD d:/lijie_tools/clion_cubemx/gcc-arm-none-eabi-10.3-2021.10/bin/../lib/gcc/arm-none-eabi/10.3.1/thumb/v7e-m/nofp/crtbegin.o
LOAD d:/lijie_tools/clion_cubemx/gcc-arm-none-eabi-10.3-2021.10/bin/../lib/gcc/arm-none-eabi/10.3.1/../../../../arm-none-eabi/lib/thumb/v7e-m/nofp/crt0.o
LOAD CMakeFiles/H750_S15909.elf.dir/APP/DS18B20.c.obj
LOAD CMakeFiles/H750_S15909.elf.dir/APP/IRIS_Method.c.obj
LOAD CMakeFiles/H750_S15909.elf.dir/APP/LED.c.obj
LOAD CMakeFiles/H750_S15909.elf.dir/APP/Shutter.c.obj
LOAD CMakeFiles/H750_S15909.elf.dir/APP/communication.c.obj
LOAD CMakeFiles/H750_S15909.elf.dir/APP/data_analyse.c.obj
LOAD CMakeFiles/H750_S15909.elf.dir/APP/delay.c.obj
LOAD CMakeFiles/H750_S15909.elf.dir/APP/mymain.c.obj
LOAD CMakeFiles/H750_S15909.elf.dir/APP/usart1_tx_dma.c.obj
LOAD CMakeFiles/H750_S15909.elf.dir/Core/Src/dma.c.obj
LOAD CMakeFiles/H750_S15909.elf.dir/Core/Src/gpio.c.obj
LOAD CMakeFiles/H750_S15909.elf.dir/Core/Src/main.c.obj
LOAD CMakeFiles/H750_S15909.elf.dir/Core/Src/stm32h7xx_hal_msp.c.obj
LOAD CMakeFiles/H750_S15909.elf.dir/Core/Src/stm32h7xx_it.c.obj
LOAD CMakeFiles/H750_S15909.elf.dir/Core/Src/syscalls.c.obj
LOAD CMakeFiles/H750_S15909.elf.dir/Core/Src/sysmem.c.obj
LOAD CMakeFiles/H750_S15909.elf.dir/Core/Src/system_stm32h7xx.c.obj
LOAD CMakeFiles/H750_S15909.elf.dir/Core/Src/tim.c.obj
LOAD CMakeFiles/H750_S15909.elf.dir/Core/Src/usart.c.obj
LOAD CMakeFiles/H750_S15909.elf.dir/Core/Startup/startup_stm32h750vbtx.s.obj
LOAD CMakeFiles/H750_S15909.elf.dir/Drivers/STM32H7xx_HAL_Driver/Src/stm32h7xx_hal.c.obj
LOAD CMakeFiles/H750_S15909.elf.dir/Drivers/STM32H7xx_HAL_Driver/Src/stm32h7xx_hal_cortex.c.obj
LOAD CMakeFiles/H750_S15909.elf.dir/Drivers/STM32H7xx_HAL_Driver/Src/stm32h7xx_hal_dma.c.obj
LOAD CMakeFiles/H750_S15909.elf.dir/Drivers/STM32H7xx_HAL_Driver/Src/stm32h7xx_hal_dma_ex.c.obj
LOAD CMakeFiles/H750_S15909.elf.dir/Drivers/STM32H7xx_HAL_Driver/Src/stm32h7xx_hal_exti.c.obj
LOAD CMakeFiles/H750_S15909.elf.dir/Drivers/STM32H7xx_HAL_Driver/Src/stm32h7xx_hal_flash.c.obj
LOAD CMakeFiles/H750_S15909.elf.dir/Drivers/STM32H7xx_HAL_Driver/Src/stm32h7xx_hal_flash_ex.c.obj
LOAD CMakeFiles/H750_S15909.elf.dir/Drivers/STM32H7xx_HAL_Driver/Src/stm32h7xx_hal_gpio.c.obj
LOAD CMakeFiles/H750_S15909.elf.dir/Drivers/STM32H7xx_HAL_Driver/Src/stm32h7xx_hal_hsem.c.obj
LOAD CMakeFiles/H750_S15909.elf.dir/Drivers/STM32H7xx_HAL_Driver/Src/stm32h7xx_hal_i2c.c.obj
LOAD CMakeFiles/H750_S15909.elf.dir/Drivers/STM32H7xx_HAL_Driver/Src/stm32h7xx_hal_i2c_ex.c.obj
LOAD CMakeFiles/H750_S15909.elf.dir/Drivers/STM32H7xx_HAL_Driver/Src/stm32h7xx_hal_mdma.c.obj
LOAD CMakeFiles/H750_S15909.elf.dir/Drivers/STM32H7xx_HAL_Driver/Src/stm32h7xx_hal_pwr.c.obj
LOAD CMakeFiles/H750_S15909.elf.dir/Drivers/STM32H7xx_HAL_Driver/Src/stm32h7xx_hal_pwr_ex.c.obj
LOAD CMakeFiles/H750_S15909.elf.dir/Drivers/STM32H7xx_HAL_Driver/Src/stm32h7xx_hal_rcc.c.obj
LOAD CMakeFiles/H750_S15909.elf.dir/Drivers/STM32H7xx_HAL_Driver/Src/stm32h7xx_hal_rcc_ex.c.obj
LOAD CMakeFiles/H750_S15909.elf.dir/Drivers/STM32H7xx_HAL_Driver/Src/stm32h7xx_hal_tim.c.obj
LOAD CMakeFiles/H750_S15909.elf.dir/Drivers/STM32H7xx_HAL_Driver/Src/stm32h7xx_hal_tim_ex.c.obj
LOAD CMakeFiles/H750_S15909.elf.dir/Drivers/STM32H7xx_HAL_Driver/Src/stm32h7xx_hal_uart.c.obj
LOAD CMakeFiles/H750_S15909.elf.dir/Drivers/STM32H7xx_HAL_Driver/Src/stm32h7xx_hal_uart_ex.c.obj
START GROUP
LOAD d:/lijie_tools/clion_cubemx/gcc-arm-none-eabi-10.3-2021.10/bin/../lib/gcc/arm-none-eabi/10.3.1/thumb/v7e-m/nofp\libgcc.a
LOAD d:/lijie_tools/clion_cubemx/gcc-arm-none-eabi-10.3-2021.10/bin/../lib/gcc/arm-none-eabi/10.3.1/../../../../arm-none-eabi/lib/thumb/v7e-m/nofp\libg.a
LOAD d:/lijie_tools/clion_cubemx/gcc-arm-none-eabi-10.3-2021.10/bin/../lib/gcc/arm-none-eabi/10.3.1/../../../../arm-none-eabi/lib/thumb/v7e-m/nofp\libc.a
END GROUP
LOAD d:/lijie_tools/clion_cubemx/gcc-arm-none-eabi-10.3-2021.10/bin/../lib/gcc/arm-none-eabi/10.3.1/thumb/v7e-m/nofp/crtend.o
LOAD d:/lijie_tools/clion_cubemx/gcc-arm-none-eabi-10.3-2021.10/bin/../lib/gcc/arm-none-eabi/10.3.1/thumb/v7e-m/nofp/crtn.o
                0x24080000                _estack = (ORIGIN (RAM_D1) + LENGTH (RAM_D1))
                0x00000200                _Min_Heap_Size = 0x200
                0x00000400                _Min_Stack_Size = 0x400

.isr_vector     0x08000000      0x298
                0x08000000                . = ALIGN (0x4)
 *(.isr_vector)
 .isr_vector    0x08000000      0x298 CMakeFiles/H750_S15909.elf.dir/Core/Startup/startup_stm32h750vbtx.s.obj
                0x08000000                g_pfnVectors
                0x08000298                . = ALIGN (0x4)

.text           0x08000298     0x9554
                0x08000298                . = ALIGN (0x4)
 *(.text)
 .text          0x08000298       0x40 d:/lijie_tools/clion_cubemx/gcc-arm-none-eabi-10.3-2021.10/bin/../lib/gcc/arm-none-eabi/10.3.1/thumb/v7e-m/nofp/crtbegin.o
 .text          0x080002d8      0x378 d:/lijie_tools/clion_cubemx/gcc-arm-none-eabi-10.3-2021.10/bin/../lib/gcc/arm-none-eabi/10.3.1/thumb/v7e-m/nofp\libgcc.a(_arm_addsubdf3.o)
                0x080002d8                __aeabi_drsub
                0x080002e0                __aeabi_dsub
                0x080002e0                __subdf3
                0x080002e4                __aeabi_dadd
                0x080002e4                __adddf3
                0x0800055c                __floatunsidf
                0x0800055c                __aeabi_ui2d
                0x0800057c                __floatsidf
                0x0800057c                __aeabi_i2d
                0x080005a0                __aeabi_f2d
                0x080005a0                __extendsfdf2
                0x080005e4                __floatundidf
                0x080005e4                __aeabi_ul2d
                0x080005f4                __floatdidf
                0x080005f4                __aeabi_l2d
 .text          0x08000650      0x424 d:/lijie_tools/clion_cubemx/gcc-arm-none-eabi-10.3-2021.10/bin/../lib/gcc/arm-none-eabi/10.3.1/thumb/v7e-m/nofp\libgcc.a(_arm_muldivdf3.o)
                0x08000650                __aeabi_dmul
                0x08000650                __muldf3
                0x080008a4                __divdf3
                0x080008a4                __aeabi_ddiv
 .text          0x08000a74      0x110 d:/lijie_tools/clion_cubemx/gcc-arm-none-eabi-10.3-2021.10/bin/../lib/gcc/arm-none-eabi/10.3.1/thumb/v7e-m/nofp\libgcc.a(_arm_cmpdf2.o)
                0x08000a74                __gtdf2
                0x08000a74                __gedf2
                0x08000a7c                __ltdf2
                0x08000a7c                __ledf2
                0x08000a84                __nedf2
                0x08000a84                __eqdf2
                0x08000a84                __cmpdf2
                0x08000b00                __aeabi_cdrcmple
                0x08000b10                __aeabi_cdcmpeq
                0x08000b10                __aeabi_cdcmple
                0x08000b20                __aeabi_dcmpeq
                0x08000b34                __aeabi_dcmplt
                0x08000b48                __aeabi_dcmple
                0x08000b5c                __aeabi_dcmpge
                0x08000b70                __aeabi_dcmpgt
 .text          0x08000b84       0x50 d:/lijie_tools/clion_cubemx/gcc-arm-none-eabi-10.3-2021.10/bin/../lib/gcc/arm-none-eabi/10.3.1/thumb/v7e-m/nofp\libgcc.a(_arm_fixdfsi.o)
                0x08000b84                __aeabi_d2iz
                0x08000b84                __fixdfsi
 .text          0x08000bd4       0x40 d:/lijie_tools/clion_cubemx/gcc-arm-none-eabi-10.3-2021.10/bin/../lib/gcc/arm-none-eabi/10.3.1/thumb/v7e-m/nofp\libgcc.a(_arm_fixunsdfsi.o)
                0x08000bd4                __aeabi_d2uiz
                0x08000bd4                __fixunsdfsi
 .text          0x08000c14       0xa0 d:/lijie_tools/clion_cubemx/gcc-arm-none-eabi-10.3-2021.10/bin/../lib/gcc/arm-none-eabi/10.3.1/thumb/v7e-m/nofp\libgcc.a(_arm_truncdfsf2.o)
                0x08000c14                __truncdfsf2
                0x08000c14                __aeabi_d2f
 .text          0x08000cb4      0x21c d:/lijie_tools/clion_cubemx/gcc-arm-none-eabi-10.3-2021.10/bin/../lib/gcc/arm-none-eabi/10.3.1/thumb/v7e-m/nofp\libgcc.a(_arm_addsubsf3.o)
                0x08000cb4                __aeabi_frsub
                0x08000cbc                __subsf3
                0x08000cbc                __aeabi_fsub
                0x08000cc0                __aeabi_fadd
                0x08000cc0                __addsf3
                0x08000e20                __aeabi_ui2f
                0x08000e20                __floatunsisf
                0x08000e28                __aeabi_i2f
                0x08000e28                __floatsisf
                0x08000e44                __aeabi_ul2f
                0x08000e44                __floatundisf
                0x08000e54                __aeabi_l2f
                0x08000e54                __floatdisf
 .text          0x08000ed0      0x2a0 d:/lijie_tools/clion_cubemx/gcc-arm-none-eabi-10.3-2021.10/bin/../lib/gcc/arm-none-eabi/10.3.1/thumb/v7e-m/nofp\libgcc.a(_arm_muldivsf3.o)
                0x08000ed0                __mulsf3
                0x08000ed0                __aeabi_fmul
                0x08001038                __aeabi_fdiv
                0x08001038                __divsf3
 .text          0x08001170       0x40 d:/lijie_tools/clion_cubemx/gcc-arm-none-eabi-10.3-2021.10/bin/../lib/gcc/arm-none-eabi/10.3.1/thumb/v7e-m/nofp\libgcc.a(_arm_fixunssfsi.o)
                0x08001170                __fixunssfsi
                0x08001170                __aeabi_f2uiz
 .text          0x080011b0       0x30 d:/lijie_tools/clion_cubemx/gcc-arm-none-eabi-10.3-2021.10/bin/../lib/gcc/arm-none-eabi/10.3.1/thumb/v7e-m/nofp\libgcc.a(_aeabi_uldivmod.o)
                0x080011b0                __aeabi_uldivmod
 .text          0x080011e0      0x2d0 d:/lijie_tools/clion_cubemx/gcc-arm-none-eabi-10.3-2021.10/bin/../lib/gcc/arm-none-eabi/10.3.1/thumb/v7e-m/nofp\libgcc.a(_udivmoddi4.o)
                0x080011e0                __udivmoddi4
 .text          0x080014b0        0x4 d:/lijie_tools/clion_cubemx/gcc-arm-none-eabi-10.3-2021.10/bin/../lib/gcc/arm-none-eabi/10.3.1/thumb/v7e-m/nofp\libgcc.a(_dvmd_tls.o)
                0x080014b0                __aeabi_idiv0
                0x080014b0                __aeabi_ldiv0
 .text          0x080014b4      0x134 d:/lijie_tools/clion_cubemx/gcc-arm-none-eabi-10.3-2021.10/bin/../lib/gcc/arm-none-eabi/10.3.1/../../../../arm-none-eabi/lib/thumb/v7e-m/nofp\libg.a(lib_a-memcpy.o)
                0x080014b4                memcpy
 *(.text*)
 .text.DS18B20_OUTPUT
                0x080015e8       0x2c CMakeFiles/H750_S15909.elf.dir/APP/DS18B20.c.obj
                0x080015e8                DS18B20_OUTPUT
 .text.DS18B20_INPUT
                0x08001614       0x28 CMakeFiles/H750_S15909.elf.dir/APP/DS18B20.c.obj
                0x08001614                DS18B20_INPUT
 .text.DS18B20_Reset
                0x0800163c       0x30 CMakeFiles/H750_S15909.elf.dir/APP/DS18B20.c.obj
                0x0800163c                DS18B20_Reset
 .text.DS18B20_Check
                0x0800166c       0x58 CMakeFiles/H750_S15909.elf.dir/APP/DS18B20.c.obj
                0x0800166c                DS18B20_Check
 .text.DS18B20_Read_Bit
                0x080016c4       0x48 CMakeFiles/H750_S15909.elf.dir/APP/DS18B20.c.obj
                0x080016c4                DS18B20_Read_Bit
 .text.DS18B20_ReadByte
                0x0800170c       0x20 CMakeFiles/H750_S15909.elf.dir/APP/DS18B20.c.obj
                0x0800170c                DS18B20_ReadByte
 .text.DS18B20_WriteByte
                0x0800172c       0x68 CMakeFiles/H750_S15909.elf.dir/APP/DS18B20.c.obj
                0x0800172c                DS18B20_WriteByte
 .text.DS18B20_Start
                0x08001794       0x18 CMakeFiles/H750_S15909.elf.dir/APP/DS18B20.c.obj
                0x08001794                DS18B20_Start
 .text.DS18B20_Init
                0x080017ac       0x68 CMakeFiles/H750_S15909.elf.dir/APP/DS18B20.c.obj
                0x080017ac                DS18B20_Init
 .text.DS18B20_Stop
                0x08001814       0x18 CMakeFiles/H750_S15909.elf.dir/APP/DS18B20.c.obj
                0x08001814                DS18B20_Stop
 .text.DS18B20_GetTemperature
                0x0800182c       0x70 CMakeFiles/H750_S15909.elf.dir/APP/DS18B20.c.obj
                0x0800182c                DS18B20_GetTemperature
 .text.IRIS_calcCRC
                0x0800189c       0x42 CMakeFiles/H750_S15909.elf.dir/APP/IRIS_Method.c.obj
                0x0800189c                IRIS_calcCRC
 .text.IRIS_Protocol_Pack
                0x080018de       0x56 CMakeFiles/H750_S15909.elf.dir/APP/IRIS_Method.c.obj
                0x080018de                IRIS_Protocol_Pack
 .text.IRIS_STM32_Protocol_Unpack
                0x08001934       0x9c CMakeFiles/H750_S15909.elf.dir/APP/IRIS_Method.c.obj
                0x08001934                IRIS_STM32_Protocol_Unpack
 .text.Shutter_Open
                0x080019d0       0x28 CMakeFiles/H750_S15909.elf.dir/APP/Shutter.c.obj
                0x080019d0                Shutter_Open
 .text.Shutter_Close
                0x080019f8       0x28 CMakeFiles/H750_S15909.elf.dir/APP/Shutter.c.obj
                0x080019f8                Shutter_Close
 .text.Send_Shutter_Time
                0x08001a20       0x4c CMakeFiles/H750_S15909.elf.dir/APP/communication.c.obj
                0x08001a20                Send_Shutter_Time
 *fill*         0x08001a6c        0x4 
 .text.Opt_Snenser
                0x08001a70       0xbc CMakeFiles/H750_S15909.elf.dir/APP/communication.c.obj
                0x08001a70                Opt_Snenser
 .text.compute_gaussian_weights
                0x08001b2c       0xb2 CMakeFiles/H750_S15909.elf.dir/APP/data_analyse.c.obj
                0x08001b2c                compute_gaussian_weights
 *fill*         0x08001bde        0x2 
 .text.sgi_smoothing
                0x08001be0       0xac CMakeFiles/H750_S15909.elf.dir/APP/data_analyse.c.obj
                0x08001be0                sgi_smoothing
 .text.sgi      0x08001c8c        0xa CMakeFiles/H750_S15909.elf.dir/APP/data_analyse.c.obj
                0x08001c8c                sgi
 *fill*         0x08001c96        0x2 
 .text.Delay_Init
                0x08001c98       0x10 CMakeFiles/H750_S15909.elf.dir/APP/delay.c.obj
                0x08001c98                Delay_Init
 .text.Delay_us
                0x08001ca8       0x3c CMakeFiles/H750_S15909.elf.dir/APP/delay.c.obj
                0x08001ca8                Delay_us
 .text.Communication_Init
                0x08001ce4       0x30 CMakeFiles/H750_S15909.elf.dir/APP/mymain.c.obj
                0x08001ce4                Communication_Init
 .text.Send_Data
                0x08001d14       0xe8 CMakeFiles/H750_S15909.elf.dir/APP/mymain.c.obj
                0x08001d14                Send_Data
 .text.HAL_UART_RxCpltCallback
                0x08001dfc       0x88 CMakeFiles/H750_S15909.elf.dir/APP/mymain.c.obj
                0x08001dfc                HAL_UART_RxCpltCallback
 .text.HAL_GPIO_EXTI_Callback
                0x08001e84       0x18 CMakeFiles/H750_S15909.elf.dir/APP/mymain.c.obj
                0x08001e84                HAL_GPIO_EXTI_Callback
 .text.commander_run
                0x08001e9c      0x210 CMakeFiles/H750_S15909.elf.dir/APP/mymain.c.obj
                0x08001e9c                commander_run
 .text.mymain   0x080020ac      0x200 CMakeFiles/H750_S15909.elf.dir/APP/mymain.c.obj
                0x080020ac                mymain
 .text.dma_init
                0x080022ac       0x90 CMakeFiles/H750_S15909.elf.dir/APP/usart1_tx_dma.c.obj
                0x080022ac                dma_init
 .text.MX_DMA_Init
                0x0800233c       0x38 CMakeFiles/H750_S15909.elf.dir/Core/Src/dma.c.obj
                0x0800233c                MX_DMA_Init
 .text.MX_GPIO_Init
                0x08002374       0xc8 CMakeFiles/H750_S15909.elf.dir/Core/Src/gpio.c.obj
                0x08002374                MX_GPIO_Init
 .text.Error_Handler
                0x0800243c        0x4 CMakeFiles/H750_S15909.elf.dir/Core/Src/main.c.obj
                0x0800243c                Error_Handler
 .text.SystemClock_Config
                0x08002440      0x114 CMakeFiles/H750_S15909.elf.dir/Core/Src/main.c.obj
                0x08002440                SystemClock_Config
 .text.main     0x08002554       0x2c CMakeFiles/H750_S15909.elf.dir/Core/Src/main.c.obj
                0x08002554                main
 .text.HAL_MspInit
                0x08002580       0x24 CMakeFiles/H750_S15909.elf.dir/Core/Src/stm32h7xx_hal_msp.c.obj
                0x08002580                HAL_MspInit
 .text.NMI_Handler
                0x080025a4        0x2 CMakeFiles/H750_S15909.elf.dir/Core/Src/stm32h7xx_it.c.obj
                0x080025a4                NMI_Handler
 .text.HardFault_Handler
                0x080025a6        0x2 CMakeFiles/H750_S15909.elf.dir/Core/Src/stm32h7xx_it.c.obj
                0x080025a6                HardFault_Handler
 .text.MemManage_Handler
                0x080025a8        0x2 CMakeFiles/H750_S15909.elf.dir/Core/Src/stm32h7xx_it.c.obj
                0x080025a8                MemManage_Handler
 .text.BusFault_Handler
                0x080025aa        0x2 CMakeFiles/H750_S15909.elf.dir/Core/Src/stm32h7xx_it.c.obj
                0x080025aa                BusFault_Handler
 .text.UsageFault_Handler
                0x080025ac        0x2 CMakeFiles/H750_S15909.elf.dir/Core/Src/stm32h7xx_it.c.obj
                0x080025ac                UsageFault_Handler
 .text.SVC_Handler
                0x080025ae        0x2 CMakeFiles/H750_S15909.elf.dir/Core/Src/stm32h7xx_it.c.obj
                0x080025ae                SVC_Handler
 .text.DebugMon_Handler
                0x080025b0        0x2 CMakeFiles/H750_S15909.elf.dir/Core/Src/stm32h7xx_it.c.obj
                0x080025b0                DebugMon_Handler
 .text.PendSV_Handler
                0x080025b2        0x2 CMakeFiles/H750_S15909.elf.dir/Core/Src/stm32h7xx_it.c.obj
                0x080025b2                PendSV_Handler
 .text.SysTick_Handler
                0x080025b4        0x8 CMakeFiles/H750_S15909.elf.dir/Core/Src/stm32h7xx_it.c.obj
                0x080025b4                SysTick_Handler
 .text.EXTI0_IRQHandler
                0x080025bc        0xa CMakeFiles/H750_S15909.elf.dir/Core/Src/stm32h7xx_it.c.obj
                0x080025bc                EXTI0_IRQHandler
 *fill*         0x080025c6        0x2 
 .text.DMA1_Stream0_IRQHandler
                0x080025c8       0x10 CMakeFiles/H750_S15909.elf.dir/Core/Src/stm32h7xx_it.c.obj
                0x080025c8                DMA1_Stream0_IRQHandler
 .text.USART1_IRQHandler
                0x080025d8       0x10 CMakeFiles/H750_S15909.elf.dir/Core/Src/stm32h7xx_it.c.obj
                0x080025d8                USART1_IRQHandler
 .text._read    0x080025e8       0x20 CMakeFiles/H750_S15909.elf.dir/Core/Src/syscalls.c.obj
                0x080025e8                _read
 .text._close   0x08002608        0x6 CMakeFiles/H750_S15909.elf.dir/Core/Src/syscalls.c.obj
                0x08002608                _close
 .text._fstat   0x0800260e        0xa CMakeFiles/H750_S15909.elf.dir/Core/Src/syscalls.c.obj
                0x0800260e                _fstat
 .text._lseek   0x08002618        0x4 CMakeFiles/H750_S15909.elf.dir/Core/Src/syscalls.c.obj
                0x08002618                _lseek
 .text._sbrk    0x0800261c       0x48 CMakeFiles/H750_S15909.elf.dir/Core/Src/sysmem.c.obj
                0x0800261c                _sbrk
 .text.SystemInit
                0x08002664       0xbc CMakeFiles/H750_S15909.elf.dir/Core/Src/system_stm32h7xx.c.obj
                0x08002664                SystemInit
 .text.MX_TIM5_Init
                0x08002720       0x70 CMakeFiles/H750_S15909.elf.dir/Core/Src/tim.c.obj
                0x08002720                MX_TIM5_Init
 .text.HAL_TIM_Base_MspInit
                0x08002790       0x34 CMakeFiles/H750_S15909.elf.dir/Core/Src/tim.c.obj
                0x08002790                HAL_TIM_Base_MspInit
 .text.MX_USART1_UART_Init
                0x080027c4       0x68 CMakeFiles/H750_S15909.elf.dir/Core/Src/usart.c.obj
                0x080027c4                MX_USART1_UART_Init
 .text.MX_USART2_UART_Init
                0x0800282c       0x68 CMakeFiles/H750_S15909.elf.dir/Core/Src/usart.c.obj
                0x0800282c                MX_USART2_UART_Init
 .text.HAL_UART_MspInit
                0x08002894      0x148 CMakeFiles/H750_S15909.elf.dir/Core/Src/usart.c.obj
                0x08002894                HAL_UART_MspInit
 .text._write   0x080029dc       0x28 CMakeFiles/H750_S15909.elf.dir/Core/Src/usart.c.obj
                0x080029dc                _write
 .text.Reset_Handler
                0x08002a04       0x50 CMakeFiles/H750_S15909.elf.dir/Core/Startup/startup_stm32h750vbtx.s.obj
                0x08002a04                Reset_Handler
 .text.Default_Handler
                0x08002a54        0x2 CMakeFiles/H750_S15909.elf.dir/Core/Startup/startup_stm32h750vbtx.s.obj
                0x08002a54                RTC_Alarm_IRQHandler
                0x08002a54                HASH_RNG_IRQHandler
                0x08002a54                EXTI2_IRQHandler
                0x08002a54                TIM8_CC_IRQHandler
                0x08002a54                HRTIM1_Master_IRQHandler
                0x08002a54                UART8_IRQHandler
                0x08002a54                SPI4_IRQHandler
                0x08002a54                TIM1_CC_IRQHandler
                0x08002a54                BDMA_Channel6_IRQHandler
                0x08002a54                DMA2_Stream5_IRQHandler
                0x08002a54                HRTIM1_FLT_IRQHandler
                0x08002a54                JPEG_IRQHandler
                0x08002a54                DMA1_Stream5_IRQHandler
                0x08002a54                BDMA_Channel1_IRQHandler
                0x08002a54                HRTIM1_TIMD_IRQHandler
                0x08002a54                TAMP_STAMP_IRQHandler
                0x08002a54                EXTI3_IRQHandler
                0x08002a54                LPTIM4_IRQHandler
                0x08002a54                TIM8_TRG_COM_TIM14_IRQHandler
                0x08002a54                LPTIM2_IRQHandler
                0x08002a54                DFSDM1_FLT1_IRQHandler
                0x08002a54                DMAMUX2_OVR_IRQHandler
                0x08002a54                TIM8_UP_TIM13_IRQHandler
                0x08002a54                I2C3_ER_IRQHandler
                0x08002a54                DFSDM1_FLT2_IRQHandler
                0x08002a54                MDMA_IRQHandler
                0x08002a54                LPTIM3_IRQHandler
                0x08002a54                HSEM1_IRQHandler
                0x08002a54                I2C2_EV_IRQHandler
                0x08002a54                DMA1_Stream2_IRQHandler
                0x08002a54                FPU_IRQHandler
                0x08002a54                OTG_HS_WKUP_IRQHandler
                0x08002a54                FDCAN1_IT1_IRQHandler
                0x08002a54                LTDC_ER_IRQHandler
                0x08002a54                DMA2_Stream2_IRQHandler
                0x08002a54                HRTIM1_TIME_IRQHandler
                0x08002a54                SPI1_IRQHandler
                0x08002a54                TIM6_DAC_IRQHandler
                0x08002a54                DCMI_IRQHandler
                0x08002a54                HRTIM1_TIMC_IRQHandler
                0x08002a54                DMA2_Stream3_IRQHandler
                0x08002a54                SAI2_IRQHandler
                0x08002a54                DFSDM1_FLT3_IRQHandler
                0x08002a54                USART6_IRQHandler
                0x08002a54                TIM17_IRQHandler
                0x08002a54                USART3_IRQHandler
                0x08002a54                BDMA_Channel7_IRQHandler
                0x08002a54                CRYP_IRQHandler
                0x08002a54                LPTIM5_IRQHandler
                0x08002a54                UART5_IRQHandler
                0x08002a54                ADC3_IRQHandler
                0x08002a54                DMA2_Stream0_IRQHandler
                0x08002a54                TIM4_IRQHandler
                0x08002a54                BDMA_Channel2_IRQHandler
                0x08002a54                QUADSPI_IRQHandler
                0x08002a54                I2C1_EV_IRQHandler
                0x08002a54                DMA1_Stream6_IRQHandler
                0x08002a54                DMAMUX1_OVR_IRQHandler
                0x08002a54                DMA1_Stream1_IRQHandler
                0x08002a54                TIM16_IRQHandler
                0x08002a54                UART4_IRQHandler
                0x08002a54                BDMA_Channel5_IRQHandler
                0x08002a54                TIM3_IRQHandler
                0x08002a54                RCC_IRQHandler
                0x08002a54                TIM8_BRK_TIM12_IRQHandler
                0x08002a54                TIM1_TRG_COM_IRQHandler
                0x08002a54                Default_Handler
                0x08002a54                ECC_IRQHandler
                0x08002a54                CEC_IRQHandler
                0x08002a54                EXTI15_10_IRQHandler
                0x08002a54                BDMA_Channel0_IRQHandler
                0x08002a54                ADC_IRQHandler
                0x08002a54                DMA1_Stream7_IRQHandler
                0x08002a54                HRTIM1_TIMA_IRQHandler
                0x08002a54                SPI5_IRQHandler
                0x08002a54                TIM7_IRQHandler
                0x08002a54                SDMMC1_IRQHandler
                0x08002a54                TIM5_IRQHandler
                0x08002a54                DMA2_Stream7_IRQHandler
                0x08002a54                TIM15_IRQHandler
                0x08002a54                PVD_AVD_IRQHandler
                0x08002a54                I2C3_EV_IRQHandler
                0x08002a54                EXTI9_5_IRQHandler
                0x08002a54                RTC_WKUP_IRQHandler
                0x08002a54                LTDC_IRQHandler
                0x08002a54                SAI3_IRQHandler
                0x08002a54                ETH_WKUP_IRQHandler
                0x08002a54                SPDIF_RX_IRQHandler
                0x08002a54                SPI2_IRQHandler
                0x08002a54                OTG_HS_EP1_IN_IRQHandler
                0x08002a54                CRS_IRQHandler
                0x08002a54                EXTI4_IRQHandler
                0x08002a54                HRTIM1_TIMB_IRQHandler
                0x08002a54                FDCAN2_IT1_IRQHandler
                0x08002a54                ETH_IRQHandler
                0x08002a54                TIM1_UP_IRQHandler
                0x08002a54                BDMA_Channel4_IRQHandler
                0x08002a54                OTG_HS_EP1_OUT_IRQHandler
                0x08002a54                WWDG_IRQHandler
                0x08002a54                SPI6_IRQHandler
                0x08002a54                MDIOS_IRQHandler
                0x08002a54                I2C4_EV_IRQHandler
                0x08002a54                FDCAN2_IT0_IRQHandler
                0x08002a54                LPUART1_IRQHandler
                0x08002a54                FDCAN1_IT0_IRQHandler
                0x08002a54                TIM2_IRQHandler
                0x08002a54                OTG_FS_WKUP_IRQHandler
                0x08002a54                OTG_HS_IRQHandler
                0x08002a54                DMA2D_IRQHandler
                0x08002a54                TIM1_BRK_IRQHandler
                0x08002a54                EXTI1_IRQHandler
                0x08002a54                SDMMC2_IRQHandler
                0x08002a54                OTG_FS_EP1_OUT_IRQHandler
                0x08002a54                BDMA_Channel3_IRQHandler
                0x08002a54                UART7_IRQHandler
                0x08002a54                MDIOS_WKUP_IRQHandler
                0x08002a54                USART2_IRQHandler
                0x08002a54                DFSDM1_FLT0_IRQHandler
                0x08002a54                SAI4_IRQHandler
                0x08002a54                I2C2_ER_IRQHandler
                0x08002a54                DMA2_Stream1_IRQHandler
                0x08002a54                FLASH_IRQHandler
                0x08002a54                DMA2_Stream4_IRQHandler
                0x08002a54                OTG_FS_IRQHandler
                0x08002a54                SPI3_IRQHandler
                0x08002a54                WAKEUP_PIN_IRQHandler
                0x08002a54                DMA1_Stream4_IRQHandler
                0x08002a54                OTG_FS_EP1_IN_IRQHandler
                0x08002a54                I2C1_ER_IRQHandler
                0x08002a54                FMC_IRQHandler
                0x08002a54                FDCAN_CAL_IRQHandler
                0x08002a54                SWPMI1_IRQHandler
                0x08002a54                COMP1_IRQHandler
                0x08002a54                LPTIM1_IRQHandler
                0x08002a54                I2C4_ER_IRQHandler
                0x08002a54                DMA2_Stream6_IRQHandler
                0x08002a54                SAI1_IRQHandler
                0x08002a54                DMA1_Stream3_IRQHandler
 *fill*         0x08002a56        0x2 
 .text.HAL_InitTick
                0x08002a58       0x50 CMakeFiles/H750_S15909.elf.dir/Drivers/STM32H7xx_HAL_Driver/Src/stm32h7xx_hal.c.obj
                0x08002a58                HAL_InitTick
 .text.HAL_Init
                0x08002aa8       0x5c CMakeFiles/H750_S15909.elf.dir/Drivers/STM32H7xx_HAL_Driver/Src/stm32h7xx_hal.c.obj
                0x08002aa8                HAL_Init
 .text.HAL_IncTick
                0x08002b04       0x18 CMakeFiles/H750_S15909.elf.dir/Drivers/STM32H7xx_HAL_Driver/Src/stm32h7xx_hal.c.obj
                0x08002b04                HAL_IncTick
 .text.HAL_GetTick
                0x08002b1c        0xc CMakeFiles/H750_S15909.elf.dir/Drivers/STM32H7xx_HAL_Driver/Src/stm32h7xx_hal.c.obj
                0x08002b1c                HAL_GetTick
 .text.HAL_Delay
                0x08002b28       0x28 CMakeFiles/H750_S15909.elf.dir/Drivers/STM32H7xx_HAL_Driver/Src/stm32h7xx_hal.c.obj
                0x08002b28                HAL_Delay
 .text.HAL_GetREVID
                0x08002b50        0xc CMakeFiles/H750_S15909.elf.dir/Drivers/STM32H7xx_HAL_Driver/Src/stm32h7xx_hal.c.obj
                0x08002b50                HAL_GetREVID
 .text.HAL_NVIC_SetPriorityGrouping
                0x08002b5c       0x24 CMakeFiles/H750_S15909.elf.dir/Drivers/STM32H7xx_HAL_Driver/Src/stm32h7xx_hal_cortex.c.obj
                0x08002b5c                HAL_NVIC_SetPriorityGrouping
 .text.HAL_NVIC_SetPriority
                0x08002b80       0x6c CMakeFiles/H750_S15909.elf.dir/Drivers/STM32H7xx_HAL_Driver/Src/stm32h7xx_hal_cortex.c.obj
                0x08002b80                HAL_NVIC_SetPriority
 .text.HAL_NVIC_EnableIRQ
                0x08002bec       0x1c CMakeFiles/H750_S15909.elf.dir/Drivers/STM32H7xx_HAL_Driver/Src/stm32h7xx_hal_cortex.c.obj
                0x08002bec                HAL_NVIC_EnableIRQ
 .text.HAL_SYSTICK_Config
                0x08002c08       0x28 CMakeFiles/H750_S15909.elf.dir/Drivers/STM32H7xx_HAL_Driver/Src/stm32h7xx_hal_cortex.c.obj
                0x08002c08                HAL_SYSTICK_Config
 .text.DMA_SetConfig
                0x08002c30      0x1b4 CMakeFiles/H750_S15909.elf.dir/Drivers/STM32H7xx_HAL_Driver/Src/stm32h7xx_hal_dma.c.obj
 .text.DMA_CalcBaseAndBitshift
                0x08002de4       0xb4 CMakeFiles/H750_S15909.elf.dir/Drivers/STM32H7xx_HAL_Driver/Src/stm32h7xx_hal_dma.c.obj
 .text.DMA_CheckFifoParam
                0x08002e98       0x92 CMakeFiles/H750_S15909.elf.dir/Drivers/STM32H7xx_HAL_Driver/Src/stm32h7xx_hal_dma.c.obj
 *fill*         0x08002f2a        0x2 
 .text.DMA_CalcDMAMUXChannelBaseAndMask
                0x08002f2c       0xb0 CMakeFiles/H750_S15909.elf.dir/Drivers/STM32H7xx_HAL_Driver/Src/stm32h7xx_hal_dma.c.obj
 .text.DMA_CalcDMAMUXRequestGenBaseAndMask
                0x08002fdc       0x7c CMakeFiles/H750_S15909.elf.dir/Drivers/STM32H7xx_HAL_Driver/Src/stm32h7xx_hal_dma.c.obj
 .text.HAL_DMA_Init
                0x08003058      0x3a4 CMakeFiles/H750_S15909.elf.dir/Drivers/STM32H7xx_HAL_Driver/Src/stm32h7xx_hal_dma.c.obj
                0x08003058                HAL_DMA_Init
 .text.HAL_DMA_DeInit
                0x080033fc      0x1d4 CMakeFiles/H750_S15909.elf.dir/Drivers/STM32H7xx_HAL_Driver/Src/stm32h7xx_hal_dma.c.obj
                0x080033fc                HAL_DMA_DeInit
 .text.HAL_DMA_Start_IT
                0x080035d0      0x298 CMakeFiles/H750_S15909.elf.dir/Drivers/STM32H7xx_HAL_Driver/Src/stm32h7xx_hal_dma.c.obj
                0x080035d0                HAL_DMA_Start_IT
 .text.HAL_DMA_Abort
                0x08003868      0x340 CMakeFiles/H750_S15909.elf.dir/Drivers/STM32H7xx_HAL_Driver/Src/stm32h7xx_hal_dma.c.obj
                0x08003868                HAL_DMA_Abort
 .text.HAL_DMA_Abort_IT
                0x08003ba8      0x270 CMakeFiles/H750_S15909.elf.dir/Drivers/STM32H7xx_HAL_Driver/Src/stm32h7xx_hal_dma.c.obj
                0x08003ba8                HAL_DMA_Abort_IT
 .text.HAL_DMA_IRQHandler
                0x08003e18      0x738 CMakeFiles/H750_S15909.elf.dir/Drivers/STM32H7xx_HAL_Driver/Src/stm32h7xx_hal_dma.c.obj
                0x08003e18                HAL_DMA_IRQHandler
 .text.HAL_DMA_GetError
                0x08004550        0x4 CMakeFiles/H750_S15909.elf.dir/Drivers/STM32H7xx_HAL_Driver/Src/stm32h7xx_hal_dma.c.obj
                0x08004550                HAL_DMA_GetError
 .text.HAL_GPIO_Init
                0x08004554      0x228 CMakeFiles/H750_S15909.elf.dir/Drivers/STM32H7xx_HAL_Driver/Src/stm32h7xx_hal_gpio.c.obj
                0x08004554                HAL_GPIO_Init
 .text.HAL_GPIO_ReadPin
                0x0800477c        0xe CMakeFiles/H750_S15909.elf.dir/Drivers/STM32H7xx_HAL_Driver/Src/stm32h7xx_hal_gpio.c.obj
                0x0800477c                HAL_GPIO_ReadPin
 .text.HAL_GPIO_WritePin
                0x0800478a        0xc CMakeFiles/H750_S15909.elf.dir/Drivers/STM32H7xx_HAL_Driver/Src/stm32h7xx_hal_gpio.c.obj
                0x0800478a                HAL_GPIO_WritePin
 .text.HAL_GPIO_EXTI_IRQHandler
                0x08004796       0x1e CMakeFiles/H750_S15909.elf.dir/Drivers/STM32H7xx_HAL_Driver/Src/stm32h7xx_hal_gpio.c.obj
                0x08004796                HAL_GPIO_EXTI_IRQHandler
 .text.HAL_PWREx_ConfigSupply
                0x080047b4       0x54 CMakeFiles/H750_S15909.elf.dir/Drivers/STM32H7xx_HAL_Driver/Src/stm32h7xx_hal_pwr_ex.c.obj
                0x080047b4                HAL_PWREx_ConfigSupply
 .text.HAL_RCC_OscConfig
                0x08004808      0x674 CMakeFiles/H750_S15909.elf.dir/Drivers/STM32H7xx_HAL_Driver/Src/stm32h7xx_hal_rcc.c.obj
                0x08004808                HAL_RCC_OscConfig
 .text.HAL_RCC_GetSysClockFreq
                0x08004e7c      0x218 CMakeFiles/H750_S15909.elf.dir/Drivers/STM32H7xx_HAL_Driver/Src/stm32h7xx_hal_rcc.c.obj
                0x08004e7c                HAL_RCC_GetSysClockFreq
 .text.HAL_RCC_ClockConfig
                0x08005094      0x294 CMakeFiles/H750_S15909.elf.dir/Drivers/STM32H7xx_HAL_Driver/Src/stm32h7xx_hal_rcc.c.obj
                0x08005094                HAL_RCC_ClockConfig
 .text.HAL_RCC_GetHCLKFreq
                0x08005328       0x44 CMakeFiles/H750_S15909.elf.dir/Drivers/STM32H7xx_HAL_Driver/Src/stm32h7xx_hal_rcc.c.obj
                0x08005328                HAL_RCC_GetHCLKFreq
 .text.HAL_RCC_GetPCLK1Freq
                0x0800536c       0x24 CMakeFiles/H750_S15909.elf.dir/Drivers/STM32H7xx_HAL_Driver/Src/stm32h7xx_hal_rcc.c.obj
                0x0800536c                HAL_RCC_GetPCLK1Freq
 .text.HAL_RCC_GetPCLK2Freq
                0x08005390       0x24 CMakeFiles/H750_S15909.elf.dir/Drivers/STM32H7xx_HAL_Driver/Src/stm32h7xx_hal_rcc.c.obj
                0x08005390                HAL_RCC_GetPCLK2Freq
 .text.RCCEx_PLL2_Config
                0x080053b4      0x10c CMakeFiles/H750_S15909.elf.dir/Drivers/STM32H7xx_HAL_Driver/Src/stm32h7xx_hal_rcc_ex.c.obj
 .text.RCCEx_PLL3_Config
                0x080054c0      0x10c CMakeFiles/H750_S15909.elf.dir/Drivers/STM32H7xx_HAL_Driver/Src/stm32h7xx_hal_rcc_ex.c.obj
 .text.HAL_RCCEx_PeriphCLKConfig
                0x080055cc      0x9c4 CMakeFiles/H750_S15909.elf.dir/Drivers/STM32H7xx_HAL_Driver/Src/stm32h7xx_hal_rcc_ex.c.obj
                0x080055cc                HAL_RCCEx_PeriphCLKConfig
 .text.HAL_RCCEx_GetD3PCLK1Freq
                0x08005f90       0x24 CMakeFiles/H750_S15909.elf.dir/Drivers/STM32H7xx_HAL_Driver/Src/stm32h7xx_hal_rcc_ex.c.obj
                0x08005f90                HAL_RCCEx_GetD3PCLK1Freq
 .text.HAL_RCCEx_GetPLL2ClockFreq
                0x08005fb4      0x234 CMakeFiles/H750_S15909.elf.dir/Drivers/STM32H7xx_HAL_Driver/Src/stm32h7xx_hal_rcc_ex.c.obj
                0x08005fb4                HAL_RCCEx_GetPLL2ClockFreq
 .text.HAL_RCCEx_GetPLL3ClockFreq
                0x080061e8      0x234 CMakeFiles/H750_S15909.elf.dir/Drivers/STM32H7xx_HAL_Driver/Src/stm32h7xx_hal_rcc_ex.c.obj
                0x080061e8                HAL_RCCEx_GetPLL3ClockFreq
 .text.TIM_TI1_ConfigInputStage
                0x0800641c       0x24 CMakeFiles/H750_S15909.elf.dir/Drivers/STM32H7xx_HAL_Driver/Src/stm32h7xx_hal_tim.c.obj
 .text.TIM_TI2_ConfigInputStage
                0x08006440       0x26 CMakeFiles/H750_S15909.elf.dir/Drivers/STM32H7xx_HAL_Driver/Src/stm32h7xx_hal_tim.c.obj
 *fill*         0x08006466        0x2 
 .text.TIM_ITRx_SetConfig
                0x08006468       0x14 CMakeFiles/H750_S15909.elf.dir/Drivers/STM32H7xx_HAL_Driver/Src/stm32h7xx_hal_tim.c.obj
 .text.HAL_TIM_Base_Start
                0x0800647c       0x88 CMakeFiles/H750_S15909.elf.dir/Drivers/STM32H7xx_HAL_Driver/Src/stm32h7xx_hal_tim.c.obj
                0x0800647c                HAL_TIM_Base_Start
 .text.TIM_Base_SetConfig
                0x08006504      0x104 CMakeFiles/H750_S15909.elf.dir/Drivers/STM32H7xx_HAL_Driver/Src/stm32h7xx_hal_tim.c.obj
                0x08006504                TIM_Base_SetConfig
 .text.HAL_TIM_Base_Init
                0x08006608       0x60 CMakeFiles/H750_S15909.elf.dir/Drivers/STM32H7xx_HAL_Driver/Src/stm32h7xx_hal_tim.c.obj
                0x08006608                HAL_TIM_Base_Init
 .text.TIM_ETR_SetConfig
                0x08006668       0x18 CMakeFiles/H750_S15909.elf.dir/Drivers/STM32H7xx_HAL_Driver/Src/stm32h7xx_hal_tim.c.obj
                0x08006668                TIM_ETR_SetConfig
 .text.HAL_TIM_ConfigClockSource
                0x08006680      0x138 CMakeFiles/H750_S15909.elf.dir/Drivers/STM32H7xx_HAL_Driver/Src/stm32h7xx_hal_tim.c.obj
                0x08006680                HAL_TIM_ConfigClockSource
 .text.HAL_TIMEx_MasterConfigSynchronization
                0x080067b8       0xa0 CMakeFiles/H750_S15909.elf.dir/Drivers/STM32H7xx_HAL_Driver/Src/stm32h7xx_hal_tim_ex.c.obj
                0x080067b8                HAL_TIMEx_MasterConfigSynchronization
 .text.UART_EndTxTransfer
                0x08006858       0x32 CMakeFiles/H750_S15909.elf.dir/Drivers/STM32H7xx_HAL_Driver/Src/stm32h7xx_hal_uart.c.obj
 *fill*         0x0800688a        0x2 
 .text.UART_EndRxTransfer
                0x0800688c       0x58 CMakeFiles/H750_S15909.elf.dir/Drivers/STM32H7xx_HAL_Driver/Src/stm32h7xx_hal_uart.c.obj
 .text.HAL_UART_Transmit_DMA
                0x080068e4       0xb8 CMakeFiles/H750_S15909.elf.dir/Drivers/STM32H7xx_HAL_Driver/Src/stm32h7xx_hal_uart.c.obj
                0x080068e4                HAL_UART_Transmit_DMA
 .text.HAL_UART_DMAStop
                0x0800699c       0xae CMakeFiles/H750_S15909.elf.dir/Drivers/STM32H7xx_HAL_Driver/Src/stm32h7xx_hal_uart.c.obj
                0x0800699c                HAL_UART_DMAStop
 .text.HAL_UART_TxCpltCallback
                0x08006a4a        0x2 CMakeFiles/H750_S15909.elf.dir/Drivers/STM32H7xx_HAL_Driver/Src/stm32h7xx_hal_uart.c.obj
                0x08006a4a                HAL_UART_TxCpltCallback
 .text.UART_DMATransmitCplt
                0x08006a4c       0x46 CMakeFiles/H750_S15909.elf.dir/Drivers/STM32H7xx_HAL_Driver/Src/stm32h7xx_hal_uart.c.obj
 .text.UART_EndTransmit_IT
                0x08006a92       0x24 CMakeFiles/H750_S15909.elf.dir/Drivers/STM32H7xx_HAL_Driver/Src/stm32h7xx_hal_uart.c.obj
 .text.HAL_UART_TxHalfCpltCallback
                0x08006ab6        0x2 CMakeFiles/H750_S15909.elf.dir/Drivers/STM32H7xx_HAL_Driver/Src/stm32h7xx_hal_uart.c.obj
                0x08006ab6                HAL_UART_TxHalfCpltCallback
 .text.UART_DMATxHalfCplt
                0x08006ab8        0xa CMakeFiles/H750_S15909.elf.dir/Drivers/STM32H7xx_HAL_Driver/Src/stm32h7xx_hal_uart.c.obj
 .text.HAL_UART_RxHalfCpltCallback
                0x08006ac2        0x2 CMakeFiles/H750_S15909.elf.dir/Drivers/STM32H7xx_HAL_Driver/Src/stm32h7xx_hal_uart.c.obj
                0x08006ac2                HAL_UART_RxHalfCpltCallback
 .text.HAL_UART_ErrorCallback
                0x08006ac4        0x2 CMakeFiles/H750_S15909.elf.dir/Drivers/STM32H7xx_HAL_Driver/Src/stm32h7xx_hal_uart.c.obj
                0x08006ac4                HAL_UART_ErrorCallback
 .text.UART_DMAError
                0x08006ac6       0x58 CMakeFiles/H750_S15909.elf.dir/Drivers/STM32H7xx_HAL_Driver/Src/stm32h7xx_hal_uart.c.obj
 .text.UART_DMAAbortOnError
                0x08006b1e       0x14 CMakeFiles/H750_S15909.elf.dir/Drivers/STM32H7xx_HAL_Driver/Src/stm32h7xx_hal_uart.c.obj
 .text.HAL_UARTEx_RxEventCallback
                0x08006b32        0x2 CMakeFiles/H750_S15909.elf.dir/Drivers/STM32H7xx_HAL_Driver/Src/stm32h7xx_hal_uart.c.obj
                0x08006b32                HAL_UARTEx_RxEventCallback
 .text.HAL_UART_IRQHandler
                0x08006b34      0x3a8 CMakeFiles/H750_S15909.elf.dir/Drivers/STM32H7xx_HAL_Driver/Src/stm32h7xx_hal_uart.c.obj
                0x08006b34                HAL_UART_IRQHandler
 .text.UART_RxISR_8BIT
                0x08006edc       0xb2 CMakeFiles/H750_S15909.elf.dir/Drivers/STM32H7xx_HAL_Driver/Src/stm32h7xx_hal_uart.c.obj
 .text.UART_RxISR_16BIT
                0x08006f8e       0xb0 CMakeFiles/H750_S15909.elf.dir/Drivers/STM32H7xx_HAL_Driver/Src/stm32h7xx_hal_uart.c.obj
 *fill*         0x0800703e        0x2 
 .text.UART_RxISR_8BIT_FIFOEN
                0x08007040      0x1a0 CMakeFiles/H750_S15909.elf.dir/Drivers/STM32H7xx_HAL_Driver/Src/stm32h7xx_hal_uart.c.obj
 .text.UART_RxISR_16BIT_FIFOEN
                0x080071e0      0x19c CMakeFiles/H750_S15909.elf.dir/Drivers/STM32H7xx_HAL_Driver/Src/stm32h7xx_hal_uart.c.obj
 .text.UART_DMARxHalfCplt
                0x0800737c       0x1c CMakeFiles/H750_S15909.elf.dir/Drivers/STM32H7xx_HAL_Driver/Src/stm32h7xx_hal_uart.c.obj
 .text.UART_DMAReceiveCplt
                0x08007398       0x8c CMakeFiles/H750_S15909.elf.dir/Drivers/STM32H7xx_HAL_Driver/Src/stm32h7xx_hal_uart.c.obj
 .text.UART_SetConfig
                0x08007424      0x5f4 CMakeFiles/H750_S15909.elf.dir/Drivers/STM32H7xx_HAL_Driver/Src/stm32h7xx_hal_uart.c.obj
                0x08007424                UART_SetConfig
 .text.UART_AdvFeatureConfig
                0x08007a18       0xca CMakeFiles/H750_S15909.elf.dir/Drivers/STM32H7xx_HAL_Driver/Src/stm32h7xx_hal_uart.c.obj
                0x08007a18                UART_AdvFeatureConfig
 .text.UART_WaitOnFlagUntilTimeout
                0x08007ae2       0xdc CMakeFiles/H750_S15909.elf.dir/Drivers/STM32H7xx_HAL_Driver/Src/stm32h7xx_hal_uart.c.obj
                0x08007ae2                UART_WaitOnFlagUntilTimeout
 .text.HAL_UART_Transmit
                0x08007bbe       0xda CMakeFiles/H750_S15909.elf.dir/Drivers/STM32H7xx_HAL_Driver/Src/stm32h7xx_hal_uart.c.obj
                0x08007bbe                HAL_UART_Transmit
 .text.UART_CheckIdleState
                0x08007c98       0x74 CMakeFiles/H750_S15909.elf.dir/Drivers/STM32H7xx_HAL_Driver/Src/stm32h7xx_hal_uart.c.obj
                0x08007c98                UART_CheckIdleState
 .text.HAL_UART_Init
                0x08007d0c       0x66 CMakeFiles/H750_S15909.elf.dir/Drivers/STM32H7xx_HAL_Driver/Src/stm32h7xx_hal_uart.c.obj
                0x08007d0c                HAL_UART_Init
 *fill*         0x08007d72        0x2 
 .text.UART_Start_Receive_IT
                0x08007d74      0x148 CMakeFiles/H750_S15909.elf.dir/Drivers/STM32H7xx_HAL_Driver/Src/stm32h7xx_hal_uart.c.obj
                0x08007d74                UART_Start_Receive_IT
 .text.HAL_UART_Receive_IT
                0x08007ebc       0x5c CMakeFiles/H750_S15909.elf.dir/Drivers/STM32H7xx_HAL_Driver/Src/stm32h7xx_hal_uart.c.obj
                0x08007ebc                HAL_UART_Receive_IT
 .text.UART_Start_Receive_DMA
                0x08007f18       0xb4 CMakeFiles/H750_S15909.elf.dir/Drivers/STM32H7xx_HAL_Driver/Src/stm32h7xx_hal_uart.c.obj
                0x08007f18                UART_Start_Receive_DMA
 .text.HAL_UART_Receive_DMA
                0x08007fcc       0x5c CMakeFiles/H750_S15909.elf.dir/Drivers/STM32H7xx_HAL_Driver/Src/stm32h7xx_hal_uart.c.obj
                0x08007fcc                HAL_UART_Receive_DMA
 .text.UARTEx_SetNbDataToProcess
                0x08008028       0x4c CMakeFiles/H750_S15909.elf.dir/Drivers/STM32H7xx_HAL_Driver/Src/stm32h7xx_hal_uart_ex.c.obj
 .text.HAL_UARTEx_WakeupCallback
                0x08008074        0x2 CMakeFiles/H750_S15909.elf.dir/Drivers/STM32H7xx_HAL_Driver/Src/stm32h7xx_hal_uart_ex.c.obj
                0x08008074                HAL_UARTEx_WakeupCallback
 .text.HAL_UARTEx_RxFifoFullCallback
                0x08008076        0x2 CMakeFiles/H750_S15909.elf.dir/Drivers/STM32H7xx_HAL_Driver/Src/stm32h7xx_hal_uart_ex.c.obj
                0x08008076                HAL_UARTEx_RxFifoFullCallback
 .text.HAL_UARTEx_TxFifoEmptyCallback
                0x08008078        0x2 CMakeFiles/H750_S15909.elf.dir/Drivers/STM32H7xx_HAL_Driver/Src/stm32h7xx_hal_uart_ex.c.obj
                0x08008078                HAL_UARTEx_TxFifoEmptyCallback
 .text.HAL_UARTEx_DisableFifoMode
                0x0800807a       0x3e CMakeFiles/H750_S15909.elf.dir/Drivers/STM32H7xx_HAL_Driver/Src/stm32h7xx_hal_uart_ex.c.obj
                0x0800807a                HAL_UARTEx_DisableFifoMode
 .text.HAL_UARTEx_SetTxFifoThreshold
                0x080080b8       0x4a CMakeFiles/H750_S15909.elf.dir/Drivers/STM32H7xx_HAL_Driver/Src/stm32h7xx_hal_uart_ex.c.obj
                0x080080b8                HAL_UARTEx_SetTxFifoThreshold
 .text.HAL_UARTEx_SetRxFifoThreshold
                0x08008102       0x4a CMakeFiles/H750_S15909.elf.dir/Drivers/STM32H7xx_HAL_Driver/Src/stm32h7xx_hal_uart_ex.c.obj
                0x08008102                HAL_UARTEx_SetRxFifoThreshold
 .text.__errno  0x0800814c        0xc d:/lijie_tools/clion_cubemx/gcc-arm-none-eabi-10.3-2021.10/bin/../lib/gcc/arm-none-eabi/10.3.1/../../../../arm-none-eabi/lib/thumb/v7e-m/nofp\libg.a(lib_a-errno.o)
                0x0800814c                __errno
 .text.__libc_init_array
                0x08008158       0x48 d:/lijie_tools/clion_cubemx/gcc-arm-none-eabi-10.3-2021.10/bin/../lib/gcc/arm-none-eabi/10.3.1/../../../../arm-none-eabi/lib/thumb/v7e-m/nofp\libg.a(lib_a-init.o)
                0x08008158                __libc_init_array
 .text.memset   0x080081a0       0xa4 d:/lijie_tools/clion_cubemx/gcc-arm-none-eabi-10.3-2021.10/bin/../lib/gcc/arm-none-eabi/10.3.1/../../../../arm-none-eabi/lib/thumb/v7e-m/nofp\libg.a(lib_a-memset.o)
                0x080081a0                memset
 .text.setvbuf  0x08008244      0x1b0 d:/lijie_tools/clion_cubemx/gcc-arm-none-eabi-10.3-2021.10/bin/../lib/gcc/arm-none-eabi/10.3.1/../../../../arm-none-eabi/lib/thumb/v7e-m/nofp\libg.a(lib_a-setvbuf.o)
                0x08008244                setvbuf
 .text.startup.register_fini
                0x080083f4       0x14 d:/lijie_tools/clion_cubemx/gcc-arm-none-eabi-10.3-2021.10/bin/../lib/gcc/arm-none-eabi/10.3.1/../../../../arm-none-eabi/lib/thumb/v7e-m/nofp\libg.a(lib_a-__call_atexit.o)
 .text.atexit   0x08008408        0xc d:/lijie_tools/clion_cubemx/gcc-arm-none-eabi-10.3-2021.10/bin/../lib/gcc/arm-none-eabi/10.3.1/../../../../arm-none-eabi/lib/thumb/v7e-m/nofp\libg.a(lib_a-atexit.o)
                0x08008408                atexit
 .text.__sflush_r
                0x08008414      0x120 d:/lijie_tools/clion_cubemx/gcc-arm-none-eabi-10.3-2021.10/bin/../lib/gcc/arm-none-eabi/10.3.1/../../../../arm-none-eabi/lib/thumb/v7e-m/nofp\libg.a(lib_a-fflush.o)
                0x08008414                __sflush_r
 .text._fflush_r
                0x08008534       0x5c d:/lijie_tools/clion_cubemx/gcc-arm-none-eabi-10.3-2021.10/bin/../lib/gcc/arm-none-eabi/10.3.1/../../../../arm-none-eabi/lib/thumb/v7e-m/nofp\libg.a(lib_a-fflush.o)
                0x08008534                _fflush_r
 .text._cleanup_r
                0x08008590        0xc d:/lijie_tools/clion_cubemx/gcc-arm-none-eabi-10.3-2021.10/bin/../lib/gcc/arm-none-eabi/10.3.1/../../../../arm-none-eabi/lib/thumb/v7e-m/nofp\libg.a(lib_a-findfp.o)
                0x08008590                _cleanup_r
 .text.__sinit  0x0800859c      0x10c d:/lijie_tools/clion_cubemx/gcc-arm-none-eabi-10.3-2021.10/bin/../lib/gcc/arm-none-eabi/10.3.1/../../../../arm-none-eabi/lib/thumb/v7e-m/nofp\libg.a(lib_a-findfp.o)
                0x0800859c                __sinit
 .text.__sfp_lock_acquire
                0x080086a8        0xc d:/lijie_tools/clion_cubemx/gcc-arm-none-eabi-10.3-2021.10/bin/../lib/gcc/arm-none-eabi/10.3.1/../../../../arm-none-eabi/lib/thumb/v7e-m/nofp\libg.a(lib_a-findfp.o)
                0x080086a8                __sfp_lock_acquire
 .text.__sfp_lock_release
                0x080086b4        0xc d:/lijie_tools/clion_cubemx/gcc-arm-none-eabi-10.3-2021.10/bin/../lib/gcc/arm-none-eabi/10.3.1/../../../../arm-none-eabi/lib/thumb/v7e-m/nofp\libg.a(lib_a-findfp.o)
                0x080086b4                __sfp_lock_release
 .text.__libc_fini_array
                0x080086c0       0x2c d:/lijie_tools/clion_cubemx/gcc-arm-none-eabi-10.3-2021.10/bin/../lib/gcc/arm-none-eabi/10.3.1/../../../../arm-none-eabi/lib/thumb/v7e-m/nofp\libg.a(lib_a-fini.o)
                0x080086c0                __libc_fini_array
 .text._malloc_trim_r
                0x080086ec       0xa0 d:/lijie_tools/clion_cubemx/gcc-arm-none-eabi-10.3-2021.10/bin/../lib/gcc/arm-none-eabi/10.3.1/../../../../arm-none-eabi/lib/thumb/v7e-m/nofp\libg.a(lib_a-freer.o)
                0x080086ec                _malloc_trim_r
 .text._free_r  0x0800878c      0x20c d:/lijie_tools/clion_cubemx/gcc-arm-none-eabi-10.3-2021.10/bin/../lib/gcc/arm-none-eabi/10.3.1/../../../../arm-none-eabi/lib/thumb/v7e-m/nofp\libg.a(lib_a-freer.o)
                0x0800878c                _free_r
 .text._fwalk_reent
                0x08008998       0x48 d:/lijie_tools/clion_cubemx/gcc-arm-none-eabi-10.3-2021.10/bin/../lib/gcc/arm-none-eabi/10.3.1/../../../../arm-none-eabi/lib/thumb/v7e-m/nofp\libg.a(lib_a-fwalk.o)
                0x08008998                _fwalk_reent
 .text.__retarget_lock_init_recursive
                0x080089e0        0x4 d:/lijie_tools/clion_cubemx/gcc-arm-none-eabi-10.3-2021.10/bin/../lib/gcc/arm-none-eabi/10.3.1/../../../../arm-none-eabi/lib/thumb/v7e-m/nofp\libg.a(lib_a-lock.o)
                0x080089e0                __retarget_lock_init_recursive
 .text.__retarget_lock_close_recursive
                0x080089e4        0x4 d:/lijie_tools/clion_cubemx/gcc-arm-none-eabi-10.3-2021.10/bin/../lib/gcc/arm-none-eabi/10.3.1/../../../../arm-none-eabi/lib/thumb/v7e-m/nofp\libg.a(lib_a-lock.o)
                0x080089e4                __retarget_lock_close_recursive
 .text.__retarget_lock_acquire_recursive
                0x080089e8        0x4 d:/lijie_tools/clion_cubemx/gcc-arm-none-eabi-10.3-2021.10/bin/../lib/gcc/arm-none-eabi/10.3.1/../../../../arm-none-eabi/lib/thumb/v7e-m/nofp\libg.a(lib_a-lock.o)
                0x080089e8                __retarget_lock_acquire_recursive
 .text.__retarget_lock_release_recursive
                0x080089ec        0x4 d:/lijie_tools/clion_cubemx/gcc-arm-none-eabi-10.3-2021.10/bin/../lib/gcc/arm-none-eabi/10.3.1/../../../../arm-none-eabi/lib/thumb/v7e-m/nofp\libg.a(lib_a-lock.o)
                0x080089ec                __retarget_lock_release_recursive
 .text.__swhatbuf_r
                0x080089f0       0x60 d:/lijie_tools/clion_cubemx/gcc-arm-none-eabi-10.3-2021.10/bin/../lib/gcc/arm-none-eabi/10.3.1/../../../../arm-none-eabi/lib/thumb/v7e-m/nofp\libg.a(lib_a-makebuf.o)
                0x080089f0                __swhatbuf_r
 .text.malloc   0x08008a50       0x10 d:/lijie_tools/clion_cubemx/gcc-arm-none-eabi-10.3-2021.10/bin/../lib/gcc/arm-none-eabi/10.3.1/../../../../arm-none-eabi/lib/thumb/v7e-m/nofp\libg.a(lib_a-malloc.o)
                0x08008a50                malloc
 .text._malloc_r
                0x08008a60      0x560 d:/lijie_tools/clion_cubemx/gcc-arm-none-eabi-10.3-2021.10/bin/../lib/gcc/arm-none-eabi/10.3.1/../../../../arm-none-eabi/lib/thumb/v7e-m/nofp\libg.a(lib_a-mallocr.o)
                0x08008a60                _malloc_r
 .text.__malloc_lock
                0x08008fc0        0xc d:/lijie_tools/clion_cubemx/gcc-arm-none-eabi-10.3-2021.10/bin/../lib/gcc/arm-none-eabi/10.3.1/../../../../arm-none-eabi/lib/thumb/v7e-m/nofp\libg.a(lib_a-mlock.o)
                0x08008fc0                __malloc_lock
 .text.__malloc_unlock
                0x08008fcc        0xc d:/lijie_tools/clion_cubemx/gcc-arm-none-eabi-10.3-2021.10/bin/../lib/gcc/arm-none-eabi/10.3.1/../../../../arm-none-eabi/lib/thumb/v7e-m/nofp\libg.a(lib_a-mlock.o)
                0x08008fcc                __malloc_unlock
 .text._sbrk_r  0x08008fd8       0x24 d:/lijie_tools/clion_cubemx/gcc-arm-none-eabi-10.3-2021.10/bin/../lib/gcc/arm-none-eabi/10.3.1/../../../../arm-none-eabi/lib/thumb/v7e-m/nofp\libg.a(lib_a-sbrkr.o)
                0x08008fd8                _sbrk_r
 .text.__sread  0x08008ffc       0x24 d:/lijie_tools/clion_cubemx/gcc-arm-none-eabi-10.3-2021.10/bin/../lib/gcc/arm-none-eabi/10.3.1/../../../../arm-none-eabi/lib/thumb/v7e-m/nofp\libg.a(lib_a-stdio.o)
                0x08008ffc                __sread
 .text.__swrite
                0x08009020       0x40 d:/lijie_tools/clion_cubemx/gcc-arm-none-eabi-10.3-2021.10/bin/../lib/gcc/arm-none-eabi/10.3.1/../../../../arm-none-eabi/lib/thumb/v7e-m/nofp\libg.a(lib_a-stdio.o)
                0x08009020                __swrite
 .text.__sseek  0x08009060       0x20 d:/lijie_tools/clion_cubemx/gcc-arm-none-eabi-10.3-2021.10/bin/../lib/gcc/arm-none-eabi/10.3.1/../../../../arm-none-eabi/lib/thumb/v7e-m/nofp\libg.a(lib_a-stdio.o)
                0x08009060                __sseek
 .text.__sclose
                0x08009080        0x8 d:/lijie_tools/clion_cubemx/gcc-arm-none-eabi-10.3-2021.10/bin/../lib/gcc/arm-none-eabi/10.3.1/../../../../arm-none-eabi/lib/thumb/v7e-m/nofp\libg.a(lib_a-stdio.o)
                0x08009080                __sclose
 .text._write_r
                0x08009088       0x2c d:/lijie_tools/clion_cubemx/gcc-arm-none-eabi-10.3-2021.10/bin/../lib/gcc/arm-none-eabi/10.3.1/../../../../arm-none-eabi/lib/thumb/v7e-m/nofp\libg.a(lib_a-writer.o)
                0x08009088                _write_r
 .text.__register_exitproc
                0x080090b4       0x8c d:/lijie_tools/clion_cubemx/gcc-arm-none-eabi-10.3-2021.10/bin/../lib/gcc/arm-none-eabi/10.3.1/../../../../arm-none-eabi/lib/thumb/v7e-m/nofp\libg.a(lib_a-__atexit.o)
                0x080090b4                __register_exitproc
 .text._close_r
                0x08009140       0x24 d:/lijie_tools/clion_cubemx/gcc-arm-none-eabi-10.3-2021.10/bin/../lib/gcc/arm-none-eabi/10.3.1/../../../../arm-none-eabi/lib/thumb/v7e-m/nofp\libg.a(lib_a-closer.o)
                0x08009140                _close_r
 .text._fclose_r
                0x08009164       0xcc d:/lijie_tools/clion_cubemx/gcc-arm-none-eabi-10.3-2021.10/bin/../lib/gcc/arm-none-eabi/10.3.1/../../../../arm-none-eabi/lib/thumb/v7e-m/nofp\libg.a(lib_a-fclose.o)
                0x08009164                _fclose_r
 .text._fstat_r
                0x08009230       0x2c d:/lijie_tools/clion_cubemx/gcc-arm-none-eabi-10.3-2021.10/bin/../lib/gcc/arm-none-eabi/10.3.1/../../../../arm-none-eabi/lib/thumb/v7e-m/nofp\libg.a(lib_a-fstatr.o)
                0x08009230                _fstat_r
 .text._lseek_r
                0x0800925c       0x2c d:/lijie_tools/clion_cubemx/gcc-arm-none-eabi-10.3-2021.10/bin/../lib/gcc/arm-none-eabi/10.3.1/../../../../arm-none-eabi/lib/thumb/v7e-m/nofp\libg.a(lib_a-lseekr.o)
                0x0800925c                _lseek_r
 .text._read_r  0x08009288       0x2c d:/lijie_tools/clion_cubemx/gcc-arm-none-eabi-10.3-2021.10/bin/../lib/gcc/arm-none-eabi/10.3.1/../../../../arm-none-eabi/lib/thumb/v7e-m/nofp\libg.a(lib_a-readr.o)
                0x08009288                _read_r
 .text.round    0x080092b4       0x94 d:/lijie_tools/clion_cubemx/gcc-arm-none-eabi-10.3-2021.10/bin/../lib/gcc/arm-none-eabi/10.3.1/../../../../arm-none-eabi/lib/thumb/v7e-m/nofp\libm.a(lib_a-s_round.o)
                0x080092b4                round
 .text.exp      0x08009348       0x74 d:/lijie_tools/clion_cubemx/gcc-arm-none-eabi-10.3-2021.10/bin/../lib/gcc/arm-none-eabi/10.3.1/../../../../arm-none-eabi/lib/thumb/v7e-m/nofp\libm.a(lib_a-w_exp.o)
                0x08009348                exp
 *fill*         0x080093bc        0x4 
 .text.__ieee754_exp
                0x080093c0      0x3a8 d:/lijie_tools/clion_cubemx/gcc-arm-none-eabi-10.3-2021.10/bin/../lib/gcc/arm-none-eabi/10.3.1/../../../../arm-none-eabi/lib/thumb/v7e-m/nofp\libm.a(lib_a-e_exp.o)
                0x080093c0                __ieee754_exp
 .text.with_errno
                0x08009768       0x18 d:/lijie_tools/clion_cubemx/gcc-arm-none-eabi-10.3-2021.10/bin/../lib/gcc/arm-none-eabi/10.3.1/../../../../arm-none-eabi/lib/thumb/v7e-m/nofp\libm.a(lib_a-math_err.o)
 .text.xflow    0x08009780       0x30 d:/lijie_tools/clion_cubemx/gcc-arm-none-eabi-10.3-2021.10/bin/../lib/gcc/arm-none-eabi/10.3.1/../../../../arm-none-eabi/lib/thumb/v7e-m/nofp\libm.a(lib_a-math_err.o)
 .text.__math_uflow
                0x080097b0        0xc d:/lijie_tools/clion_cubemx/gcc-arm-none-eabi-10.3-2021.10/bin/../lib/gcc/arm-none-eabi/10.3.1/../../../../arm-none-eabi/lib/thumb/v7e-m/nofp\libm.a(lib_a-math_err.o)
                0x080097b0                __math_uflow
 .text.__math_oflow
                0x080097bc        0xc d:/lijie_tools/clion_cubemx/gcc-arm-none-eabi-10.3-2021.10/bin/../lib/gcc/arm-none-eabi/10.3.1/../../../../arm-none-eabi/lib/thumb/v7e-m/nofp\libm.a(lib_a-math_err.o)
                0x080097bc                __math_oflow
 .text.finite   0x080097c8        0xc d:/lijie_tools/clion_cubemx/gcc-arm-none-eabi-10.3-2021.10/bin/../lib/gcc/arm-none-eabi/10.3.1/../../../../arm-none-eabi/lib/thumb/v7e-m/nofp\libm.a(lib_a-s_finite.o)
                0x080097c8                finite
 *(.glue_7)
 .glue_7        0x080097d4        0x0 linker stubs
 *(.glue_7t)
 .glue_7t       0x080097d4        0x0 linker stubs
 *(.eh_frame)
 .eh_frame      0x080097d4        0x0 d:/lijie_tools/clion_cubemx/gcc-arm-none-eabi-10.3-2021.10/bin/../lib/gcc/arm-none-eabi/10.3.1/thumb/v7e-m/nofp/crtbegin.o
 *(.init)
 .init          0x080097d4        0x4 d:/lijie_tools/clion_cubemx/gcc-arm-none-eabi-10.3-2021.10/bin/../lib/gcc/arm-none-eabi/10.3.1/thumb/v7e-m/nofp/crti.o
                0x080097d4                _init
 .init          0x080097d8        0x8 d:/lijie_tools/clion_cubemx/gcc-arm-none-eabi-10.3-2021.10/bin/../lib/gcc/arm-none-eabi/10.3.1/thumb/v7e-m/nofp/crtn.o
 *(.fini)
 .fini          0x080097e0        0x4 d:/lijie_tools/clion_cubemx/gcc-arm-none-eabi-10.3-2021.10/bin/../lib/gcc/arm-none-eabi/10.3.1/thumb/v7e-m/nofp/crti.o
                0x080097e0                _fini
 .fini          0x080097e4        0x8 d:/lijie_tools/clion_cubemx/gcc-arm-none-eabi-10.3-2021.10/bin/../lib/gcc/arm-none-eabi/10.3.1/thumb/v7e-m/nofp/crtn.o
                0x080097ec                . = ALIGN (0x4)
                0x080097ec                _etext = .

.vfp11_veneer   0x080097ec        0x0
 .vfp11_veneer  0x080097ec        0x0 linker stubs

.v4_bx          0x080097ec        0x0
 .v4_bx         0x080097ec        0x0 linker stubs

.iplt           0x080097ec        0x0
 .iplt          0x080097ec        0x0 d:/lijie_tools/clion_cubemx/gcc-arm-none-eabi-10.3-2021.10/bin/../lib/gcc/arm-none-eabi/10.3.1/thumb/v7e-m/nofp/crtbegin.o

.rodata         0x080097f0       0x78
                0x080097f0                . = ALIGN (0x4)
 *(.rodata)
 *(.rodata*)
 .rodata.D1CorePrescTable
                0x080097f0       0x10 CMakeFiles/H750_S15909.elf.dir/Core/Src/system_stm32h7xx.c.obj
                0x080097f0                D1CorePrescTable
 .rodata.flagBitshiftOffset.0
                0x08009800        0x8 CMakeFiles/H750_S15909.elf.dir/Drivers/STM32H7xx_HAL_Driver/Src/stm32h7xx_hal_dma.c.obj
 .rodata.UARTPrescTable
                0x08009808       0x18 CMakeFiles/H750_S15909.elf.dir/Drivers/STM32H7xx_HAL_Driver/Src/stm32h7xx_hal_uart.c.obj
                0x08009808                UARTPrescTable
 .rodata.denominator.0
                0x08009820        0x8 CMakeFiles/H750_S15909.elf.dir/Drivers/STM32H7xx_HAL_Driver/Src/stm32h7xx_hal_uart_ex.c.obj
 .rodata.numerator.1
                0x08009828        0x8 CMakeFiles/H750_S15909.elf.dir/Drivers/STM32H7xx_HAL_Driver/Src/stm32h7xx_hal_uart_ex.c.obj
 .rodata._global_impure_ptr
                0x08009830        0x4 d:/lijie_tools/clion_cubemx/gcc-arm-none-eabi-10.3-2021.10/bin/../lib/gcc/arm-none-eabi/10.3.1/../../../../arm-none-eabi/lib/thumb/v7e-m/nofp\libg.a(lib_a-impure.o)
                0x08009830                _global_impure_ptr
 *fill*         0x08009834        0x4 
 .rodata.halF   0x08009838       0x10 d:/lijie_tools/clion_cubemx/gcc-arm-none-eabi-10.3-2021.10/bin/../lib/gcc/arm-none-eabi/10.3.1/../../../../arm-none-eabi/lib/thumb/v7e-m/nofp\libm.a(lib_a-e_exp.o)
 .rodata.ln2HI  0x08009848       0x10 d:/lijie_tools/clion_cubemx/gcc-arm-none-eabi-10.3-2021.10/bin/../lib/gcc/arm-none-eabi/10.3.1/../../../../arm-none-eabi/lib/thumb/v7e-m/nofp\libm.a(lib_a-e_exp.o)
 .rodata.ln2LO  0x08009858       0x10 d:/lijie_tools/clion_cubemx/gcc-arm-none-eabi-10.3-2021.10/bin/../lib/gcc/arm-none-eabi/10.3.1/../../../../arm-none-eabi/lib/thumb/v7e-m/nofp\libm.a(lib_a-e_exp.o)
                0x08009868                . = ALIGN (0x4)

.ARM.extab
 *(.ARM.extab* .gnu.linkonce.armextab.*)

.ARM            0x08009868        0x8
                0x08009868                __exidx_start = .
 *(.ARM.exidx*)
 .ARM.exidx     0x08009868        0x8 d:/lijie_tools/clion_cubemx/gcc-arm-none-eabi-10.3-2021.10/bin/../lib/gcc/arm-none-eabi/10.3.1/thumb/v7e-m/nofp\libgcc.a(_udivmoddi4.o)
                0x08009870                __exidx_end = .

.rel.dyn        0x08009870        0x0
 .rel.iplt      0x08009870        0x0 d:/lijie_tools/clion_cubemx/gcc-arm-none-eabi-10.3-2021.10/bin/../lib/gcc/arm-none-eabi/10.3.1/thumb/v7e-m/nofp/crtbegin.o

.preinit_array  0x08009870        0x0
                0x08009870                PROVIDE (__preinit_array_start = .)
 *(.preinit_array*)
                0x08009870                PROVIDE (__preinit_array_end = .)

.init_array     0x08009870        0x8
                0x08009870                PROVIDE (__init_array_start = .)
 *(SORT_BY_NAME(.init_array.*))
 .init_array.00000
                0x08009870        0x4 d:/lijie_tools/clion_cubemx/gcc-arm-none-eabi-10.3-2021.10/bin/../lib/gcc/arm-none-eabi/10.3.1/../../../../arm-none-eabi/lib/thumb/v7e-m/nofp\libg.a(lib_a-__call_atexit.o)
 *(.init_array*)
 .init_array    0x08009874        0x4 d:/lijie_tools/clion_cubemx/gcc-arm-none-eabi-10.3-2021.10/bin/../lib/gcc/arm-none-eabi/10.3.1/thumb/v7e-m/nofp/crtbegin.o
                0x08009878                PROVIDE (__init_array_end = .)

.fini_array     0x08009878        0x4
                0x08009878                PROVIDE (__fini_array_start = .)
 *(SORT_BY_NAME(.fini_array.*))
 *(.fini_array*)
 .fini_array    0x08009878        0x4 d:/lijie_tools/clion_cubemx/gcc-arm-none-eabi-10.3-2021.10/bin/../lib/gcc/arm-none-eabi/10.3.1/thumb/v7e-m/nofp/crtbegin.o
                0x0800987c                PROVIDE (__fini_array_end = .)
                0x0800987c                _sidata = LOADADDR (.data)

.data           0x24000000      0x85c load address 0x0800987c
                0x24000000                . = ALIGN (0x4)
                0x24000000                _sdata = .
 *(.data)
 *(.data*)
 .data.Target_Average_Times
                0x24000000        0x1 CMakeFiles/H750_S15909.elf.dir/APP/mymain.c.obj
                0x24000000                Target_Average_Times
 *fill*         0x24000001        0x3 
 .data.shutter_time
                0x24000004        0x4 CMakeFiles/H750_S15909.elf.dir/APP/mymain.c.obj
                0x24000004                shutter_time
 .data.sn       0x24000008        0x4 CMakeFiles/H750_S15909.elf.dir/APP/mymain.c.obj
                0x24000008                sn
 .data.SystemCoreClock
                0x2400000c        0x4 CMakeFiles/H750_S15909.elf.dir/Core/Src/system_stm32h7xx.c.obj
                0x2400000c                SystemCoreClock
 .data.SystemD2Clock
                0x24000010        0x4 CMakeFiles/H750_S15909.elf.dir/Core/Src/system_stm32h7xx.c.obj
                0x24000010                SystemD2Clock
 .data.uwTickFreq
                0x24000014        0x1 CMakeFiles/H750_S15909.elf.dir/Drivers/STM32H7xx_HAL_Driver/Src/stm32h7xx_hal.c.obj
                0x24000014                uwTickFreq
 *fill*         0x24000015        0x3 
 .data.uwTickPrio
                0x24000018        0x4 CMakeFiles/H750_S15909.elf.dir/Drivers/STM32H7xx_HAL_Driver/Src/stm32h7xx_hal.c.obj
                0x24000018                uwTickPrio
 .data._impure_ptr
                0x2400001c        0x4 d:/lijie_tools/clion_cubemx/gcc-arm-none-eabi-10.3-2021.10/bin/../lib/gcc/arm-none-eabi/10.3.1/../../../../arm-none-eabi/lib/thumb/v7e-m/nofp\libg.a(lib_a-impure.o)
                0x2400001c                _impure_ptr
 .data.impure_data
                0x24000020      0x428 d:/lijie_tools/clion_cubemx/gcc-arm-none-eabi-10.3-2021.10/bin/../lib/gcc/arm-none-eabi/10.3.1/../../../../arm-none-eabi/lib/thumb/v7e-m/nofp\libg.a(lib_a-impure.o)
 .data.__atexit_recursive_mutex
                0x24000448        0x4 d:/lijie_tools/clion_cubemx/gcc-arm-none-eabi-10.3-2021.10/bin/../lib/gcc/arm-none-eabi/10.3.1/../../../../arm-none-eabi/lib/thumb/v7e-m/nofp\libg.a(lib_a-__call_atexit.o)
                0x24000448                __atexit_recursive_mutex
 .data.__malloc_av_
                0x2400044c      0x408 d:/lijie_tools/clion_cubemx/gcc-arm-none-eabi-10.3-2021.10/bin/../lib/gcc/arm-none-eabi/10.3.1/../../../../arm-none-eabi/lib/thumb/v7e-m/nofp\libg.a(lib_a-mallocr.o)
                0x2400044c                __malloc_av_
 .data.__malloc_sbrk_base
                0x24000854        0x4 d:/lijie_tools/clion_cubemx/gcc-arm-none-eabi-10.3-2021.10/bin/../lib/gcc/arm-none-eabi/10.3.1/../../../../arm-none-eabi/lib/thumb/v7e-m/nofp\libg.a(lib_a-mallocr.o)
                0x24000854                __malloc_sbrk_base
 .data.__malloc_trim_threshold
                0x24000858        0x4 d:/lijie_tools/clion_cubemx/gcc-arm-none-eabi-10.3-2021.10/bin/../lib/gcc/arm-none-eabi/10.3.1/../../../../arm-none-eabi/lib/thumb/v7e-m/nofp\libg.a(lib_a-mallocr.o)
                0x24000858                __malloc_trim_threshold
 *(.RamFunc)
 *(.RamFunc*)
                0x2400085c                . = ALIGN (0x4)
                0x2400085c                _edata = .

.igot.plt       0x2400085c        0x0 load address 0x0800a0d8
 .igot.plt      0x2400085c        0x0 d:/lijie_tools/clion_cubemx/gcc-arm-none-eabi-10.3-2021.10/bin/../lib/gcc/arm-none-eabi/10.3.1/thumb/v7e-m/nofp/crtbegin.o
                0x2400085c                . = ALIGN (0x4)

.bss            0x2400085c     0x3c08 load address 0x0800a0d8
                0x2400085c                _sbss = .
                0x2400085c                __bss_start__ = _sbss
 *(.bss)
 .bss           0x2400085c       0x1c d:/lijie_tools/clion_cubemx/gcc-arm-none-eabi-10.3-2021.10/bin/../lib/gcc/arm-none-eabi/10.3.1/thumb/v7e-m/nofp/crtbegin.o
 *(.bss*)
 .bss.Average_Buffer
                0x24000878      0x406 CMakeFiles/H750_S15909.elf.dir/APP/mymain.c.obj
                0x24000878                Average_Buffer
 *fill*         0x24000c7e        0x2 
 .bss.Last_Receive_Data_Count
                0x24000c80        0x4 CMakeFiles/H750_S15909.elf.dir/APP/mymain.c.obj
                0x24000c80                Last_Receive_Data_Count
 .bss.Moving_Average_Buffer
                0x24000c84      0x406 CMakeFiles/H750_S15909.elf.dir/APP/mymain.c.obj
                0x24000c84                Moving_Average_Buffer
 *fill*         0x2400108a        0x2 
 .bss.Moving_Buffer
                0x2400108c     0x283c CMakeFiles/H750_S15909.elf.dir/APP/mymain.c.obj
                0x2400108c                Moving_Buffer
 .bss.Receive_Data_Buffer
                0x240038c8      0x406 CMakeFiles/H750_S15909.elf.dir/APP/mymain.c.obj
                0x240038c8                Receive_Data_Buffer
 *fill*         0x24003cce        0x2 
 .bss.Receive_Data_Count
                0x24003cd0        0x4 CMakeFiles/H750_S15909.elf.dir/APP/mymain.c.obj
                0x24003cd0                Receive_Data_Count
 .bss.Send_Data_Type
                0x24003cd4        0x4 CMakeFiles/H750_S15909.elf.dir/APP/mymain.c.obj
                0x24003cd4                Send_Data_Type
 .bss.Temperature
                0x24003cd8        0x4 CMakeFiles/H750_S15909.elf.dir/APP/mymain.c.obj
                0x24003cd8                Temperature
 .bss.USART2_RX_Buffer
                0x24003cdc      0x408 CMakeFiles/H750_S15909.elf.dir/APP/mymain.c.obj
                0x24003cdc                USART2_RX_Buffer
 .bss.g_rx_buffer
                0x240040e4        0x1 CMakeFiles/H750_S15909.elf.dir/APP/mymain.c.obj
                0x240040e4                g_rx_buffer
 *fill*         0x240040e5        0x3 
 .bss.g_usart_rx_buf
                0x240040e8       0xc8 CMakeFiles/H750_S15909.elf.dir/APP/mymain.c.obj
                0x240040e8                g_usart_rx_buf
 .bss.g_usart_rx_sta
                0x240041b0        0x2 CMakeFiles/H750_S15909.elf.dir/APP/mymain.c.obj
                0x240041b0                g_usart_rx_sta
 *fill*         0x240041b2        0x2 
 .bss.mode      0x240041b4        0x4 CMakeFiles/H750_S15909.elf.dir/APP/mymain.c.obj
                0x240041b4                mode
 .bss.g_dma_handle
                0x240041b8       0x78 CMakeFiles/H750_S15909.elf.dir/APP/usart1_tx_dma.c.obj
                0x240041b8                g_dma_handle
 .bss.__sbrk_heap_end
                0x24004230        0x4 CMakeFiles/H750_S15909.elf.dir/Core/Src/sysmem.c.obj
 .bss.htim5     0x24004234       0x4c CMakeFiles/H750_S15909.elf.dir/Core/Src/tim.c.obj
                0x24004234                htim5
 .bss.hdma_usart2_rx
                0x24004280       0x78 CMakeFiles/H750_S15909.elf.dir/Core/Src/usart.c.obj
                0x24004280                hdma_usart2_rx
 .bss.huart1    0x240042f8       0x90 CMakeFiles/H750_S15909.elf.dir/Core/Src/usart.c.obj
                0x240042f8                huart1
 .bss.huart2    0x24004388       0x90 CMakeFiles/H750_S15909.elf.dir/Core/Src/usart.c.obj
                0x24004388                huart2
 .bss.uwTick    0x24004418        0x4 CMakeFiles/H750_S15909.elf.dir/Drivers/STM32H7xx_HAL_Driver/Src/stm32h7xx_hal.c.obj
                0x24004418                uwTick
 .bss.__lock___atexit_recursive_mutex
                0x2400441c        0x1 d:/lijie_tools/clion_cubemx/gcc-arm-none-eabi-10.3-2021.10/bin/../lib/gcc/arm-none-eabi/10.3.1/../../../../arm-none-eabi/lib/thumb/v7e-m/nofp\libg.a(lib_a-lock.o)
                0x2400441c                __lock___atexit_recursive_mutex
 *fill*         0x2400441d        0x3 
 .bss.__lock___malloc_recursive_mutex
                0x24004420        0x1 d:/lijie_tools/clion_cubemx/gcc-arm-none-eabi-10.3-2021.10/bin/../lib/gcc/arm-none-eabi/10.3.1/../../../../arm-none-eabi/lib/thumb/v7e-m/nofp\libg.a(lib_a-lock.o)
                0x24004420                __lock___malloc_recursive_mutex
 *fill*         0x24004421        0x3 
 .bss.__lock___sfp_recursive_mutex
                0x24004424        0x1 d:/lijie_tools/clion_cubemx/gcc-arm-none-eabi-10.3-2021.10/bin/../lib/gcc/arm-none-eabi/10.3.1/../../../../arm-none-eabi/lib/thumb/v7e-m/nofp\libg.a(lib_a-lock.o)
                0x24004424                __lock___sfp_recursive_mutex
 *fill*         0x24004425        0x3 
 .bss.__lock___sinit_recursive_mutex
                0x24004428        0x1 d:/lijie_tools/clion_cubemx/gcc-arm-none-eabi-10.3-2021.10/bin/../lib/gcc/arm-none-eabi/10.3.1/../../../../arm-none-eabi/lib/thumb/v7e-m/nofp\libg.a(lib_a-lock.o)
                0x24004428                __lock___sinit_recursive_mutex
 *fill*         0x24004429        0x3 
 .bss.__malloc_current_mallinfo
                0x2400442c       0x28 d:/lijie_tools/clion_cubemx/gcc-arm-none-eabi-10.3-2021.10/bin/../lib/gcc/arm-none-eabi/10.3.1/../../../../arm-none-eabi/lib/thumb/v7e-m/nofp\libg.a(lib_a-mallocr.o)
                0x2400442c                __malloc_current_mallinfo
 .bss.__malloc_max_sbrked_mem
                0x24004454        0x4 d:/lijie_tools/clion_cubemx/gcc-arm-none-eabi-10.3-2021.10/bin/../lib/gcc/arm-none-eabi/10.3.1/../../../../arm-none-eabi/lib/thumb/v7e-m/nofp\libg.a(lib_a-mallocr.o)
                0x24004454                __malloc_max_sbrked_mem
 .bss.__malloc_max_total_mem
                0x24004458        0x4 d:/lijie_tools/clion_cubemx/gcc-arm-none-eabi-10.3-2021.10/bin/../lib/gcc/arm-none-eabi/10.3.1/../../../../arm-none-eabi/lib/thumb/v7e-m/nofp\libg.a(lib_a-mallocr.o)
                0x24004458                __malloc_max_total_mem
 .bss.__malloc_top_pad
                0x2400445c        0x4 d:/lijie_tools/clion_cubemx/gcc-arm-none-eabi-10.3-2021.10/bin/../lib/gcc/arm-none-eabi/10.3.1/../../../../arm-none-eabi/lib/thumb/v7e-m/nofp\libg.a(lib_a-mallocr.o)
                0x2400445c                __malloc_top_pad
 .bss.errno     0x24004460        0x4 d:/lijie_tools/clion_cubemx/gcc-arm-none-eabi-10.3-2021.10/bin/../lib/gcc/arm-none-eabi/10.3.1/../../../../arm-none-eabi/lib/thumb/v7e-m/nofp\libg.a(lib_a-reent.o)
                0x24004460                errno
 *(COMMON)
                0x24004464                . = ALIGN (0x4)
                0x24004464                _ebss = .
                0x24004464                __bss_end__ = _ebss

._user_heap_stack
                0x24004464      0x604 load address 0x0800a0d8
                0x24004468                . = ALIGN (0x8)
 *fill*         0x24004464        0x4 
                [!provide]                PROVIDE (end = .)
                0x24004468                PROVIDE (_end = .)
                0x24004668                . = (. + _Min_Heap_Size)
 *fill*         0x24004468      0x200 
                0x24004a68                . = (. + _Min_Stack_Size)
 *fill*         0x24004668      0x400 
                0x24004a68                . = ALIGN (0x8)

/DISCARD/
 libc.a(*)
 libm.a(*)
 libgcc.a(*)

.ARM.attributes
                0x00000000       0x2a
 *(.ARM.attributes)
 .ARM.attributes
                0x00000000       0x1e d:/lijie_tools/clion_cubemx/gcc-arm-none-eabi-10.3-2021.10/bin/../lib/gcc/arm-none-eabi/10.3.1/thumb/v7e-m/nofp/crti.o
 .ARM.attributes
                0x0000001e       0x2e d:/lijie_tools/clion_cubemx/gcc-arm-none-eabi-10.3-2021.10/bin/../lib/gcc/arm-none-eabi/10.3.1/thumb/v7e-m/nofp/crtbegin.o
 .ARM.attributes
                0x0000004c       0x2e CMakeFiles/H750_S15909.elf.dir/APP/DS18B20.c.obj
 .ARM.attributes
                0x0000007a       0x2e CMakeFiles/H750_S15909.elf.dir/APP/IRIS_Method.c.obj
 .ARM.attributes
                0x000000a8       0x2e CMakeFiles/H750_S15909.elf.dir/APP/Shutter.c.obj
 .ARM.attributes
                0x000000d6       0x2e CMakeFiles/H750_S15909.elf.dir/APP/communication.c.obj
 .ARM.attributes
                0x00000104       0x2e CMakeFiles/H750_S15909.elf.dir/APP/data_analyse.c.obj
 .ARM.attributes
                0x00000132       0x2e CMakeFiles/H750_S15909.elf.dir/APP/delay.c.obj
 .ARM.attributes
                0x00000160       0x2e CMakeFiles/H750_S15909.elf.dir/APP/mymain.c.obj
 .ARM.attributes
                0x0000018e       0x2e CMakeFiles/H750_S15909.elf.dir/APP/usart1_tx_dma.c.obj
 .ARM.attributes
                0x000001bc       0x2e CMakeFiles/H750_S15909.elf.dir/Core/Src/dma.c.obj
 .ARM.attributes
                0x000001ea       0x2e CMakeFiles/H750_S15909.elf.dir/Core/Src/gpio.c.obj
 .ARM.attributes
                0x00000218       0x2e CMakeFiles/H750_S15909.elf.dir/Core/Src/main.c.obj
 .ARM.attributes
                0x00000246       0x2e CMakeFiles/H750_S15909.elf.dir/Core/Src/stm32h7xx_hal_msp.c.obj
 .ARM.attributes
                0x00000274       0x2e CMakeFiles/H750_S15909.elf.dir/Core/Src/stm32h7xx_it.c.obj
 .ARM.attributes
                0x000002a2       0x2e CMakeFiles/H750_S15909.elf.dir/Core/Src/syscalls.c.obj
 .ARM.attributes
                0x000002d0       0x2e CMakeFiles/H750_S15909.elf.dir/Core/Src/sysmem.c.obj
 .ARM.attributes
                0x000002fe       0x2e CMakeFiles/H750_S15909.elf.dir/Core/Src/system_stm32h7xx.c.obj
 .ARM.attributes
                0x0000032c       0x2e CMakeFiles/H750_S15909.elf.dir/Core/Src/tim.c.obj
 .ARM.attributes
                0x0000035a       0x2e CMakeFiles/H750_S15909.elf.dir/Core/Src/usart.c.obj
 .ARM.attributes
                0x00000388       0x21 CMakeFiles/H750_S15909.elf.dir/Core/Startup/startup_stm32h750vbtx.s.obj
 .ARM.attributes
                0x000003a9       0x2e CMakeFiles/H750_S15909.elf.dir/Drivers/STM32H7xx_HAL_Driver/Src/stm32h7xx_hal.c.obj
 .ARM.attributes
                0x000003d7       0x2e CMakeFiles/H750_S15909.elf.dir/Drivers/STM32H7xx_HAL_Driver/Src/stm32h7xx_hal_cortex.c.obj
 .ARM.attributes
                0x00000405       0x2e CMakeFiles/H750_S15909.elf.dir/Drivers/STM32H7xx_HAL_Driver/Src/stm32h7xx_hal_dma.c.obj
 .ARM.attributes
                0x00000433       0x2e CMakeFiles/H750_S15909.elf.dir/Drivers/STM32H7xx_HAL_Driver/Src/stm32h7xx_hal_gpio.c.obj
 .ARM.attributes
                0x00000461       0x2e CMakeFiles/H750_S15909.elf.dir/Drivers/STM32H7xx_HAL_Driver/Src/stm32h7xx_hal_pwr_ex.c.obj
 .ARM.attributes
                0x0000048f       0x2e CMakeFiles/H750_S15909.elf.dir/Drivers/STM32H7xx_HAL_Driver/Src/stm32h7xx_hal_rcc.c.obj
 .ARM.attributes
                0x000004bd       0x2e CMakeFiles/H750_S15909.elf.dir/Drivers/STM32H7xx_HAL_Driver/Src/stm32h7xx_hal_rcc_ex.c.obj
 .ARM.attributes
                0x000004eb       0x2e CMakeFiles/H750_S15909.elf.dir/Drivers/STM32H7xx_HAL_Driver/Src/stm32h7xx_hal_tim.c.obj
 .ARM.attributes
                0x00000519       0x2e CMakeFiles/H750_S15909.elf.dir/Drivers/STM32H7xx_HAL_Driver/Src/stm32h7xx_hal_tim_ex.c.obj
 .ARM.attributes
                0x00000547       0x2e CMakeFiles/H750_S15909.elf.dir/Drivers/STM32H7xx_HAL_Driver/Src/stm32h7xx_hal_uart.c.obj
 .ARM.attributes
                0x00000575       0x2e CMakeFiles/H750_S15909.elf.dir/Drivers/STM32H7xx_HAL_Driver/Src/stm32h7xx_hal_uart_ex.c.obj
 .ARM.attributes
                0x000005a3       0x1e d:/lijie_tools/clion_cubemx/gcc-arm-none-eabi-10.3-2021.10/bin/../lib/gcc/arm-none-eabi/10.3.1/thumb/v7e-m/nofp\libgcc.a(_arm_addsubdf3.o)
 .ARM.attributes
                0x000005c1       0x1e d:/lijie_tools/clion_cubemx/gcc-arm-none-eabi-10.3-2021.10/bin/../lib/gcc/arm-none-eabi/10.3.1/thumb/v7e-m/nofp\libgcc.a(_arm_muldivdf3.o)
 .ARM.attributes
                0x000005df       0x1e d:/lijie_tools/clion_cubemx/gcc-arm-none-eabi-10.3-2021.10/bin/../lib/gcc/arm-none-eabi/10.3.1/thumb/v7e-m/nofp\libgcc.a(_arm_cmpdf2.o)
 .ARM.attributes
                0x000005fd       0x1e d:/lijie_tools/clion_cubemx/gcc-arm-none-eabi-10.3-2021.10/bin/../lib/gcc/arm-none-eabi/10.3.1/thumb/v7e-m/nofp\libgcc.a(_arm_fixdfsi.o)
 .ARM.attributes
                0x0000061b       0x1e d:/lijie_tools/clion_cubemx/gcc-arm-none-eabi-10.3-2021.10/bin/../lib/gcc/arm-none-eabi/10.3.1/thumb/v7e-m/nofp\libgcc.a(_arm_fixunsdfsi.o)
 .ARM.attributes
                0x00000639       0x1e d:/lijie_tools/clion_cubemx/gcc-arm-none-eabi-10.3-2021.10/bin/../lib/gcc/arm-none-eabi/10.3.1/thumb/v7e-m/nofp\libgcc.a(_arm_truncdfsf2.o)
 .ARM.attributes
                0x00000657       0x1e d:/lijie_tools/clion_cubemx/gcc-arm-none-eabi-10.3-2021.10/bin/../lib/gcc/arm-none-eabi/10.3.1/thumb/v7e-m/nofp\libgcc.a(_arm_addsubsf3.o)
 .ARM.attributes
                0x00000675       0x1e d:/lijie_tools/clion_cubemx/gcc-arm-none-eabi-10.3-2021.10/bin/../lib/gcc/arm-none-eabi/10.3.1/thumb/v7e-m/nofp\libgcc.a(_arm_muldivsf3.o)
 .ARM.attributes
                0x00000693       0x1e d:/lijie_tools/clion_cubemx/gcc-arm-none-eabi-10.3-2021.10/bin/../lib/gcc/arm-none-eabi/10.3.1/thumb/v7e-m/nofp\libgcc.a(_arm_fixunssfsi.o)
 .ARM.attributes
                0x000006b1       0x1e d:/lijie_tools/clion_cubemx/gcc-arm-none-eabi-10.3-2021.10/bin/../lib/gcc/arm-none-eabi/10.3.1/thumb/v7e-m/nofp\libgcc.a(_aeabi_uldivmod.o)
 .ARM.attributes
                0x000006cf       0x2e d:/lijie_tools/clion_cubemx/gcc-arm-none-eabi-10.3-2021.10/bin/../lib/gcc/arm-none-eabi/10.3.1/thumb/v7e-m/nofp\libgcc.a(_udivmoddi4.o)
 .ARM.attributes
                0x000006fd       0x1e d:/lijie_tools/clion_cubemx/gcc-arm-none-eabi-10.3-2021.10/bin/../lib/gcc/arm-none-eabi/10.3.1/thumb/v7e-m/nofp\libgcc.a(_dvmd_tls.o)
 .ARM.attributes
                0x0000071b       0x2e d:/lijie_tools/clion_cubemx/gcc-arm-none-eabi-10.3-2021.10/bin/../lib/gcc/arm-none-eabi/10.3.1/../../../../arm-none-eabi/lib/thumb/v7e-m/nofp\libg.a(lib_a-errno.o)
 .ARM.attributes
                0x00000749       0x2e d:/lijie_tools/clion_cubemx/gcc-arm-none-eabi-10.3-2021.10/bin/../lib/gcc/arm-none-eabi/10.3.1/../../../../arm-none-eabi/lib/thumb/v7e-m/nofp\libg.a(lib_a-impure.o)
 .ARM.attributes
                0x00000777       0x2e d:/lijie_tools/clion_cubemx/gcc-arm-none-eabi-10.3-2021.10/bin/../lib/gcc/arm-none-eabi/10.3.1/../../../../arm-none-eabi/lib/thumb/v7e-m/nofp\libg.a(lib_a-init.o)
 .ARM.attributes
                0x000007a5       0x1c d:/lijie_tools/clion_cubemx/gcc-arm-none-eabi-10.3-2021.10/bin/../lib/gcc/arm-none-eabi/10.3.1/../../../../arm-none-eabi/lib/thumb/v7e-m/nofp\libg.a(lib_a-memcpy.o)
 .ARM.attributes
                0x000007c1       0x2e d:/lijie_tools/clion_cubemx/gcc-arm-none-eabi-10.3-2021.10/bin/../lib/gcc/arm-none-eabi/10.3.1/../../../../arm-none-eabi/lib/thumb/v7e-m/nofp\libg.a(lib_a-memset.o)
 .ARM.attributes
                0x000007ef       0x2e d:/lijie_tools/clion_cubemx/gcc-arm-none-eabi-10.3-2021.10/bin/../lib/gcc/arm-none-eabi/10.3.1/../../../../arm-none-eabi/lib/thumb/v7e-m/nofp\libg.a(lib_a-setvbuf.o)
 .ARM.attributes
                0x0000081d       0x2e d:/lijie_tools/clion_cubemx/gcc-arm-none-eabi-10.3-2021.10/bin/../lib/gcc/arm-none-eabi/10.3.1/../../../../arm-none-eabi/lib/thumb/v7e-m/nofp\libg.a(lib_a-__call_atexit.o)
 .ARM.attributes
                0x0000084b       0x2e d:/lijie_tools/clion_cubemx/gcc-arm-none-eabi-10.3-2021.10/bin/../lib/gcc/arm-none-eabi/10.3.1/../../../../arm-none-eabi/lib/thumb/v7e-m/nofp\libg.a(lib_a-atexit.o)
 .ARM.attributes
                0x00000879       0x2e d:/lijie_tools/clion_cubemx/gcc-arm-none-eabi-10.3-2021.10/bin/../lib/gcc/arm-none-eabi/10.3.1/../../../../arm-none-eabi/lib/thumb/v7e-m/nofp\libg.a(lib_a-fflush.o)
 .ARM.attributes
                0x000008a7       0x2e d:/lijie_tools/clion_cubemx/gcc-arm-none-eabi-10.3-2021.10/bin/../lib/gcc/arm-none-eabi/10.3.1/../../../../arm-none-eabi/lib/thumb/v7e-m/nofp\libg.a(lib_a-findfp.o)
 .ARM.attributes
                0x000008d5       0x2e d:/lijie_tools/clion_cubemx/gcc-arm-none-eabi-10.3-2021.10/bin/../lib/gcc/arm-none-eabi/10.3.1/../../../../arm-none-eabi/lib/thumb/v7e-m/nofp\libg.a(lib_a-fini.o)
 .ARM.attributes
                0x00000903       0x2e d:/lijie_tools/clion_cubemx/gcc-arm-none-eabi-10.3-2021.10/bin/../lib/gcc/arm-none-eabi/10.3.1/../../../../arm-none-eabi/lib/thumb/v7e-m/nofp\libg.a(lib_a-freer.o)
 .ARM.attributes
                0x00000931       0x2e d:/lijie_tools/clion_cubemx/gcc-arm-none-eabi-10.3-2021.10/bin/../lib/gcc/arm-none-eabi/10.3.1/../../../../arm-none-eabi/lib/thumb/v7e-m/nofp\libg.a(lib_a-fwalk.o)
 .ARM.attributes
                0x0000095f       0x2e d:/lijie_tools/clion_cubemx/gcc-arm-none-eabi-10.3-2021.10/bin/../lib/gcc/arm-none-eabi/10.3.1/../../../../arm-none-eabi/lib/thumb/v7e-m/nofp\libg.a(lib_a-lock.o)
 .ARM.attributes
                0x0000098d       0x2e d:/lijie_tools/clion_cubemx/gcc-arm-none-eabi-10.3-2021.10/bin/../lib/gcc/arm-none-eabi/10.3.1/../../../../arm-none-eabi/lib/thumb/v7e-m/nofp\libg.a(lib_a-makebuf.o)
 .ARM.attributes
                0x000009bb       0x2e d:/lijie_tools/clion_cubemx/gcc-arm-none-eabi-10.3-2021.10/bin/../lib/gcc/arm-none-eabi/10.3.1/../../../../arm-none-eabi/lib/thumb/v7e-m/nofp\libg.a(lib_a-malloc.o)
 .ARM.attributes
                0x000009e9       0x2e d:/lijie_tools/clion_cubemx/gcc-arm-none-eabi-10.3-2021.10/bin/../lib/gcc/arm-none-eabi/10.3.1/../../../../arm-none-eabi/lib/thumb/v7e-m/nofp\libg.a(lib_a-mallocr.o)
 .ARM.attributes
                0x00000a17       0x2e d:/lijie_tools/clion_cubemx/gcc-arm-none-eabi-10.3-2021.10/bin/../lib/gcc/arm-none-eabi/10.3.1/../../../../arm-none-eabi/lib/thumb/v7e-m/nofp\libg.a(lib_a-mlock.o)
 .ARM.attributes
                0x00000a45       0x2e d:/lijie_tools/clion_cubemx/gcc-arm-none-eabi-10.3-2021.10/bin/../lib/gcc/arm-none-eabi/10.3.1/../../../../arm-none-eabi/lib/thumb/v7e-m/nofp\libg.a(lib_a-sbrkr.o)
 .ARM.attributes
                0x00000a73       0x2e d:/lijie_tools/clion_cubemx/gcc-arm-none-eabi-10.3-2021.10/bin/../lib/gcc/arm-none-eabi/10.3.1/../../../../arm-none-eabi/lib/thumb/v7e-m/nofp\libg.a(lib_a-stdio.o)
 .ARM.attributes
                0x00000aa1       0x2e d:/lijie_tools/clion_cubemx/gcc-arm-none-eabi-10.3-2021.10/bin/../lib/gcc/arm-none-eabi/10.3.1/../../../../arm-none-eabi/lib/thumb/v7e-m/nofp\libg.a(lib_a-writer.o)
 .ARM.attributes
                0x00000acf       0x2e d:/lijie_tools/clion_cubemx/gcc-arm-none-eabi-10.3-2021.10/bin/../lib/gcc/arm-none-eabi/10.3.1/../../../../arm-none-eabi/lib/thumb/v7e-m/nofp\libg.a(lib_a-__atexit.o)
 .ARM.attributes
                0x00000afd       0x2e d:/lijie_tools/clion_cubemx/gcc-arm-none-eabi-10.3-2021.10/bin/../lib/gcc/arm-none-eabi/10.3.1/../../../../arm-none-eabi/lib/thumb/v7e-m/nofp\libg.a(lib_a-closer.o)
 .ARM.attributes
                0x00000b2b       0x2e d:/lijie_tools/clion_cubemx/gcc-arm-none-eabi-10.3-2021.10/bin/../lib/gcc/arm-none-eabi/10.3.1/../../../../arm-none-eabi/lib/thumb/v7e-m/nofp\libg.a(lib_a-fclose.o)
 .ARM.attributes
                0x00000b59       0x2e d:/lijie_tools/clion_cubemx/gcc-arm-none-eabi-10.3-2021.10/bin/../lib/gcc/arm-none-eabi/10.3.1/../../../../arm-none-eabi/lib/thumb/v7e-m/nofp\libg.a(lib_a-fstatr.o)
 .ARM.attributes
                0x00000b87       0x2e d:/lijie_tools/clion_cubemx/gcc-arm-none-eabi-10.3-2021.10/bin/../lib/gcc/arm-none-eabi/10.3.1/../../../../arm-none-eabi/lib/thumb/v7e-m/nofp\libg.a(lib_a-lseekr.o)
 .ARM.attributes
                0x00000bb5       0x2e d:/lijie_tools/clion_cubemx/gcc-arm-none-eabi-10.3-2021.10/bin/../lib/gcc/arm-none-eabi/10.3.1/../../../../arm-none-eabi/lib/thumb/v7e-m/nofp\libg.a(lib_a-readr.o)
 .ARM.attributes
                0x00000be3       0x2e d:/lijie_tools/clion_cubemx/gcc-arm-none-eabi-10.3-2021.10/bin/../lib/gcc/arm-none-eabi/10.3.1/../../../../arm-none-eabi/lib/thumb/v7e-m/nofp\libg.a(lib_a-reent.o)
 .ARM.attributes
                0x00000c11       0x1e d:/lijie_tools/clion_cubemx/gcc-arm-none-eabi-10.3-2021.10/bin/../lib/gcc/arm-none-eabi/10.3.1/thumb/v7e-m/nofp/crtn.o
OUTPUT(H750_S15909.elf elf32-littlearm)
LOAD linker stubs
LOAD d:/lijie_tools/clion_cubemx/gcc-arm-none-eabi-10.3-2021.10/bin/../lib/gcc/arm-none-eabi/10.3.1/../../../../arm-none-eabi/lib/thumb/v7e-m/nofp\libc.a
LOAD d:/lijie_tools/clion_cubemx/gcc-arm-none-eabi-10.3-2021.10/bin/../lib/gcc/arm-none-eabi/10.3.1/../../../../arm-none-eabi/lib/thumb/v7e-m/nofp\libm.a
LOAD d:/lijie_tools/clion_cubemx/gcc-arm-none-eabi-10.3-2021.10/bin/../lib/gcc/arm-none-eabi/10.3.1/thumb/v7e-m/nofp\libgcc.a

.debug_info     0x00000000    0x21de8
 .debug_info    0x00000000      0xd4c CMakeFiles/H750_S15909.elf.dir/APP/DS18B20.c.obj
 .debug_info    0x00000d4c      0x542 CMakeFiles/H750_S15909.elf.dir/APP/IRIS_Method.c.obj
 .debug_info    0x0000128e      0x6ed CMakeFiles/H750_S15909.elf.dir/APP/Shutter.c.obj
 .debug_info    0x0000197b      0x983 CMakeFiles/H750_S15909.elf.dir/APP/communication.c.obj
 .debug_info    0x000022fe      0x3aa CMakeFiles/H750_S15909.elf.dir/APP/data_analyse.c.obj
 .debug_info    0x000026a8      0x83f CMakeFiles/H750_S15909.elf.dir/APP/delay.c.obj
 .debug_info    0x00002ee7     0x1a46 CMakeFiles/H750_S15909.elf.dir/APP/mymain.c.obj
 .debug_info    0x0000492d      0xcd4 CMakeFiles/H750_S15909.elf.dir/APP/usart1_tx_dma.c.obj
 .debug_info    0x00005601      0x87b CMakeFiles/H750_S15909.elf.dir/Core/Src/dma.c.obj
 .debug_info    0x00005e7c      0xa9e CMakeFiles/H750_S15909.elf.dir/Core/Src/gpio.c.obj
 .debug_info    0x0000691a      0xb67 CMakeFiles/H750_S15909.elf.dir/Core/Src/main.c.obj
 .debug_info    0x00007481      0x4a0 CMakeFiles/H750_S15909.elf.dir/Core/Src/stm32h7xx_hal_msp.c.obj
 .debug_info    0x00007921      0x8ca CMakeFiles/H750_S15909.elf.dir/Core/Src/stm32h7xx_it.c.obj
 .debug_info    0x000081eb      0x7af CMakeFiles/H750_S15909.elf.dir/Core/Src/syscalls.c.obj
 .debug_info    0x0000899a      0x174 CMakeFiles/H750_S15909.elf.dir/Core/Src/sysmem.c.obj
 .debug_info    0x00008b0e      0xaf5 CMakeFiles/H750_S15909.elf.dir/Core/Src/system_stm32h7xx.c.obj
 .debug_info    0x00009603      0xd53 CMakeFiles/H750_S15909.elf.dir/Core/Src/tim.c.obj
 .debug_info    0x0000a356     0x1801 CMakeFiles/H750_S15909.elf.dir/Core/Src/usart.c.obj
 .debug_info    0x0000bb57       0x22 CMakeFiles/H750_S15909.elf.dir/Core/Startup/startup_stm32h750vbtx.s.obj
 .debug_info    0x0000bb79     0x16a6 CMakeFiles/H750_S15909.elf.dir/Drivers/STM32H7xx_HAL_Driver/Src/stm32h7xx_hal.c.obj
 .debug_info    0x0000d21f     0x13f0 CMakeFiles/H750_S15909.elf.dir/Drivers/STM32H7xx_HAL_Driver/Src/stm32h7xx_hal_cortex.c.obj
 .debug_info    0x0000e60f      0xfeb CMakeFiles/H750_S15909.elf.dir/Drivers/STM32H7xx_HAL_Driver/Src/stm32h7xx_hal_dma.c.obj
 .debug_info    0x0000f5fa      0xd66 CMakeFiles/H750_S15909.elf.dir/Drivers/STM32H7xx_HAL_Driver/Src/stm32h7xx_hal_gpio.c.obj
 .debug_info    0x00010360     0x122e CMakeFiles/H750_S15909.elf.dir/Drivers/STM32H7xx_HAL_Driver/Src/stm32h7xx_hal_pwr_ex.c.obj
 .debug_info    0x0001158e     0x13b3 CMakeFiles/H750_S15909.elf.dir/Drivers/STM32H7xx_HAL_Driver/Src/stm32h7xx_hal_rcc.c.obj
 .debug_info    0x00012941     0x1f48 CMakeFiles/H750_S15909.elf.dir/Drivers/STM32H7xx_HAL_Driver/Src/stm32h7xx_hal_rcc_ex.c.obj
 .debug_info    0x00014889     0x3fcf CMakeFiles/H750_S15909.elf.dir/Drivers/STM32H7xx_HAL_Driver/Src/stm32h7xx_hal_tim.c.obj
 .debug_info    0x00018858     0x1e53 CMakeFiles/H750_S15909.elf.dir/Drivers/STM32H7xx_HAL_Driver/Src/stm32h7xx_hal_tim_ex.c.obj
 .debug_info    0x0001a6ab     0x652f CMakeFiles/H750_S15909.elf.dir/Drivers/STM32H7xx_HAL_Driver/Src/stm32h7xx_hal_uart.c.obj
 .debug_info    0x00020bda     0x120e CMakeFiles/H750_S15909.elf.dir/Drivers/STM32H7xx_HAL_Driver/Src/stm32h7xx_hal_uart_ex.c.obj

.debug_abbrev   0x00000000     0x3b97
 .debug_abbrev  0x00000000      0x253 CMakeFiles/H750_S15909.elf.dir/APP/DS18B20.c.obj
 .debug_abbrev  0x00000253      0x10f CMakeFiles/H750_S15909.elf.dir/APP/IRIS_Method.c.obj
 .debug_abbrev  0x00000362      0x179 CMakeFiles/H750_S15909.elf.dir/APP/Shutter.c.obj
 .debug_abbrev  0x000004db      0x209 CMakeFiles/H750_S15909.elf.dir/APP/communication.c.obj
 .debug_abbrev  0x000006e4      0x163 CMakeFiles/H750_S15909.elf.dir/APP/data_analyse.c.obj
 .debug_abbrev  0x00000847      0x1c2 CMakeFiles/H750_S15909.elf.dir/APP/delay.c.obj
 .debug_abbrev  0x00000a09      0x362 CMakeFiles/H750_S15909.elf.dir/APP/mymain.c.obj
 .debug_abbrev  0x00000d6b      0x1df CMakeFiles/H750_S15909.elf.dir/APP/usart1_tx_dma.c.obj
 .debug_abbrev  0x00000f4a      0x137 CMakeFiles/H750_S15909.elf.dir/Core/Src/dma.c.obj
 .debug_abbrev  0x00001081      0x18a CMakeFiles/H750_S15909.elf.dir/Core/Src/gpio.c.obj
 .debug_abbrev  0x0000120b      0x1e8 CMakeFiles/H750_S15909.elf.dir/Core/Src/main.c.obj
 .debug_abbrev  0x000013f3       0xd7 CMakeFiles/H750_S15909.elf.dir/Core/Src/stm32h7xx_hal_msp.c.obj
 .debug_abbrev  0x000014ca      0x172 CMakeFiles/H750_S15909.elf.dir/Core/Src/stm32h7xx_it.c.obj
 .debug_abbrev  0x0000163c      0x1a3 CMakeFiles/H750_S15909.elf.dir/Core/Src/syscalls.c.obj
 .debug_abbrev  0x000017df       0xe7 CMakeFiles/H750_S15909.elf.dir/Core/Src/sysmem.c.obj
 .debug_abbrev  0x000018c6      0x162 CMakeFiles/H750_S15909.elf.dir/Core/Src/system_stm32h7xx.c.obj
 .debug_abbrev  0x00001a28      0x1e5 CMakeFiles/H750_S15909.elf.dir/Core/Src/tim.c.obj
 .debug_abbrev  0x00001c0d      0x290 CMakeFiles/H750_S15909.elf.dir/Core/Src/usart.c.obj
 .debug_abbrev  0x00001e9d       0x12 CMakeFiles/H750_S15909.elf.dir/Core/Startup/startup_stm32h750vbtx.s.obj
 .debug_abbrev  0x00001eaf      0x264 CMakeFiles/H750_S15909.elf.dir/Drivers/STM32H7xx_HAL_Driver/Src/stm32h7xx_hal.c.obj
 .debug_abbrev  0x00002113      0x37d CMakeFiles/H750_S15909.elf.dir/Drivers/STM32H7xx_HAL_Driver/Src/stm32h7xx_hal_cortex.c.obj
 .debug_abbrev  0x00002490      0x298 CMakeFiles/H750_S15909.elf.dir/Drivers/STM32H7xx_HAL_Driver/Src/stm32h7xx_hal_dma.c.obj
 .debug_abbrev  0x00002728      0x239 CMakeFiles/H750_S15909.elf.dir/Drivers/STM32H7xx_HAL_Driver/Src/stm32h7xx_hal_gpio.c.obj
 .debug_abbrev  0x00002961      0x29b CMakeFiles/H750_S15909.elf.dir/Drivers/STM32H7xx_HAL_Driver/Src/stm32h7xx_hal_pwr_ex.c.obj
 .debug_abbrev  0x00002bfc      0x28c CMakeFiles/H750_S15909.elf.dir/Drivers/STM32H7xx_HAL_Driver/Src/stm32h7xx_hal_rcc.c.obj
 .debug_abbrev  0x00002e88      0x285 CMakeFiles/H750_S15909.elf.dir/Drivers/STM32H7xx_HAL_Driver/Src/stm32h7xx_hal_rcc_ex.c.obj
 .debug_abbrev  0x0000310d      0x22b CMakeFiles/H750_S15909.elf.dir/Drivers/STM32H7xx_HAL_Driver/Src/stm32h7xx_hal_tim.c.obj
 .debug_abbrev  0x00003338      0x241 CMakeFiles/H750_S15909.elf.dir/Drivers/STM32H7xx_HAL_Driver/Src/stm32h7xx_hal_tim_ex.c.obj
 .debug_abbrev  0x00003579      0x337 CMakeFiles/H750_S15909.elf.dir/Drivers/STM32H7xx_HAL_Driver/Src/stm32h7xx_hal_uart.c.obj
 .debug_abbrev  0x000038b0      0x2e7 CMakeFiles/H750_S15909.elf.dir/Drivers/STM32H7xx_HAL_Driver/Src/stm32h7xx_hal_uart_ex.c.obj

.debug_loc      0x00000000    0x1484a
 .debug_loc     0x00000000      0x232 CMakeFiles/H750_S15909.elf.dir/APP/DS18B20.c.obj
 .debug_loc     0x00000232      0x875 CMakeFiles/H750_S15909.elf.dir/APP/IRIS_Method.c.obj
 .debug_loc     0x00000aa7       0xbe CMakeFiles/H750_S15909.elf.dir/APP/Shutter.c.obj
 .debug_loc     0x00000b65      0x197 CMakeFiles/H750_S15909.elf.dir/APP/communication.c.obj
 .debug_loc     0x00000cfc      0x30c CMakeFiles/H750_S15909.elf.dir/APP/data_analyse.c.obj
 .debug_loc     0x00001008       0x69 CMakeFiles/H750_S15909.elf.dir/APP/delay.c.obj
 .debug_loc     0x00001071      0x295 CMakeFiles/H750_S15909.elf.dir/APP/mymain.c.obj
 .debug_loc     0x00001306       0x75 CMakeFiles/H750_S15909.elf.dir/APP/usart1_tx_dma.c.obj
 .debug_loc     0x0000137b      0x3c5 CMakeFiles/H750_S15909.elf.dir/Core/Src/syscalls.c.obj
 .debug_loc     0x00001740       0x64 CMakeFiles/H750_S15909.elf.dir/Core/Src/sysmem.c.obj
 .debug_loc     0x000017a4      0x21e CMakeFiles/H750_S15909.elf.dir/Core/Src/system_stm32h7xx.c.obj
 .debug_loc     0x000019c2      0x122 CMakeFiles/H750_S15909.elf.dir/Core/Src/usart.c.obj
 .debug_loc     0x00001ae4      0x3fa CMakeFiles/H750_S15909.elf.dir/Drivers/STM32H7xx_HAL_Driver/Src/stm32h7xx_hal.c.obj
 .debug_loc     0x00001ede      0x726 CMakeFiles/H750_S15909.elf.dir/Drivers/STM32H7xx_HAL_Driver/Src/stm32h7xx_hal_cortex.c.obj
 .debug_loc     0x00002604      0xe96 CMakeFiles/H750_S15909.elf.dir/Drivers/STM32H7xx_HAL_Driver/Src/stm32h7xx_hal_dma.c.obj
 .debug_loc     0x0000349a      0x3c6 CMakeFiles/H750_S15909.elf.dir/Drivers/STM32H7xx_HAL_Driver/Src/stm32h7xx_hal_gpio.c.obj
 .debug_loc     0x00003860      0x4df CMakeFiles/H750_S15909.elf.dir/Drivers/STM32H7xx_HAL_Driver/Src/stm32h7xx_hal_pwr_ex.c.obj
 .debug_loc     0x00003d3f      0x96f CMakeFiles/H750_S15909.elf.dir/Drivers/STM32H7xx_HAL_Driver/Src/stm32h7xx_hal_rcc.c.obj
 .debug_loc     0x000046ae     0x1bfb CMakeFiles/H750_S15909.elf.dir/Drivers/STM32H7xx_HAL_Driver/Src/stm32h7xx_hal_rcc_ex.c.obj
 .debug_loc     0x000062a9     0x567b CMakeFiles/H750_S15909.elf.dir/Drivers/STM32H7xx_HAL_Driver/Src/stm32h7xx_hal_tim.c.obj
 .debug_loc     0x0000b924     0x257f CMakeFiles/H750_S15909.elf.dir/Drivers/STM32H7xx_HAL_Driver/Src/stm32h7xx_hal_tim_ex.c.obj
 .debug_loc     0x0000dea3     0x5d9b CMakeFiles/H750_S15909.elf.dir/Drivers/STM32H7xx_HAL_Driver/Src/stm32h7xx_hal_uart.c.obj
 .debug_loc     0x00013c3e      0xc0c CMakeFiles/H750_S15909.elf.dir/Drivers/STM32H7xx_HAL_Driver/Src/stm32h7xx_hal_uart_ex.c.obj

.debug_aranges  0x00000000     0x12d0
 .debug_aranges
                0x00000000       0x78 CMakeFiles/H750_S15909.elf.dir/APP/DS18B20.c.obj
 .debug_aranges
                0x00000078       0x48 CMakeFiles/H750_S15909.elf.dir/APP/IRIS_Method.c.obj
 .debug_aranges
                0x000000c0       0x30 CMakeFiles/H750_S15909.elf.dir/APP/Shutter.c.obj
 .debug_aranges
                0x000000f0       0x28 CMakeFiles/H750_S15909.elf.dir/APP/communication.c.obj
 .debug_aranges
                0x00000118       0x30 CMakeFiles/H750_S15909.elf.dir/APP/data_analyse.c.obj
 .debug_aranges
                0x00000148       0x28 CMakeFiles/H750_S15909.elf.dir/APP/delay.c.obj
 .debug_aranges
                0x00000170       0x48 CMakeFiles/H750_S15909.elf.dir/APP/mymain.c.obj
 .debug_aranges
                0x000001b8       0x20 CMakeFiles/H750_S15909.elf.dir/APP/usart1_tx_dma.c.obj
 .debug_aranges
                0x000001d8       0x20 CMakeFiles/H750_S15909.elf.dir/Core/Src/dma.c.obj
 .debug_aranges
                0x000001f8       0x20 CMakeFiles/H750_S15909.elf.dir/Core/Src/gpio.c.obj
 .debug_aranges
                0x00000218       0x30 CMakeFiles/H750_S15909.elf.dir/Core/Src/main.c.obj
 .debug_aranges
                0x00000248       0x20 CMakeFiles/H750_S15909.elf.dir/Core/Src/stm32h7xx_hal_msp.c.obj
 .debug_aranges
                0x00000268       0x78 CMakeFiles/H750_S15909.elf.dir/Core/Src/stm32h7xx_it.c.obj
 .debug_aranges
                0x000002e0       0xa8 CMakeFiles/H750_S15909.elf.dir/Core/Src/syscalls.c.obj
 .debug_aranges
                0x00000388       0x20 CMakeFiles/H750_S15909.elf.dir/Core/Src/sysmem.c.obj
 .debug_aranges
                0x000003a8       0x28 CMakeFiles/H750_S15909.elf.dir/Core/Src/system_stm32h7xx.c.obj
 .debug_aranges
                0x000003d0       0x30 CMakeFiles/H750_S15909.elf.dir/Core/Src/tim.c.obj
 .debug_aranges
                0x00000400       0x40 CMakeFiles/H750_S15909.elf.dir/Core/Src/usart.c.obj
 .debug_aranges
                0x00000440       0x28 CMakeFiles/H750_S15909.elf.dir/Core/Startup/startup_stm32h750vbtx.s.obj
 .debug_aranges
                0x00000468      0x198 CMakeFiles/H750_S15909.elf.dir/Drivers/STM32H7xx_HAL_Driver/Src/stm32h7xx_hal.c.obj
 .debug_aranges
                0x00000600       0xb0 CMakeFiles/H750_S15909.elf.dir/Drivers/STM32H7xx_HAL_Driver/Src/stm32h7xx_hal_cortex.c.obj
 .debug_aranges
                0x000006b0       0xa0 CMakeFiles/H750_S15909.elf.dir/Drivers/STM32H7xx_HAL_Driver/Src/stm32h7xx_hal_dma.c.obj
 .debug_aranges
                0x00000750       0x58 CMakeFiles/H750_S15909.elf.dir/Drivers/STM32H7xx_HAL_Driver/Src/stm32h7xx_hal_gpio.c.obj
 .debug_aranges
                0x000007a8      0x158 CMakeFiles/H750_S15909.elf.dir/Drivers/STM32H7xx_HAL_Driver/Src/stm32h7xx_hal_pwr_ex.c.obj
 .debug_aranges
                0x00000900       0x88 CMakeFiles/H750_S15909.elf.dir/Drivers/STM32H7xx_HAL_Driver/Src/stm32h7xx_hal_rcc.c.obj
 .debug_aranges
                0x00000988       0xf8 CMakeFiles/H750_S15909.elf.dir/Drivers/STM32H7xx_HAL_Driver/Src/stm32h7xx_hal_rcc_ex.c.obj
 .debug_aranges
                0x00000a80      0x3e0 CMakeFiles/H750_S15909.elf.dir/Drivers/STM32H7xx_HAL_Driver/Src/stm32h7xx_hal_tim.c.obj
 .debug_aranges
                0x00000e60      0x188 CMakeFiles/H750_S15909.elf.dir/Drivers/STM32H7xx_HAL_Driver/Src/stm32h7xx_hal_tim_ex.c.obj
 .debug_aranges
                0x00000fe8      0x248 CMakeFiles/H750_S15909.elf.dir/Drivers/STM32H7xx_HAL_Driver/Src/stm32h7xx_hal_uart.c.obj
 .debug_aranges
                0x00001230       0xa0 CMakeFiles/H750_S15909.elf.dir/Drivers/STM32H7xx_HAL_Driver/Src/stm32h7xx_hal_uart_ex.c.obj

.debug_ranges   0x00000000     0x1398
 .debug_ranges  0x00000000       0x80 CMakeFiles/H750_S15909.elf.dir/APP/DS18B20.c.obj
 .debug_ranges  0x00000080       0x80 CMakeFiles/H750_S15909.elf.dir/APP/IRIS_Method.c.obj
 .debug_ranges  0x00000100       0x20 CMakeFiles/H750_S15909.elf.dir/APP/Shutter.c.obj
 .debug_ranges  0x00000120       0x30 CMakeFiles/H750_S15909.elf.dir/APP/communication.c.obj
 .debug_ranges  0x00000150       0x70 CMakeFiles/H750_S15909.elf.dir/APP/data_analyse.c.obj
 .debug_ranges  0x000001c0       0x18 CMakeFiles/H750_S15909.elf.dir/APP/delay.c.obj
 .debug_ranges  0x000001d8       0xc8 CMakeFiles/H750_S15909.elf.dir/APP/mymain.c.obj
 .debug_ranges  0x000002a0       0x10 CMakeFiles/H750_S15909.elf.dir/APP/usart1_tx_dma.c.obj
 .debug_ranges  0x000002b0       0x10 CMakeFiles/H750_S15909.elf.dir/Core/Src/dma.c.obj
 .debug_ranges  0x000002c0       0x10 CMakeFiles/H750_S15909.elf.dir/Core/Src/gpio.c.obj
 .debug_ranges  0x000002d0       0x20 CMakeFiles/H750_S15909.elf.dir/Core/Src/main.c.obj
 .debug_ranges  0x000002f0       0x10 CMakeFiles/H750_S15909.elf.dir/Core/Src/stm32h7xx_hal_msp.c.obj
 .debug_ranges  0x00000300       0x68 CMakeFiles/H750_S15909.elf.dir/Core/Src/stm32h7xx_it.c.obj
 .debug_ranges  0x00000368       0x98 CMakeFiles/H750_S15909.elf.dir/Core/Src/syscalls.c.obj
 .debug_ranges  0x00000400       0x10 CMakeFiles/H750_S15909.elf.dir/Core/Src/sysmem.c.obj
 .debug_ranges  0x00000410       0x18 CMakeFiles/H750_S15909.elf.dir/Core/Src/system_stm32h7xx.c.obj
 .debug_ranges  0x00000428       0x20 CMakeFiles/H750_S15909.elf.dir/Core/Src/tim.c.obj
 .debug_ranges  0x00000448       0x30 CMakeFiles/H750_S15909.elf.dir/Core/Src/usart.c.obj
 .debug_ranges  0x00000478       0x20 CMakeFiles/H750_S15909.elf.dir/Core/Startup/startup_stm32h750vbtx.s.obj
 .debug_ranges  0x00000498      0x188 CMakeFiles/H750_S15909.elf.dir/Drivers/STM32H7xx_HAL_Driver/Src/stm32h7xx_hal.c.obj
 .debug_ranges  0x00000620      0x100 CMakeFiles/H750_S15909.elf.dir/Drivers/STM32H7xx_HAL_Driver/Src/stm32h7xx_hal_cortex.c.obj
 .debug_ranges  0x00000720       0xa8 CMakeFiles/H750_S15909.elf.dir/Drivers/STM32H7xx_HAL_Driver/Src/stm32h7xx_hal_dma.c.obj
 .debug_ranges  0x000007c8       0x48 CMakeFiles/H750_S15909.elf.dir/Drivers/STM32H7xx_HAL_Driver/Src/stm32h7xx_hal_gpio.c.obj
 .debug_ranges  0x00000810      0x1a8 CMakeFiles/H750_S15909.elf.dir/Drivers/STM32H7xx_HAL_Driver/Src/stm32h7xx_hal_pwr_ex.c.obj
 .debug_ranges  0x000009b8       0xe8 CMakeFiles/H750_S15909.elf.dir/Drivers/STM32H7xx_HAL_Driver/Src/stm32h7xx_hal_rcc.c.obj
 .debug_ranges  0x00000aa0       0xe8 CMakeFiles/H750_S15909.elf.dir/Drivers/STM32H7xx_HAL_Driver/Src/stm32h7xx_hal_rcc_ex.c.obj
 .debug_ranges  0x00000b88      0x3d0 CMakeFiles/H750_S15909.elf.dir/Drivers/STM32H7xx_HAL_Driver/Src/stm32h7xx_hal_tim.c.obj
 .debug_ranges  0x00000f58      0x178 CMakeFiles/H750_S15909.elf.dir/Drivers/STM32H7xx_HAL_Driver/Src/stm32h7xx_hal_tim_ex.c.obj
 .debug_ranges  0x000010d0      0x238 CMakeFiles/H750_S15909.elf.dir/Drivers/STM32H7xx_HAL_Driver/Src/stm32h7xx_hal_uart.c.obj
 .debug_ranges  0x00001308       0x90 CMakeFiles/H750_S15909.elf.dir/Drivers/STM32H7xx_HAL_Driver/Src/stm32h7xx_hal_uart_ex.c.obj

.debug_line     0x00000000    0x19b5b
 .debug_line    0x00000000      0x4f8 CMakeFiles/H750_S15909.elf.dir/APP/DS18B20.c.obj
 .debug_line    0x000004f8      0x51c CMakeFiles/H750_S15909.elf.dir/APP/IRIS_Method.c.obj
 .debug_line    0x00000a14      0x249 CMakeFiles/H750_S15909.elf.dir/APP/Shutter.c.obj
 .debug_line    0x00000c5d      0x309 CMakeFiles/H750_S15909.elf.dir/APP/communication.c.obj
 .debug_line    0x00000f66      0x32f CMakeFiles/H750_S15909.elf.dir/APP/data_analyse.c.obj
 .debug_line    0x00001295      0x247 CMakeFiles/H750_S15909.elf.dir/APP/delay.c.obj
 .debug_line    0x000014dc      0x7e8 CMakeFiles/H750_S15909.elf.dir/APP/mymain.c.obj
 .debug_line    0x00001cc4      0x346 CMakeFiles/H750_S15909.elf.dir/APP/usart1_tx_dma.c.obj
 .debug_line    0x0000200a      0x1c9 CMakeFiles/H750_S15909.elf.dir/Core/Src/dma.c.obj
 .debug_line    0x000021d3      0x25a CMakeFiles/H750_S15909.elf.dir/Core/Src/gpio.c.obj
 .debug_line    0x0000242d      0x435 CMakeFiles/H750_S15909.elf.dir/Core/Src/main.c.obj
 .debug_line    0x00002862      0x188 CMakeFiles/H750_S15909.elf.dir/Core/Src/stm32h7xx_hal_msp.c.obj
 .debug_line    0x000029ea      0x360 CMakeFiles/H750_S15909.elf.dir/Core/Src/stm32h7xx_it.c.obj
 .debug_line    0x00002d4a      0x40f CMakeFiles/H750_S15909.elf.dir/Core/Src/syscalls.c.obj
 .debug_line    0x00003159      0x1ec CMakeFiles/H750_S15909.elf.dir/Core/Src/sysmem.c.obj
 .debug_line    0x00003345      0x43c CMakeFiles/H750_S15909.elf.dir/Core/Src/system_stm32h7xx.c.obj
 .debug_line    0x00003781      0x30a CMakeFiles/H750_S15909.elf.dir/Core/Src/tim.c.obj
 .debug_line    0x00003a8b      0x5d4 CMakeFiles/H750_S15909.elf.dir/Core/Src/usart.c.obj
 .debug_line    0x0000405f       0x97 CMakeFiles/H750_S15909.elf.dir/Core/Startup/startup_stm32h750vbtx.s.obj
 .debug_line    0x000040f6      0x914 CMakeFiles/H750_S15909.elf.dir/Drivers/STM32H7xx_HAL_Driver/Src/stm32h7xx_hal.c.obj
 .debug_line    0x00004a0a      0x7df CMakeFiles/H750_S15909.elf.dir/Drivers/STM32H7xx_HAL_Driver/Src/stm32h7xx_hal_cortex.c.obj
 .debug_line    0x000051e9     0x247d CMakeFiles/H750_S15909.elf.dir/Drivers/STM32H7xx_HAL_Driver/Src/stm32h7xx_hal_dma.c.obj
 .debug_line    0x00007666      0x6f9 CMakeFiles/H750_S15909.elf.dir/Drivers/STM32H7xx_HAL_Driver/Src/stm32h7xx_hal_gpio.c.obj
 .debug_line    0x00007d5f      0xad4 CMakeFiles/H750_S15909.elf.dir/Drivers/STM32H7xx_HAL_Driver/Src/stm32h7xx_hal_pwr_ex.c.obj
 .debug_line    0x00008833     0x1244 CMakeFiles/H750_S15909.elf.dir/Drivers/STM32H7xx_HAL_Driver/Src/stm32h7xx_hal_rcc.c.obj
 .debug_line    0x00009a77     0x1d9c CMakeFiles/H750_S15909.elf.dir/Drivers/STM32H7xx_HAL_Driver/Src/stm32h7xx_hal_rcc_ex.c.obj
 .debug_line    0x0000b813     0x5064 CMakeFiles/H750_S15909.elf.dir/Drivers/STM32H7xx_HAL_Driver/Src/stm32h7xx_hal_tim.c.obj
 .debug_line    0x00010877     0x1f6b CMakeFiles/H750_S15909.elf.dir/Drivers/STM32H7xx_HAL_Driver/Src/stm32h7xx_hal_tim_ex.c.obj
 .debug_line    0x000127e2     0x6646 CMakeFiles/H750_S15909.elf.dir/Drivers/STM32H7xx_HAL_Driver/Src/stm32h7xx_hal_uart.c.obj
 .debug_line    0x00018e28      0xd33 CMakeFiles/H750_S15909.elf.dir/Drivers/STM32H7xx_HAL_Driver/Src/stm32h7xx_hal_uart_ex.c.obj

.debug_str      0x00000000     0x6c08
 .debug_str     0x00000000      0x59d CMakeFiles/H750_S15909.elf.dir/APP/DS18B20.c.obj
                                0x611 (size before relaxing)
 .debug_str     0x0000059d      0x155 CMakeFiles/H750_S15909.elf.dir/APP/IRIS_Method.c.obj
                                0x328 (size before relaxing)
 .debug_str     0x000006f2       0x50 CMakeFiles/H750_S15909.elf.dir/APP/Shutter.c.obj
                                0x4d8 (size before relaxing)
 .debug_str     0x00000742      0x5d4 CMakeFiles/H750_S15909.elf.dir/APP/communication.c.obj
                                0x835 (size before relaxing)
 .debug_str     0x00000d16       0x88 CMakeFiles/H750_S15909.elf.dir/APP/data_analyse.c.obj
                                0x272 (size before relaxing)
 .debug_str     0x00000d9e      0x32d CMakeFiles/H750_S15909.elf.dir/APP/delay.c.obj
                                0x865 (size before relaxing)
 .debug_str     0x000010cb      0x5fe CMakeFiles/H750_S15909.elf.dir/APP/mymain.c.obj
                                0xe92 (size before relaxing)
 .debug_str     0x000016c9       0x54 CMakeFiles/H750_S15909.elf.dir/APP/usart1_tx_dma.c.obj
                                0xa02 (size before relaxing)
 .debug_str     0x0000171d      0x859 CMakeFiles/H750_S15909.elf.dir/Core/Src/dma.c.obj
                                0xc56 (size before relaxing)
 .debug_str     0x00001f76       0x2f CMakeFiles/H750_S15909.elf.dir/Core/Src/gpio.c.obj
                                0xd27 (size before relaxing)
 .debug_str     0x00001fa5      0x30d CMakeFiles/H750_S15909.elf.dir/Core/Src/main.c.obj
                                0x729 (size before relaxing)
 .debug_str     0x000022b2       0x3b CMakeFiles/H750_S15909.elf.dir/Core/Src/stm32h7xx_hal_msp.c.obj
                                0x410 (size before relaxing)
 .debug_str     0x000022ed      0x150 CMakeFiles/H750_S15909.elf.dir/Core/Src/stm32h7xx_it.c.obj
                                0x87a (size before relaxing)
 .debug_str     0x0000243d      0x20e CMakeFiles/H750_S15909.elf.dir/Core/Src/syscalls.c.obj
                                0x415 (size before relaxing)
 .debug_str     0x0000264b       0x84 CMakeFiles/H750_S15909.elf.dir/Core/Src/sysmem.c.obj
                                0x241 (size before relaxing)
 .debug_str     0x000026cf      0x292 CMakeFiles/H750_S15909.elf.dir/Core/Src/system_stm32h7xx.c.obj
                                0x686 (size before relaxing)
 .debug_str     0x00002961      0x151 CMakeFiles/H750_S15909.elf.dir/Core/Src/tim.c.obj
                                0xbbc (size before relaxing)
 .debug_str     0x00002ab2      0x430 CMakeFiles/H750_S15909.elf.dir/Core/Src/usart.c.obj
                               0x1734 (size before relaxing)
 .debug_str     0x00002ee2       0x45 CMakeFiles/H750_S15909.elf.dir/Core/Startup/startup_stm32h750vbtx.s.obj
                                 0x75 (size before relaxing)
 .debug_str     0x00002f27      0x721 CMakeFiles/H750_S15909.elf.dir/Drivers/STM32H7xx_HAL_Driver/Src/stm32h7xx_hal.c.obj
                               0x14dd (size before relaxing)
 .debug_str     0x00003648      0x545 CMakeFiles/H750_S15909.elf.dir/Drivers/STM32H7xx_HAL_Driver/Src/stm32h7xx_hal_cortex.c.obj
                               0x1075 (size before relaxing)
 .debug_str     0x00003b8d      0x3c0 CMakeFiles/H750_S15909.elf.dir/Drivers/STM32H7xx_HAL_Driver/Src/stm32h7xx_hal_dma.c.obj
                                0x9e9 (size before relaxing)
 .debug_str     0x00003f4d       0xad CMakeFiles/H750_S15909.elf.dir/Drivers/STM32H7xx_HAL_Driver/Src/stm32h7xx_hal_gpio.c.obj
                                0x6f2 (size before relaxing)
 .debug_str     0x00003ffa      0x55c CMakeFiles/H750_S15909.elf.dir/Drivers/STM32H7xx_HAL_Driver/Src/stm32h7xx_hal_pwr_ex.c.obj
                                0xa67 (size before relaxing)
 .debug_str     0x00004556      0x1a1 CMakeFiles/H750_S15909.elf.dir/Drivers/STM32H7xx_HAL_Driver/Src/stm32h7xx_hal_rcc.c.obj
                                0xa7a (size before relaxing)
 .debug_str     0x000046f7      0x5d4 CMakeFiles/H750_S15909.elf.dir/Drivers/STM32H7xx_HAL_Driver/Src/stm32h7xx_hal_rcc_ex.c.obj
                                0xf5c (size before relaxing)
 .debug_str     0x00004ccb      0xe94 CMakeFiles/H750_S15909.elf.dir/Drivers/STM32H7xx_HAL_Driver/Src/stm32h7xx_hal_tim.c.obj
                               0x1841 (size before relaxing)
 .debug_str     0x00005b5f      0x630 CMakeFiles/H750_S15909.elf.dir/Drivers/STM32H7xx_HAL_Driver/Src/stm32h7xx_hal_tim_ex.c.obj
                               0x115e (size before relaxing)
 .debug_str     0x0000618f      0x842 CMakeFiles/H750_S15909.elf.dir/Drivers/STM32H7xx_HAL_Driver/Src/stm32h7xx_hal_uart.c.obj
                               0x14a9 (size before relaxing)
 .debug_str     0x000069d1      0x237 CMakeFiles/H750_S15909.elf.dir/Drivers/STM32H7xx_HAL_Driver/Src/stm32h7xx_hal_uart_ex.c.obj
                                0xb78 (size before relaxing)

.comment        0x00000000       0x49
 .comment       0x00000000       0x49 CMakeFiles/H750_S15909.elf.dir/APP/DS18B20.c.obj
                                 0x4a (size before relaxing)
 .comment       0x00000049       0x4a CMakeFiles/H750_S15909.elf.dir/APP/IRIS_Method.c.obj
 .comment       0x00000049       0x4a CMakeFiles/H750_S15909.elf.dir/APP/Shutter.c.obj
 .comment       0x00000049       0x4a CMakeFiles/H750_S15909.elf.dir/APP/communication.c.obj
 .comment       0x00000049       0x4a CMakeFiles/H750_S15909.elf.dir/APP/data_analyse.c.obj
 .comment       0x00000049       0x4a CMakeFiles/H750_S15909.elf.dir/APP/delay.c.obj
 .comment       0x00000049       0x4a CMakeFiles/H750_S15909.elf.dir/APP/mymain.c.obj
 .comment       0x00000049       0x4a CMakeFiles/H750_S15909.elf.dir/APP/usart1_tx_dma.c.obj
 .comment       0x00000049       0x4a CMakeFiles/H750_S15909.elf.dir/Core/Src/dma.c.obj
 .comment       0x00000049       0x4a CMakeFiles/H750_S15909.elf.dir/Core/Src/gpio.c.obj
 .comment       0x00000049       0x4a CMakeFiles/H750_S15909.elf.dir/Core/Src/main.c.obj
 .comment       0x00000049       0x4a CMakeFiles/H750_S15909.elf.dir/Core/Src/stm32h7xx_hal_msp.c.obj
 .comment       0x00000049       0x4a CMakeFiles/H750_S15909.elf.dir/Core/Src/stm32h7xx_it.c.obj
 .comment       0x00000049       0x4a CMakeFiles/H750_S15909.elf.dir/Core/Src/syscalls.c.obj
 .comment       0x00000049       0x4a CMakeFiles/H750_S15909.elf.dir/Core/Src/sysmem.c.obj
 .comment       0x00000049       0x4a CMakeFiles/H750_S15909.elf.dir/Core/Src/system_stm32h7xx.c.obj
 .comment       0x00000049       0x4a CMakeFiles/H750_S15909.elf.dir/Core/Src/tim.c.obj
 .comment       0x00000049       0x4a CMakeFiles/H750_S15909.elf.dir/Core/Src/usart.c.obj
 .comment       0x00000049       0x4a CMakeFiles/H750_S15909.elf.dir/Drivers/STM32H7xx_HAL_Driver/Src/stm32h7xx_hal.c.obj
 .comment       0x00000049       0x4a CMakeFiles/H750_S15909.elf.dir/Drivers/STM32H7xx_HAL_Driver/Src/stm32h7xx_hal_cortex.c.obj
 .comment       0x00000049       0x4a CMakeFiles/H750_S15909.elf.dir/Drivers/STM32H7xx_HAL_Driver/Src/stm32h7xx_hal_dma.c.obj
 .comment       0x00000049       0x4a CMakeFiles/H750_S15909.elf.dir/Drivers/STM32H7xx_HAL_Driver/Src/stm32h7xx_hal_gpio.c.obj
 .comment       0x00000049       0x4a CMakeFiles/H750_S15909.elf.dir/Drivers/STM32H7xx_HAL_Driver/Src/stm32h7xx_hal_pwr_ex.c.obj
 .comment       0x00000049       0x4a CMakeFiles/H750_S15909.elf.dir/Drivers/STM32H7xx_HAL_Driver/Src/stm32h7xx_hal_rcc.c.obj
 .comment       0x00000049       0x4a CMakeFiles/H750_S15909.elf.dir/Drivers/STM32H7xx_HAL_Driver/Src/stm32h7xx_hal_rcc_ex.c.obj
 .comment       0x00000049       0x4a CMakeFiles/H750_S15909.elf.dir/Drivers/STM32H7xx_HAL_Driver/Src/stm32h7xx_hal_tim.c.obj
 .comment       0x00000049       0x4a CMakeFiles/H750_S15909.elf.dir/Drivers/STM32H7xx_HAL_Driver/Src/stm32h7xx_hal_tim_ex.c.obj
 .comment       0x00000049       0x4a CMakeFiles/H750_S15909.elf.dir/Drivers/STM32H7xx_HAL_Driver/Src/stm32h7xx_hal_uart.c.obj
 .comment       0x00000049       0x4a CMakeFiles/H750_S15909.elf.dir/Drivers/STM32H7xx_HAL_Driver/Src/stm32h7xx_hal_uart_ex.c.obj

.debug_frame    0x00000000     0x3b7c
 .debug_frame   0x00000000      0x150 CMakeFiles/H750_S15909.elf.dir/APP/DS18B20.c.obj
 .debug_frame   0x00000150       0xe8 CMakeFiles/H750_S15909.elf.dir/APP/IRIS_Method.c.obj
 .debug_frame   0x00000238       0x5c CMakeFiles/H750_S15909.elf.dir/APP/Shutter.c.obj
 .debug_frame   0x00000294       0x50 CMakeFiles/H750_S15909.elf.dir/APP/communication.c.obj
 .debug_frame   0x000002e4       0x80 CMakeFiles/H750_S15909.elf.dir/APP/data_analyse.c.obj
 .debug_frame   0x00000364       0x44 CMakeFiles/H750_S15909.elf.dir/APP/delay.c.obj
 .debug_frame   0x000003a8       0xc4 CMakeFiles/H750_S15909.elf.dir/APP/mymain.c.obj
 .debug_frame   0x0000046c       0x30 CMakeFiles/H750_S15909.elf.dir/APP/usart1_tx_dma.c.obj
 .debug_frame   0x0000049c       0x2c CMakeFiles/H750_S15909.elf.dir/Core/Src/dma.c.obj
 .debug_frame   0x000004c8       0x34 CMakeFiles/H750_S15909.elf.dir/Core/Src/gpio.c.obj
 .debug_frame   0x000004fc       0x58 CMakeFiles/H750_S15909.elf.dir/Core/Src/main.c.obj
 .debug_frame   0x00000554       0x28 CMakeFiles/H750_S15909.elf.dir/Core/Src/stm32h7xx_hal_msp.c.obj
 .debug_frame   0x0000057c       0xf0 CMakeFiles/H750_S15909.elf.dir/Core/Src/stm32h7xx_it.c.obj
 .debug_frame   0x0000066c      0x190 CMakeFiles/H750_S15909.elf.dir/Core/Src/syscalls.c.obj
 .debug_frame   0x000007fc       0x28 CMakeFiles/H750_S15909.elf.dir/Core/Src/sysmem.c.obj
 .debug_frame   0x00000824       0x40 CMakeFiles/H750_S15909.elf.dir/Core/Src/system_stm32h7xx.c.obj
 .debug_frame   0x00000864       0x58 CMakeFiles/H750_S15909.elf.dir/Core/Src/tim.c.obj
 .debug_frame   0x000008bc       0x8c CMakeFiles/H750_S15909.elf.dir/Core/Src/usart.c.obj
 .debug_frame   0x00000948      0x360 CMakeFiles/H750_S15909.elf.dir/Drivers/STM32H7xx_HAL_Driver/Src/stm32h7xx_hal.c.obj
 .debug_frame   0x00000ca8      0x158 CMakeFiles/H750_S15909.elf.dir/Drivers/STM32H7xx_HAL_Driver/Src/stm32h7xx_hal_cortex.c.obj
 .debug_frame   0x00000e00      0x1fc CMakeFiles/H750_S15909.elf.dir/Drivers/STM32H7xx_HAL_Driver/Src/stm32h7xx_hal_dma.c.obj
 .debug_frame   0x00000ffc       0xd0 CMakeFiles/H750_S15909.elf.dir/Drivers/STM32H7xx_HAL_Driver/Src/stm32h7xx_hal_gpio.c.obj
 .debug_frame   0x000010cc      0x2f4 CMakeFiles/H750_S15909.elf.dir/Drivers/STM32H7xx_HAL_Driver/Src/stm32h7xx_hal_pwr_ex.c.obj
 .debug_frame   0x000013c0      0x188 CMakeFiles/H750_S15909.elf.dir/Drivers/STM32H7xx_HAL_Driver/Src/stm32h7xx_hal_rcc.c.obj
 .debug_frame   0x00001548      0x284 CMakeFiles/H750_S15909.elf.dir/Drivers/STM32H7xx_HAL_Driver/Src/stm32h7xx_hal_rcc_ex.c.obj
 .debug_frame   0x000017cc      0xb64 CMakeFiles/H750_S15909.elf.dir/Drivers/STM32H7xx_HAL_Driver/Src/stm32h7xx_hal_tim.c.obj
 .debug_frame   0x00002330      0x480 CMakeFiles/H750_S15909.elf.dir/Drivers/STM32H7xx_HAL_Driver/Src/stm32h7xx_hal_tim_ex.c.obj
 .debug_frame   0x000027b0      0x688 CMakeFiles/H750_S15909.elf.dir/Drivers/STM32H7xx_HAL_Driver/Src/stm32h7xx_hal_uart.c.obj
 .debug_frame   0x00002e38      0x1c8 CMakeFiles/H750_S15909.elf.dir/Drivers/STM32H7xx_HAL_Driver/Src/stm32h7xx_hal_uart_ex.c.obj
 .debug_frame   0x00003000       0xac d:/lijie_tools/clion_cubemx/gcc-arm-none-eabi-10.3-2021.10/bin/../lib/gcc/arm-none-eabi/10.3.1/thumb/v7e-m/nofp\libgcc.a(_arm_addsubdf3.o)
 .debug_frame   0x000030ac       0x50 d:/lijie_tools/clion_cubemx/gcc-arm-none-eabi-10.3-2021.10/bin/../lib/gcc/arm-none-eabi/10.3.1/thumb/v7e-m/nofp\libgcc.a(_arm_muldivdf3.o)
 .debug_frame   0x000030fc       0xc4 d:/lijie_tools/clion_cubemx/gcc-arm-none-eabi-10.3-2021.10/bin/../lib/gcc/arm-none-eabi/10.3.1/thumb/v7e-m/nofp\libgcc.a(_arm_cmpdf2.o)
 .debug_frame   0x000031c0       0x24 d:/lijie_tools/clion_cubemx/gcc-arm-none-eabi-10.3-2021.10/bin/../lib/gcc/arm-none-eabi/10.3.1/thumb/v7e-m/nofp\libgcc.a(_arm_fixdfsi.o)
 .debug_frame   0x000031e4       0x24 d:/lijie_tools/clion_cubemx/gcc-arm-none-eabi-10.3-2021.10/bin/../lib/gcc/arm-none-eabi/10.3.1/thumb/v7e-m/nofp\libgcc.a(_arm_fixunsdfsi.o)
 .debug_frame   0x00003208       0x24 d:/lijie_tools/clion_cubemx/gcc-arm-none-eabi-10.3-2021.10/bin/../lib/gcc/arm-none-eabi/10.3.1/thumb/v7e-m/nofp\libgcc.a(_arm_truncdfsf2.o)
 .debug_frame   0x0000322c       0x4c d:/lijie_tools/clion_cubemx/gcc-arm-none-eabi-10.3-2021.10/bin/../lib/gcc/arm-none-eabi/10.3.1/thumb/v7e-m/nofp\libgcc.a(_arm_addsubsf3.o)
 .debug_frame   0x00003278       0x38 d:/lijie_tools/clion_cubemx/gcc-arm-none-eabi-10.3-2021.10/bin/../lib/gcc/arm-none-eabi/10.3.1/thumb/v7e-m/nofp\libgcc.a(_arm_muldivsf3.o)
 .debug_frame   0x000032b0       0x24 d:/lijie_tools/clion_cubemx/gcc-arm-none-eabi-10.3-2021.10/bin/../lib/gcc/arm-none-eabi/10.3.1/thumb/v7e-m/nofp\libgcc.a(_arm_fixunssfsi.o)
 .debug_frame   0x000032d4       0x2c d:/lijie_tools/clion_cubemx/gcc-arm-none-eabi-10.3-2021.10/bin/../lib/gcc/arm-none-eabi/10.3.1/thumb/v7e-m/nofp\libgcc.a(_aeabi_uldivmod.o)
 .debug_frame   0x00003300       0x34 d:/lijie_tools/clion_cubemx/gcc-arm-none-eabi-10.3-2021.10/bin/../lib/gcc/arm-none-eabi/10.3.1/thumb/v7e-m/nofp\libgcc.a(_udivmoddi4.o)
 .debug_frame   0x00003334       0x20 d:/lijie_tools/clion_cubemx/gcc-arm-none-eabi-10.3-2021.10/bin/../lib/gcc/arm-none-eabi/10.3.1/../../../../arm-none-eabi/lib/thumb/v7e-m/nofp\libg.a(lib_a-errno.o)
 .debug_frame   0x00003354       0x2c d:/lijie_tools/clion_cubemx/gcc-arm-none-eabi-10.3-2021.10/bin/../lib/gcc/arm-none-eabi/10.3.1/../../../../arm-none-eabi/lib/thumb/v7e-m/nofp\libg.a(lib_a-init.o)
 .debug_frame   0x00003380       0x2c d:/lijie_tools/clion_cubemx/gcc-arm-none-eabi-10.3-2021.10/bin/../lib/gcc/arm-none-eabi/10.3.1/../../../../arm-none-eabi/lib/thumb/v7e-m/nofp\libg.a(lib_a-memset.o)
 .debug_frame   0x000033ac       0x48 d:/lijie_tools/clion_cubemx/gcc-arm-none-eabi-10.3-2021.10/bin/../lib/gcc/arm-none-eabi/10.3.1/../../../../arm-none-eabi/lib/thumb/v7e-m/nofp\libg.a(lib_a-setvbuf.o)
 .debug_frame   0x000033f4       0x5c d:/lijie_tools/clion_cubemx/gcc-arm-none-eabi-10.3-2021.10/bin/../lib/gcc/arm-none-eabi/10.3.1/../../../../arm-none-eabi/lib/thumb/v7e-m/nofp\libg.a(lib_a-__call_atexit.o)
 .debug_frame   0x00003450       0x20 d:/lijie_tools/clion_cubemx/gcc-arm-none-eabi-10.3-2021.10/bin/../lib/gcc/arm-none-eabi/10.3.1/../../../../arm-none-eabi/lib/thumb/v7e-m/nofp\libg.a(lib_a-atexit.o)
 .debug_frame   0x00003470       0x70 d:/lijie_tools/clion_cubemx/gcc-arm-none-eabi-10.3-2021.10/bin/../lib/gcc/arm-none-eabi/10.3.1/../../../../arm-none-eabi/lib/thumb/v7e-m/nofp\libg.a(lib_a-fflush.o)
 .debug_frame   0x000034e0      0x154 d:/lijie_tools/clion_cubemx/gcc-arm-none-eabi-10.3-2021.10/bin/../lib/gcc/arm-none-eabi/10.3.1/../../../../arm-none-eabi/lib/thumb/v7e-m/nofp\libg.a(lib_a-findfp.o)
 .debug_frame   0x00003634       0x34 d:/lijie_tools/clion_cubemx/gcc-arm-none-eabi-10.3-2021.10/bin/../lib/gcc/arm-none-eabi/10.3.1/../../../../arm-none-eabi/lib/thumb/v7e-m/nofp\libg.a(lib_a-fini.o)
 .debug_frame   0x00003668       0x8c d:/lijie_tools/clion_cubemx/gcc-arm-none-eabi-10.3-2021.10/bin/../lib/gcc/arm-none-eabi/10.3.1/../../../../arm-none-eabi/lib/thumb/v7e-m/nofp\libg.a(lib_a-freer.o)
 .debug_frame   0x000036f4       0x54 d:/lijie_tools/clion_cubemx/gcc-arm-none-eabi-10.3-2021.10/bin/../lib/gcc/arm-none-eabi/10.3.1/../../../../arm-none-eabi/lib/thumb/v7e-m/nofp\libg.a(lib_a-fwalk.o)
 .debug_frame   0x00003748       0xb0 d:/lijie_tools/clion_cubemx/gcc-arm-none-eabi-10.3-2021.10/bin/../lib/gcc/arm-none-eabi/10.3.1/../../../../arm-none-eabi/lib/thumb/v7e-m/nofp\libg.a(lib_a-lock.o)
 .debug_frame   0x000037f8       0x70 d:/lijie_tools/clion_cubemx/gcc-arm-none-eabi-10.3-2021.10/bin/../lib/gcc/arm-none-eabi/10.3.1/../../../../arm-none-eabi/lib/thumb/v7e-m/nofp\libg.a(lib_a-makebuf.o)
 .debug_frame   0x00003868       0x30 d:/lijie_tools/clion_cubemx/gcc-arm-none-eabi-10.3-2021.10/bin/../lib/gcc/arm-none-eabi/10.3.1/../../../../arm-none-eabi/lib/thumb/v7e-m/nofp\libg.a(lib_a-malloc.o)
 .debug_frame   0x00003898       0x4c d:/lijie_tools/clion_cubemx/gcc-arm-none-eabi-10.3-2021.10/bin/../lib/gcc/arm-none-eabi/10.3.1/../../../../arm-none-eabi/lib/thumb/v7e-m/nofp\libg.a(lib_a-mallocr.o)
 .debug_frame   0x000038e4       0x30 d:/lijie_tools/clion_cubemx/gcc-arm-none-eabi-10.3-2021.10/bin/../lib/gcc/arm-none-eabi/10.3.1/../../../../arm-none-eabi/lib/thumb/v7e-m/nofp\libg.a(lib_a-mlock.o)
 .debug_frame   0x00003914       0x2c d:/lijie_tools/clion_cubemx/gcc-arm-none-eabi-10.3-2021.10/bin/../lib/gcc/arm-none-eabi/10.3.1/../../../../arm-none-eabi/lib/thumb/v7e-m/nofp\libg.a(lib_a-sbrkr.o)
 .debug_frame   0x00003940       0x8c d:/lijie_tools/clion_cubemx/gcc-arm-none-eabi-10.3-2021.10/bin/../lib/gcc/arm-none-eabi/10.3.1/../../../../arm-none-eabi/lib/thumb/v7e-m/nofp\libg.a(lib_a-stdio.o)
 .debug_frame   0x000039cc       0x2c d:/lijie_tools/clion_cubemx/gcc-arm-none-eabi-10.3-2021.10/bin/../lib/gcc/arm-none-eabi/10.3.1/../../../../arm-none-eabi/lib/thumb/v7e-m/nofp\libg.a(lib_a-writer.o)
 .debug_frame   0x000039f8       0x34 d:/lijie_tools/clion_cubemx/gcc-arm-none-eabi-10.3-2021.10/bin/../lib/gcc/arm-none-eabi/10.3.1/../../../../arm-none-eabi/lib/thumb/v7e-m/nofp\libg.a(lib_a-__atexit.o)
 .debug_frame   0x00003a2c       0x2c d:/lijie_tools/clion_cubemx/gcc-arm-none-eabi-10.3-2021.10/bin/../lib/gcc/arm-none-eabi/10.3.1/../../../../arm-none-eabi/lib/thumb/v7e-m/nofp\libg.a(lib_a-closer.o)
 .debug_frame   0x00003a58       0x3c d:/lijie_tools/clion_cubemx/gcc-arm-none-eabi-10.3-2021.10/bin/../lib/gcc/arm-none-eabi/10.3.1/../../../../arm-none-eabi/lib/thumb/v7e-m/nofp\libg.a(lib_a-fclose.o)
 .debug_frame   0x00003a94       0x2c d:/lijie_tools/clion_cubemx/gcc-arm-none-eabi-10.3-2021.10/bin/../lib/gcc/arm-none-eabi/10.3.1/../../../../arm-none-eabi/lib/thumb/v7e-m/nofp\libg.a(lib_a-fstatr.o)
 .debug_frame   0x00003ac0       0x2c d:/lijie_tools/clion_cubemx/gcc-arm-none-eabi-10.3-2021.10/bin/../lib/gcc/arm-none-eabi/10.3.1/../../../../arm-none-eabi/lib/thumb/v7e-m/nofp\libg.a(lib_a-lseekr.o)
 .debug_frame   0x00003aec       0x2c d:/lijie_tools/clion_cubemx/gcc-arm-none-eabi-10.3-2021.10/bin/../lib/gcc/arm-none-eabi/10.3.1/../../../../arm-none-eabi/lib/thumb/v7e-m/nofp\libg.a(lib_a-readr.o)
 .debug_frame   0x00003b18       0x64 d:/lijie_tools/clion_cubemx/gcc-arm-none-eabi-10.3-2021.10/bin/../lib/gcc/arm-none-eabi/10.3.1/../../../../arm-none-eabi/lib/thumb/v7e-m/nofp\libg.a(lib_a-reent.o)
